 eboot

 Timestamp is 4da2a544 (Mon Apr 11 18:52:52 2011)

 Preferred load address is 00010000

 Start         Length     Name                   Class
 0001:00000000 000002f8H .astart                 CODE
 0001:00000300 0000fdfcH .rdata                  CODE
 0001:000100fc 00000022H .rdata$debug            CODE
 0001:00010120 00042258H .text                   CODE
 0001:00052378 000000d0H .xdata                  CODE
 0001:00052448 00000000H .edata                  CODE
 0002:00000000 00005a0cH .data                   DATA
 0002:00005a20 0001efecH .bss                    DATA
 0003:00000000 00001418H .pdata                  DATA

  Address         Publics by Value              Rva+Base       Lib:Object

 0000:00000000       ___safe_se_handler_count   00000000     <absolute>
 0000:00000000       ___safe_se_handler_table   00000000     <absolute>
 0001:00000000       StartUp                    00011000 f   bootcmn:startup.obj
 0001:000000f4       g_oalAddressTable          000110f4     bootcmn:startup.obj
 0001:0000016c       KernelStart                0001116c f   bootcmn:startup.obj
 0001:00000260       Launch                     00011260 f   bootcmn:startup.obj
 0001:00000320       ??_C@_0EK@BLGPAFDM@Microsoft?5Windows?5CE?5Ethernet?5Bo@ 00011320     eboot.obj
 0001:0000036c       ??_C@_0M@CJGCCEJL@Apr?511?52011?$AA@ 0001136c     eboot.obj
 0001:00000378       ??_C@_08MGEMPJAC@18?350?353?$AA@ 00011378     eboot.obj
 0001:00000384       ??_C@_05DFLKGENG@Topaz?$AA@ 00011384     eboot.obj
 0001:0000038c       ??_C@_0DO@GKLPKMK@ERROR?3?5Failed?5to?5detect?5and?5init@ 0001138c     eboot.obj
 0001:000003cc       ??_C@_0CJ@HMMHCENL@ERROR?3?5EbootWaitForHostConnect?5f@ 000113cc     eboot.obj
 0001:000003f8       ??_C@_0FA@OIIAKJBG@INFO?3?5EbootWaitForHostConnect?5?$CII@ 000113f8     eboot.obj
 0001:00000448       ??_C@_0EO@OMICEANL@INFO?3?5ResetDefaultBootCFG?3?5facto@ 00011448     eboot.obj
 0001:00000498       ??_C@_0EE@DJCDNEKB@WARNING?3?5ResetDefaultBootCFG?3?5sa@ 00011498     eboot.obj
 0001:000004e0       ??_C@_0EP@NEFDNHFP@WARNING?3?5ResetDefaultBootCFG?3?5fa@ 000114e0     eboot.obj
 0001:00000530       ??_C@_0EL@KFPIALJM@INFO?3?5ResetDefaultBootCFG?3?5facto@ 00011530     eboot.obj
 0001:00000580       ??_C@_0EG@GKGGEOCH@ERROR?3?5ResetDefaultBootCFG?3?5fail@ 00011580     eboot.obj
 0001:000005c8       ??_C@_07OHKHACFK@0?40?40?40?$AA@ 000115c8     eboot.obj
 0001:000005d0       ??_C@_0CP@LKBEOLND@?$AN?6Resetting?5factory?5default?5conf@ 000115d0     eboot.obj
 0001:00000600       ??_C@_0CM@PEMGPOKC@INFO?3?5OEMEthSendFrame?3?5retrying?5@ 00011600     eboot.obj
 0001:0000062c       ??_C@_1BM@MOEMNNDE@?$AAS?$AAa?$AAv?$AAe?$AA?5?$AAS?$AAe?$AAt?$AAt?$AAi?$AAn?$AAg?$AAs?$AA?$AA@ 0001162c     menu.obj
 0001:00000648       ??_C@_1M@PNBPANGG@?$AAR?$AAe?$AAs?$AAe?$AAt?$AA?$AA@ 00011648     menu.obj
 0001:00000654       ??_C@_1CK@DKDIBGID@?$AAM?$AAM?$AAC?$AA?5?$AAa?$AAn?$AAd?$AA?5?$AAS?$AAD?$AA?5?$AAU?$AAt?$AAi?$AAl?$AAi?$AAt?$AAi?$AAe?$AAs?$AA?$AA@ 00011654     menu.obj
 0001:00000680       ??_C@_1FC@NIGCHAIH@?$AAL?$AAa?$AAu?$AAn?$AAc?$AAh?$AA?5?$AAE?$AAx?$AAi?$AAs?$AAt?$AAi?$AAn?$AAg?$AA?5?$AAF?$AAl?$AAa?$AAs?$AAh?$AA?5?$AAR?$AAe?$AAs?$AAi?$AAd?$AAe?$AAn?$AAt?$AA?5?$AAI@ 00011680     menu.obj
 0001:000006d4       ??_C@_1CG@PPAMDBLA@?$AAD?$AAo?$AAw?$AAn?$AAl?$AAo?$AAa?$AAd?$AA?5?$AAI?$AAm?$AAa?$AAg?$AAe?$AA?5?$AAN?$AAo?$AAw?$AA?$AA@ 000116d4     menu.obj
 0001:000006fc       ??_C@_1DK@CJENBLML@?$AAS?$AAe?$AAl?$AAe?$AAc?$AAt?$AA?5?$AAW?$AAi?$AAn?$AAd?$AAo?$AAw?$AAs?$AA?5?$AAC?$AAE?$AA?5?$AAD?$AAe?$AAb?$AAu?$AAg?$AA?5?$AAU?$AAA?$AAR?$AAT?$AA?$AA@ 000116fc     menu.obj
 0001:00000738       ??_C@_1CI@MLMJOJI@?$AAS?$AAe?$AAl?$AAe?$AAc?$AAt?$AA?5?$AAE?$AAt?$AAh?$AAe?$AAr?$AA?5?$AAD?$AAe?$AAv?$AAi?$AAc?$AAe?$AA?$AA@ 00011738     menu.obj
 0001:00000760       ??_C@_1CE@PKBKOLCO@?$AAK?$AAI?$AAT?$AAL?$AA?5?$AAP?$AAa?$AAs?$AAs?$AAi?$AAv?$AAe?$AA?5?$AAM?$AAo?$AAd?$AAe?$AA?$AA@ 00011760     menu.obj
 0001:00000784       ??_C@_1CC@DBLKBKOG@?$AAK?$AAI?$AAT?$AAL?$AA?5?$AAE?$AAn?$AAa?$AAb?$AAl?$AAe?$AA?5?$AAM?$AAo?$AAd?$AAe?$AA?$AA@ 00011784     menu.obj
 0001:000007a8       ??_C@_1BO@PABCHCBJ@?$AAK?$AAI?$AAT?$AAL?$AA?5?$AAW?$AAo?$AAr?$AAk?$AA?5?$AAM?$AAo?$AAd?$AAe?$AA?$AA@ 000117a8     menu.obj
 0001:000007c8       ??_C@_1CC@PFDHOAOM@?$AAB?$AAo?$AAo?$AAt?$AAl?$AAo?$AAa?$AAd?$AAe?$AAr?$AA?5?$AAS?$AAh?$AAe?$AAl?$AAl?$AA?$AA@ 000117c8     menu.obj
 0001:000007ec       ??_C@_1DG@JKEDBFOF@?$AAC?$AAl?$AAe?$AAa?$AAn?$AA?5?$AAr?$AAe?$AAg?$AAi?$AAs?$AAt?$AAr?$AAy?$AA?5?$AA?$CG?$AA?5?$AAd?$AAa?$AAt?$AAa?$AAb?$AAa?$AAs?$AAe?$AAs?$AA?$AA@ 000117ec     menu.obj
 0001:00000824       ??_C@_1DA@JJAMJFOD@?$AAF?$AAo?$AAr?$AAm?$AAa?$AAt?$AA?5?$AAA?$AAl?$AAl?$AA?5?$AAN?$AAA?$AAN?$AAD?$AA?5?$AAR?$AAe?$AAg?$AAi?$AAo?$AAn?$AAs?$AA?$AA@ 00011824     menu.obj
 0001:00000854       ??_C@_1CM@MOIDFHOM@?$AAF?$AAo?$AAr?$AAm?$AAa?$AAt?$AA?5?$AAO?$AAS?$AA?5?$AAN?$AAA?$AAN?$AAD?$AA?5?$AAR?$AAe?$AAg?$AAi?$AAo?$AAn?$AA?$AA@ 00011854     menu.obj
 0001:00000880       ??_C@_1EO@JEPFIEIH@?$AAR?$AAe?$AAs?$AAe?$AAt?$AA?5?$AAt?$AAo?$AA?5?$AAF?$AAa?$AAc?$AAt?$AAo?$AAr?$AAy?$AA?5?$AAD?$AAe?$AAf?$AAa?$AAu?$AAl?$AAt?$AA?5?$AAC?$AAo?$AAn?$AAf?$AAi?$AAg?$AAu@ 00011880     menu.obj
 0001:000008d0       ??_C@_1CG@BBALNGAE@?$AAS?$AAe?$AAl?$AAe?$AAc?$AAt?$AA?5?$AAB?$AAo?$AAo?$AAt?$AA?5?$AAD?$AAe?$AAv?$AAi?$AAc?$AAe?$AA?$AA@ 000118d0     menu.obj
 0001:000008f8       ??_C@_1BG@GBKEAKLM@?$AAB?$AAo?$AAo?$AAt?$AA?5?$AAD?$AAe?$AAl?$AAa?$AAy?$AA?$AA@ 000118f8     menu.obj
 0001:00000910       ??_C@_19DDJNJOGL@?$AAD?$AAH?$AAC?$AAP?$AA?$AA@ 00011910     menu.obj
 0001:0000091c       ??_C@_1BI@PKAFKBAO@?$AAM?$AAA?$AAC?$AA?5?$AAA?$AAd?$AAd?$AAr?$AAe?$AAs?$AAs?$AA?$AA@ 0001191c     menu.obj
 0001:00000934       ??_C@_1CA@BMIKHDOB@?$AAS?$AAe?$AAt?$AA?5?$AAM?$AAA?$AAC?$AA?5?$AAA?$AAd?$AAd?$AAr?$AAe?$AAs?$AAs?$AA?$AA@ 00011934     menu.obj
 0001:00000954       ??_C@_1BA@LCJJAKKF@?$AAG?$AAa?$AAt?$AAe?$AAw?$AAa?$AAy?$AA?$AA@ 00011954     menu.obj
 0001:00000964       ??_C@_1BI@CJHLOJOF@?$AAS?$AAe?$AAt?$AA?5?$AAG?$AAa?$AAt?$AAe?$AAw?$AAa?$AAy?$AA?$AA@ 00011964     menu.obj
 0001:0000097c       ??_C@_1BA@MJOPHPLD@?$AAI?$AAP?$AA?5?$AAM?$AAa?$AAs?$AAk?$AA?$AA@ 0001197c     menu.obj
 0001:0000098c       ??_C@_1BI@FCANJMPD@?$AAS?$AAe?$AAt?$AA?5?$AAI?$AAP?$AA?5?$AAM?$AAa?$AAs?$AAk?$AA?$AA@ 0001198c     menu.obj
 0001:000009a4       ??_C@_1BG@BLDDCHFC@?$AAI?$AAP?$AA?5?$AAA?$AAd?$AAd?$AAr?$AAe?$AAs?$AAs?$AA?$AA@ 000119a4     menu.obj
 0001:000009bc       ??_C@_0CH@HJFHFGIJ@INFO?3?5MAC?5address?3?5?$CFx?9?$CFx?9?$CFx?9?$CFx?9?$CF@ 000119bc     menu.obj
 0001:000009e8       ??_C@_0EA@OMKEPEHK@ERROR?3?5Invalid?5Ethernet?5address?5@ 000119e8     menu.obj
 0001:00000a28       ??_C@_0CA@OPBDBDDP@?$AN?6Starting?5auto?5download?5?4?4?4?5?$AN?6?$AA@ 00011a28     menu.obj
 0001:00000a48       ??_C@_0CA@CLDGGJMD@?$AN?6Launching?5flash?5image?5?5?4?4?4?5?$AN?6?$AA@ 00011a48     menu.obj
 0001:00000a68       ??_C@_0N@FLJDAHIC@?$CFd?5seconds?4?5?$AA@ 00011a68     menu.obj
 0001:00000a78       ??_C@_0CM@MPOIFBJA@?$AN?6Initiating?5image?5download?5in?5?$CF@ 00011a78     menu.obj
 0001:00000aa4       ??_C@_0DI@JNGDCJGH@?$AN?6Press?5?$FLENTER?$FN?5to?5download?5now?5@ 00011aa4     menu.obj
 0001:00000ae0       ??_C@_0EJ@LBCIGPCN@?$AN?6Press?5?$FLENTER?$FN?5to?5launch?5image?5@ 00011ae0     menu.obj
 0001:00000b2c       ??_C@_0CK@PCOCDPAP@?$AN?6Initiating?5image?5launch?5in?5?$CFd?5@ 00011b2c     menu.obj
 0001:00000b58       ??_C@_0EN@KBHLEBPN@?$AN?6Press?5?$FLENTER?$FN?5to?5launch?5image?5@ 00011b58     menu.obj
 0001:00000ba8       ??_C@_0EJ@NPNOADG@WARNING?3?5?5Uninitialized?5MAC?5addr@ 00011ba8     menu.obj
 0001:00000bf4       ??_C@_02PCIJFNDE@?$AN?6?$AA@ 00011bf4     menu.obj
 0001:00000bf8       ??_C@_0BE@PKINMFFD@?5?3?5Invalid?5Device?$AN?6?$AA@ 00011bf8     menu.obj
 0001:00000c0c       ??_C@_0BA@FMMDOFML@?5?3?5USB?5Serial?$AN?6?$AA@ 00011c0c     menu.obj
 0001:00000c1c       ??_C@_0P@NONOIHBD@?5?3?5USB?5RNDIS?$AN?6?$AA@ 00011c1c     menu.obj
 0001:00000c2c       ??_C@_08HCDDKNJJ@?5?3?5FEC?$AN?6?$AA@ 00011c2c     menu.obj
 0001:00000c38       ??_C@_0L@IMACDOJI@?5?3?5UART3?$AN?6?$AA@ 00011c38     menu.obj
 0001:00000c44       ??_C@_0L@DELOFJPN@?5?3?5UART2?$AN?6?$AA@ 00011c44     menu.obj
 0001:00000c50       ??_C@_0L@CGALPGBD@?5?3?5UART1?$AN?6?$AA@ 00011c50     menu.obj
 0001:00000c5c       ??_C@_0O@CMIFMFKO@?5?3?5Disabled?$AN?6?$AA@ 00011c5c     menu.obj
 0001:00000c6c       ??_C@_0BE@IIODHDMP@?5?3?5NK?5from?5SD?1MMC?$AN?6?$AA@ 00011c6c     menu.obj
 0001:00000c80       ??_C@_0BC@IHBBJPDE@?5?3?5NK?5from?5NAND?$AN?6?$AA@ 00011c80     menu.obj
 0001:00000c94       ??_C@_0M@CDHNGIPM@?$CFu?4?$CFu?4?$CFu?4?$CFu?$AA@ 00011c94     oal_blnk:ipformata.obj
 0001:00000ca0       ??_C@_1O@INIEDEDF@?$AA?$CI?$AAN?$AAU?$AAL?$AAL?$AA?$CJ?$AA?$AA@ 00011ca0     oal_blnk:formata.obj
 0001:00000cb0       ??_C@_06LHGEHABH@?$CINULL?$CJ?$AA@ 00011cb0     oal_blnk:formata.obj
 0001:00000cb8       ??_C@_1DE@DAHNLBLJ@?$AA?9?$AAO?$AAA?$AAL?$AAP?$AAA?$AAt?$AAo?$AAV?$AAA?$AA?$CI?$AAv?$AAa?$AA?5?$AA?$DN?$AA?5?$AA0?$AAx?$AA?$CF?$AA0?$AA8?$AAx?$AA?$CJ?$AA?$AN?$AA?6?$AA?$AA@ 00011cb8     oal_blmemory_arm:memory.obj
 0001:00000cec       ??_C@_1CO@JEIJEAKF@?$AA?$CL?$AAO?$AAA?$AAL?$AAP?$AAA?$AAt?$AAo?$AAV?$AAA?$AA?$CI?$AA0?$AAx?$AA?$CF?$AAx?$AA?0?$AA?5?$AA?$CF?$AAd?$AA?$CJ?$AA?$AN?$AA?6?$AA?$AA@ 00011cec     oal_blmemory_arm:memory.obj
 0001:00000d1c       ??_C@_1DA@BBOHBBNH@?$AA?9?$AAO?$AAA?$AAL?$AAV?$AAA?$AAt?$AAo?$AAP?$AAA?$AA?$CI?$AAp?$AAa?$AA?5?$AA?$DN?$AA?5?$AA0?$AAx?$AA?$CF?$AAx?$AA?$CJ?$AA?$AN?$AA?6?$AA?$AA@ 00011d1c     oal_blmemory_arm:memory.obj
 0001:00000d50       ??_C@_1GE@IPLNFFII@?$AAE?$AAR?$AAR?$AAO?$AAR?$AA?3?$AAO?$AAA?$AAL?$AAV?$AAA?$AAt?$AAo?$AAP?$AAA?$AA?3?$AA?5?$AAi?$AAn?$AAv?$AAa?$AAl?$AAi?$AAd?$AA?5?$AAv?$AAi?$AAr?$AAt?$AAu?$AAa?$AAl@ 00011d50     oal_blmemory_arm:memory.obj
 0001:00000db4       ??_C@_1CK@LKNIEAFP@?$AA?$CL?$AAO?$AAA?$AAL?$AAV?$AAA?$AAt?$AAo?$AAP?$AAA?$AA?$CI?$AA0?$AAx?$AA?$CF?$AA0?$AA8?$AAx?$AA?$CJ?$AA?$AN?$AA?6?$AA?$AA@ 00011db4     oal_blmemory_arm:memory.obj
 0001:00000de0       ??_C@_1DM@OCLJLKJN@?$AA?5?$AA?5?$AA?5?$AA?5?$AAP?$AAe?$AAr?$AAi?$AAp?$AAh?$AA?5?$AAC?$AAl?$AAk?$AA?5?$AAU?$AAA?$AAR?$AAT?$AA?5?$AA?$DN?$AA?5?$AA?$CF?$AAd?$AA?5?$AAH?$AAz?$AA?$AN?$AA?6?$AA?$AA@ 00011de0     bspcmn:bspargs.obj
 0001:00000e1c       ??_C@_1DM@BGNEBGOE@?$AA?5?$AA?5?$AA?5?$AA?5?$AAP?$AAe?$AAr?$AAi?$AAp?$AAh?$AA?5?$AAC?$AAl?$AAk?$AA?5?$AAS?$AAS?$AAI?$AA2?$AA?5?$AA?$DN?$AA?5?$AA?$CF?$AAd?$AA?5?$AAH?$AAz?$AA?$AN?$AA?6?$AA?$AA@ 00011e1c     bspcmn:bspargs.obj
 0001:00000e58       ??_C@_1DM@EOMKLPMM@?$AA?5?$AA?5?$AA?5?$AA?5?$AAP?$AAe?$AAr?$AAi?$AAp?$AAh?$AA?5?$AAC?$AAl?$AAk?$AA?5?$AAS?$AAS?$AAI?$AA1?$AA?5?$AA?$DN?$AA?5?$AA?$CF?$AAd?$AA?5?$AAH?$AAz?$AA?$AN?$AA?6?$AA?$AA@ 00011e58     bspcmn:bspargs.obj
 0001:00000e94       ??_C@_1DM@CJNLEDDI@?$AA?5?$AA?5?$AA?5?$AA?5?$AAP?$AAe?$AAr?$AAi?$AAp?$AAh?$AA?5?$AAC?$AAl?$AAk?$AA?5?$AAS?$AAI?$AAM?$AA2?$AA?5?$AA?$DN?$AA?5?$AA?$CF?$AAd?$AA?5?$AAH?$AAz?$AA?$AN?$AA?6?$AA?$AA@ 00011e94     bspcmn:bspargs.obj
 0001:00000ed0       ??_C@_1DM@HBMFOKBA@?$AA?5?$AA?5?$AA?5?$AA?5?$AAP?$AAe?$AAr?$AAi?$AAp?$AAh?$AA?5?$AAC?$AAl?$AAk?$AA?5?$AAS?$AAI?$AAM?$AA1?$AA?5?$AA?$DN?$AA?5?$AA?$CF?$AAd?$AA?5?$AAH?$AAz?$AA?$AN?$AA?6?$AA?$AA@ 00011ed0     bspcmn:bspargs.obj
 0001:00000f0c       ??_C@_1DK@MIDNNIPL@?$AA?5?$AA?5?$AA?5?$AA?5?$AAP?$AAe?$AAr?$AAi?$AAp?$AAh?$AA?5?$AAC?$AAl?$AAk?$AA?5?$AAP?$AAW?$AAM?$AA?5?$AA?$DN?$AA?5?$AA?$CF?$AAd?$AA?5?$AAH?$AAz?$AA?$AN?$AA?6?$AA?$AA@ 00011f0c     bspcmn:bspargs.obj
 0001:00000f48       ??_C@_1DO@GMICDJDG@?$AA?5?$AA?5?$AA?5?$AA?5?$AAP?$AAe?$AAr?$AAi?$AAp?$AAh?$AA?5?$AAC?$AAl?$AAk?$AA?5?$AAO?$AAW?$AAI?$AAR?$AAE?$AA?5?$AA?$DN?$AA?5?$AA?$CF?$AAd?$AA?5?$AAH?$AAz?$AA?$AN?$AA?6?$AA?$AA@ 00011f48     bspcmn:bspargs.obj
 0001:00000f88       ??_C@_1DK@PEAOHMIM@?$AA?5?$AA?5?$AA?5?$AA?5?$AAP?$AAe?$AAr?$AAi?$AAp?$AAh?$AA?5?$AAC?$AAl?$AAk?$AA?5?$AAN?$AAF?$AAC?$AA?5?$AA?$DN?$AA?5?$AA?$CF?$AAd?$AA?5?$AAH?$AAz?$AA?$AN?$AA?6?$AA?$AA@ 00011f88     bspcmn:bspargs.obj
 0001:00000fc4       ??_C@_1DM@EONHEPCP@?$AA?5?$AA?5?$AA?5?$AA?5?$AAP?$AAe?$AAr?$AAi?$AAp?$AAh?$AA?5?$AAC?$AAl?$AAk?$AA?5?$AAL?$AAC?$AAD?$AAC?$AA?5?$AA?$DN?$AA?5?$AA?$CF?$AAd?$AA?5?$AAH?$AAz?$AA?$AN?$AA?6?$AA?$AA@ 00011fc4     bspcmn:bspargs.obj
 0001:00001000       ??_C@_1DK@DLMOJFOL@?$AA?5?$AA?5?$AA?5?$AA?5?$AAP?$AAe?$AAr?$AAi?$AAp?$AAh?$AA?5?$AAC?$AAl?$AAk?$AA?5?$AAI?$AA2?$AAC?$AA?5?$AA?$DN?$AA?5?$AA?$CF?$AAd?$AA?5?$AAH?$AAz?$AA?$AN?$AA?6?$AA?$AA@ 00012000     bspcmn:bspargs.obj
 0001:0000103c       ??_C@_1DK@CDOLKHPK@?$AA?5?$AA?5?$AA?5?$AA?5?$AAP?$AAe?$AAr?$AAi?$AAp?$AAh?$AA?5?$AAC?$AAl?$AAk?$AA?5?$AAG?$AAP?$AAT?$AA?5?$AA?$DN?$AA?5?$AA?$CF?$AAd?$AA?5?$AAH?$AAz?$AA?$AN?$AA?6?$AA?$AA@ 0001203c     bspcmn:bspargs.obj
 0001:00001078       ??_C@_1EA@MPFCNGCJ@?$AA?5?$AA?5?$AA?5?$AA?5?$AAP?$AAe?$AAr?$AAi?$AAp?$AAh?$AA?5?$AAC?$AAl?$AAk?$AA?5?$AAE?$AAS?$AAD?$AAH?$AAC?$AA2?$AA?5?$AA?$DN?$AA?5?$AA?$CF?$AAd?$AA?5?$AAH?$AAz?$AA?$AN?$AA?6?$AA?$AA@ 00012078     bspcmn:bspargs.obj
 0001:000010b8       ??_C@_1EA@JHEMHPAB@?$AA?5?$AA?5?$AA?5?$AA?5?$AAP?$AAe?$AAr?$AAi?$AAp?$AAh?$AA?5?$AAC?$AAl?$AAk?$AA?5?$AAE?$AAS?$AAD?$AAH?$AAC?$AA1?$AA?5?$AA?$DN?$AA?5?$AA?$CF?$AAd?$AA?5?$AAH?$AAz?$AA?$AN?$AA?6?$AA?$AA@ 000120b8     bspcmn:bspargs.obj
 0001:000010f8       ??_C@_1DM@JHCBKDAO@?$AA?5?$AA?5?$AA?5?$AA?5?$AAP?$AAe?$AAr?$AAi?$AAp?$AAh?$AA?5?$AAC?$AAl?$AAk?$AA?5?$AAE?$AAS?$AAA?$AAI?$AA?5?$AA?$DN?$AA?5?$AA?$CF?$AAd?$AA?5?$AAH?$AAz?$AA?$AN?$AA?6?$AA?$AA@ 000120f8     bspcmn:bspargs.obj
 0001:00001134       ??_C@_1DM@IFJDDBGO@?$AA?5?$AA?5?$AA?5?$AA?5?$AAP?$AAe?$AAr?$AAi?$AAp?$AAh?$AA?5?$AAC?$AAl?$AAk?$AA?5?$AAE?$AAP?$AAI?$AAT?$AA?5?$AA?$DN?$AA?5?$AA?$CF?$AAd?$AA?5?$AAH?$AAz?$AA?$AN?$AA?6?$AA?$AA@ 00012134     bspcmn:bspargs.obj
 0001:00001170       ??_C@_1DK@JCCOAGIN@?$AA?5?$AA?5?$AA?5?$AA?5?$AAP?$AAe?$AAr?$AAi?$AAp?$AAh?$AA?5?$AAC?$AAl?$AAk?$AA?5?$AAC?$AAS?$AAI?$AA?5?$AA?$DN?$AA?5?$AA?$CF?$AAd?$AA?5?$AAH?$AAz?$AA?$AN?$AA?6?$AA?$AA@ 00012170     bspcmn:bspargs.obj
 0001:000011ac       ??_C@_1DA@OBKCEEDF@?$AA?5?$AA?5?$AA?5?$AA?5?$AAU?$AAS?$AAB?$AA?5?$AAC?$AAL?$AAO?$AAC?$AAK?$AA?5?$AA?$DN?$AA?5?$AA?$CF?$AAd?$AA?5?$AAH?$AAz?$AA?$AN?$AA?6?$AA?$AA@ 000121ac     bspcmn:bspargs.obj
 0001:000011dc       ??_C@_1DC@HLPKBKNH@?$AA?5?$AA?5?$AA?5?$AA?5?$AAI?$AAP?$AAG?$AA?5?$AAC?$AAL?$AAO?$AAC?$AAK?$AA?5?$AA?5?$AA?$DN?$AA?5?$AA?$CF?$AAd?$AA?5?$AAH?$AAz?$AA?$AN?$AA?6?$AA?$AA@ 000121dc     bspcmn:bspargs.obj
 0001:00001210       ??_C@_1DC@CKMNKMMI@?$AA?5?$AA?5?$AA?5?$AA?5?$AAA?$AAH?$AAB?$AA?5?$AAC?$AAL?$AAO?$AAC?$AAK?$AA?5?$AA?5?$AA?$DN?$AA?5?$AA?$CF?$AAd?$AA?5?$AAH?$AAz?$AA?$AN?$AA?6?$AA?$AA@ 00012210     bspcmn:bspargs.obj
 0001:00001244       ??_C@_1DC@IAJIALLM@?$AA?5?$AA?5?$AA?5?$AA?5?$AAA?$AAR?$AAM?$AA?5?$AAC?$AAL?$AAO?$AAC?$AAK?$AA?5?$AA?5?$AA?$DN?$AA?5?$AA?$CF?$AAd?$AA?5?$AAH?$AAz?$AA?$AN?$AA?6?$AA?$AA@ 00012244     bspcmn:bspargs.obj
 0001:00001278       ??_C@_1CO@IOOCOMMB@?$AA?5?$AA?5?$AA?5?$AA?5?$AAU?$AAS?$AAB?$AA?5?$AAP?$AAL?$AAL?$AA?5?$AA?5?$AA?$DN?$AA?5?$AA?$CF?$AAd?$AA?5?$AAH?$AAz?$AA?$AN?$AA?6?$AA?$AA@ 00012278     bspcmn:bspargs.obj
 0001:000012a8       ??_C@_1CO@LHEJCJEH@?$AA?5?$AA?5?$AA?5?$AA?5?$AAM?$AAC?$AAU?$AA?5?$AAP?$AAL?$AAL?$AA?5?$AA?5?$AA?$DN?$AA?5?$AA?$CF?$AAd?$AA?5?$AAH?$AAz?$AA?$AN?$AA?6?$AA?$AA@ 000122a8     bspcmn:bspargs.obj
 0001:000012d8       ??_C@_1DG@IJHKIPGD@?$AAB?$AAS?$AAP?$AA?5?$AAC?$AAl?$AAo?$AAc?$AAk?$AA?5?$AAC?$AAo?$AAn?$AAf?$AAi?$AAg?$AAu?$AAr?$AAa?$AAt?$AAi?$AAo?$AAn?$AA?3?$AA?$AN?$AA?6?$AA?$AA@ 000122d8     bspcmn:bspargs.obj
 0001:00001310       ??_C@_0EL@BJCJJOHF@WARNING?3?5Could?5not?5find?5the?5boot@ 00012310     bootcmn:main.obj
 0001:0000135c       ??_C@_0DI@FJCDBJCA@INFO?3?5OEMPlatformInit?3?5Initializ@ 0001235c     bootcmn:main.obj
 0001:00001398       ??_C@_0EE@KIMOANOM@WARNING?3?5OEMPlatformInit?3?5Failed@ 00012398     bootcmn:main.obj
 0001:000013dc       ??_C@_0CO@DOGAJLCC@INFO?3?5FAKING?5?5Bootloader?5launche@ 000123dc     bootcmn:main.obj
 0001:0000140c       ??_C@_0CM@NHECMJBH@INFO?3?5?5Bootloader?5launched?5from?5@ 0001240c     bootcmn:main.obj
 0001:00001438       ??_C@_0EI@DPIDEJBF@INFO?3?5?5XLDR?5launched?5from?5I2C?5EE@ 00012438     bootcmn:main.obj
 0001:00001480       ??_C@_0CI@BBFNIMIB@INFO?3?5?5Bootloader?5launched?5from?5@ 00012480     bootcmn:main.obj
 0001:000014a8       ??_C@_0CH@OFHLFLCP@INFO?3?5?5Bootloader?5launched?5from?5@ 000124a8     bootcmn:main.obj
 0001:000014d0       ??_C@_0CO@CLCHIGDN@ERROR?3?5Failed?5to?5load?5OS?5image?5f@ 000124d0     bootcmn:main.obj
 0001:00001500       ??_C@_0CN@MKBLLODK@ERROR?3?5Failed?5to?5load?5IPL?5image?5@ 00012500     bootcmn:main.obj
 0001:00001530       ??_C@_0CM@HCKAPHGI@ERROR?3?5Failed?5to?5load?5OS?5image?5f@ 00012530     bootcmn:main.obj
 0001:0000155c       ??_C@_0DB@OPLKFPCH@Received?5boot?5request?5ack?4?4?4?5sta@ 0001255c     bootcmn:main.obj
 0001:00001590       ??_C@_0DA@MDAAKDGO@Received?5boot?5request?5ack?4?4?4?5jum@ 00012590     bootcmn:main.obj
 0001:000015c0       ??_C@_0BO@GOCJJNNJ@Failed?5to?5send?5boot?5request?$AN?6?$AA@ 000125c0     bootcmn:main.obj
 0001:000015e0       ??_C@_0BK@KJKLPNKO@Sending?5boot?5request?4?4?4?$AN?6?$AA@ 000125e0     bootcmn:main.obj
 0001:000015fc       ??_C@_0BP@KFHIKLKI@INFO?3?5Using?5device?5name?3?5?8?$CFs?8?6?$AA@ 000125fc     bootcmn:main.obj
 0001:0000161c       ??_C@_05ENGOENAF@IMX25?$AA@ 0001261c     bootcmn:main.obj
 0001:00001624       ??_C@_06MHMFDNCL@?$AN?6?$AN?6?$AN?6?$AA@ 00012624     bootcmn:main.obj
 0001:00001630       ??_C@_0EE@NJJIECID@Download?5successful?$CB?5?5Jumping?5to@ 00012630     bootcmn:main.obj
 0001:00001674       ??_C@_0DA@NOPADPHG@?$AN?6INFO?3?5DIO?5image?5with?5starting?5@ 00012674     bootcmn:main.obj
 0001:000016a4       ??_C@_0DN@EFKGNOEL@?$AN?6WARNING?3?5Unsupported?5binary?5fo@ 000126a4     bootcmn:main.obj
 0001:000016e4       ??_C@_0CD@BDBOCALK@?$AN?6INFO?3?5NK?5NB0?5remapped?5to?50x?$CFx?4@ 000126e4     bootcmn:main.obj
 0001:00001708       ??_C@_0EB@DDOPHGII@Specify?5destination?5for?5NK?5NB0?5?$FL@ 00012708     bootcmn:main.obj
 0001:0000174c       ??_C@_04IMADAAK@?4nb0?$AA@ 0001274c     bootcmn:main.obj
 0001:00001754       ??_C@_0CM@PFPHHIOP@?$AN?6INFO?3?5EBOOT?1SBOOT?5NB0?5remapped@ 00012754     bootcmn:main.obj
 0001:00001780       ??_C@_0EK@NNMIMOMC@Specify?5destination?5for?5EBOOT?1SB@ 00012780     bootcmn:main.obj
 0001:000017cc       ??_C@_09KGAFPJBE@sboot?4nb0?$AA@ 000127cc     bootcmn:main.obj
 0001:000017d8       ??_C@_09IMLFAILL@eboot?4nb0?$AA@ 000127d8     bootcmn:main.obj
 0001:000017e4       ??_C@_0CD@IJDCBNHD@INFO?3?5XLDR?5NB0?5remapped?5to?50x?$CFx?4@ 000127e4     bootcmn:main.obj
 0001:00001808       ??_C@_0EK@CJLNKEGP@Specify?5destination?5for?5XLDR?5NB0@ 00012808     bootcmn:main.obj
 0001:00001854       ??_C@_08NNMHMDLM@xldr?4nb0?$AA@ 00012854     bootcmn:main.obj
 0001:00001860       ??_C@_0EF@MBMCDLHM@INFO?3?5OEMMultiBINNotify?5?$CIdwNumRe@ 00012860     bootcmn:main.obj
 0001:000018a8       ??_C@_0CD@ELMGDNGD@INFO?3?5OEMReportError?5Reason?50x?$CFx@ 000128a8     bootcmn:main.obj
 0001:000018cc       ??_C@_0CA@OFFHNLCK@ERROR?3?5Invalid?5address?5range?4?$AN?6?$AA@ 000128cc     bootcmn:main.obj
 0001:000018ec       ??_C@_0CP@JDGPIHPA@INFO?3?5Downloading?5EBOOT?1SBOOT?5fo@ 000128ec     bootcmn:main.obj
 0001:0000191c       ??_C@_0CE@HMABAKKF@INFO?3?5Downloading?5XLDR?5SPI?5image@ 0001291c     bootcmn:main.obj
 0001:00001940       ??_C@_0CL@LNJKHKKB@INFO?3?5Downloading?5XLDR?5I2C?5EEPRO@ 00012940     bootcmn:main.obj
 0001:0000196c       ??_C@_0CF@HCMGOJNF@INFO?3?5Downloading?5NK?5SD?1MMC?5imag@ 0001296c     bootcmn:main.obj
 0001:00001994       ??_C@_0DC@PIMDAHJO@INFO?3?5Downloading?5EBOOT?1SBOOT?5fo@ 00012994     bootcmn:main.obj
 0001:000019c8       ??_C@_0CH@LGJDEBHD@INFO?3?5Downloading?5XLDR?5SD?1MMC?5im@ 000129c8     bootcmn:main.obj
 0001:000019f0       ??_C@_0CC@JCIKJLGP@INFO?3?5Downloading?5NK?5RAM?5image?4?$AN@ 000129f0     bootcmn:main.obj
 0001:00001a14       ??_C@_0CD@CCLLAHMG@INFO?3?5Downloading?5NK?5NAND?5image?4@ 00012a14     bootcmn:main.obj
 0001:00001a38       ??_C@_0CM@BDOCNOGM@INFO?3?5Downloading?5EBOOT?1SBOOT?5NA@ 00012a38     bootcmn:main.obj
 0001:00001a64       ??_C@_0CF@KOHMACKP@INFO?3?5Downloading?5XLDR?5NAND?5imag@ 00012a64     bootcmn:main.obj
 0001:00001a8c       ??_C@_0DO@IAHEPFAH@INFO?3?5OEMVerifyMemory?5?$CICA?5?$DN?50x?$CFx@ 00012a8c     bootcmn:main.obj
 0001:00001acc       ??_C@_0CE@PDFEDJGG@INFO?3?5Downloading?5DIO?5NAND?5image@ 00012acc     bootcmn:main.obj
 0001:00001af0       ??_C@_0DG@PBAIANGJ@ERROR?3?5StoreBootCFG?3?5failed?5to?5w@ 00012af0     bootcmn:main.obj
 0001:00001b28       ??_C@_0FG@GFJDGOLO@ERROR?3?5LoadBootCFG?3?5ConfigMagicN@ 00012b28     bootcmn:main.obj
 0001:00001b80       ??_C@_0DE@GGGDJLON@ERROR?3?5LoadBootCFG?3?5failed?5to?5lo@ 00012b80     bootcmn:main.obj
 0001:00001bb8       ??_C@_0EJ@OHBNOOGC@ERROR?3?5Failed?5to?5initialize?5unkn@ 00012bb8     bootcmn:ether.obj
 0001:00001c08       ??_C@_0EC@PJLCGLI@ERROR?3?5Failed?5to?5detect?5and?5init@ 00012c08     bootcmn:ether.obj
 0001:00001c4c       ??_C@_0DM@EJPJMAEJ@ERROR?3?5Failed?5to?5initialize?5USB?5@ 00012c4c     bootcmn:ether.obj
 0001:00001c88       ??_C@_0DH@NMDABBIN@ERROR?3?5Failed?5to?5initialize?5Fast@ 00012c88     bootcmn:ether.obj
 0001:00001cc0       ??_C@_0CO@JBGBMPAB@INFO?3?5Fast?5Ethernet?5controller?5i@ 00012cc0     bootcmn:ether.obj
 0001:00001cf0       ??_C@_0DH@HPMFHNO@ERROR?3?5Failed?5to?5initialize?5Fast@ 00012cf0     bootcmn:ether.obj
 0001:00001d28       ??_C@_0EA@JPDHBOGB@ERROR?3?5Failed?5to?5initialize?5ARC?5@ 00012d28     bootcmn:ether.obj
 0001:00001d68       ??_C@_0CK@CODIHID@INFO?3?5Trying?5to?5initialize?5USB?5R@ 00012d68     bootcmn:ether.obj
 0001:00001d94       ??_C@_0BO@LOAGLJOJ@Do?5you?5want?5to?5reset?5?$FLY?2N?$FN?5?$AN?6?$AA@ 00012d94     bootcmn:utils.obj
 0001:00001db4       ??_C@_0BB@MEBHIIAP@SpinForever?4?4?4?$AN?6?$AA@ 00012db4     bootcmn:utils.obj
 0001:00001dc8       ??_C@_0CG@DBIMOJLH@BootTimerInit?3?5EPIT?5mapping?5fail@ 00012dc8     bootcmn:utils.obj
 0001:00001df0       ??_C@_0DK@HFAHLAPK@Enter?5maximum?5number?5of?5boot?5me?5@ 00012df0     bootcmn:utils.obj
 0001:00001e2c       ??_C@_0CL@OJFDJCGB@?$AN?6Use?50?5for?5continuous?5boot?5me?5p@ 00012e2c     bootcmn:utils.obj
 0001:00001e58       ??_C@_0DF@JLKFBNBO@?$AN?6Enter?5maximum?5number?5of?5second@ 00012e58     bootcmn:utils.obj
 0001:00001e90       ??_C@_0CA@PFBHAHMM@Reboot?5the?5device?5manually?4?4?4?$AN?6?$AA@ 00012e90     bootcmn:flash.obj
 0001:00001eb0       ??_C@_0CC@GOAJDIEC@Flash?5update?5has?5been?5canceled?4?$AN@ 00012eb0     bootcmn:flash.obj
 0001:00001ed4       ??_C@_0CA@IKNJPMAI@Do?5you?5want?5to?5continue?5?$CIy?1n?$CJ?$DP?5?$AA@ 00012ed4     bootcmn:flash.obj
 0001:00001ef4       ??_C@_0CG@MMBMGINJ@?$AN?6WARNING?3?5?5Flash?5update?5request@ 00012ef4     bootcmn:flash.obj
 0001:00001f1c       ??_C@_0CP@IFDOEFCL@INFO?3?5Update?5of?5XLDR?5completed?5s@ 00012f1c     bootcmn:cspi_flash.obj
 0001:00001f4c       ??_C@_0CC@DMLNFECM@WARNING?3?5Failed?5to?5verify?5XLDR?4?$AN@ 00012f4c     bootcmn:cspi_flash.obj
 0001:00001f70       ??_C@_0DB@BAMNCDJA@WARNING?3?5Failed?5to?5read?5XLDR?5in?5@ 00012f70     bootcmn:cspi_flash.obj
 0001:00001fa4       ??_C@_0CO@MHLLIGAH@WARNING?3?5Failed?5to?5write?5XLDR?5in@ 00012fa4     bootcmn:cspi_flash.obj
 0001:00001fd4       ??_C@_0CO@OOFAPEAH@WARNING?3?5Unable?5to?5erase?5SPI?5fla@ 00012fd4     bootcmn:cspi_flash.obj
 0001:00002008       ??_C@_0EC@IKNNGHEA@INFO?3?5Using?5XLDR?5image?5from?5flas@ 00013008     bootcmn:cspi_flash.obj
 0001:0000204c       ??_C@_0CF@GABMJBPB@ERROR?3?5XLDR?5exceeds?5allocated?5si@ 0001304c     bootcmn:cspi_flash.obj
 0001:00002074       ??_C@_0CO@DBDCEEDI@ERROR?3?5Unable?5to?5get?5SPI?5flash?5i@ 00013074     bootcmn:cspi_flash.obj
 0001:000020a4       ??_C@_0DJ@LJDMMIHA@INFO?3?5Writing?5XLDR?5image?5to?5SPI?5@ 000130a4     bootcmn:cspi_flash.obj
 0001:000020e0       ??_C@_0ED@HJBHPIPI@WARNING?3?5SPI?5Flash?5device?5doesn?8@ 000130e0     bootcmn:cspi_flash.obj
 0001:00002124       ??_C@_0DG@PNOMNNHB@INFO?3?5Update?5of?5EBOOT?1SBOOT?5comp@ 00013124     bootcmn:cspi_flash.obj
 0001:0000215c       ??_C@_0CH@NDFCJD@ERROR?3?5Failed?5to?5verify?5EBOOT?1SB@ 0001315c     bootcmn:cspi_flash.obj
 0001:00002184       ??_C@_0BJ@DHAKPJOJ@INFO?3?5Verifying?5image?4?$AN?6?$AA@ 00013184     bootcmn:cspi_flash.obj
 0001:000021a0       ??_C@_0CH@DLBGIHNI@ERROR?3?5Failed?5to?5update?5EBOOT?1SB@ 000131a0     bootcmn:cspi_flash.obj
 0001:000021c8       ??_C@_0EP@OHKPPMNH@INFO?3?5Programming?5EBOOT?1SBOOT?5im@ 000131c8     bootcmn:cspi_flash.obj
 0001:00002218       ??_C@_0DB@OLFBJNHF@ERROR?3?5Unable?5to?5erase?5SPI?5flash@ 00013218     bootcmn:cspi_flash.obj
 0001:0000224c       ??_C@_0CK@NHLALAMN@INFO?3?5Found?5bad?5SPI?5flash?5block?5@ 0001324c     bootcmn:cspi_flash.obj
 0001:00002278       ??_C@_0DA@NIELMACL@INFO?3?5Erasing?5SPI?5flash?5blocks?5?$FL@ 00013278     bootcmn:cspi_flash.obj
 0001:000022a8       ??_C@_0DN@HEEIMBBG@ERROR?3?5Boot?5size?5exceeds?5reserve@ 000132a8     bootcmn:cspi_flash.obj
 0001:000022e8       ??_C@_0DJ@MKEMIADH@INFO?3?5Writing?5Boot?5image?5to?5SPI?5@ 000132e8     bootcmn:cspi_flash.obj
 0001:00002324       ??_C@_0DN@OKBNDMKM@WARNING?3?5SPI?5device?5doesn?8t?5exis@ 00013324     bootcmn:cspi_flash.obj
 0001:00002364       ??_C@_0DE@MHADHDG@ERROR?3?5Failed?5to?5load?5boot?5confi@ 00013364     bootcmn:cspi_flash.obj
 0001:00002398       ??_C@_0CM@KBCPGLLJ@INFO?3?5Loading?5boot?5configuration@ 00013398     bootcmn:cspi_flash.obj
 0001:000023c4       ??_C@_0DG@PDOHILLO@INFO?3?5Successfully?5stored?5boot?5c@ 000133c4     bootcmn:cspi_flash.obj
 0001:000023fc       ??_C@_0CB@FMPGMDDB@ERROR?3?5Failed?5to?5update?5EBOOT?4?$AN?6@ 000133fc     bootcmn:cspi_flash.obj
 0001:00002420       ??_C@_0CK@EKCHFDOP@INFO?3?5Storing?5boot?5configuration@ 00013420     bootcmn:cspi_flash.obj
 0001:00002450       ??_C@_1EO@DICLCFIH@?$AAI?$AA2?$AAC?$AA?5?$AAE?$AAE?$AAP?$AAR?$AAO?$AAM?$AA?5?$AAX?$AAl?$AAd?$AAr?$AA?5?$AAW?$AAr?$AAi?$AAt?$AAt?$AAe?$AAn?$AA?5?$AAS?$AAu?$AAc?$AAc?$AAe?$AAs?$AAs?$AAf@ 00013450     bootcmn:i2c_eeprom.obj
 0001:000024a0       ??_C@_0EN@EEDEPJBE@ERROR?3?5I2CEEPROMWriteXldr?3?5Read?5@ 000134a0     bootcmn:i2c_eeprom.obj
 0001:000024f0       ??_C@_0CN@OKPHLHJF@ERROR?3?5I2CEEPROMWriteXldr?3?5PageR@ 000134f0     bootcmn:i2c_eeprom.obj
 0001:00002520       ??_C@_0CO@FJCGKCNG@ERROR?3?5I2CEEPROMWriteXldr?3?5PageW@ 00013520     bootcmn:i2c_eeprom.obj
 0001:00002550       ??_C@_0BO@GCKLILNE@ERROR?3?5XLDR?5exceeds?564KByte?$AN?6?$AA@ 00013550     bootcmn:i2c_eeprom.obj
 0001:00002570       ??_C@_0CG@MJIEOAAL@I2CEEPROMWriteXldr?3?5dwLength?5?$DN?50@ 00013570     bootcmn:i2c_eeprom.obj
 0001:00002598       ??_C@_0CL@BBJPJLKF@ERROR?3?5PageWrite?3?5Write?5EEPROM?5D@ 00013598     bootcmn:i2c_eeprom.obj
 0001:000025c4       ??_C@_0CO@HGEGHFHG@ERROR?3?5PageWrite?3?5Write?5EEPROM?5a@ 000135c4     bootcmn:i2c_eeprom.obj
 0001:000025f4       ??_C@_0CI@CPBFGIJF@ERROR?3?5PageWrite?3?5Generate?5Start@ 000135f4     bootcmn:i2c_eeprom.obj
 0001:0000261c       ??_C@_0CJ@FGNAPIED@ERROR?3?5PageRead?3?5Read?5EEPROM?5dat@ 0001361c     bootcmn:i2c_eeprom.obj
 0001:00002648       ??_C@_0CH@PHKPBEHO@ERROR?3?5PageRead?3?5Repeated?5Start?5@ 00013648     bootcmn:i2c_eeprom.obj
 0001:00002670       ??_C@_0CN@IHAHJMEC@ERROR?3?5PageRead?3?5Write?5EEPROM?5ad@ 00013670     bootcmn:i2c_eeprom.obj
 0001:000026a0       ??_C@_0CH@DKIBMJNB@ERROR?3?5PageRead?3?5Generate?5Start?5@ 000136a0     bootcmn:i2c_eeprom.obj
 0001:000026c8       ??_C@_1FE@FFNPEPPH@?$AAH?$AAa?$AAr?$AAd?$AAw?$AAa?$AAr?$AAe?$AA?5?$AAf?$AAl?$AAo?$AAw?$AA?5?$AAc?$AAo?$AAn?$AAt?$AAr?$AAo?$AAl?$AA?5?$AAi?$AAs?$AA?5?$AAn?$AAo?$AAt?$AA?5?$AAs?$AAu?$AAp@ 000136c8     serialutils:serialutils.obj
 0001:0000271c       ??_C@_1CI@OHCJFJPM@?$AAE?$AAR?$AAR?$AAO?$AAR?$AA?3?$AA?5?$AA?$CF?$AAs?$AA?5?$AAl?$AAi?$AAn?$AAe?$AA?5?$AA?$CF?$AAd?$AA?3?$AA?5?$AA?$AA@ 0001371c     serialutils:serialutils.obj
 0001:00002748       ??_C@_1KC@BPCNHDLN@?$AAc?$AA?3?$AA?2?$AAw?$AAi?$AAn?$AAc?$AAe?$AAr?$AAo?$AAo?$AAt?$AAs?$AA?2?$AAt?$AAo?$AAp?$AAa?$AAz?$AA?2?$AAw?$AAi?$AAn?$AAc?$AAe?$AA7?$AA0?$AA0?$AA?2?$AAp?$AAl?$AAa@ 00013748     serialutils:serialutils.obj
 0001:000027ec       ??_C@_0CB@KKLHFGEJ@OALStall?3?5EPIT?5mapping?5failed?$CB?$AN?6@ 000137ec     ethdrv:ethdrv.obj
 0001:00002810       ??_C@_1CI@KDDHFOOJ@?$AAR?$AAe?$AAt?$AAu?$AAr?$AAn?$AA?5?$AAt?$AAo?$AA?5?$AAM?$AAa?$AAi?$AAn?$AA?5?$AAM?$AAe?$AAn?$AAu?$AA?$AA@ 00013810     blmenu_common_topaz_v1:menu.obj
 0001:00002838       ??_C@_1DE@CJJMFMLM@?$AAF?$AAo?$AAr?$AAm?$AAa?$AAt?$AA?5?$AAA?$AAl?$AAl?$AA?5?$AAS?$AAD?$AA?1?$AAM?$AAM?$AAC?$AA?5?$AAR?$AAe?$AAg?$AAi?$AAo?$AAn?$AAs?$AA?$AA@ 00013838     blmenu_common_topaz_v1:menu.obj
 0001:00002870       ??_C@_1GC@OMHINPHG@?$AAC?$AAr?$AAe?$AAa?$AAt?$AAe?$AA?5?$AAF?$AAi?$AAl?$AAe?$AA?5?$AAS?$AAy?$AAs?$AAt?$AAe?$AAm?$AA?5?$AAP?$AAa?$AAr?$AAt?$AAi?$AAt?$AAi?$AAo?$AAn?$AA?5?$AAo?$AAn?$AA?5@ 00013870     blmenu_common_topaz_v1:menu.obj
 0001:000028d4       ??_C@_1DI@CHPLHBGN@?$AAe?$AAS?$AAD?$AA?5?$AA2?$AA?4?$AA1?$AA?5?$AAB?$AAo?$AAo?$AAt?$AA?5?$AAP?$AAa?$AAr?$AAt?$AAi?$AAt?$AAi?$AAo?$AAn?$AA?5?$AAS?$AAi?$AAz?$AAe?$AA?$AA@ 000138d4     blmenu_common_topaz_v1:menu.obj
 0001:0000290c       ??_C@_1CO@KMCKFBEK@?$AAe?$AAS?$AAD?$AA?5?$AA2?$AA?4?$AA1?$AA?5?$AAB?$AAo?$AAo?$AAt?$AA?5?$AAP?$AAa?$AAr?$AAt?$AAi?$AAt?$AAi?$AAo?$AAn?$AA?$AA@ 0001390c     blmenu_common_topaz_v1:menu.obj
 0001:0000293c       ??_C@_1DK@IFGBMPID@?$AAe?$AAM?$AAM?$AAC?$AA?5?$AA4?$AA?4?$AA3?$AA?5?$AAB?$AAo?$AAo?$AAt?$AA?5?$AAP?$AAa?$AAr?$AAt?$AAi?$AAt?$AAi?$AAo?$AAn?$AA?5?$AAS?$AAi?$AAz?$AAe?$AA?$AA@ 0001393c     blmenu_common_topaz_v1:menu.obj
 0001:00002978       ??_C@_1DA@CKPOEKDC@?$AAe?$AAM?$AAM?$AAC?$AA?5?$AA4?$AA?4?$AA3?$AA?5?$AAB?$AAo?$AAo?$AAt?$AA?5?$AAP?$AAa?$AAr?$AAt?$AAi?$AAt?$AAi?$AAo?$AAn?$AA?$AA@ 00013978     blmenu_common_topaz_v1:menu.obj
 0001:000029a8       ??_C@_19DIEGALPP@?$AA?$CF?$AAc?$AA?$AN?$AA?6?$AA?$AA@ 000139a8     blmenu_common_topaz_v1:menu.obj
 0001:000029b4       ??_C@_1BO@MKGCCJBG@?$AA?$AN?$AA?6?$AA?5?$AAS?$AAe?$AAl?$AAe?$AAc?$AAt?$AAi?$AAo?$AAn?$AA?3?$AA?5?$AA?$AA@ 000139b4     blmenu_common_topaz_v1:menu.obj
 0001:000029d4       ??_C@_1BC@NKFMDHEP@?$AA?5?$AA?$FL?$AA?$CF?$AAc?$AA?$FN?$AA?5?$AA?$CF?$AAs?$AA?$AA@ 000139d4     blmenu_common_topaz_v1:menu.obj
 0001:000029e8       ??_C@_1BI@MGJPENDP@?$AA?5?$AA?$FL?$AA?$CF?$AAc?$AA?$FN?$AA?5?$AA?$CF?$AAs?$AA?5?$AA?$AN?$AA?6?$AA?$AA@ 000139e8     blmenu_common_topaz_v1:menu.obj
 0001:00002a00       ??_C@_1DE@DMLMOHKE@?$AAT?$AAo?$AAp?$AAa?$AAz?$AA?5?$AAi?$AA?4?$AAM?$AAX?$AA2?$AA5?$AA?5?$AAB?$AAo?$AAo?$AAt?$AA?5?$AAM?$AAe?$AAn?$AAu?$AA?5?$AA?$CF?$AAs?$AA?$AA@ 00013a00     blmenu_common_topaz_v1:menu.obj
 0001:00002a34       ??_C@_11LOCGONAA@?$AA?$AA@ 00013a34     blmenu_common_topaz_v1:menu.obj
 0001:00002a38       ??_C@_1CE@DHIEGFHF@?$AA?$CI?$AAU?$AAN?$AAS?$AAA?$AAV?$AAE?$AAD?$AA?5?$AAC?$AAH?$AAA?$AAN?$AAG?$AAE?$AAS?$AA?$CJ?$AA?$AA@ 00013a38     blmenu_common_topaz_v1:menu.obj
 0001:00002a60       ??_C@_1KE@LKPJEGMN@?$AA?$AN?$AA?6?$AA?9?$AA?9?$AA?9?$AA?9?$AA?9?$AA?9?$AA?9?$AA?9?$AA?9?$AA?9?$AA?9?$AA?9?$AA?9?$AA?9?$AA?9?$AA?9?$AA?9?$AA?9?$AA?9?$AA?9?$AA?9?$AA?9?$AA?9?$AA?9?$AA?9?$AA?9?$AA?9?$AA?9?$AA?9?$AA?9@ 00013a60     blmenu_common_topaz_v1:menu.obj
 0001:00002b08       ??_C@_1FC@OJBLOANL@?$AAE?$AAR?$AAR?$AAO?$AAR?$AA?3?$AA?5?$AAB?$AAL?$AAM?$AAe?$AAn?$AAu?$AAE?$AAn?$AAa?$AAb?$AAl?$AAe?$AA?3?$AA?5?$AAI?$AAn?$AAv?$AAa?$AAl?$AAi?$AAd?$AA?5?$AAp?$AAa?$AAr@ 00013b08     blmenu_common_topaz_v1:menu.obj
 0001:00002b5c       ??_C@_1CA@IGABMMKB@?$AA?5?$AA?$CF?$AAs?$AA?5?$AAs?$AAe?$AAt?$AA?5?$AAt?$AAo?$AA?5?$AA?$CF?$AAs?$AA?$AN?$AA?6?$AA?$AA@ 00013b5c     blmenu_common_topaz_v1:menu.obj
 0001:00002b80       ??_C@_1EA@HMINENJO@?$AA?5?$AA?8?$AA?$CF?$AAs?$AA?8?$AA?5?$AAi?$AAs?$AAn?$AA?8?$AAt?$AA?5?$AAv?$AAa?$AAl?$AAi?$AAd?$AA?5?$AAM?$AAA?$AAC?$AA?5?$AAa?$AAd?$AAd?$AAr?$AAe?$AAs?$AAs?$AA?$AN?$AA?6?$AA?$AA@ 00013b80     blmenu_common_topaz_v1:menu.obj
 0001:00002bc0       ??_C@_1DA@CFLFOOLN@?$AA?5?$AAE?$AAn?$AAt?$AAe?$AAr?$AA?5?$AA?$CF?$AAs?$AA?5?$AA?$CI?$AAa?$AAc?$AAt?$AAu?$AAa?$AAl?$AA?5?$AA?$CF?$AAs?$AA?$CJ?$AA?3?$AA?5?$AA?$AA@ 00013bc0     blmenu_common_topaz_v1:menu.obj
 0001:00002bf0       ??_C@_1GG@KAOMNNAE@?$AAE?$AAR?$AAR?$AAO?$AAR?$AA?3?$AA?5?$AAO?$AAA?$AAL?$AAB?$AAL?$AAM?$AAe?$AAn?$AAu?$AAS?$AAe?$AAt?$AAM?$AAa?$AAc?$AAA?$AAd?$AAd?$AAr?$AAe?$AAs?$AAs?$AA?3?$AA?5?$AAI@ 00013bf0     blmenu_common_topaz_v1:menu.obj
 0001:00002c58       ??_C@_1DO@PNGPKAIC@?$AA?5?$AA?8?$AA?$CF?$AAs?$AA?8?$AA?5?$AAi?$AAs?$AAn?$AA?8?$AAt?$AA?5?$AAv?$AAa?$AAl?$AAi?$AAd?$AA?5?$AAI?$AAP?$AA?5?$AAa?$AAd?$AAd?$AAr?$AAe?$AAs?$AAs?$AA?$AN?$AA?6?$AA?$AA@ 00013c58     blmenu_common_topaz_v1:menu.obj
 0001:00002c98       ??_C@_1GA@DANHOIAN@?$AAE?$AAR?$AAR?$AAO?$AAR?$AA?3?$AA?5?$AAB?$AAL?$AAM?$AAe?$AAn?$AAu?$AAS?$AAe?$AAt?$AAI?$AAp?$AAA?$AAd?$AAd?$AAr?$AAe?$AAs?$AAs?$AA?3?$AA?5?$AAI?$AAn?$AAv?$AAa?$AAl@ 00013c98     blmenu_common_topaz_v1:menu.obj
 0001:00002cf8       ??_C@_1DI@NFENBBKL@?$AA?5?$AA?8?$AA?$CF?$AAs?$AA?8?$AA?5?$AAi?$AAs?$AAn?$AA?8?$AAt?$AA?5?$AAv?$AAa?$AAl?$AAi?$AAd?$AA?5?$AAI?$AAP?$AA?5?$AAm?$AAa?$AAs?$AAk?$AA?$AN?$AA?6?$AA?$AA@ 00013cf8     blmenu_common_topaz_v1:menu.obj
 0001:00002d30       ??_C@_1FK@HDEECBIC@?$AAE?$AAR?$AAR?$AAO?$AAR?$AA?3?$AA?5?$AAB?$AAL?$AAM?$AAe?$AAn?$AAu?$AAS?$AAe?$AAt?$AAI?$AAp?$AAM?$AAa?$AAs?$AAk?$AA?3?$AA?5?$AAI?$AAn?$AAv?$AAa?$AAl?$AAi?$AAd?$AA?5@ 00013d30     blmenu_common_topaz_v1:menu.obj
 0001:00002d8c       ??_C@_15DAMPJCDE@?$AA?$CF?$AAc?$AA?$AA@ 00013d8c     blmenu_common_topaz_v1:menu.obj
 0001:00002d94       ??_C@_17ILCABGPK@?$AA?$AI?$AA?5?$AA?$AI?$AA?$AA@ 00013d94     blmenu_common_topaz_v1:menu.obj
 0001:00002d9c       ??_C@_15JNBOKNOG@?$AA?$AN?$AA?6?$AA?$AA@ 00013d9c     blmenu_common_topaz_v1:menu.obj
 0001:00002da4       ??_C@_0N@LPLKOEJA@?5?3?5Enabled?$AN?6?$AA@ 00013da4     blmenu_common_topaz_v1:menu.obj
 0001:00002db4       ??_C@_0P@LIJBDBHL@?5?3?5?$CFd?5Kbytes?$AN?6?$AA@ 00013db4     blmenu_common_topaz_v1:menu.obj
 0001:00002dc4       ??_C@_0BP@GBDFDBJI@?5?3?5Boot?5part?52?0?5r?1w?5usr?5part?$AN?6?$AA@ 00013dc4     blmenu_common_topaz_v1:menu.obj
 0001:00002de4       ??_C@_0BJ@NELEKEFH@?5?3?5Boot?5and?5r?1w?5part?52?$AN?6?$AA@ 00013de4     blmenu_common_topaz_v1:menu.obj
 0001:00002e00       ??_C@_0BP@ILLDOMPK@?5?3?5Boot?5part?51?0?5r?1w?5usr?5part?$AN?6?$AA@ 00013e00     blmenu_common_topaz_v1:menu.obj
 0001:00002e20       ??_C@_0BJ@MGABALLJ@?5?3?5Boot?5and?5r?1w?5part?51?$AN?6?$AA@ 00013e20     blmenu_common_topaz_v1:menu.obj
 0001:00002e3c       ??_C@_0BO@BCOIFLKC@?5?3?5Disabled?5?1?5Not?5Available?$AN?6?$AA@ 00013e3c     blmenu_common_topaz_v1:menu.obj
 0001:00002e5c       ??_C@_07LPCKBJPC@Polling?$AA@ 00013e5c     blmenu_common_topaz_v1:menu.obj
 0001:00002e64       ??_C@_09JNFEIGJE@Interrupt?$AA@ 00013e64     blmenu_common_topaz_v1:menu.obj
 0001:00002e70       ??_C@_07CHEGAGBD@?5?3?5?$CFd?$AN?6?$AA@ 00013e70     blmenu_common_topaz_v1:menu.obj
 0001:00002e78       ??_C@_07DOAOMMKG@Enabled?$AA@ 00013e78     blmenu_common_topaz_v1:menu.obj
 0001:00002e80       ??_C@_08JGILNPHN@Disabled?$AA@ 00013e80     blmenu_common_topaz_v1:menu.obj
 0001:00002e8c       ??_C@_0BH@IMLFGHDI@?5?3?5?$CFx?9?$CFx?9?$CFx?9?$CFx?9?$CFx?9?$CFx?$AN?6?$AA@ 00013e8c     blmenu_common_topaz_v1:menu.obj
 0001:00002ea4       ??_C@_07OKIIGJDF@?5?3?5?$CFs?$AN?6?$AA@ 00013ea4     blmenu_common_topaz_v1:menu.obj
 0001:00002eac       ??_C@_0DC@JJHEEFDO@?$AN?6WARNING?3?5?5Format?5of?5OS?5NAND?5re@ 00013eac     blmenu_common_topaz_v1:menu.obj
 0001:00002ee0       ??_C@_0DP@POLFEJAN@Boot?5loader?5and?5boot?5configurati@ 00013ee0     blmenu_common_topaz_v1:menu.obj
 0001:00002f20       ??_C@_0DE@FMHJGPFH@?$AN?6WARNING?3?5?5Format?5of?5all?5NAND?5r@ 00013f20     blmenu_common_topaz_v1:menu.obj
 0001:00002f54       ??_C@_0CO@BBPEEJNH@ERROR?3?5Unable?5to?5read?5EXT_CSD?5fr@ 00013f54     blmenu_common_topaz_v1:menu.obj
 0001:00002f84       ??_C@_0DH@CLNMIBLA@Data?5on?5all?5partitions?5on?5the?5ca@ 00013f84     blmenu_common_topaz_v1:menu.obj
 0001:00002fbc       ??_C@_0DJ@KCKGNILM@?$AN?6WARNING?3?5?5Change?5in?5boot?5parti@ 00013fbc     blmenu_common_topaz_v1:menu.obj
 0001:00002ff8       ??_C@_0CM@EGMJHFG@ERROR?3?5Unable?5to?5set?5partition?5a@ 00013ff8     blmenu_common_topaz_v1:menu.obj
 0001:00003028       ??_C@_0ED@JCEMHIBN@Boot?5loader?0?5OS?5and?5boot?5configu@ 00014028     blmenu_common_topaz_v1:menu.obj
 0001:0000306c       ??_C@_0DG@NJPLKEB@?$AN?6WARNING?3?5?5Format?5of?5all?5SD?1MMC@ 0001406c     blmenu_common_topaz_v1:menu.obj
 0001:000030a8       ??_C@_0HI@PJONFHDK@?$AN?6If?5partition?5creation?5was?5succ@ 000140a8     blmenu_common_topaz_v1:menu.obj
 0001:00003120       ??_C@_0DL@GLMCHJMJ@All?5previous?5file?5system?5data?5on@ 00014120     blmenu_common_topaz_v1:menu.obj
 0001:00003160       ??_C@_0ED@ENHEEIGF@?$AN?6WARNING?3?5?5SD?1MMC?5File?5System?5p@ 00014160     blmenu_common_topaz_v1:menu.obj
 0001:000031a4       ??_C@_0BE@OIKALELC@Unknown?5command?$CB?5?$AN?6?$AA@ 000141a4     bsp_bootshell:bspbootshell.obj
 0001:000031b8       ??_C@_0CJ@BKEGJFOI@Invalid?5parameter?0Please?5Input?5A@ 000141b8     bsp_bootshell:bspbootshell.obj
 0001:000031e4       ??_C@_0M@PDNKHPIC@command?5?9?9?5?$AA@ 000141e4     bsp_bootshell:bspbootshell.obj
 0001:000031f0       ??_C@_0BC@JOKBLNPI@type?5?$DP?5for?5help?$AN?6?$AA@ 000141f0     bsp_bootshell:bspbootshell.obj
 0001:00003204       ??_C@_0DD@HEBPMLJO@?9?9?9?9?9?9?9?9?9?9?9?5?5Topaz?5i?4MX25?5Boot?5S@ 00014204     bsp_bootshell:bspbootshell.obj
 0001:00003238       ??_C@_1CC@KBABDHEI@?$AA?9?$AAF?$AAE?$AAC?$AAE?$AAn?$AAa?$AAb?$AAl?$AAe?$AAI?$AAn?$AAt?$AAs?$AA?$AN?$AA?6?$AA?$AA@ 00014238     oal_ethdrv_fec_common_topaz_v1:fec.obj
 0001:0000325c       ??_C@_1CC@HKAMNBPM@?$AA?$CL?$AAF?$AAE?$AAC?$AAE?$AAn?$AAa?$AAb?$AAl?$AAe?$AAI?$AAn?$AAt?$AAs?$AA?$AN?$AA?6?$AA?$AA@ 0001425c     oal_ethdrv_fec_common_topaz_v1:fec.obj
 0001:00003280       ??_C@_1CE@PAJNDNPH@?$AA?9?$AAF?$AAE?$AAC?$AAD?$AAi?$AAs?$AAa?$AAb?$AAl?$AAe?$AAI?$AAn?$AAt?$AAs?$AA?$AN?$AA?6?$AA?$AA@ 00014280     oal_ethdrv_fec_common_topaz_v1:fec.obj
 0001:000032a4       ??_C@_1CE@DJFNMKAL@?$AA?$CL?$AAF?$AAE?$AAC?$AAD?$AAi?$AAs?$AAa?$AAb?$AAl?$AAe?$AAI?$AAn?$AAt?$AAs?$AA?$AN?$AA?6?$AA?$AA@ 000142a4     oal_ethdrv_fec_common_topaz_v1:fec.obj
 0001:000032c8       ??_C@_1DK@CHFIODGD@?$AA?9?$AAF?$AAE?$AAC?$AAI?$AAn?$AAi?$AAt?$AAD?$AAM?$AAA?$AAB?$AAu?$AAf?$AAf?$AAe?$AAr?$AA?$CI?$AAr?$AAc?$AA?5?$AA?$DN?$AA?5?$AA?$CF?$AAd?$AA?$CJ?$AA?$AN?$AA?6?$AA?$AA@ 000142c8     oal_ethdrv_fec_common_topaz_v1:fec.obj
 0001:00003308       ??_C@_1GA@LFAILOCH@?$AAE?$AAR?$AAR?$AAO?$AAR?$AA?3?$AA?5?$AAF?$AAE?$AAC?$AAI?$AAn?$AAi?$AAt?$AAD?$AAM?$AAA?$AAB?$AAu?$AAf?$AAf?$AAe?$AAr?$AA?3?$AA?5?$AAD?$AAM?$AAA?$AA?5?$AAB?$AAu?$AAf@ 00014308     oal_ethdrv_fec_common_topaz_v1:fec.obj
 0001:00003368       ??_C@_0CI@KMIJHHBB@FECInitDMABuffer?5DMA?5Buffer?5too?5@ 00014368     oal_ethdrv_fec_common_topaz_v1:fec.obj
 0001:00003390       ??_C@_1EA@MDNGEOGF@?$AA?$CL?$AAF?$AAE?$AAC?$AAI?$AAn?$AAi?$AAt?$AAD?$AAM?$AAA?$AAB?$AAu?$AAf?$AAf?$AAe?$AAr?$AA?$CI?$AA0?$AAx?$AA?$CF?$AAX?$AA?0?$AA?5?$AA0?$AAx?$AA?$CF?$AAX?$AA?$CJ?$AA?$AN?$AA?6?$AA?$AA@ 00014390     oal_ethdrv_fec_common_topaz_v1:fec.obj
 0001:000033d0       ??_C@_1CI@LLGKHLKN@?$AA?9?$AAF?$AAE?$AAC?$AAI?$AAn?$AAi?$AAt?$AA?$CI?$AAr?$AAc?$AA?5?$AA?$DN?$AA?5?$AA?$CF?$AAd?$AA?$CJ?$AA?$AN?$AA?6?$AA?$AA@ 000143d0     oal_ethdrv_fec_common_topaz_v1:fec.obj
 0001:000033f8       ??_C@_0CN@NECAPPEM@FEC?5is?5linked?0?5speed?510?5Mbps?0?5ha@ 000143f8     oal_ethdrv_fec_common_topaz_v1:fec.obj
 0001:00003428       ??_C@_0CN@KMHKLMCP@FEC?5is?5linked?0?5speed?510?5Mbps?0?5fu@ 00014428     oal_ethdrv_fec_common_topaz_v1:fec.obj
 0001:00003458       ??_C@_0CO@NCDNBHO@FEC?5is?5linked?0?5speed?5100?5Mbps?0?5h@ 00014458     oal_ethdrv_fec_common_topaz_v1:fec.obj
 0001:00003488       ??_C@_0CO@HFHJJCBN@FEC?5is?5linked?0?5speed?5100?5Mbps?0?5f@ 00014488     oal_ethdrv_fec_common_topaz_v1:fec.obj
 0001:000034b8       ??_C@_0CB@DFINIDFK@Failed?5to?5get?5the?5external?5PHY?$AN?6@ 000144b8     oal_ethdrv_fec_common_topaz_v1:fec.obj
 0001:000034e0       ??_C@_1EM@PFHKNHEN@?$AAT?$AAh?$AAe?$AA?5?$AAn?$AAa?$AAm?$AAe?$AA?5?$AAf?$AAo?$AAr?$AA?5?$AAt?$AAh?$AAe?$AA?5?$AAe?$AAx?$AAt?$AAe?$AAr?$AAn?$AAa?$AAl?$AA?5?$AAP?$AAH?$AAY?$AA?5?$AAi?$AAs@ 000144e0     oal_ethdrv_fec_common_topaz_v1:fec.obj
 0001:0000352c       ??_C@_1DM@PNEAGLBJ@?$AAM?$AAI?$AAI?$AA_?$AAR?$AAE?$AAG?$AA_?$AAP?$AAH?$AAY?$AAI?$AAR?$AA1?$AA?5?$AAR?$AAE?$AAA?$AAD?$AA?5?$AAF?$AAa?$AAi?$AAl?$AAe?$AAd?$AA?5?$AA?$AN?$AA?6?$AA?$AA@ 0001452c     oal_ethdrv_fec_common_topaz_v1:fec.obj
 0001:00003568       ??_C@_1HC@KIHIPIBC@?$AAF?$AAE?$AAC?$AAI?$AAn?$AAi?$AAt?$AA?$CI?$AA0?$AAx?$AA?$CF?$AA0?$AA8?$AAx?$AA?0?$AA?5?$AA0?$AAx?$AA?$CF?$AA0?$AA8?$AAx?$AA?0?$AA?5?$AA?$CF?$AA0?$AA2?$AAx?$AA?3?$AA?$CF?$AA0?$AA2@ 00014568     oal_ethdrv_fec_common_topaz_v1:fec.obj
 0001:000035dc       ??_C@_0BL@PCLOMCF@Initializing?5Ethernet?4?4?4?$AN?6?$AA@ 000145dc     oal_ethdrv_fec_common_topaz_v1:fec.obj
 0001:000035f8       ??_C@_1DC@PKJNHKDJ@?$AA?9?$AAF?$AAE?$AAC?$AAS?$AAe?$AAn?$AAd?$AAF?$AAr?$AAa?$AAm?$AAe?$AA?$CI?$AAr?$AAc?$AA?5?$AA?$DN?$AA?5?$AA?$CF?$AAd?$AA?$CJ?$AA?$AN?$AA?6?$AA?$AA@ 000145f8     oal_ethdrv_fec_common_topaz_v1:fec.obj
 0001:00003630       ??_C@_1EI@KKGEKELM@?$AAE?$AAR?$AAR?$AAO?$AAR?$AA?3?$AA?5?$AAF?$AAE?$AAC?$AAS?$AAe?$AAn?$AAd?$AAF?$AAr?$AAa?$AAm?$AAe?$AA?3?$AA?5?$AAS?$AAe?$AAn?$AAd?$AA?5?$AAt?$AAi?$AAm?$AAe?$AAo?$AAu@ 00014630     oal_ethdrv_fec_common_topaz_v1:fec.obj
 0001:00003678       ??_C@_1CE@KCCCDJJH@?$AA?$CL?$AAS?$AA?5?$AA?$CI?$AA0?$AAx?$AA?$CF?$AA0?$AA8?$AAx?$AA?0?$AA?5?$AA?$CF?$AAd?$AA?$CJ?$AA?$AN?$AA?6?$AA?$AA@ 00014678     oal_ethdrv_fec_common_topaz_v1:fec.obj
 0001:000036a0       ??_C@_1EA@BEFHLOEB@?$AA?9?$AAF?$AAE?$AAC?$AAG?$AAe?$AAt?$AAF?$AAr?$AAa?$AAm?$AAe?$AA?$CI?$AAP?$AAa?$AAc?$AAk?$AAe?$AAt?$AAS?$AAi?$AAz?$AAe?$AA?5?$AA?$DN?$AA?5?$AA?$CF?$AAd?$AA?$CJ?$AA?$AN?$AA?6?$AA?$AA@ 000146a0     oal_ethdrv_fec_common_topaz_v1:fec.obj
 0001:000036e0       ??_C@_1DG@LJFMBLGF@?$AA?$CL?$AAF?$AAE?$AAC?$AAG?$AAe?$AAt?$AAF?$AAr?$AAa?$AAm?$AAe?$AA?$CI?$AA0?$AAx?$AA?$CF?$AA0?$AA8?$AAx?$AA?0?$AA?5?$AA?$CF?$AAd?$AA?$CJ?$AA?$AN?$AA?6?$AA?$AA@ 000146e0     oal_ethdrv_fec_common_topaz_v1:fec.obj
 0001:00003718       ??_C@_1DE@NJHDJGOC@?$AA?9?$AAF?$AAE?$AAC?$AAC?$AAu?$AAr?$AAr?$AAe?$AAn?$AAt?$AAP?$AAa?$AAc?$AAk?$AAe?$AAt?$AAF?$AAi?$AAl?$AAt?$AAe?$AAr?$AA?$AN?$AA?6?$AA?$AA@ 00014718     oal_ethdrv_fec_common_topaz_v1:fec.obj
 0001:00003750       ??_C@_1EE@EDJFMPFC@?$AA?$CL?$AAF?$AAE?$AAC?$AAC?$AAu?$AAr?$AAr?$AAe?$AAn?$AAt?$AAP?$AAa?$AAc?$AAk?$AAe?$AAt?$AAF?$AAi?$AAl?$AAt?$AAe?$AAr?$AA?$CI?$AA0?$AAx?$AA?$CF?$AA0?$AA8?$AAx?$AA?$CJ?$AA?$AN@ 00014750     oal_ethdrv_fec_common_topaz_v1:fec.obj
 0001:00003794       ??_C@_1DI@GJINCFOM@?$AA?9?$AAF?$AAE?$AAC?$AAM?$AAu?$AAl?$AAt?$AAi?$AAc?$AAa?$AAs?$AAt?$AAL?$AAi?$AAs?$AAt?$AA?$CI?$AAr?$AAc?$AA?5?$AA?$DN?$AA?5?$AA1?$AA?$CJ?$AA?$AN?$AA?6?$AA?$AA@ 00014794     oal_ethdrv_fec_common_topaz_v1:fec.obj
 0001:000037d0       ??_C@_1EA@CKJMHDOG@?$AA?$CL?$AAF?$AAE?$AAC?$AAM?$AAu?$AAl?$AAt?$AAi?$AAc?$AAa?$AAs?$AAt?$AAL?$AAi?$AAs?$AAt?$AA?$CI?$AA0?$AAx?$AA?$CF?$AA0?$AA8?$AAx?$AA?0?$AA?5?$AA?$CF?$AAd?$AA?$CJ?$AA?$AN?$AA?6?$AA?$AA@ 000147d0     oal_ethdrv_fec_common_topaz_v1:fec.obj
 0001:00003810       ??_C@_1FC@MIIBOMPK@?$AAO?$AAA?$AAL?$AAK?$AAi?$AAt?$AAl?$AAF?$AAE?$AAC?$AAB?$AAS?$AAP?$AAI?$AAn?$AAi?$AAt?$AA?3?$AA?5?$AAG?$AAP?$AAI?$AAO?$AA3?$AA?5?$AAn?$AAu?$AAl?$AAl?$AA?5?$AAp?$AAo@ 00014810     bspfec:bspfec.obj
 0001:00003868       ??_C@_1FC@JEDBMPJD@?$AAO?$AAA?$AAL?$AAK?$AAi?$AAt?$AAl?$AAF?$AAE?$AAC?$AAB?$AAS?$AAP?$AAI?$AAn?$AAi?$AAt?$AA?3?$AA?5?$AAG?$AAP?$AAI?$AAO?$AA4?$AA?5?$AAn?$AAu?$AAl?$AAl?$AA?5?$AAp?$AAo@ 00014868     bspfec:bspfec.obj
 0001:000038c0       ??_C@_1FI@GIMIACCK@?$AAO?$AAA?$AAL?$AAK?$AAi?$AAt?$AAl?$AAF?$AAE?$AAC?$AAB?$AAS?$AAP?$AAI?$AAn?$AAi?$AAt?$AA?3?$AA?5?$AAI?$AAO?$AAM?$AAU?$AAX?$AAC?$AA?5?$AAm?$AAa?$AAp?$AAp?$AAi?$AAn@ 000148c0     bspfec:bspfec.obj
 0001:00003918       ??_C@_0BK@FGOBGFEM@RNDISMINI?5?9?9?9?5RESET?5?9?9?9?$AN?6?$AA@ 00014918     fsl_rne_mdd_common_topaz_v1:rndis.obj
 0001:00003934       ??_C@_0CK@HCFNMAPL@RNdis?3?3?5Too?5much?5outgoing?0?5baili@ 00014934     fsl_rne_mdd_common_topaz_v1:rndis.obj
 0001:00003960       ??_C@_0DK@LOJODLJL@ASSERT?$CB?5Rndis?3?3MddSendRndisMessa@ 00014960     fsl_rne_mdd_common_topaz_v1:rndis.obj
 0001:0000399c       ??_C@_0BN@MJFOLLBM@RNdis?3?3?5Should?5not?5happen?$CB?$AN?6?$AA@ 0001499c     fsl_rne_mdd_common_topaz_v1:rndis.obj
 0001:000039bc       ??_C@_0CK@BEACHKGH@RNdis?3?3?5No?5mem?5for?5INITIALIZE_CO@ 000149bc     fsl_rne_mdd_common_topaz_v1:rndis.obj
 0001:000039e8       ??_C@_0DI@ELIDGGNF@ASSERT?5Fail?5at?5uiMessageSize?$CI?$CFd?$CJ@ 000149e8     fsl_rne_mdd_common_topaz_v1:rndis.obj
 0001:00003a20       ??_C@_0DA@CMCBBBCA@RNdis?3?3?5Unknown?5RNDIS?5msg?0?5buff?$FL@ 00014a20     fsl_rne_mdd_common_topaz_v1:rndis.obj
 0001:00003a50       ??_C@_0DB@PAFHLFPB@RndisMini?5rcv?5REMOTE_NDIS_RESET_@ 00014a50     fsl_rne_mdd_common_topaz_v1:rndis.obj
 0001:00003a84       ??_C@_0DB@NGCDHJGD@RndisMini?5recv?5REMOTE_NDIS_HALT_@ 00014a84     fsl_rne_mdd_common_topaz_v1:rndis.obj
 0001:00003ab8       ??_C@_0CP@HEPIJLKK@RndisMdd?3?3?5PDD?8s?5max?5RX?5buffer?5?$DN@ 00014ab8     fsl_rne_mdd_common_topaz_v1:rndis.obj
 0001:00003ae8       ??_C@_0BP@HHOMIKAO@ASSERT?5at?5File?$CI?$CFs?$CJ?5line?5?$CI?$CFd?$CJ?$AN?6?$AA@ 00014ae8     fsl_rne_mdd_common_topaz_v1:rndis.obj
 0001:00003b08       ??_C@_09JBPNJICM@rndis?4cpp?$AA@ 00014b08     fsl_rne_mdd_common_topaz_v1:rndis.obj
 0001:00003b14       ??_C@_0CK@JCOPOCLM@ERROR?$CB?5RndisInitialize?5msg?5recei@ 00014b14     fsl_rne_mdd_common_topaz_v1:rndis.obj
 0001:00003b40       ??_C@_0CO@JHJMPDCG@RNDISMINI?5Err?$CB?$CB?5unsupported?5RNDI@ 00014b40     fsl_rne_mdd_common_topaz_v1:rndis.obj
 0001:00003b70       ??_C@_0P@BDJJIKDL@Overrun?$DN0x?$CFx?6?$AN?$AA@ 00014b70     fsl_rne_mdd_common_topaz_v1:rndis.obj
 0001:00003b80       ??_C@_0BJ@IJMDONAK@Buffer?5is?5too?5big?50x?$CFx?6?$AN?$AA@ 00014b80     fsl_rne_mdd_common_topaz_v1:rndis.obj
 0001:00003b9c       ??_C@_0CK@LKMHPIGI@Wrong?5Data?5DataLength?5Msg?$DN0x?$CFx?0P@ 00014b9c     fsl_rne_mdd_common_topaz_v1:rndis.obj
 0001:00003bc8       ??_C@_0CN@OHNGADLJ@RNdis?3?3?5Invalid?5RndisPacket?5l?$FL?$CFd@ 00014bc8     fsl_rne_mdd_common_topaz_v1:rndis.obj
 0001:00003bf8       ??_C@_0BH@HBKBIINO@Wrong?5Data?5Type?50x?$CFx?$AN?6?$AA@ 00014bf8     fsl_rne_mdd_common_topaz_v1:rndis.obj
 0001:00003c10       ??_C@_0CA@IBGOHNCO@Rndis?3?3?5initialization?3?5Fail?$CB?$AN?6?$AA@ 00014c10     fsl_rne_mdd_common_topaz_v1:rndis.obj
 0001:00003c30       ??_C@_0CC@EELLDCCI@Rndis?3?3?5initialization?3?5Success?$AN@ 00014c30     fsl_rne_mdd_common_topaz_v1:rndis.obj
 0001:00003c54       ??_C@_0CD@EOFHIDOL@Rndis?3?3?5Get?5MAC?5address?5?$CFx?0?$CFx?0?$CFx@ 00014c54     fsl_rne_mdd_common_topaz_v1:rndis.obj
 0001:00003c78       ??_C@_0CM@KLOLOCDD@Rndis?3?3?5Err?5no?5MAC?5address?5read?5@ 00014c78     fsl_rne_mdd_common_topaz_v1:rndis.obj
 0001:00003ca4       ??_C@_0BL@EINAHMEI@Rndis?3?3?5PDDInit?5Success?$CB?$AN?6?$AA@ 00014ca4     fsl_rne_mdd_common_topaz_v1:rndis.obj
 0001:00003cc0       ??_C@_0BK@BFGGBGMH@Rndis?3?3?5initialization?$CB?$AN?6?$AA@ 00014cc0     fsl_rne_mdd_common_topaz_v1:rndis.obj
 0001:00003cdc       ??_C@_0CI@PFDJABBD@Rndis?3?3?5Address?5static?5map?5to?5ad@ 00014cdc     fsl_rne_mdd_common_topaz_v1:rndis.obj
 0001:00003d04       ??_C@_0CH@LBCKJEJO@Rndis?3?3?5initialization?3?5with?5add@ 00014d04     fsl_rne_mdd_common_topaz_v1:rndis.obj
 0001:00003d2c       ??_C@_0BP@JDIDIKNB@OID?$FL?$CFx?$FN?5not?5yet?5implemented?$CB?$AN?6?$AA@ 00014d2c     fsl_rne_mdd_common_topaz_v1:hostmini.obj
 0001:00003d4c       ??_C@_0CP@MKNOHPIM@HostMini?3?3?5New?5filter?5set?3?5?$FL0x?$CFx@ 00014d4c     fsl_rne_mdd_common_topaz_v1:hostmini.obj
 0001:00003d80       ??_C@_1FK@FNONLNGN@?$AA?$CF?$AAs?$AA?3?$AA?5?$AAD?$AAE?$AAB?$AAU?$AAG?$AAC?$AAH?$AAK?$AA?5?$AAf?$AAa?$AAi?$AAl?$AAe?$AAd?$AA?5?$AAi?$AAn?$AA?5?$AAf?$AAi?$AAl?$AAe?$AA?5?$AA?$CF?$AAs?$AA?5?$AAa@ 00014d80     fsl_rne_mdd_common_topaz_v1:hostmini.obj
 0001:00003ddc       ??_C@_1BA@LEPJIIOK@?$AAU?$AAn?$AAk?$AAn?$AAo?$AAw?$AAn?$AA?$AA@ 00014ddc     fsl_rne_mdd_common_topaz_v1:hostmini.obj
 0001:00003df0       ??_C@_1LG@MGEOLHMC@?$AAc?$AA?3?$AA?2?$AAw?$AAi?$AAn?$AAc?$AAe?$AAr?$AAo?$AAo?$AAt?$AAs?$AA?2?$AAt?$AAo?$AAp?$AAa?$AAz?$AA?2?$AAw?$AAi?$AAn?$AAc?$AAe?$AA7?$AA0?$AA0?$AA?2?$AAp?$AAl?$AAa@ 00014df0     fsl_rne_mdd_common_topaz_v1:hostmini.obj
 0001:00003ea8       ??_C@_0BN@DGLONFMO@HostMini?3?3?5MddDisconnect?$CB?$CB?$AN?6?$AA@ 00014ea8     fsl_rne_mdd_common_topaz_v1:hostmini.obj
 0001:00003ec8       ??_C@_0BE@LPGPNKBH@HostMiniInit?3?3?5?$CB?$CB?$AN?6?$AA@ 00014ec8     fsl_rne_mdd_common_topaz_v1:hostmini.obj
 0001:00003edc       ??_C@_1O@NJEHEHHO@?$AAu?$AAt?$AAi?$AAl?$AA?4?$AAc?$AA?$AA@ 00014edc     fsl_rne_mdd_common_topaz_v1:util.obj
 0001:00003ef0       ??_C@_1FA@PHGBNLGM@?$AAM?$AAi?$AAc?$AAr?$AAo?$AAs?$AAo?$AAf?$AAt?$AA?5?$AAR?$AAN?$AAD?$AAI?$AAS?$AA?5?$AAK?$AAI?$AAT?$AAL?$AA?5?$AAf?$AAo?$AAr?$AA?5?$AAF?$AAS?$AAL?$AA?5?$AAH?$AAS?$AA?5@ 00014ef0     fsl_rne_pdd_common_topaz_v1:rndis_pdd.obj
 0001:00003f40       ??_C@_1BE@DEAPIJA@?$AAM?$AAi?$AAc?$AAr?$AAo?$AAs?$AAo?$AAf?$AAt?$AA?$AA@ 00014f40     fsl_rne_pdd_common_topaz_v1:rndis_pdd.obj
 0001:00003f68       DigitTable                 00014f68     fsl_rne_pdd_common_topaz_v1:rndis_pdd.obj
 0001:00003f90       ??_C@_1FE@MMFBADFF@?$AA?$CK?$AA?$CK?$AA?$CK?$AA?5?$AAU?$AAn?$AAk?$AAn?$AAo?$AAw?$AAn?$AA?5?$AAG?$AAE?$AAT?$AA_?$AAD?$AAE?$AAS?$AAC?$AAR?$AAI?$AAP?$AAT?$AAO?$AAR?$AA?5?$AAr?$AAe?$AAq?$AAu?$AAe@ 00014f90     fsl_rne_pdd_common_topaz_v1:rndis_pdd.obj
 0001:00003fe4       ??_C@_1DM@FCMMONGE@?$AA?$CK?$AA?$CK?$AA?$CK?$AA?5?$AAU?$AAn?$AAk?$AAn?$AAo?$AAw?$AAn?$AA?5?$AAS?$AAT?$AAR?$AAI?$AAN?$AAG?$AA?5?$AAi?$AAn?$AAd?$AAe?$AAx?$AA?5?$AA?$CF?$AAd?$AA?$AN?$AA?6?$AA?$AA@ 00014fe4     fsl_rne_pdd_common_topaz_v1:rndis_pdd.obj
 0001:00004020       ??_C@_1HM@BPDLPCOO@?$AAc?$AA?3?$AA?2?$AAw?$AAi?$AAn?$AAc?$AAe?$AAr?$AAo?$AAo?$AAt?$AAs?$AA?2?$AAt?$AAo?$AAp?$AAa?$AAz?$AA?2?$AAw?$AAi?$AAn?$AAc?$AAe?$AA7?$AA0?$AA0?$AA?2?$AAp?$AAu?$AAb@ 00015020     fsl_rne_pdd_common_topaz_v1:rndis_pdd.obj
 0001:000040a0       ??_C@_1ME@MKHPGGPI@?$AAc?$AA?3?$AA?2?$AAw?$AAi?$AAn?$AAc?$AAe?$AAr?$AAo?$AAo?$AAt?$AAs?$AA?2?$AAt?$AAo?$AAp?$AAa?$AAz?$AA?2?$AAw?$AAi?$AAn?$AAc?$AAe?$AA7?$AA0?$AA0?$AA?2?$AAp?$AAl?$AAa@ 000150a0     fsl_rne_pdd_common_topaz_v1:rndis_pdd.obj
 0001:00004164       ??_C@_1CK@OLHEFDLK@?$AAN?$AAo?$AA?5?$AAm?$AAe?$AAm?$AA?5?$AAf?$AAo?$AAr?$AA?5?$AAR?$AAX?$AA?5?$AAd?$AAa?$AAt?$AAa?$AA?$AN?$AA?6?$AA?$AA@ 00015164     fsl_rne_pdd_common_topaz_v1:rndis_pdd.obj
 0001:00004190       ??_C@_1DI@FELDACDH@?$AAN?$AAo?$AA?5?$AAm?$AAe?$AAm?$AA?5?$AAf?$AAo?$AAr?$AA?5?$AAR?$AAX?$AA?5?$AAD?$AAa?$AAt?$AAa?$AAW?$AAr?$AAa?$AAp?$AAp?$AAe?$AAr?$AA?$AN?$AA?6?$AA?$AA@ 00015190     fsl_rne_pdd_common_topaz_v1:rndis_pdd.obj
 0001:000041c8       ??_C@_1DG@HDGBABFG@?$AA?$CK?$AA?$CK?$AA?$CK?$AA?5?$AAU?$AAn?$AAk?$AAn?$AAo?$AAw?$AAn?$AA?5?$AAr?$AAe?$AAq?$AAu?$AAe?$AAs?$AAt?$AA?5?$AA0?$AAx?$AA?$CF?$AAx?$AA?$AN?$AA?6?$AA?$AA@ 000151c8     fsl_rne_pdd_common_topaz_v1:rndis_pdd.obj
 0001:00004200       ??_C@_1FI@GLILKAEG@?$AA?$CK?$AA?$CK?$AA?$CK?$AA?5?$AAU?$AAn?$AAH?$AAa?$AAn?$AAd?$AAl?$AAe?$AAd?$AA?5?$AAG?$AAE?$AAT?$AA_?$AAD?$AAE?$AAS?$AAC?$AAR?$AAI?$AAP?$AAT?$AAO?$AAR?$AA?5?$AAr?$AAe?$AAq@ 00015200     fsl_rne_pdd_common_topaz_v1:rndis_pdd.obj
 0001:00004258       ??_C@_1CO@NANJHOKH@?$AA?$CK?$AA?$CK?$AA?$CK?$AAR?$AAe?$AAq?$AAu?$AAe?$AAs?$AAt?$AAT?$AAy?$AAp?$AAe?$AA?$DN?$AA?$DN?$AA0?$AAx?$AA0?$AA2?$AA?$AN?$AA?6?$AA?$AA@ 00015258     fsl_rne_pdd_common_topaz_v1:rndis_pdd.obj
 0001:00004288       ??_C@_1CO@MDAODOFD@?$AA?$CK?$AA?$CK?$AA?$CK?$AAR?$AAe?$AAq?$AAu?$AAe?$AAs?$AAt?$AAT?$AAy?$AAp?$AAe?$AA?$DN?$AA?$DN?$AA0?$AAx?$AA8?$AA2?$AA?$AN?$AA?6?$AA?$AA@ 00015288     fsl_rne_pdd_common_topaz_v1:rndis_pdd.obj
 0001:000042b8       ??_C@_1EM@PLFMLLKO@?$AA?$CK?$AA?$CK?$AA?$CK?$AA?$CK?$AA?5?$AAU?$AAn?$AAh?$AAa?$AAn?$AAd?$AAl?$AAe?$AAd?$AA?5?$AAv?$AAe?$AAr?$AAn?$AAd?$AAo?$AAr?$AA?5?$AAc?$AAo?$AAm?$AAm?$AAa?$AAn?$AAd?$AA?5?$AA0@ 000152b8     fsl_rne_pdd_common_topaz_v1:rndis_pdd.obj
 0001:00004304       ??_C@_1O@KIJBGEAN@?$AAD?$AAo?$AAn?$AAe?$AA?$AN?$AA?6?$AA?$AA@ 00015304     fsl_rne_pdd_common_topaz_v1:rndis_pdd.obj
 0001:00004318       ??_C@_1FG@LFHLPLMG@?$AAS?$AAe?$AAn?$AAd?$AAP?$AAa?$AAc?$AAk?$AAe?$AAt?$AA?5?$AAr?$AAe?$AAq?$AAu?$AAe?$AAs?$AAt?$AA?5?$AAc?$AAo?$AAm?$AAp?$AAl?$AAe?$AAt?$AAe?$AAd?$AA?$CB?$AA?5?$AA?$FL?$AA?$CF@ 00015318     fsl_rne_pdd_common_topaz_v1:rndis_pdd.obj
 0001:00004370       ??_C@_0CB@HAHFALKI@Unexpected?5Msg?5in?5NotifyHandler?$CB@ 00015370     fsl_rne_pdd_common_topaz_v1:rndis_pdd.obj
 0001:00004394       ??_C@_0BG@MPFHNHOK@Unexpected?5bus?5event?$CB?$AA@ 00015394     fsl_rne_pdd_common_topaz_v1:rndis_pdd.obj
 0001:000043ac       ??_C@_1DO@PFNPIHHC@?$AAU?$AAn?$AAe?$AAx?$AAp?$AAe?$AAc?$AAt?$AAe?$AAd?$AA?5?$AAE?$AAP?$AA2?$AA?5?$AAt?$AAr?$AAa?$AAn?$AAs?$AAf?$AAe?$AAr?$AA?5?$AAs?$AAt?$AAa?$AAt?$AAe?$AA?$CB?$AA?$AA@ 000153ac     fsl_rne_pdd_common_topaz_v1:rndis_pdd.obj
 0001:000043f0       ??_C@_1EG@NEPEKMDB@?$AAS?$AAe?$AAn?$AAd?$AAP?$AAa?$AAc?$AAk?$AAe?$AAt?$AA?5?$AAN?$AAU?$AAL?$AAL?$AA?5?$AAt?$AAe?$AAr?$AAm?$AAi?$AAn?$AAa?$AAt?$AAo?$AAr?$AA?5?$AAs?$AAe?$AAn?$AAt?$AA?$CB@ 000153f0     fsl_rne_pdd_common_topaz_v1:rndis_pdd.obj
 0001:00004438       ??_C@_1FI@KOMJGPLF@?$AAS?$AAe?$AAn?$AAd?$AAi?$AAn?$AAg?$AA?5?$AAN?$AAU?$AAL?$AAL?$AA?5?$AAt?$AAe?$AAr?$AAm?$AAi?$AAn?$AAa?$AAt?$AAo?$AAr?$AA?5?$AAf?$AAo?$AAr?$AA?5?$AAt?$AAh?$AAe?$AA?5@ 00015438     fsl_rne_pdd_common_topaz_v1:rndis_pdd.obj
 0001:00004490       ??_C@_1EA@ODINLGJJ@?$AAR?$AAe?$AAc?$AAe?$AAi?$AAv?$AAe?$AAd?$AA?5?$AAa?$AA?5?$AAp?$AAa?$AAc?$AAk?$AAe?$AAt?$AA?5?$AA?$FL?$AA?$CF?$AAd?$AA?5?$AAb?$AAy?$AAt?$AAe?$AAs?$AA?$FN?$AA?$CB?$AA?$AN?$AA?6?$AA?$AA@ 00015490     fsl_rne_pdd_common_topaz_v1:rndis_pdd.obj
 0001:000044d0       ??_C@_1EC@LJDGALBJ@?$AAS?$AAe?$AAn?$AAd?$AAM?$AAe?$AAs?$AAs?$AAa?$AAg?$AAe?$AA?5?$AAr?$AAe?$AAq?$AAu?$AAe?$AAs?$AAt?$AA?5?$AAc?$AAo?$AAm?$AAp?$AAl?$AAe?$AAt?$AAe?$AAd?$AA?$CB?$AA?$AN?$AA?6@ 000154d0     fsl_rne_pdd_common_topaz_v1:rndis_pdd.obj
 0001:00004514       ??_C@_1CK@FEGGBLDE@?$AAD?$AAo?$AAn?$AAe?$AA?5?$AAs?$AAe?$AAn?$AAd?$AAi?$AAn?$AAg?$AA?5?$AAd?$AAa?$AAt?$AAa?$AA?4?$AA?$AN?$AA?6?$AA?$AA@ 00015514     fsl_rne_pdd_common_topaz_v1:rndis_pdd.obj
 0001:00004540       ??_C@_1CM@FNJKEBIB@?$AAR?$AAe?$AAc?$AAe?$AAi?$AAv?$AAe?$AAd?$AA?5?$AAa?$AA?5?$AAm?$AAe?$AAs?$AAs?$AAa?$AAg?$AAe?$AA?$CB?$AA?$AN?$AA?6?$AA?$AA@ 00015540     fsl_rne_pdd_common_topaz_v1:rndis_pdd.obj
 0001:0000456c       ??_C@_1CO@MJKBFNNP@?$AAD?$AAo?$AAn?$AAe?$AA?5?$AAr?$AAe?$AAc?$AAe?$AAi?$AAv?$AAi?$AAn?$AAg?$AA?5?$AAd?$AAa?$AAt?$AAa?$AA?4?$AA?$AN?$AA?6?$AA?$AA@ 0001556c     fsl_rne_pdd_common_topaz_v1:rndis_pdd.obj
 0001:000045a0       ??_C@_1FM@FDJOONCJ@?$AAG?$AAo?$AAt?$AA?5?$AAS?$AAE?$AAT?$AAU?$AAP?$AA?5?$AA?$DM?$AAN?$AAO?$AA?5?$AAD?$AAA?$AAT?$AAA?$AA?3?$AA?5?$AA?$CF?$AAx?$AA?5?$AA?$CF?$AAx?$AA?5?$AA?$CF?$AAx?$AA?5?$AA?$CF?$AAx?$AA?5@ 000155a0     fsl_rne_pdd_common_topaz_v1:rndis_pdd.obj
 0001:000045fc       ??_C@_1DA@MJLPENBD@?$AAG?$AAo?$AAt?$AA?5?$AAS?$AAE?$AAT?$AAU?$AAP?$AA?5?$AAO?$AAU?$AAT?$AA?5?$AAp?$AAa?$AAc?$AAk?$AAe?$AAt?$AA?4?$AA?$AN?$AA?6?$AA?$AA@ 000155fc     fsl_rne_pdd_common_topaz_v1:rndis_pdd.obj
 0001:0000462c       ??_C@_1CM@NHNGDKFM@?$AAG?$AAo?$AAt?$AA?5?$AAS?$AAE?$AAT?$AAU?$AAP?$AA?5?$AAI?$AAN?$AA?5?$AAp?$AAa?$AAc?$AAk?$AAe?$AAt?$AA?$AN?$AA?6?$AA?$AA@ 0001562c     fsl_rne_pdd_common_topaz_v1:rndis_pdd.obj
 0001:00004658       ??_C@_1DK@CJOHLCDF@?$AAE?$AAR?$AAR?$AAO?$AAR?$AA?5?$AAP?$AAA?$AAR?$AAS?$AAI?$AAN?$AAG?$AA?5?$AAS?$AAE?$AAT?$AAU?$AAP?$AA?5?$AAP?$AAA?$AAC?$AAK?$AAE?$AAT?$AA?$AN?$AA?6?$AA?$AA@ 00015658     fsl_rne_pdd_common_topaz_v1:rndis_pdd.obj
 0001:00004694       ??_C@_1CO@MPAJKINN@?$AA?9?$AAR?$AAN?$AAD?$AAI?$AAS?$AA_?$AAU?$AAS?$AAB?$AAF?$AAN?$AA_?$AAP?$AAD?$AAD?$AAI?$AAn?$AAi?$AAt?$AA?$AN?$AA?6?$AA?$AA@ 00015694     fsl_rne_pdd_common_topaz_v1:rndis_pdd.obj
 0001:000046c8       ??_C@_1GC@COEDNCDC@?$AA?5?$AAR?$AAN?$AAD?$AAI?$AAS?$AA_?$AAU?$AAS?$AAB?$AAF?$AAN?$AA_?$AAP?$AAD?$AAD?$AAI?$AAn?$AAi?$AAt?$AA?3?$AA?5?$AAi?$AAn?$AAi?$AAt?$AAi?$AAa?$AAl?$AAi?$AAz?$AAa@ 000156c8     fsl_rne_pdd_common_topaz_v1:rndis_pdd.obj
 0001:0000472c       ??_C@_1CM@CGCNDLMD@?$AAU?$AAf?$AAn?$AAP?$AAd?$AAd?$AA_?$AAI?$AAn?$AAi?$AAt?$AA?5?$AAf?$AAa?$AAi?$AAl?$AAe?$AAd?$AA?$CB?$AA?$AN?$AA?6?$AA?$AA@ 0001572c     fsl_rne_pdd_common_topaz_v1:rndis_pdd.obj
 0001:00004758       ??_C@_1DA@MNIGJPIF@?$AA?9?$AAR?$AAN?$AAD?$AAI?$AAS?$AA_?$AAU?$AAS?$AAB?$AAF?$AAN?$AA_?$AAP?$AAD?$AAD?$AAD?$AAe?$AAn?$AAi?$AAt?$AA?$AN?$AA?6?$AA?$AA@ 00015758     fsl_rne_pdd_common_topaz_v1:rndis_pdd.obj
 0001:00004788       ??_C@_1DA@EACCPFEN@?$AA?$CL?$AAR?$AAN?$AAD?$AAI?$AAS?$AA_?$AAU?$AAS?$AAB?$AAF?$AAN?$AA_?$AAP?$AAD?$AAD?$AAD?$AAe?$AAn?$AAi?$AAt?$AA?$AN?$AA?6?$AA?$AA@ 00015788     fsl_rne_pdd_common_topaz_v1:rndis_pdd.obj
 0001:000047b8       ??_C@_1EI@ONHOMNHJ@?$AA?9?$AAR?$AAN?$AAD?$AAI?$AAS?$AA_?$AAU?$AAS?$AAB?$AAF?$AAN?$AA_?$AAP?$AAD?$AAD?$AA_?$AAS?$AAe?$AAn?$AAd?$AAR?$AAn?$AAd?$AAi?$AAs?$AAM?$AAe?$AAs?$AAs?$AAa?$AAg@ 000157b8     fsl_rne_pdd_common_topaz_v1:rndis_pdd.obj
 0001:00004800       ??_C@_1HE@PDJOEOPK@?$AA?$CL?$AAR?$AAN?$AAD?$AAI?$AAS?$AA_?$AAU?$AAS?$AAB?$AAF?$AAN?$AA_?$AAP?$AAD?$AAD?$AA_?$AAS?$AAe?$AAn?$AAd?$AAR?$AAn?$AAd?$AAi?$AAs?$AAM?$AAe?$AAs?$AAs?$AAa?$AAg@ 00015800     fsl_rne_pdd_common_topaz_v1:rndis_pdd.obj
 0001:00004878       ??_C@_1GK@OCDDHLML@?$AA?$CL?$AAR?$AAN?$AAD?$AAI?$AAS?$AA_?$AAU?$AAS?$AAB?$AAF?$AAN?$AA_?$AAP?$AAD?$AAD?$AA_?$AAS?$AAe?$AAn?$AAd?$AAR?$AAn?$AAd?$AAi?$AAs?$AAM?$AAe?$AAs?$AAs?$AAa?$AAg@ 00015878     fsl_rne_pdd_common_topaz_v1:rndis_pdd.obj
 0001:000048e8       ??_C@_1EI@LPKHCIID@?$AA?$CL?$AAR?$AAN?$AAD?$AAI?$AAS?$AA_?$AAU?$AAS?$AAB?$AAF?$AAN?$AA_?$AAP?$AAD?$AAD?$AA_?$AAS?$AAe?$AAn?$AAd?$AAR?$AAn?$AAd?$AAi?$AAs?$AAM?$AAe?$AAs?$AAs?$AAa?$AAg@ 000158e8     fsl_rne_pdd_common_topaz_v1:rndis_pdd.obj
 0001:00004930       ??_C@_1EG@FPFPIBJG@?$AA?9?$AAR?$AAN?$AAD?$AAI?$AAS?$AA_?$AAU?$AAS?$AAB?$AAF?$AAN?$AA_?$AAP?$AAD?$AAD?$AA_?$AAS?$AAe?$AAn?$AAd?$AAR?$AAn?$AAd?$AAi?$AAs?$AAP?$AAa?$AAc?$AAk?$AAe?$AAt@ 00015930     fsl_rne_pdd_common_topaz_v1:rndis_pdd.obj
 0001:00004978       ??_C@_1FG@MIKLDILD@?$AA?$CK?$AA?$CK?$AA?$CK?$AA?$CK?$AAM?$AAu?$AAl?$AAt?$AAi?$AAp?$AAl?$AAe?$AA?5?$AAp?$AAe?$AAn?$AAd?$AAi?$AAn?$AAg?$AA?5?$AAs?$AAe?$AAn?$AAd?$AA?5?$AAr?$AAn?$AAd?$AAi?$AAs?$AA?5@ 00015978     fsl_rne_pdd_common_topaz_v1:rndis_pdd.obj
 0001:000049d0       ??_C@_1EI@PJCOBAOE@?$AAG?$AAo?$AAt?$AA?5?$AAS?$AAe?$AAn?$AAd?$AAP?$AAa?$AAc?$AAk?$AAe?$AAt?$AA?5?$AAR?$AAe?$AAq?$AAu?$AAe?$AAs?$AAt?$AA?5?$AA?$FL?$AA?$CF?$AAd?$AA?5?$AAb?$AAy?$AAt?$AAe?$AAs@ 000159d0     fsl_rne_pdd_common_topaz_v1:rndis_pdd.obj
 0001:00004a18       ??_C@_1EG@FDHKBGKN@?$AA?$CL?$AAR?$AAN?$AAD?$AAI?$AAS?$AA_?$AAU?$AAS?$AAB?$AAF?$AAN?$AA_?$AAP?$AAD?$AAD?$AA_?$AAS?$AAe?$AAn?$AAd?$AAR?$AAn?$AAd?$AAi?$AAs?$AAP?$AAa?$AAc?$AAk?$AAe?$AAt@ 00015a18     fsl_rne_pdd_common_topaz_v1:rndis_pdd.obj
 0001:00004a60       ??_C@_1CO@MBMDAIGD@?$AA?9?$AAR?$AAN?$AAD?$AAI?$AAS?$AA_?$AAU?$AAS?$AAB?$AAF?$AAN?$AA_?$AAP?$AAD?$AAD?$AA_?$AAS?$AAe?$AAt?$AA?$AN?$AA?6?$AA?$AA@ 00015a60     fsl_rne_pdd_common_topaz_v1:rndis_pdd.obj
 0001:00004a90       ??_C@_1DO@PIKCPFME@?$AAP?$AAD?$AAD?$AA_?$AAS?$AAe?$AAt?$AA?3?$AAU?$AAn?$AAk?$AAn?$AAo?$AAw?$AAn?$AA?5?$AAr?$AAe?$AAq?$AAu?$AAe?$AAs?$AAt?$AA?3?$AA0?$AAx?$AA?$CF?$AAx?$AA?$AN?$AA?6?$AA?$AA@ 00015a90     fsl_rne_pdd_common_topaz_v1:rndis_pdd.obj
 0001:00004ad0       ??_C@_1DK@PGGKHLLK@?$AAP?$AAD?$AAD?$AA_?$AAS?$AAe?$AAt?$AA?3?$AAR?$AAE?$AAQ?$AA_?$AAI?$AAD?$AA_?$AAD?$AAI?$AAS?$AAA?$AAB?$AAL?$AAE?$AA_?$AAI?$AAN?$AAT?$AA?$AN?$AA?6?$AA?$AA@ 00015ad0     fsl_rne_pdd_common_topaz_v1:rndis_pdd.obj
 0001:00004b0c       ??_C@_1DI@KFPGHMKG@?$AAP?$AAD?$AAD?$AA_?$AAS?$AAe?$AAt?$AA?3?$AAR?$AAE?$AAQ?$AA_?$AAI?$AAD?$AA_?$AAE?$AAN?$AAA?$AAB?$AAL?$AAE?$AA_?$AAI?$AAN?$AAT?$AA?$AN?$AA?6?$AA?$AA@ 00015b0c     fsl_rne_pdd_common_topaz_v1:rndis_pdd.obj
 0001:00004b44       ??_C@_1DI@MFNCMIPE@?$AAP?$AAD?$AAD?$AA_?$AAS?$AAe?$AAt?$AA?3?$AAR?$AAE?$AAQ?$AA_?$AAI?$AAD?$AA_?$AAS?$AAO?$AAF?$AAT?$AA_?$AAR?$AAE?$AAS?$AAE?$AAT?$AA?$AN?$AA?6?$AA?$AA@ 00015b44     fsl_rne_pdd_common_topaz_v1:rndis_pdd.obj
 0001:00004b7c       ??_C@_1DI@LPFOEPEC@?$AAP?$AAD?$AAD?$AA_?$AAS?$AAe?$AAt?$AA?3?$AAR?$AAE?$AAQ?$AA_?$AAI?$AAD?$AA_?$AAH?$AAA?$AAR?$AAD?$AA_?$AAR?$AAE?$AAS?$AAE?$AAT?$AA?$AN?$AA?6?$AA?$AA@ 00015b7c     fsl_rne_pdd_common_topaz_v1:rndis_pdd.obj
 0001:00004bb4       ??_C@_1CO@BKAHFHEI@?$AA?$CL?$AAR?$AAN?$AAD?$AAI?$AAS?$AA_?$AAU?$AAS?$AAB?$AAF?$AAN?$AA_?$AAP?$AAD?$AAD?$AA_?$AAS?$AAe?$AAt?$AA?$AN?$AA?6?$AA?$AA@ 00015bb4     fsl_rne_pdd_common_topaz_v1:rndis_pdd.obj
 0001:00004be4       ??_C@_0BO@FJNCJEJP@Discard?5?$CFd?5Pending?5Messages?$AN?6?$AA@ 00015be4     fsl_rne_pdd_common_topaz_v1:rndis_pdd.obj
 0001:00004c04       ??_C@_1CO@MONNNOOA@?$AA?9?$AAR?$AAN?$AAD?$AAI?$AAS?$AA_?$AAU?$AAS?$AAB?$AAF?$AAN?$AA_?$AAP?$AAD?$AAD?$AA_?$AAG?$AAe?$AAt?$AA?$AN?$AA?6?$AA?$AA@ 00015c04     fsl_rne_pdd_common_topaz_v1:rndis_pdd.obj
 0001:00004c38       ??_C@_1EC@FCCAEHJA@?$AA?9?$AAP?$AAD?$AAD?$AA_?$AAG?$AAe?$AAt?$AA?3?$AA?5?$AAu?$AAn?$AAk?$AAn?$AAo?$AAw?$AAn?$AA?5?$AAr?$AAe?$AAq?$AAu?$AAe?$AAs?$AAt?$AA?5?$AA0?$AAx?$AA?$CF?$AAx?$AA?$AN?$AA?6@ 00015c38     fsl_rne_pdd_common_topaz_v1:rndis_pdd.obj
 0001:00004c7c       ??_C@_1CO@BFBJIBML@?$AA?$CL?$AAR?$AAN?$AAD?$AAI?$AAS?$AA_?$AAU?$AAS?$AAB?$AAF?$AAN?$AA_?$AAP?$AAD?$AAD?$AA_?$AAG?$AAe?$AAt?$AA?$AN?$AA?6?$AA?$AA@ 00015c7c     fsl_rne_pdd_common_topaz_v1:rndis_pdd.obj
 0001:00004cb0       ??_C@_1FO@HIPGBBGN@?$AA?9?$AAR?$AAN?$AAD?$AAI?$AAS?$AA_?$AAU?$AAS?$AAB?$AAF?$AAN?$AA_?$AAP?$AAD?$AAD?$AA_?$AAI?$AAn?$AAd?$AAi?$AAc?$AAa?$AAt?$AAe?$AAR?$AAn?$AAd?$AAi?$AAs?$AAP?$AAa@ 00015cb0     fsl_rne_pdd_common_topaz_v1:rndis_pdd.obj
 0001:00004d10       ??_C@_1FO@PLBKEBPA@?$AA?$CL?$AAR?$AAN?$AAD?$AAI?$AAS?$AA_?$AAU?$AAS?$AAB?$AAF?$AAN?$AA_?$AAP?$AAD?$AAD?$AA_?$AAI?$AAn?$AAd?$AAi?$AAc?$AAa?$AAt?$AAe?$AAR?$AAn?$AAd?$AAi?$AAs?$AAP?$AAa@ 00015d10     fsl_rne_pdd_common_topaz_v1:rndis_pdd.obj
 0001:00004d70       ??_C@_1DG@LOIHLLKG@?$AAR?$AAN?$AAD?$AAI?$AAS?$AA?5?$AAS?$AAe?$AAr?$AAi?$AAa?$AAl?$AA?5?$AAN?$AAu?$AAm?$AAb?$AAe?$AAr?$AA?$DN?$AA?$FL?$AA?$CF?$AAs?$AA?$FN?$AA?$AN?$AA?6?$AA?$AA@ 00015d70     fsl_rne_pdd_common_topaz_v1:rndis_pdd.obj
 0001:00004da8       ??_C@_1BC@GDFGLIEL@?$AAO?$AAT?$AAG?$AAG?$AAr?$AAo?$AAu?$AAp?$AA?$AA@ 00015da8     usb_usbfn_mx25_topaz_v1:i_pdd.obj
 0001:00004dbc       ??_C@_1BG@HHFAGDDC@?$AAO?$AAT?$AAG?$AAS?$AAu?$AAp?$AAp?$AAo?$AAr?$AAt?$AA?$AA@ 00015dbc     usb_usbfn_mx25_topaz_v1:i_pdd.obj
 0001:00004dd4       ??_C@_1BI@BHLBGEOK@?$AAP?$AAr?$AAi?$AAo?$AAr?$AAi?$AAt?$AAy?$AA2?$AA5?$AA6?$AA?$AA@ 00015dd4     usb_usbfn_mx25_topaz_v1:i_pdd.obj
 0001:00004dec       ??_C@_17DJGGJCGD@?$AAI?$AAr?$AAq?$AA?$AA@ 00015dec     usb_usbfn_mx25_topaz_v1:i_pdd.obj
 0001:00004df4       ??_C@_1O@LBBNFMDB@?$AAM?$AAe?$AAm?$AAL?$AAe?$AAn?$AA?$AA@ 00015df4     usb_usbfn_mx25_topaz_v1:i_pdd.obj
 0001:00004e04       ??_C@_1BA@INLDIDEN@?$AAM?$AAe?$AAm?$AAB?$AAa?$AAs?$AAe?$AA?$AA@ 00015e04     usb_usbfn_mx25_topaz_v1:i_pdd.obj
 0001:00004ea8       ??_C@_1CM@IKIIJOLF@?$AAP?$AAo?$AAw?$AAe?$AAr?$AAD?$AAo?$AAw?$AAn?$AA?5?$AAc?$AAo?$AAm?$AAp?$AAl?$AAe?$AAt?$AAe?$AAd?$AA?$AN?$AA?6?$AA?$AA@ 00015ea8     usb_usbfn_mx25_topaz_v1:i_pdd.obj
 0001:00004ed4       ??_C@_1CC@OEGDFOPI@?$AAU?$AAS?$AAB?$AA?5?$AAC?$AAl?$AAo?$AAc?$AAk?$AA?5?$AAs?$AAt?$AAo?$AAp?$AA?$AN?$AA?6?$AA?$AA@ 00015ed4     usb_usbfn_mx25_topaz_v1:i_pdd.obj
 0001:00004ef8       ??_C@_1DC@MJCJJIDL@?$AAP?$AAo?$AAw?$AAe?$AAr?$AAD?$AAo?$AAw?$AAn?$AA?5?$AAU?$AAS?$AAB?$AAC?$AAT?$AAR?$AAL?$AA?$DN?$AA0?$AAx?$AA?$CF?$AAx?$AA?$AN?$AA?6?$AA?$AA@ 00015ef8     usb_usbfn_mx25_topaz_v1:i_pdd.obj
 0001:00004f2c       ??_C@_1DC@NJODNJCA@?$AAP?$AAo?$AAw?$AAe?$AAr?$AAD?$AAo?$AAw?$AAn?$AA?5?$AAP?$AAO?$AAR?$AAT?$AAS?$AAC?$AA?$DN?$AA?5?$AA0?$AAx?$AA?$CF?$AAx?$AA?$AN?$AA?6?$AA?$AA@ 00015f2c     usb_usbfn_mx25_topaz_v1:i_pdd.obj
 0001:00004f60       ??_C@_1DG@NJOCHJMF@?$AAP?$AAo?$AAw?$AAe?$AAr?$AAD?$AAo?$AAw?$AAn?$AA?5?$AAU?$AAS?$AAB?$AAI?$AAN?$AAT?$AAR?$AA?5?$AA?$DN?$AA?5?$AA0?$AAx?$AA?$CF?$AAx?$AA?$AN?$AA?6?$AA?$AA@ 00015f60     usb_usbfn_mx25_topaz_v1:i_pdd.obj
 0001:00004f98       ??_C@_1DE@CFOAAIJP@?$AAP?$AAo?$AAw?$AAe?$AAr?$AAD?$AAo?$AAw?$AAn?$AA?5?$AAU?$AAS?$AAB?$AAC?$AAM?$AAD?$AA?5?$AA?$DN?$AA?5?$AA0?$AAx?$AA?$CF?$AAx?$AA?$AN?$AA?6?$AA?$AA@ 00015f98     usb_usbfn_mx25_topaz_v1:i_pdd.obj
 0001:00004fd0       ??_C@_1EM@IEDMFFDN@?$AAU?$AAf?$AAn?$AAP?$AAd?$AAd?$AA_?$AAP?$AAo?$AAw?$AAe?$AAr?$AAD?$AAo?$AAw?$AAn?$AA?5?$AAn?$AAo?$AA?5?$AAa?$AAc?$AAt?$AAi?$AAo?$AAn?$AA?5?$AAr?$AAe?$AAq?$AAu?$AAi@ 00015fd0     usb_usbfn_mx25_topaz_v1:i_pdd.obj
 0001:0000501c       ??_C@_1CG@OIILOOGO@?$AAU?$AAs?$AAb?$AAP?$AAd?$AAd?$AA_?$AAP?$AAo?$AAw?$AAe?$AAr?$AAD?$AAo?$AAw?$AAn?$AA?$AN?$AA?6?$AA?$AA@ 0001601c     usb_usbfn_mx25_topaz_v1:i_pdd.obj
 0001:00005044       ??_C@_1DA@KMOKCFJD@?$AAP?$AAo?$AAw?$AAe?$AAr?$AAU?$AAp?$AA?5?$AAU?$AAS?$AAB?$AAC?$AAM?$AAD?$AA?5?$AA?$DN?$AA?5?$AA0?$AAx?$AA?$CF?$AAx?$AA?$AN?$AA?6?$AA?$AA@ 00016044     usb_usbfn_mx25_topaz_v1:i_pdd.obj
 0001:00005078       ??_C@_1EA@HIDFOGGD@?$AAW?$AAa?$AAk?$AAe?$AAu?$AAp?$AA?5?$AAI?$AAn?$AAt?$AAe?$AAr?$AAr?$AAu?$AAp?$AAt?$AA?5?$AAS?$AAe?$AAt?$AAt?$AAi?$AAn?$AAg?$AA?5?$AA0?$AAx?$AA?$CF?$AAx?$AA?$AN?$AA?6?$AA?$AA@ 00016078     usb_usbfn_mx25_topaz_v1:i_pdd.obj
 0001:000050b8       ??_C@_1DA@ODLPFKGM@?$AAP?$AAo?$AAw?$AAe?$AAr?$AAU?$AAp?$AA?5?$AAw?$AAa?$AAk?$AAe?$AAu?$AAp?$AA?5?$AA?$DN?$AA?5?$AA0?$AAx?$AA?$CF?$AAx?$AA?$AN?$AA?6?$AA?$AA@ 000160b8     usb_usbfn_mx25_topaz_v1:i_pdd.obj
 0001:000050e8       ??_C@_1BO@JBMLODEA@?$AAF?$AAo?$AAr?$AAc?$AAe?$AA?5?$AAr?$AAe?$AAs?$AAu?$AAm?$AAe?$AA?$AN?$AA?6?$AA?$AA@ 000160e8     usb_usbfn_mx25_topaz_v1:i_pdd.obj
 0001:00005108       ??_C@_1EI@LEEJEJNJ@?$AAP?$AAo?$AAw?$AAe?$AAr?$AAU?$AAp?$AA?3?$AAU?$AAS?$AAB?$AAS?$AAT?$AAS?$AA?$CI?$AA0?$AAx?$AA?$CF?$AAx?$AA?$CJ?$AA?5?$AAP?$AAO?$AAR?$AAT?$AAS?$AAC?$AA?$CI?$AA0?$AAx?$AA?$CF?$AAx@ 00016108     usb_usbfn_mx25_topaz_v1:i_pdd.obj
 0001:00005150       ??_C@_1CE@HMNFKKGB@?$AAU?$AAS?$AAB?$AA?5?$AAC?$AAl?$AAo?$AAc?$AAk?$AA?5?$AAs?$AAt?$AAa?$AAr?$AAt?$AA?$AN?$AA?6?$AA?$AA@ 00016150     usb_usbfn_mx25_topaz_v1:i_pdd.obj
 0001:00005178       ??_C@_1EE@FMEOMODP@?$AAU?$AAs?$AAb?$AAP?$AAd?$AAd?$AA_?$AAP?$AAo?$AAw?$AAe?$AAr?$AAU?$AAp?$AA?5?$AAw?$AAi?$AAt?$AAh?$AA?5?$AAb?$AAI?$AAn?$AAU?$AAS?$AAB?$AAF?$AAN?$AA?5?$AA?$CF?$AAd?$AA?$AN@ 00016178     usb_usbfn_mx25_topaz_v1:i_pdd.obj
 0001:000051c0       ??_C@_1EC@POPMIGGA@?$AAU?$AAp?$AAd?$AAa?$AAt?$AAe?$AAD?$AAe?$AAv?$AAi?$AAc?$AAe?$AAP?$AAo?$AAw?$AAe?$AAr?$AA?5?$AAt?$AAo?$AA?5?$AAp?$AAo?$AAw?$AAe?$AAr?$AAd?$AAo?$AAw?$AAn?$AA?$AN?$AA?6@ 000161c0     usb_usbfn_mx25_topaz_v1:i_pdd.obj
 0001:00005204       ??_C@_1DO@CFDCODDO@?$AAU?$AAp?$AAd?$AAa?$AAt?$AAe?$AAD?$AAe?$AAv?$AAi?$AAc?$AAe?$AAP?$AAo?$AAw?$AAe?$AAr?$AA?5?$AAt?$AAo?$AA?5?$AAp?$AAo?$AAw?$AAe?$AAr?$AAu?$AAp?$AA?$AN?$AA?6?$AA?$AA@ 00016204     usb_usbfn_mx25_topaz_v1:i_pdd.obj
 0001:00005248       ??_C@_1FE@DIHLBJLK@?$AAU?$AAp?$AAd?$AAa?$AAt?$AAe?$AAD?$AAe?$AAv?$AAi?$AAc?$AAe?$AAP?$AAo?$AAw?$AAe?$AAr?$AA?5?$AAG?$AAo?$AAi?$AAn?$AAg?$AA?5?$AAf?$AAr?$AAo?$AAm?$AA?5?$AAD?$AA?$CF?$AAd@ 00016248     usb_usbfn_mx25_topaz_v1:i_pdd.obj
 0001:000052a0       ??_C@_1KO@EOAMMFLK@?$AAc?$AA?3?$AA?2?$AAw?$AAi?$AAn?$AAc?$AAe?$AAr?$AAo?$AAo?$AAt?$AAs?$AA?2?$AAt?$AAo?$AAp?$AAa?$AAz?$AA?2?$AAw?$AAi?$AAn?$AAc?$AAe?$AA7?$AA0?$AA0?$AA?2?$AAp?$AAl?$AAa@ 000162a0     usb_usbfn_mx25_topaz_v1:i_pdd.obj
 0001:00005350       ??_C@_1BO@LJJCCAKA@?$AAS?$AAe?$AAt?$AAu?$AAp?$AA?3?$AA?5?$AA?$CF?$AAx?$AA?5?$AA?$CF?$AAx?$AA?$AN?$AA?6?$AA?$AA@ 00016350     usb_usbfn_mx25_topaz_v1:i_pdd.obj
 0001:00005370       ??_C@_1CA@NAJOELH@?$AAD?$AAe?$AAv?$AAi?$AAc?$AAe?$AA?5?$AAA?$AAt?$AAt?$AAa?$AAc?$AAh?$AA?$AN?$AA?6?$AA?$AA@ 00016370     usb_usbfn_mx25_topaz_v1:i_pdd.obj
 0001:00005390       ??_C@_1IE@MBNKMJA@?$AA?$CD?$AA?$CD?$AA?$CD?$AA?$CD?$AA?$CD?$AA?$CD?$AA?$CD?$AA?5?$AAG?$AAe?$AAt?$AAS?$AAe?$AAt?$AAu?$AAp?$AAP?$AAa?$AAc?$AAk?$AAe?$AAt?$AA?3?$AA?5?$AAF?$AAl?$AAu?$AAs?$AAh?$AAi?$AAn?$AAg@ 00016390     usb_usbfn_mx25_topaz_v1:i_pdd.obj
 0001:00005418       ??_C@_1KK@KOKNNFID@?$AA?$CD?$AA?$CD?$AA?$CD?$AA?$CD?$AA?$CD?$AA?$CD?$AA?$CD?$AA?5?$AAG?$AAe?$AAt?$AAS?$AAe?$AAt?$AAu?$AAp?$AAP?$AAa?$AAc?$AAk?$AAe?$AAt?$AA?3?$AA?5?$AAT?$AAr?$AAa?$AAn?$AAs?$AAf?$AAe?$AAr@ 00016418     usb_usbfn_mx25_topaz_v1:i_pdd.obj
 0001:000054c4       ??_C@_1DM@JOKNMMI@?$AAG?$AAe?$AAt?$AAS?$AAe?$AAt?$AAu?$AAp?$AAP?$AAa?$AAc?$AAk?$AAe?$AAt?$AA?5?$AA?$CF?$AA8?$AA?4?$AA8?$AAl?$AAx?$AA?$CF?$AA8?$AA?4?$AA8?$AAl?$AAx?$AA?$AN?$AA?6?$AA?$AA@ 000164c4     usb_usbfn_mx25_topaz_v1:i_pdd.obj
 0001:00005500       ??_C@_1DM@PINNGIJL@?$AA?7?$AA?7?$AA?7?$AAS?$AAe?$AAr?$AAi?$AAa?$AAl?$AA?1?$AA1?$AA?4?$AA1?$AA?5?$AAP?$AAH?$AAY?$AA?5?$AA?$CI?$AAF?$AAS?$AA?5?$AAO?$AAn?$AAl?$AAy?$AA?$CJ?$AA?$AN?$AA?6?$AA?$AA@ 00016500     usb_usbfn_mx25_topaz_v1:i_pdd.obj
 0001:0000553c       ??_C@_1BE@OHMKGMAA@?$AA?7?$AA?7?$AA?7?$AAU?$AAL?$AAP?$AAI?$AA?$AN?$AA?6?$AA?$AA@ 0001653c     usb_usbfn_mx25_topaz_v1:i_pdd.obj
 0001:00005550       ??_C@_1CK@JDCKMGFE@?$AA?7?$AA?7?$AA?7?$AAP?$AAh?$AAi?$AAl?$AAi?$AAp?$AAs?$AA?5?$AAC?$AAl?$AAa?$AAs?$AAs?$AAi?$AAc?$AA?$AN?$AA?6?$AA?$AA@ 00016550     usb_usbfn_mx25_topaz_v1:i_pdd.obj
 0001:0000557c       ??_C@_1CA@GIFIBBC@?$AA?7?$AA?7?$AA?7?$AAU?$AAT?$AAM?$AAI?$AA?1?$AAU?$AAT?$AAM?$AAI?$AA?$CL?$AA?$AN?$AA?6?$AA?$AA@ 0001657c     usb_usbfn_mx25_topaz_v1:i_pdd.obj
 0001:000055a0       ??_C@_1EG@GEPPEHI@?$AA?7?$AA?7?$AAP?$AAa?$AAr?$AAa?$AAl?$AAl?$AAe?$AAl?$AA?5?$AAT?$AAr?$AAa?$AAn?$AAs?$AAc?$AAe?$AAi?$AAv?$AAe?$AAr?$AA?5?$AAS?$AAe?$AAl?$AAe?$AAc?$AAt?$AA?3?$AA?$CF?$AAx@ 000165a0     usb_usbfn_mx25_topaz_v1:i_pdd.obj
 0001:000055e8       ??_C@_1DO@GOALHOBG@?$AA?7?$AA?7?$AAS?$AAe?$AAr?$AAi?$AAa?$AAl?$AA?5?$AAT?$AAr?$AAa?$AAn?$AAs?$AAc?$AAe?$AAi?$AAv?$AAe?$AAr?$AA?5?$AAS?$AAe?$AAl?$AAe?$AAc?$AAt?$AA?5?$AA?$AN?$AA?6?$AA?$AA@ 000165e8     usb_usbfn_mx25_topaz_v1:i_pdd.obj
 0001:00005628       ??_C@_1BI@PMFMKPBN@?$AA?7?$AA?7?$AA?7?$AA8?$AA?5?$AAb?$AAi?$AAt?$AAs?$AA?$AN?$AA?6?$AA?$AA@ 00016628     usb_usbfn_mx25_topaz_v1:i_pdd.obj
 0001:00005640       ??_C@_1BK@DMIJGPDB@?$AA?7?$AA?7?$AA?7?$AA1?$AA6?$AA?5?$AAb?$AAi?$AAt?$AAs?$AA?$AN?$AA?6?$AA?$AA@ 00016640     usb_usbfn_mx25_topaz_v1:i_pdd.obj
 0001:00005660       ??_C@_1EE@PJPHJMEN@?$AA?7?$AA?7?$AAP?$AAa?$AAr?$AAa?$AAl?$AAl?$AAe?$AAl?$AA?5?$AAT?$AAr?$AAa?$AAn?$AAs?$AAc?$AAe?$AAi?$AAv?$AAe?$AAr?$AA?5?$AAW?$AAi?$AAd?$AAt?$AAh?$AA?3?$AA?$CF?$AAx?$AA?9@ 00016660     usb_usbfn_mx25_topaz_v1:i_pdd.obj
 0001:000056a4       ??_C@_1CA@CFDEDDEG@?$AA?7?$AA?7?$AA?7?$AAH?$AAi?$AAg?$AAh?$AA?5?$AAS?$AAp?$AAe?$AAe?$AAd?$AA?$AN?$AA?6?$AA?$AA@ 000166a4     usb_usbfn_mx25_topaz_v1:i_pdd.obj
 0001:000056c4       ??_C@_1BO@DONMFABC@?$AA?7?$AA?7?$AA?7?$AAL?$AAo?$AAw?$AA?5?$AAS?$AAp?$AAe?$AAe?$AAd?$AA?$AN?$AA?6?$AA?$AA@ 000166c4     usb_usbfn_mx25_topaz_v1:i_pdd.obj
 0001:000056e4       ??_C@_1CA@EFHFHOIO@?$AA?7?$AA?7?$AA?7?$AAF?$AAu?$AAl?$AAl?$AA?5?$AAS?$AAp?$AAe?$AAe?$AAd?$AA?$AN?$AA?6?$AA?$AA@ 000166e4     usb_usbfn_mx25_topaz_v1:i_pdd.obj
 0001:00005704       ??_C@_1CG@DLDJDNPN@?$AA?7?$AA?7?$AAP?$AAo?$AAr?$AAt?$AA?5?$AAS?$AAp?$AAe?$AAe?$AAd?$AA?3?$AA?5?$AA?$CF?$AAx?$AA?9?$AA?$DO?$AA?$AA@ 00016704     usb_usbfn_mx25_topaz_v1:i_pdd.obj
 0001:00005730       ??_C@_1EG@FLKCNOK@?$AA?7?$AA?7?$AAP?$AAo?$AAr?$AAt?$AA?5?$AAF?$AAo?$AAr?$AAc?$AAe?$AA?5?$AAF?$AAu?$AAl?$AAl?$AA?5?$AAS?$AAp?$AAe?$AAe?$AAd?$AA?5?$AAC?$AAo?$AAn?$AAn?$AAe?$AAc?$AAt?$AA?5@ 00016730     usb_usbfn_mx25_topaz_v1:i_pdd.obj
 0001:00005778       ??_C@_1GI@HKEGLKNC@?$AA?7?$AA?7?$AAP?$AAH?$AAY?$AA?5?$AAL?$AAo?$AAw?$AA?5?$AAP?$AAo?$AAw?$AAe?$AAr?$AA?5?$AAS?$AAu?$AAs?$AAp?$AAe?$AAn?$AAd?$AA?5?$AA?9?$AA?5?$AAC?$AAl?$AAo?$AAc?$AAk?$AA?5@ 00016778     usb_usbfn_mx25_topaz_v1:i_pdd.obj
 0001:000057e0       ??_C@_1FE@PECIMICA@?$AA?7?$AA?7?$AAW?$AAa?$AAk?$AAe?$AA?5?$AAo?$AAn?$AA?5?$AAO?$AAv?$AAe?$AAr?$AA?9?$AAc?$AAu?$AAr?$AAr?$AAe?$AAn?$AAt?$AA?5?$AAE?$AAn?$AAa?$AAb?$AAl?$AAe?$AA?5?$AA?$CI?$AAW@ 000167e0     usb_usbfn_mx25_topaz_v1:i_pdd.obj
 0001:00005838       ??_C@_1FI@KPMEKFHG@?$AA?7?$AA?7?$AAW?$AAa?$AAk?$AAe?$AA?5?$AAo?$AAn?$AA?5?$AAD?$AAi?$AAs?$AAc?$AAo?$AAn?$AAn?$AAe?$AAc?$AAt?$AA?5?$AAE?$AAn?$AAa?$AAb?$AAl?$AAe?$AA?5?$AA?$CI?$AAW?$AAK?$AAD@ 00016838     usb_usbfn_mx25_topaz_v1:i_pdd.obj
 0001:00005890       ??_C@_1EM@HPIOFCNI@?$AA?7?$AA?7?$AAW?$AAa?$AAk?$AAe?$AA?5?$AAo?$AAn?$AA?5?$AAC?$AAo?$AAn?$AAn?$AAe?$AAc?$AAt?$AA?5?$AAE?$AAn?$AAa?$AAb?$AAl?$AAe?$AA?5?$AA?$CI?$AAW?$AAK?$AAC?$AAN?$AAN?$AAT@ 00016890     usb_usbfn_mx25_topaz_v1:i_pdd.obj
 0001:000058dc       ??_C@_1DE@NJCPBMGI@?$AA?7?$AA?7?$AAP?$AAo?$AAr?$AAt?$AA?5?$AAT?$AAe?$AAs?$AAt?$AA?5?$AAC?$AAo?$AAn?$AAt?$AAr?$AAo?$AAl?$AA?3?$AA?5?$AA?$CF?$AAx?$AA?$AN?$AA?6?$AA?$AA@ 000168dc     usb_usbfn_mx25_topaz_v1:i_pdd.obj
 0001:00005910       ??_C@_1BG@LAPJBFLO@?$AA?7?$AA?7?$AA?7?$AAG?$AAr?$AAe?$AAe?$AAn?$AA?$AN?$AA?6?$AA?$AA@ 00016910     usb_usbfn_mx25_topaz_v1:i_pdd.obj
 0001:00005928       ??_C@_1BG@IMMCDJCL@?$AA?7?$AA?7?$AA?7?$AAA?$AAm?$AAb?$AAe?$AAr?$AA?$AN?$AA?6?$AA?$AA@ 00016928     usb_usbfn_mx25_topaz_v1:i_pdd.obj
 0001:00005940       ??_C@_1DC@IPGABND@?$AA?7?$AA?7?$AAP?$AAo?$AAr?$AAt?$AA?5?$AAI?$AAn?$AAd?$AAi?$AAc?$AAa?$AAt?$AAo?$AAr?$AA?5?$AAC?$AAo?$AAn?$AAt?$AAr?$AAo?$AAl?$AA?$AA@ 00016940     usb_usbfn_mx25_topaz_v1:i_pdd.obj
 0001:00005974       ??_C@_1BO@FPLCLNEP@?$AA?7?$AA?7?$AAP?$AAo?$AAr?$AAt?$AA?5?$AAO?$AAw?$AAn?$AAe?$AAr?$AA?$AN?$AA?6?$AA?$AA@ 00016974     usb_usbfn_mx25_topaz_v1:i_pdd.obj
 0001:00005994       ??_C@_1DO@MCLJLJA@?$AA?7?$AA?7?$AA?$DP?$AA?$DP?$AA?$DP?$AA?5?$AAS?$AAh?$AAo?$AAu?$AAl?$AAd?$AA?5?$AAb?$AAe?$AA?5?$AA0?$AA?5?$AAf?$AAo?$AAr?$AA?5?$AAd?$AAe?$AAv?$AAi?$AAc?$AAe?$AA?$AN?$AA?6?$AA?$AA@ 00016994     usb_usbfn_mx25_topaz_v1:i_pdd.obj
 0001:000059d4       ??_C@_1BO@CGJIBKMJ@?$AA?7?$AA?7?$AA?7?$AAU?$AAn?$AAd?$AAe?$AAf?$AAi?$AAn?$AAe?$AAd?$AA?$AN?$AA?6?$AA?$AA@ 000169d4     usb_usbfn_mx25_topaz_v1:i_pdd.obj
 0001:000059f4       ??_C@_1BK@LEBDPOFP@?$AA?7?$AA?7?$AA?7?$AAK?$AA?9?$AAs?$AAt?$AAa?$AAt?$AAe?$AA?$AN?$AA?6?$AA?$AA@ 000169f4     usb_usbfn_mx25_topaz_v1:i_pdd.obj
 0001:00005a10       ??_C@_1BK@NBHEMFBJ@?$AA?7?$AA?7?$AA?7?$AAJ?$AA?9?$AAs?$AAt?$AAa?$AAt?$AAe?$AA?$AN?$AA?6?$AA?$AA@ 00016a10     usb_usbfn_mx25_topaz_v1:i_pdd.obj
 0001:00005a2c       ??_C@_1BC@HGFCDNBO@?$AA?7?$AA?7?$AA?7?$AAS?$AAE?$AA0?$AA?$AN?$AA?6?$AA?$AA@ 00016a2c     usb_usbfn_mx25_topaz_v1:i_pdd.obj
 0001:00005a40       ??_C@_1CE@HKBMNK@?$AA?7?$AA?7?$AAL?$AAi?$AAn?$AAe?$AA?5?$AAS?$AAt?$AAa?$AAt?$AAu?$AAs?$AA?3?$AA?5?$AA?$CF?$AAx?$AA?$AA@ 00016a40     usb_usbfn_mx25_topaz_v1:i_pdd.obj
 0001:00005a64       ??_C@_1CK@KAKGINHH@?$AA?7?$AA?7?$AAH?$AAi?$AAg?$AAh?$AA?9?$AAS?$AAp?$AAe?$AAe?$AAd?$AA?5?$AAP?$AAo?$AAr?$AAt?$AA?5?$AA?$AN?$AA?6?$AA?$AA@ 00016a64     usb_usbfn_mx25_topaz_v1:i_pdd.obj
 0001:00005a90       ??_C@_1BO@GDNLNMNM@?$AA?7?$AA?7?$AAP?$AAo?$AAr?$AAt?$AA?5?$AAR?$AAe?$AAs?$AAe?$AAt?$AA?$AN?$AA?6?$AA?$AA@ 00016a90     usb_usbfn_mx25_topaz_v1:i_pdd.obj
 0001:00005ab0       ??_C@_1BI@BCOEFLFO@?$AA?7?$AA?7?$AAS?$AAu?$AAs?$AAp?$AAe?$AAn?$AAd?$AA?$AN?$AA?6?$AA?$AA@ 00016ab0     usb_usbfn_mx25_topaz_v1:i_pdd.obj
 0001:00005ac8       ??_C@_1CM@LOGLIGHF@?$AA?7?$AA?7?$AAF?$AAo?$AAr?$AAc?$AAe?$AA?5?$AAP?$AAo?$AAr?$AAt?$AA?5?$AAR?$AAe?$AAs?$AAu?$AAm?$AAe?$AA?$AN?$AA?6?$AA?$AA@ 00016ac8     usb_usbfn_mx25_topaz_v1:i_pdd.obj
 0001:00005af4       ??_C@_1DA@IPBKEGAM@?$AA?7?$AA?7?$AAO?$AAv?$AAe?$AAr?$AA?9?$AAc?$AAu?$AAr?$AAr?$AAe?$AAn?$AAt?$AA?5?$AAC?$AAh?$AAa?$AAn?$AAg?$AAe?$AA?$AN?$AA?6?$AA?$AA@ 00016af4     usb_usbfn_mx25_topaz_v1:i_pdd.obj
 0001:00005b24       ??_C@_1DA@IOPAFHGK@?$AA?7?$AA?7?$AAO?$AAv?$AAe?$AAr?$AA?9?$AAc?$AAu?$AAr?$AAr?$AAe?$AAn?$AAt?$AA?5?$AAA?$AAc?$AAt?$AAi?$AAv?$AAe?$AA?$AN?$AA?6?$AA?$AA@ 00016b24     usb_usbfn_mx25_topaz_v1:i_pdd.obj
 0001:00005b54       ??_C@_1DO@IDEEGAC@?$AA?7?$AA?7?$AAP?$AAo?$AAr?$AAt?$AA?5?$AAE?$AAn?$AAa?$AAb?$AAl?$AAe?$AA?1?$AAD?$AAi?$AAs?$AAa?$AAb?$AAl?$AAe?$AA?5?$AAC?$AAh?$AAa?$AAn?$AAg?$AAe?$AA?$AN?$AA?6?$AA?$AA@ 00016b54     usb_usbfn_mx25_topaz_v1:i_pdd.obj
 0001:00005b94       ??_C@_1CC@HIBPLHBD@?$AA?7?$AA?7?$AAP?$AAo?$AAr?$AAt?$AA?5?$AAE?$AAn?$AAa?$AAb?$AAl?$AAe?$AAd?$AA?$AN?$AA?6?$AA?$AA@ 00016b94     usb_usbfn_mx25_topaz_v1:i_pdd.obj
 0001:00005bb8       ??_C@_1EG@CHIFACHN@?$AA?7?$AA?7?$AAC?$AAo?$AAn?$AAn?$AAe?$AAc?$AAt?$AA?5?$AAS?$AAt?$AAa?$AAt?$AAu?$AAs?$AA?5?$AAC?$AAh?$AAa?$AAn?$AAg?$AAe?$AA?3?$AA?5?$AAC?$AAh?$AAa?$AAn?$AAg?$AAe?$AAd@ 00016bb8     usb_usbfn_mx25_topaz_v1:i_pdd.obj
 0001:00005c00       ??_C@_1EK@CIGPBIFB@?$AA?7?$AA?7?$AAC?$AAu?$AAr?$AAr?$AAe?$AAn?$AAt?$AA?5?$AAC?$AAo?$AAn?$AAn?$AAe?$AAc?$AAt?$AA?5?$AAS?$AAt?$AAa?$AAt?$AAu?$AAs?$AA?3?$AA?5?$AAA?$AAt?$AAt?$AAa?$AAc?$AAh@ 00016c00     usb_usbfn_mx25_topaz_v1:i_pdd.obj
 0001:00005c50       ??_C@_1EE@NKEDAIOG@?$AA?7?$AAA?$AAs?$AAy?$AAn?$AAc?$AAh?$AAr?$AAo?$AAn?$AAo?$AAu?$AAs?$AA?5?$AAS?$AAc?$AAh?$AAe?$AAd?$AAu?$AAl?$AAe?$AA?5?$AAS?$AAt?$AAa?$AAt?$AAu?$AAs?$AA?4?$AA?5?$AA?$AN@ 00016c50     usb_usbfn_mx25_topaz_v1:i_pdd.obj
 0001:00005c94       ??_C@_1DM@OLIDMOLB@?$AA?7?$AAP?$AAe?$AAr?$AAi?$AAo?$AAd?$AAi?$AAc?$AA?5?$AAS?$AAc?$AAh?$AAe?$AAd?$AAu?$AAl?$AAe?$AA?5?$AAS?$AAt?$AAa?$AAt?$AAu?$AAs?$AA?4?$AA?5?$AA?$AN?$AA?6?$AA?$AA@ 00016c94     usb_usbfn_mx25_topaz_v1:i_pdd.obj
 0001:00005cd0       ??_C@_1GE@JMEHEIAD@?$AA?7?$AAR?$AAe?$AAc?$AAl?$AAa?$AAm?$AAa?$AAt?$AAi?$AAo?$AAn?$AA?0?$AAO?$AAn?$AAl?$AAy?$AA?5?$AAu?$AAs?$AAe?$AAd?$AA?5?$AAb?$AAy?$AA?5?$AAt?$AAh?$AAe?$AA?5?$AAh?$AAo@ 00016cd0     usb_usbfn_mx25_topaz_v1:i_pdd.obj
 0001:00005d34       ??_C@_1BK@HBEGAPL@?$AA?7?$AAH?$AAC?$AAH?$AAa?$AAI?$AAt?$AAe?$AAd?$AA?5?$AA?$AN?$AA?6?$AA?$AA@ 00016d34     usb_usbfn_mx25_topaz_v1:i_pdd.obj
 0001:00005d50       ??_C@_1CE@IIMNHGIF@?$AA?7?$AAU?$AAL?$AAP?$AAI?$AA?5?$AAI?$AAn?$AAt?$AAe?$AAr?$AAr?$AAu?$AAp?$AAt?$AA?$AN?$AA?6?$AA?$AA@ 00016d50     usb_usbfn_mx25_topaz_v1:i_pdd.obj
 0001:00005d74       ??_C@_1BM@JKFMOBOF@?$AA?7?$AAD?$AAC?$AAS?$AAu?$AAs?$AAp?$AAe?$AAn?$AAd?$AA?5?$AA?$AN?$AA?6?$AA?$AA@ 00016d74     usb_usbfn_mx25_topaz_v1:i_pdd.obj
 0001:00005d90       ??_C@_1CC@ILIGGFI@?$AA?7?$AAS?$AAO?$AAF?$AA?5?$AAR?$AAe?$AAc?$AAe?$AAi?$AAv?$AAe?$AAd?$AA?5?$AA?$AN?$AA?6?$AA?$AA@ 00016d90     usb_usbfn_mx25_topaz_v1:i_pdd.obj
 0001:00005db4       ??_C@_1CO@KLBBIGDH@?$AA?7?$AAU?$AAS?$AAB?$AA?5?$AAR?$AAe?$AAs?$AAe?$AAt?$AA?5?$AAR?$AAe?$AAc?$AAe?$AAi?$AAv?$AAe?$AAd?$AA?5?$AA?$AN?$AA?6?$AA?$AA@ 00016db4     usb_usbfn_mx25_topaz_v1:i_pdd.obj
 0001:00005de4       ??_C@_1DM@GMIDHHHN@?$AA?7?$AAI?$AAn?$AAt?$AAe?$AAr?$AAr?$AAu?$AAp?$AAt?$AA?5?$AAo?$AAn?$AA?5?$AAA?$AAs?$AAy?$AAn?$AAc?$AA?5?$AAA?$AAd?$AAv?$AAa?$AAn?$AAc?$AAe?$AA?$AN?$AA?6?$AA?$AA@ 00016de4     usb_usbfn_mx25_topaz_v1:i_pdd.obj
 0001:00005e20       ??_C@_1CA@OPJKBAE@?$AA?7?$AAS?$AAy?$AAs?$AAt?$AAe?$AAm?$AA?5?$AAE?$AAr?$AAr?$AAo?$AAr?$AA?$AN?$AA?6?$AA?$AA@ 00016e20     usb_usbfn_mx25_topaz_v1:i_pdd.obj
 0001:00005e40       ??_C@_1CO@ONBPMBE@?$AA?7?$AAF?$AAr?$AAa?$AAm?$AAe?$AA?5?$AAL?$AAi?$AAs?$AAt?$AA?5?$AAR?$AAo?$AAl?$AAl?$AAo?$AAv?$AAe?$AAr?$AA?$AN?$AA?6?$AA?$AA@ 00016e40     usb_usbfn_mx25_topaz_v1:i_pdd.obj
 0001:00005e70       ??_C@_1CM@BOJMIELL@?$AA?7?$AAP?$AAo?$AAr?$AAt?$AA?5?$AAC?$AAh?$AAa?$AAn?$AAg?$AAe?$AA?5?$AAD?$AAe?$AAt?$AAe?$AAc?$AAt?$AA?$AN?$AA?6?$AA?$AA@ 00016e70     usb_usbfn_mx25_topaz_v1:i_pdd.obj
 0001:00005ea0       ??_C@_1EG@JNFJCNAA@?$AA?7?$AAU?$AAS?$AAB?$AA?5?$AAE?$AAr?$AAr?$AAo?$AAr?$AA?5?$AAI?$AAn?$AAt?$AAe?$AAr?$AAr?$AAu?$AAp?$AAt?$AA?5?$AA?$CI?$AAU?$AAS?$AAB?$AAE?$AAR?$AAR?$AAI?$AAN?$AAT?$AA?$CJ@ 00016ea0     usb_usbfn_mx25_topaz_v1:i_pdd.obj
 0001:00005ee8       ??_C@_1DE@KHLIMFPA@?$AA?7?$AAU?$AAS?$AAB?$AA?5?$AAI?$AAn?$AAt?$AAe?$AAr?$AAr?$AAu?$AAp?$AAt?$AA?5?$AA?$CI?$AAU?$AAS?$AAB?$AAI?$AAN?$AAT?$AA?$CJ?$AA?$AN?$AA?6?$AA?$AA@ 00016ee8     usb_usbfn_mx25_topaz_v1:i_pdd.obj
 0001:00005f1c       ??_C@_1DG@EIGILMMI@?$AAI?$AAN?$AA?5?$AA?$CF?$AAs?$AA?5?$AAC?$AAo?$AAm?$AAp?$AAl?$AAe?$AAt?$AAe?$AAd?$AA?5?$AAa?$AAt?$AA?5?$AAe?$AAp?$AA?5?$AA?$CF?$AAd?$AA?$AN?$AA?6?$AA?$AA@ 00016f1c     usb_usbfn_mx25_topaz_v1:i_pdd.obj
 0001:00005f58       ??_C@_1FA@KBGDHCDA@?$AAS?$AAe?$AAn?$AAd?$AA?5?$AAe?$AAr?$AAr?$AAo?$AAr?$AA?$DP?$AA?$DP?$AA?5?$AAl?$AAe?$AAn?$AA?$DN?$AA?$CF?$AAx?$AA?0?$AA?5?$AAs?$AAt?$AAa?$AAt?$AAu?$AAs?$AA?$DN?$AA?$CF?$AAx?$AA?0?$AA?5@ 00016f58     usb_usbfn_mx25_topaz_v1:i_pdd.obj
 0001:00005fa8       ??_C@_1EC@ONAPCMHH@?$AAS?$AAt?$AAa?$AAt?$AAu?$AAs?$AA?5?$AAi?$AAs?$AA?5?$AAn?$AAo?$AAt?$AA?5?$AA0?$AA?5?$AAo?$AAn?$AA?5?$AAs?$AAe?$AAn?$AAt?$AA?5?$AA?$CF?$AAx?$AA?5?$AA?$DN?$AA?$CF?$AAx?$AA?$AN?$AA?6@ 00016fa8     usb_usbfn_mx25_topaz_v1:i_pdd.obj
 0001:00005ff0       ??_C@_1GI@DMJOJCJK@?$AAC?$AAh?$AAe?$AAc?$AAk?$AAE?$AAn?$AAd?$AAp?$AAo?$AAi?$AAn?$AAt?$AA?3?$AAS?$AAe?$AAt?$AA?5?$AAA?$AAd?$AAd?$AAr?$AAe?$AAs?$AAs?$AA?3?$AA?5?$AA?$CF?$AAx?$AA?$CI?$AA?$CF?$AAx@ 00016ff0     usb_usbfn_mx25_topaz_v1:i_pdd.obj
 0001:00006058       ??_C@_1FO@LDFIJMJF@?$AAC?$AAh?$AAe?$AAc?$AAk?$AAE?$AAn?$AAd?$AAp?$AAo?$AAi?$AAn?$AAt?$AA?3?$AAE?$AAP?$AA0?$AA?5?$AAO?$AAU?$AAT?$AA?5?$AAN?$AAU?$AAL?$AAL?$AA?5?$AAt?$AAr?$AAa?$AAn?$AAs@ 00017058     usb_usbfn_mx25_topaz_v1:i_pdd.obj
 0001:000060b8       ??_C@_1FG@MIJKNENI@?$AAC?$AAh?$AAe?$AAc?$AAk?$AAE?$AAn?$AAd?$AAp?$AAo?$AAi?$AAn?$AAt?$AA?3?$AAE?$AAP?$AA0?$AA?5?$AAO?$AAU?$AAT?$AA?5?$AA?$CF?$AAd?$AA?5?$AAb?$AAy?$AAt?$AAe?$AAs?$AA?5?$AAc@ 000170b8     usb_usbfn_mx25_topaz_v1:i_pdd.obj
 0001:00006110       ??_C@_1FK@DOJLLFPC@?$AAC?$AAh?$AAe?$AAc?$AAk?$AAE?$AAn?$AAd?$AAp?$AAo?$AAi?$AAn?$AAt?$AA?3?$AAE?$AAP?$AA0?$AA?5?$AAO?$AAU?$AAT?$AA?5?$AA?$CF?$AAd?$AA?5?$AAb?$AAy?$AAt?$AAe?$AAs?$AA?5?$AAn@ 00017110     usb_usbfn_mx25_topaz_v1:i_pdd.obj
 0001:00006170       ??_C@_1GA@IAMKOKAN@?$AA?$CD?$AA?$CD?$AA?$CD?$AA?$CD?$AA?$CD?$AA?5?$AAm?$AAo?$AAr?$AAe?$AA?5?$AAd?$AAa?$AAt?$AAa?$AA?5?$AAt?$AAo?$AA?5?$AAr?$AAe?$AAc?$AAe?$AAi?$AAv?$AAe?$AA?5?$AAo?$AAn?$AA?5?$AAE?$AAP@ 00017170     usb_usbfn_mx25_topaz_v1:i_pdd.obj
 0001:000061d0       ??_C@_1IM@GIGJCFIB@?$AA?$CD?$AA?$CD?$AA?$CD?$AA?$CD?$AA?$CD?$AA?$CD?$AA?$CD?$AA?$CD?$AA?$CD?$AA?$CD?$AA?$CD?$AA?$CD?$AA?$CD?$AA?5?$AAE?$AAN?$AAD?$AAP?$AAT?$AAC?$AAO?$AAM?$AAP?$AAL?$AAE?$AAT?$AAE?$AA?5?$AA?$CF?$AAx?$AA?5?$AAN@ 000171d0     usb_usbfn_mx25_topaz_v1:i_pdd.obj
 0001:00006260       ??_C@_1EG@NDHBBAAH@?$AAO?$AAU?$AAT?$AA?5?$AA?$CF?$AAs?$AA?5?$AAC?$AAo?$AAm?$AAp?$AAl?$AAe?$AAt?$AAe?$AAd?$AA?5?$AAf?$AAo?$AAr?$AA?5?$AAe?$AAn?$AAd?$AAp?$AAo?$AAi?$AAn?$AAt?$AA?5?$AA?$CF?$AAd@ 00017260     usb_usbfn_mx25_topaz_v1:i_pdd.obj
 0001:000062a8       ??_C@_1O@BIOIDBLM@?$AAC?$AAa?$AAn?$AAc?$AAe?$AAl?$AA?$AA@ 000172a8     usb_usbfn_mx25_topaz_v1:i_pdd.obj
 0001:000062b8       ??_C@_1O@PFKKKDLL@?$AAN?$AAo?$AAr?$AAm?$AAa?$AAl?$AA?$AA@ 000172b8     usb_usbfn_mx25_topaz_v1:i_pdd.obj
 0001:000062c8       ??_C@_1EK@JNBLLHDF@?$AAC?$AAh?$AAe?$AAc?$AAk?$AAE?$AAn?$AAd?$AAp?$AAo?$AAi?$AAn?$AAt?$AA?$CI?$AAe?$AAp?$AA?$DN?$AA?$CF?$AAd?$AA?$CJ?$AA?3?$AA?5?$AAB?$AAU?$AAF?$AAF?$AAE?$AAR?$AA_?$AAE?$AAR?$AAR@ 000172c8     usb_usbfn_mx25_topaz_v1:i_pdd.obj
 0001:00006314       ??_C@_1CG@FAGAAPBN@?$AAE?$AAN?$AAD?$AAP?$AAT?$AAC?$AAO?$AAM?$AAP?$AAL?$AAE?$AAT?$AAE?$AA?5?$AA?$CF?$AAx?$AA?$AN?$AA?6?$AA?$AA@ 00017314     usb_usbfn_mx25_topaz_v1:i_pdd.obj
 0001:0000633c       ??_C@_1DO@LDKDDFPP@?$AAS?$AAt?$AAa?$AAt?$AAu?$AAs?$AA?5?$AAi?$AAs?$AA?5?$AAn?$AAo?$AAt?$AA?5?$AA0?$AA?5?$AAo?$AAn?$AA?5?$AAr?$AAe?$AAc?$AAv?$AA?5?$AA?$CF?$AAx?$AA?5?$AA?$DN?$AA?$CF?$AAx?$AA?$AA@ 0001733c     usb_usbfn_mx25_topaz_v1:i_pdd.obj
 0001:00006380       ??_C@_1EO@FDNJCHA@?$AAD?$AAe?$AAv?$AAi?$AAc?$AAe?$AA?5?$AAD?$AAe?$AAt?$AAa?$AAc?$AAh?$AA?0?$AA?5?$AAw?$AAi?$AAt?$AAh?$AA?5?$AAs?$AAu?$AAs?$AAp?$AA?$CI?$AA?$CF?$AAd?$AA?$CJ?$AA?0?$AA?5?$AAi?$AAd@ 00017380     usb_usbfn_mx25_topaz_v1:i_pdd.obj
 0001:000063d0       ??_C@_1BO@PIPKGBKA@?$AA?$CK?$AAt?$AAe?$AAm?$AAp?$AA3?$AA?5?$AA0?$AAx?$AA?$CF?$AAx?$AA?5?$AA?$AN?$AA?6?$AA?$AA@ 000173d0     usb_usbfn_mx25_topaz_v1:i_pdd.obj
 0001:000063f0       ??_C@_1CI@HKDMKLGF@?$AAD?$AAe?$AAt?$AAa?$AAc?$AAh?$AA?3?$AA?5?$AAP?$AAO?$AAR?$AAT?$AAS?$AAC?$AA?5?$AA0?$AAx?$AA?$CF?$AAx?$AA?$AA@ 000173f0     usb_usbfn_mx25_topaz_v1:i_pdd.obj
 0001:00006418       ??_C@_1CK@LPGMAHKL@?$AA?9?$AAU?$AAF?$AAN?$AA_?$AAD?$AAE?$AAT?$AAA?$AAC?$AAH?$AA?5?$AAc?$AAa?$AAl?$AAl?$AAe?$AAd?$AA?$AN?$AA?6?$AA?$AA@ 00017418     usb_usbfn_mx25_topaz_v1:i_pdd.obj
 0001:00006444       ??_C@_1CK@MPBLBBEN@?$AA?$CL?$AAU?$AAF?$AAN?$AA_?$AAD?$AAE?$AAT?$AAA?$AAC?$AAH?$AA?5?$AAc?$AAa?$AAl?$AAl?$AAe?$AAd?$AA?$AN?$AA?6?$AA?$AA@ 00017444     usb_usbfn_mx25_topaz_v1:i_pdd.obj
 0001:00006470       ??_C@_1O@BJIMCIMK@?$AAR?$AAe?$AAs?$AAu?$AAm?$AAe?$AA?$AA@ 00017470     usb_usbfn_mx25_topaz_v1:i_pdd.obj
 0001:00006480       ??_C@_1BC@MHKABCGD@?$AAB?$AAr?$AAe?$AAa?$AAk?$AA?5?$AA?$AN?$AA?6?$AA?$AA@ 00017480     usb_usbfn_mx25_topaz_v1:i_pdd.obj
 0001:00006494       ??_C@_1BE@JNFMNJIM@?$AAI?$AAn?$AAt?$AAr?$AA?3?$AAD?$AAo?$AAn?$AAe?$AA?$AA@ 00017494     usb_usbfn_mx25_topaz_v1:i_pdd.obj
 0001:000064a8       ??_C@_1CC@IFAPINEE@?$AAS?$AAe?$AAt?$AAu?$AAp?$AAE?$AAv?$AAe?$AAn?$AAt?$AA?5?$AA?4?$AA?4?$AA?4?$AA?$AN?$AA?6?$AA?$AA@ 000174a8     usb_usbfn_mx25_topaz_v1:i_pdd.obj
 0001:000064d0       ??_C@_1EE@JAFGGGNF@?$AAI?$AAn?$AAt?$AAr?$AA?3?$AAU?$AAI?$AA?5?$AAS?$AAE?$AAT?$AAU?$AAP?$AAS?$AAT?$AAA?$AAT?$AA?5?$AA?$CF?$AAx?$AA?5?$AAE?$AAN?$AAD?$AAP?$AAT?$AAC?$AAO?$AAM?$AAP?$AA?5?$AA?$CF@ 000174d0     usb_usbfn_mx25_topaz_v1:i_pdd.obj
 0001:00006514       ??_C@_1BC@MCOFDLFC@?$AAI?$AAn?$AAt?$AAr?$AA?3?$AAS?$AAL?$AAI?$AA?$AA@ 00017514     usb_usbfn_mx25_topaz_v1:i_pdd.obj
 0001:00006528       ??_C@_1BO@EGKDOEEI@?$AAI?$AAn?$AAt?$AAr?$AA?3?$AAS?$AAi?$AAg?$AAn?$AAa?$AAl?$AAl?$AAe?$AAd?$AA?$AA@ 00017528     usb_usbfn_mx25_topaz_v1:i_pdd.obj
 0001:00006548       ??_C@_1CA@FFAPNJLP@?$AAP?$AAD?$AAD?$AA?5?$AA?9?$AA?5?$AAS?$AAU?$AAS?$AAP?$AAE?$AAN?$AAD?$AA?$AN?$AA?6?$AA?$AA@ 00017548     usb_usbfn_mx25_topaz_v1:i_pdd.obj
 0001:00006568       ??_C@_1CC@NCLEKMLF@?$AA?5?$AAs?$AAt?$AAa?$AAt?$AAe?$AA?4?$AAP?$AAS?$AAP?$AAD?$AA?5?$AA?$CF?$AAx?$AA?$AN?$AA?6?$AA?$AA@ 00017568     usb_usbfn_mx25_topaz_v1:i_pdd.obj
 0001:0000658c       ??_C@_1CM@GCFNPFKO@?$AA?5?$AAB?$AAS?$AA_?$AAF?$AAU?$AAL?$AAL?$AA_?$AAS?$AAP?$AAE?$AAE?$AAD?$AA?5?$AA?5?$AA?5?$AA?$CF?$AAx?$AA?$AN?$AA?6?$AA?$AA@ 0001758c     usb_usbfn_mx25_topaz_v1:i_pdd.obj
 0001:000065b8       ??_C@_1CM@EIGJNBDN@?$AA?5?$AAB?$AAS?$AA_?$AAH?$AAI?$AAG?$AAH?$AA_?$AAS?$AAP?$AAE?$AAE?$AAD?$AA?5?$AA?5?$AA?5?$AA?$CF?$AAx?$AA?$AN?$AA?6?$AA?$AA@ 000175b8     usb_usbfn_mx25_topaz_v1:i_pdd.obj
 0001:000065e8       ??_C@_1JI@KKCMHPHI@?$AAH?$AAa?$AAn?$AAd?$AAl?$AAe?$AAU?$AAS?$AAB?$AAR?$AAe?$AAs?$AAe?$AAt?$AA?3?$AA?5?$AAN?$AAo?$AAt?$AA?5?$AAs?$AAt?$AAi?$AAl?$AAl?$AA?5?$AAi?$AAn?$AA?5?$AAr?$AAe?$AAs@ 000175e8     usb_usbfn_mx25_topaz_v1:i_pdd.obj
 0001:00006680       ??_C@_1CA@KBLMCKFP@?$AAD?$AAe?$AAv?$AAi?$AAc?$AAe?$AA?5?$AAD?$AAe?$AAt?$AAa?$AAc?$AAh?$AA?$AN?$AA?6?$AA?$AA@ 00017680     usb_usbfn_mx25_topaz_v1:i_pdd.obj
 0001:000066a0       ??_C@_1FO@DFNLJIPA@?$AAU?$AAS?$AAB?$AAC?$AAo?$AAn?$AAt?$AAr?$AAo?$AAl?$AAl?$AAe?$AAr?$AAR?$AAu?$AAn?$AA?$CI?$AA?$CF?$AAd?$AA?$CJ?$AA?3?$AA?5?$AAf?$AAa?$AAi?$AAl?$AAe?$AAd?$AA?5?$AAt?$AAo?$AA?5@ 000176a0     usb_usbfn_mx25_topaz_v1:i_pdd.obj
 0001:00006700       ??_C@_1HI@FMJPDAIJ@?$AAU?$AAS?$AAB?$AAC?$AAo?$AAn?$AAt?$AAr?$AAo?$AAl?$AAl?$AAe?$AAr?$AAR?$AAu?$AAn?$AA?$CI?$AA1?$AA?$CJ?$AA?3?$AA?5?$AAE?$AAR?$AAR?$AAO?$AAR?$AA?5?$AA?$CD?$AA?$CD?$AA?$CD?$AA?$CD?$AA?$CD@ 00017700     usb_usbfn_mx25_topaz_v1:i_pdd.obj
 0001:00006778       ??_C@_1EM@BBPKMFPI@?$AAS?$AAt?$AAo?$AAp?$AA?5?$AAU?$AAS?$AAB?$AA?5?$AAc?$AAo?$AAn?$AAt?$AAr?$AAo?$AAl?$AAl?$AAe?$AAr?$AA?5?$AA?$CI?$AAR?$AAS?$AA?$DN?$AA?$CF?$AAd?$AA?5?$AA?9?$AA?$DO?$AA?5?$AAR?$AAS@ 00017778     usb_usbfn_mx25_topaz_v1:i_pdd.obj
 0001:000067c8       ??_C@_1EO@GGMICPAJ@?$AAS?$AAt?$AAa?$AAr?$AAt?$AA?5?$AAU?$AAS?$AAB?$AA?5?$AAc?$AAo?$AAn?$AAt?$AAr?$AAo?$AAl?$AAl?$AAe?$AAr?$AA?5?$AA?$CI?$AAR?$AAS?$AA?$DN?$AA?$CF?$AAd?$AA?5?$AA?9?$AA?$DO?$AA?5?$AAR@ 000177c8     usb_usbfn_mx25_topaz_v1:i_pdd.obj
 0001:00006818       ??_C@_1IO@CBIPFBFK@?$AA?$CD?$AA?$CD?$AA?$CD?$AA?$CD?$AA?$CD?$AA?$CD?$AA?$CD?$AA?$CD?$AA?$CD?$AA?$CD?$AA?$CD?$AA?$CD?$AA?$CD?$AA?5?$AAP?$AAr?$AAi?$AAm?$AAe?$AA?5?$AAF?$AAa?$AAi?$AAl?$AAe?$AAd?$AA?5?$AAf?$AAo?$AAr?$AA?5?$AAe@ 00017818     usb_usbfn_mx25_topaz_v1:i_pdd.obj
 0001:000068a8       ??_C@_1FO@BKKPAEJB@?$AAI?$AAs?$AAs?$AAu?$AAe?$AAT?$AAr?$AAa?$AAn?$AAs?$AAf?$AAe?$AAr?$AA?5?$AAS?$AAE?$AAT?$AAU?$AAP?$AAS?$AAT?$AAA?$AAT?$AA?5?$AAr?$AAe?$AAc?$AAe?$AAi?$AAv?$AAe?$AAd@ 000178a8     usb_usbfn_mx25_topaz_v1:i_pdd.obj
 0001:00006908       ??_C@_1EK@PGGCKEHJ@?$AAU?$AAf?$AAn?$AAP?$AAd?$AAd?$AA?3?$AA?5?$AAn?$AAe?$AAw?$AA?5?$AAs?$AAe?$AAt?$AAu?$AAp?$AA?5?$AAr?$AAe?$AAq?$AAu?$AAe?$AAs?$AAt?$AA?5?$AAd?$AAe?$AAt?$AAe?$AAc?$AAt@ 00017908     usb_usbfn_mx25_topaz_v1:i_pdd.obj
 0001:00006958       ??_C@_1HI@CDKGKFCF@?$AAE?$AAR?$AAR?$AAO?$AAR?$AA?3?$AA?5?$AAU?$AAf?$AAn?$AAP?$AAd?$AAd?$AA_?$AAI?$AAs?$AAs?$AAu?$AAe?$AAT?$AAr?$AAa?$AAn?$AAs?$AAf?$AAe?$AAr?$AA?3?$AA?5?$AAC?$AAe?$AAC@ 00017958     usb_usbfn_mx25_topaz_v1:i_pdd.obj
 0001:000069d0       ??_C@_1FK@CELBMJI@?$AAU?$AAf?$AAn?$AAP?$AAd?$AAd?$AA?3?$AA?5?$AAP?$AAa?$AAg?$AAe?$AA?5?$AAt?$AAr?$AAa?$AAn?$AAs?$AAl?$AAa?$AAt?$AAi?$AAo?$AAn?$AA?5?$AAf?$AAa?$AAi?$AAl?$AAe?$AAd?$AA?4@ 000179d0     usb_usbfn_mx25_topaz_v1:i_pdd.obj
 0001:00006a30       ??_C@_1HA@DFAMLEOB@?$AAU?$AAf?$AAn?$AAP?$AAd?$AAd?$AA_?$AAI?$AAs?$AAs?$AAu?$AAe?$AAT?$AAr?$AAa?$AAn?$AAs?$AAf?$AAe?$AAr?$AA?3?$AA?5?$AAB?$AAu?$AAf?$AAf?$AAe?$AAr?$AA?5?$AAP?$AAa?$AAg@ 00017a30     usb_usbfn_mx25_topaz_v1:i_pdd.obj
 0001:00006aa0       ??_C@_1KA@JGAAJONG@?$AAU?$AAf?$AAn?$AAP?$AAd?$AAd?$AA_?$AAI?$AAs?$AAs?$AAu?$AAe?$AAT?$AAr?$AAa?$AAn?$AAs?$AAf?$AAe?$AAr?$AA?3?$AA?5?$AAF?$AAa?$AAi?$AAl?$AAe?$AAd?$AA?5?$AAt?$AAo?$AA?5@ 00017aa0     usb_usbfn_mx25_topaz_v1:i_pdd.obj
 0001:00006b40       ??_C@_1HG@OBGGAFFH@?$AAE?$AAR?$AAR?$AAO?$AAR?$AA?3?$AA?5?$AAU?$AAf?$AAn?$AAP?$AAd?$AAd?$AA_?$AAI?$AAs?$AAs?$AAu?$AAe?$AAT?$AAr?$AAa?$AAn?$AAs?$AAf?$AAe?$AAr?$AA?3?$AA?5?$AAC?$AAe?$AAO@ 00017b40     usb_usbfn_mx25_topaz_v1:i_pdd.obj
 0001:00006bb8       ??_C@_1FA@PGOEGLMA@?$AAU?$AAf?$AAn?$AAP?$AAd?$AAd?$AA_?$AAI?$AAs?$AAs?$AAu?$AAe?$AAT?$AAr?$AAa?$AAn?$AAs?$AAf?$AAe?$AAr?$AA?5?$AAf?$AAi?$AAr?$AAs?$AAt?$AA?5?$AAt?$AAi?$AAm?$AAe?$AA?$CI@ 00017bb8     usb_usbfn_mx25_topaz_v1:i_pdd.obj
 0001:00006c08       ??_C@_1JO@PEEOMCDL@?$AAI?$AAs?$AAs?$AAT?$AAr?$AAa?$AAn?$AA?5?$AA?$CI?$AA?$CF?$AAd?$AA?$CJ?$AA?3?$AA?5?$AA?$CF?$AAs?$AA?5?$AA?$CI?$AAp?$AAT?$AAr?$AAa?$AAn?$AAs?$AAf?$AAe?$AAr?$AA?$DN?$AA0?$AAx?$AA?$CF?$AAx@ 00017c08     usb_usbfn_mx25_topaz_v1:i_pdd.obj
 0001:00006ca8       ??_C@_1EA@GOCNCOIC@?$AAI?$AAs?$AAs?$AAu?$AAe?$AAT?$AAr?$AAa?$AAn?$AAs?$AAf?$AAe?$AAr?$AA?3?$AA?5?$AA?$CF?$AAs?$AA?5?$AAw?$AAi?$AAt?$AAh?$AA?5?$AA?$CF?$AAd?$AA?5?$AAb?$AAy?$AAt?$AAe?$AAs?$AA?$AA@ 00017ca8     usb_usbfn_mx25_topaz_v1:i_pdd.obj
 0001:00006ce8       ??_C@_19CIJIHAKK@?$AAN?$AAU?$AAL?$AAL?$AA?$AA@ 00017ce8     usb_usbfn_mx25_topaz_v1:i_pdd.obj
 0001:00006cf4       ??_C@_17HCEMPBGG@?$AAO?$AAU?$AAT?$AA?$AA@ 00017cf4     usb_usbfn_mx25_topaz_v1:i_pdd.obj
 0001:00006cfc       ??_C@_15BNKBCKPG@?$AAI?$AAN?$AA?$AA@ 00017cfc     usb_usbfn_mx25_topaz_v1:i_pdd.obj
 0001:00006d08       ??_C@_1EG@CKENHIMK@?$AAU?$AAs?$AAb?$AAF?$AAn?$AAP?$AAd?$AAd?$AA_?$AAA?$AAb?$AAo?$AAr?$AAt?$AAT?$AAr?$AAa?$AAn?$AAs?$AAf?$AAe?$AAr?$AA?9?$AA?5?$AA?$CI?$AAE?$AAP?$AA?$DN?$AA?5?$AA?$CF?$AAd?$AA?$CJ@ 00017d08     usb_usbfn_mx25_topaz_v1:i_pdd.obj
 0001:00006d50       ??_C@_1FA@PHGGDELL@?$AAA?$AAb?$AAo?$AAr?$AAt?$AA?$CI?$AA?$CF?$AAd?$AA?$CJ?$AA?5?$AAs?$AAk?$AAi?$AAp?$AAp?$AAe?$AAd?$AA?5?$AA?$CI?$AAT?$AAr?$AAa?$AAn?$AA?5?$AA0?$AAx?$AA?$CF?$AAx?$AA?5?$AA?$CB?$AA?$DN?$AA?5@ 00017d50     usb_usbfn_mx25_topaz_v1:i_pdd.obj
 0001:00006da0       ??_C@_1FK@ENKBNDBL@?$AA?$CD?$AA?$CD?$AA?$CD?$AA?$CD?$AA?$CD?$AA?$CD?$AA?$CD?$AA?$CD?$AA?$CD?$AA?$CD?$AA?$CD?$AA?5?$AAA?$AAb?$AAo?$AAr?$AAt?$AAT?$AAr?$AAa?$AAn?$AAs?$AAf?$AAe?$AAr?$AA?$CI?$AA?$CF?$AAd?$AA?$CJ?$AA?5?$AAD?$AAe@ 00017da0     usb_usbfn_mx25_topaz_v1:i_pdd.obj
 0001:00006e00       ??_C@_1GK@BJNDOLBF@?$AAU?$AAs?$AAb?$AAF?$AAn?$AAP?$AAd?$AAd?$AA_?$AAA?$AAb?$AAo?$AAr?$AAt?$AAT?$AAr?$AAa?$AAn?$AAs?$AAf?$AAe?$AAr?$AA?3?$AA?5?$AAp?$AAT?$AAr?$AAa?$AAn?$AAs?$AAf?$AAe@ 00017e00     usb_usbfn_mx25_topaz_v1:i_pdd.obj
 0001:00006e6c       ??_C@_1DA@JMEFNML@?$AAA?$AAb?$AAo?$AAr?$AAt?$AAT?$AAr?$AAa?$AAn?$AAs?$AAf?$AAe?$AAr?$AA?5?$AA?$CI?$AA?$CF?$AAs?$AA?5?$AAE?$AAP?$AA?$CF?$AAd?$AA?$CJ?$AA?$AA@ 00017e6c     usb_usbfn_mx25_topaz_v1:i_pdd.obj
 0001:00006ea0       ??_C@_1EG@BFJDKFHL@?$AAU?$AAs?$AAb?$AAF?$AAn?$AAP?$AAd?$AAd?$AA_?$AAA?$AAb?$AAo?$AAr?$AAt?$AAT?$AAr?$AAa?$AAn?$AAs?$AAf?$AAe?$AAr?$AA?$CL?$AA?5?$AA?$CI?$AAE?$AAP?$AA?$DN?$AA?5?$AA?$CF?$AAd?$AA?$CJ@ 00017ea0     usb_usbfn_mx25_topaz_v1:i_pdd.obj
 0001:00006ee8       ??_C@_1DI@FFFNHHBF@?$AAU?$AAs?$AAb?$AAF?$AAn?$AAP?$AAd?$AAd?$AA_?$AAS?$AAt?$AAa?$AAl?$AAl?$AAE?$AAn?$AAd?$AAp?$AAo?$AAi?$AAn?$AAt?$AA?5?$AA?$CF?$AAd?$AA?$AN?$AA?6?$AA?$AA@ 00017ee8     usb_usbfn_mx25_topaz_v1:i_pdd.obj
 0001:00006f20       ??_C@_1DI@EBJLFADF@?$AAU?$AAs?$AAb?$AAF?$AAn?$AAP?$AAd?$AAd?$AA_?$AAC?$AAl?$AAe?$AAa?$AAr?$AAE?$AAn?$AAd?$AAp?$AAo?$AAi?$AAn?$AAt?$AA?5?$AA?$CF?$AAd?$AA?$AN?$AA?6?$AA?$AA@ 00017f20     usb_usbfn_mx25_topaz_v1:i_pdd.obj
 0001:00006f58       ??_C@_1EA@DIDLDIBI@?$AA?9?$AAU?$AAs?$AAb?$AAF?$AAn?$AAP?$AAd?$AAd?$AA_?$AAI?$AAs?$AAE?$AAn?$AAd?$AAp?$AAo?$AAi?$AAn?$AAt?$AAH?$AAa?$AAl?$AAt?$AAe?$AAd?$AA?5?$AA?$CF?$AAd?$AA?$AN?$AA?6?$AA?$AA@ 00017f58     usb_usbfn_mx25_topaz_v1:i_pdd.obj
 0001:00006f98       ??_C@_1DO@MLIBPKBI@?$AAU?$AAs?$AAb?$AAF?$AAn?$AAP?$AAd?$AAd?$AA_?$AAI?$AAs?$AAE?$AAn?$AAd?$AAp?$AAo?$AAi?$AAn?$AAt?$AAH?$AAa?$AAl?$AAt?$AAe?$AAd?$AA?5?$AA?$CF?$AAd?$AA?$AN?$AA?6?$AA?$AA@ 00017f98     usb_usbfn_mx25_topaz_v1:i_pdd.obj
 0001:00006fd8       ??_C@_1CA@HMLLGPGC@?$AA?9?$AAS?$AAe?$AAn?$AAd?$AAC?$AAS?$AAH?$AA?5?$AA?$CI?$AAE?$AAP?$AA?$CF?$AAd?$AA?$CJ?$AA?$AA@ 00017fd8     usb_usbfn_mx25_topaz_v1:i_pdd.obj
 0001:00006ff8       ??_C@_1CE@MAHEKDJP@?$AAS?$AAe?$AAn?$AAd?$AAC?$AAS?$AAH?$AA?5?$AAI?$AAN?$AA?5?$AA?$CI?$AA?$CF?$AAd?$AA?$CJ?$AA?$AN?$AA?6?$AA?$AA@ 00017ff8     usb_usbfn_mx25_topaz_v1:i_pdd.obj
 0001:0000701c       ??_C@_1CG@NAGMKJIL@?$AAS?$AAe?$AAn?$AAd?$AAC?$AAS?$AAH?$AA?5?$AAO?$AAU?$AAT?$AA?5?$AA?$CI?$AA?$CF?$AAd?$AA?$CJ?$AA?$AN?$AA?6?$AA?$AA@ 0001801c     usb_usbfn_mx25_topaz_v1:i_pdd.obj
 0001:00007044       ??_C@_1CA@DFPEHIFN@?$AA?$CL?$AAS?$AAe?$AAn?$AAd?$AAC?$AAS?$AAH?$AA?5?$AA?$CI?$AAE?$AAP?$AA?$CF?$AAd?$AA?$CJ?$AA?$AA@ 00018044     usb_usbfn_mx25_topaz_v1:i_pdd.obj
 0001:00007068       ??_C@_1FM@FGGEPKIB@?$AA?$CD?$AA?$CD?$AA?$CD?$AA?$CD?$AA?$CD?$AA?$CD?$AA?$CD?$AA?$CD?$AA?$CD?$AA?$CD?$AA?$CD?$AA?$CD?$AA?$CD?$AA?$CD?$AA?$CD?$AA?$CD?$AA?5?$AAF?$AAa?$AAi?$AAl?$AAe?$AAd?$AA?5?$AAt?$AAo?$AA?5?$AAp?$AAr?$AAi?$AAm?$AAe@ 00018068     usb_usbfn_mx25_topaz_v1:i_pdd.obj
 0001:000070c8       ??_C@_1EG@KGILPPEC@?$AAC?$AAa?$AAn?$AA?5?$AAn?$AAo?$AAt?$AA?5?$AAp?$AAr?$AAi?$AAm?$AAe?$AA?5?$AAf?$AAo?$AAr?$AA?5?$AAZ?$AAL?$AAT?$AA?5?$AA?$CI?$AA?$CF?$AAs?$AA?$CJ?$AA?3?$AA?5?$AAb?$AAu?$AAs?$AAy@ 000180c8     usb_usbfn_mx25_topaz_v1:i_pdd.obj
 0001:00007110       ??_C@_1BM@LGGJJGMB@?$AAP?$AAr?$AAi?$AAm?$AAe?$AAF?$AAZ?$AAL?$AAT?$AA?3?$AA?5?$AA?$CF?$AAs?$AA?$AA@ 00018110     usb_usbfn_mx25_topaz_v1:i_pdd.obj
 0001:00007130       ??_C@_1EA@KNMJPPBI@?$AAU?$AAs?$AAb?$AAF?$AAn?$AAP?$AAd?$AAd?$AA_?$AAI?$AAn?$AAi?$AAt?$AAi?$AAa?$AAt?$AAe?$AAR?$AAe?$AAm?$AAo?$AAt?$AAe?$AAW?$AAa?$AAk?$AAe?$AAu?$AAp?$AA?$AN?$AA?6?$AA?$AA@ 00018130     usb_usbfn_mx25_topaz_v1:i_pdd.obj
 0001:00007170       ??_C@_1CO@LFIHBCKN@?$AAS?$AAe?$AAt?$AAP?$AAo?$AAw?$AAe?$AAr?$AAS?$AAt?$AAa?$AAt?$AAe?$AA?5?$AA?$DN?$AA?5?$AA0?$AAx?$AA?$CF?$AAx?$AA?$AN?$AA?6?$AA?$AA@ 00018170     usb_usbfn_mx25_topaz_v1:i_pdd.obj
 0001:000071a0       ??_C@_1HC@FEAKGGLP@?$AAP?$AAD?$AAD?$AA?3?$AA?5?$AAS?$AAe?$AAt?$AA?5?$AAF?$AAe?$AAa?$AAt?$AAu?$AAr?$AAe?$AA?5?$AA?$CI?$AAT?$AAE?$AAS?$AAT?$AA?5?$AAM?$AAO?$AAD?$AAE?$AA?$CJ?$AA?5?$AAO?$AAT?$AAG@ 000181a0     usb_usbfn_mx25_topaz_v1:i_pdd.obj
 0001:00007218       ??_C@_1HC@GBFNHNAG@?$AAI?$AAO?$AAC?$AAT?$AAL?$AA_?$AAB?$AAU?$AAS?$AA_?$AAS?$AAE?$AAT?$AA_?$AAP?$AAO?$AAW?$AAE?$AAR?$AA_?$AAS?$AAT?$AAA?$AAT?$AAE?$AA?3?$AA?5?$AAC?$AAe?$AAO?$AAp?$AAe@ 00018218     usb_usbfn_mx25_topaz_v1:i_pdd.obj
 0001:00007290       ??_C@_1HE@NONILAAF@?$AAI?$AAO?$AAC?$AAT?$AAL?$AA_?$AAB?$AAU?$AAS?$AA_?$AAS?$AAE?$AAT?$AA_?$AAP?$AAO?$AAW?$AAE?$AAR?$AA_?$AAS?$AAT?$AAA?$AAT?$AAE?$AA?3?$AA?5?$AAC?$AAe?$AAC?$AAl?$AAo@ 00018290     usb_usbfn_mx25_topaz_v1:i_pdd.obj
 0001:00007308       ??_C@_1EG@GJIKGHF@?$AAI?$AAO?$AAC?$AAT?$AAL?$AA_?$AAB?$AAU?$AAS?$AA_?$AAS?$AAE?$AAT?$AA_?$AAP?$AAO?$AAW?$AAE?$AAR?$AA_?$AAS?$AAT?$AAA?$AAT?$AAE?$AA?5?$AAc?$AAa?$AAl?$AAl?$AAe?$AAd@ 00018308     usb_usbfn_mx25_topaz_v1:i_pdd.obj
 0001:00007350       ??_C@_1HC@NPNGJCMK@?$AAI?$AAO?$AAC?$AAT?$AAL?$AA_?$AAB?$AAU?$AAS?$AA_?$AAG?$AAE?$AAT?$AA_?$AAP?$AAO?$AAW?$AAE?$AAR?$AA_?$AAS?$AAT?$AAA?$AAT?$AAE?$AA?3?$AA?5?$AAC?$AAe?$AAO?$AAp?$AAe@ 00018350     usb_usbfn_mx25_topaz_v1:i_pdd.obj
 0001:000073c8       ??_C@_1HE@IJCCGJCF@?$AAI?$AAO?$AAC?$AAT?$AAL?$AA_?$AAB?$AAU?$AAS?$AA_?$AAG?$AAE?$AAT?$AA_?$AAP?$AAO?$AAW?$AAE?$AAR?$AA_?$AAS?$AAT?$AAA?$AAT?$AAE?$AA?3?$AA?5?$AAC?$AAe?$AAC?$AAl?$AAo@ 000183c8     usb_usbfn_mx25_topaz_v1:i_pdd.obj
 0001:00007440       ??_C@_1EG@FFODHJCP@?$AAI?$AAO?$AAC?$AAT?$AAL?$AA_?$AAB?$AAU?$AAS?$AA_?$AAG?$AAE?$AAT?$AA_?$AAP?$AAO?$AAW?$AAE?$AAR?$AA_?$AAS?$AAT?$AAA?$AAT?$AAE?$AA?5?$AAc?$AAa?$AAl?$AAl?$AAe?$AAd@ 00018440     usb_usbfn_mx25_topaz_v1:i_pdd.obj
 0001:00007488       ??_C@_1BM@ELBPNMDN@?$AAU?$AAf?$AAn?$AAP?$AAd?$AAd?$AA_?$AAS?$AAt?$AAo?$AAp?$AA?$AN?$AA?6?$AA?$AA@ 00018488     usb_usbfn_mx25_topaz_v1:i_pdd.obj
 0001:000074a4       ??_C@_1DK@CCAICBIP@?$AA?$CL?$AAU?$AAf?$AAn?$AAP?$AAd?$AAd?$AA_?$AAD?$AAe?$AAi?$AAn?$AAi?$AAt?$AAE?$AAn?$AAd?$AAp?$AAo?$AAi?$AAn?$AAt?$AA?3?$AA?5?$AA?$CF?$AAd?$AA?$AN?$AA?6?$AA?$AA@ 000184a4     usb_usbfn_mx25_topaz_v1:i_pdd.obj
 0001:000074e0       ??_C@_1DK@MHIAFBPJ@?$AAI?$AAn?$AAi?$AAt?$AA?5?$AAE?$AAn?$AAd?$AAp?$AAo?$AAi?$AAn?$AAt?$AA?3?$AA?5?$AA?$CF?$AAx?$AA?0?$AA?5?$AAc?$AAt?$AAr?$AAl?$AA?$DN?$AA?$CF?$AAx?$AA?$AN?$AA?6?$AA?$AA@ 000184e0     usb_usbfn_mx25_topaz_v1:i_pdd.obj
 0001:00007520       ??_C@_1EK@HMBFBNAN@?$AAU?$AAf?$AAn?$AAP?$AAd?$AAd?$AA_?$AAI?$AAn?$AAi?$AAt?$AAE?$AAn?$AAd?$AAp?$AAo?$AAi?$AAn?$AAt?$AA?3?$AA?5?$AA?$CF?$AAd?$AA?5?$AAA?$AAt?$AAt?$AAr?$AAi?$AAb?$AA?$CI?$AA?$CF@ 00018520     usb_usbfn_mx25_topaz_v1:i_pdd.obj
 0001:0000756c       ??_C@_1CA@IJBGFJAE@?$AA?9?$AAU?$AAf?$AAn?$AAP?$AAd?$AAd?$AA_?$AAS?$AAt?$AAa?$AAr?$AAt?$AA?$AN?$AA?6?$AA?$AA@ 0001856c     usb_usbfn_mx25_topaz_v1:i_pdd.obj
 0001:0000758c       ??_C@_1CA@MAFJEODL@?$AA?$CL?$AAU?$AAf?$AAn?$AAP?$AAd?$AAd?$AA_?$AAS?$AAt?$AAa?$AAr?$AAt?$AA?$AN?$AA?6?$AA?$AA@ 0001858c     usb_usbfn_mx25_topaz_v1:i_pdd.obj
 0001:000075ac       ??_C@_1DG@EEIHMJOF@?$AAS?$AAt?$AAa?$AAt?$AAu?$AAs?$AA?5?$AAf?$AAo?$AAr?$AA?5?$AAt?$AAd?$AA0?$AA?$DN?$AA?$CF?$AAx?$AA?0?$AA?5?$AAt?$AAb?$AA?$DN?$AA?$CF?$AAx?$AA?$AN?$AA?6?$AA?$AA@ 000185ac     usb_usbfn_mx25_topaz_v1:i_pdd.obj
 0001:000075e4       ??_C@_1CM@FGGAHLIL@?$AAP?$AAR?$AAI?$AAM?$AAE?$AA?5?$AAf?$AAa?$AAi?$AAl?$AAe?$AAd?$AA?5?$AAo?$AAn?$AA?5?$AAE?$AAP?$AA0?$AA?$AN?$AA?6?$AA?$AA@ 000185e4     usb_usbfn_mx25_topaz_v1:i_pdd.obj
 0001:00007610       ??_C@_1FC@FLIFOJB@?$AAN?$AAe?$AAw?$AA?5?$AAs?$AAe?$AAt?$AAu?$AAp?$AA?5?$AAr?$AAe?$AAc?$AAe?$AAi?$AAv?$AAe?$AAd?$AA?5?$AAw?$AAh?$AAe?$AAn?$AA?5?$AAp?$AAr?$AAi?$AAm?$AAi?$AAn?$AAg?$AA?$DN@ 00018610     usb_usbfn_mx25_topaz_v1:i_pdd.obj
 0001:00007668       ??_C@_1GC@FCEGAELL@?$AAS?$AAe?$AAt?$AAu?$AAp?$AA?5?$AAn?$AAo?$AAt?$AA?5?$AAp?$AAr?$AAo?$AAc?$AAe?$AAs?$AAs?$AAe?$AAd?$AA?5?$AA?$CI?$AAS?$AAE?$AAT?$AAU?$AAP?$AAS?$AAT?$AAA?$AAT?$AA?$DN?$AA0@ 00018668     usb_usbfn_mx25_topaz_v1:i_pdd.obj
 0001:000076cc       ??_C@_1BI@DKIPBNLN@?$AAI?$AAn?$AAi?$AAt?$AAq?$AAh?$AA0?$AA?0?$AA?5?$AA?$CF?$AAx?$AA?$AA@ 000186cc     usb_usbfn_mx25_topaz_v1:i_pdd.obj
 0001:000076e4       ??_C@_1BK@PALAPBNH@?$AA?4?$AA?4?$AAc?$AAo?$AAu?$AAn?$AAt?$AA?5?$AA?$CF?$AAd?$AA?$AN?$AA?6?$AA?$AA@ 000186e4     usb_usbfn_mx25_topaz_v1:i_pdd.obj
 0001:00007700       ??_C@_1HA@BIGHAGHK@?$AAD?$AAi?$AAs?$AAa?$AAb?$AAl?$AAe?$AA?5?$AAI?$AAn?$AAt?$AAe?$AAr?$AAr?$AAu?$AAp?$AAt?$AA?5?$AAa?$AAn?$AAd?$AA?5?$AAl?$AAe?$AAt?$AA?5?$AAt?$AAh?$AAe?$AA?5?$AAT?$AAr@ 00018700     usb_usbfn_mx25_topaz_v1:i_pdd.obj
 0001:00007770       ??_C@_1DC@LGPAELOO@?$AAS?$AAi?$AAz?$AAe?$AAo?$AAf?$AA?5?$AAq?$AAh?$AAb?$AAu?$AAf?$AAf?$AAe?$AAr?$AA?5?$AA?$DN?$AA?5?$AA0?$AAx?$AA?$CF?$AAx?$AA?$AN?$AA?6?$AA?$AA@ 00018770     usb_usbfn_mx25_topaz_v1:i_pdd.obj
 0001:000077a8       ??_C@_1HE@JFIJHLAK@?$AAE?$AAR?$AAR?$AAO?$AAR?$AA?3?$AA?5?$AAU?$AAf?$AAn?$AAP?$AAd?$AAd?$AA_?$AAI?$AAn?$AAi?$AAt?$AA?3?$AA?5?$AAC?$AAo?$AAn?$AAt?$AAr?$AAo?$AAl?$AAl?$AAe?$AAr?$AA?5?$AAr@ 000187a8     usb_usbfn_mx25_topaz_v1:i_pdd.obj
 0001:00007820       ??_C@_1FK@EMBOCJKF@?$AAE?$AAR?$AAR?$AAO?$AAR?$AA?3?$AA?5?$AAU?$AAf?$AAn?$AAP?$AAd?$AAd?$AA_?$AAI?$AAn?$AAi?$AAt?$AA?3?$AA?5?$AAF?$AAa?$AAi?$AAl?$AAe?$AAd?$AA?5?$AAo?$AAp?$AAe?$AAn?$AA?5@ 00018820     usb_usbfn_mx25_topaz_v1:i_pdd.obj
 0001:00007880       ??_C@_1GM@LIECJJPD@?$AAE?$AAR?$AAR?$AAO?$AAR?$AA?3?$AA?5?$AAU?$AAf?$AAn?$AAP?$AAd?$AAd?$AA_?$AAI?$AAn?$AAi?$AAt?$AA?3?$AA?5?$AAF?$AAa?$AAi?$AAl?$AAe?$AAd?$AA?5?$AAr?$AAe?$AAa?$AAd?$AA?5@ 00018880     usb_usbfn_mx25_topaz_v1:i_pdd.obj
 0001:000078f0       ??_C@_1EG@BDFMMKKK@?$AAU?$AAf?$AAn?$AAP?$AAd?$AAd?$AA_?$AAI?$AAn?$AAi?$AAt?$AA?5?$AAp?$AAP?$AAd?$AAd?$AA?5?$AAa?$AAl?$AAl?$AAo?$AAc?$AAa?$AAt?$AAe?$AA?5?$AAf?$AAa?$AAi?$AAl?$AAe?$AAd@ 000188f0     usb_usbfn_mx25_topaz_v1:i_pdd.obj
 0001:00007938       ??_C@_1GG@IILKAMAB@?$AAU?$AAS?$AAB?$AA?5?$AAD?$AAr?$AAi?$AAv?$AAe?$AAr?$AA?5?$AAl?$AAo?$AAa?$AAd?$AA?5?$AAf?$AAa?$AAi?$AAl?$AAu?$AAr?$AAe?$AA?5?$AAb?$AAe?$AAc?$AAa?$AAu?$AAs?$AAe?$AA?5@ 00018938     usb_usbfn_mx25_topaz_v1:i_pdd.obj
 0001:000079a4       ??_C@_0CJ@CHGIGMLG@received?5non?9download?5packet?5typ@ 000189a4     oal_blserial:serfuncs.obj
 0001:000079d0       ??_C@_0BE@KEIPDPMM@Expected?5block?5?$CFu?$AN?6?$AA@ 000189d0     oal_blserial:serfuncs.obj
 0001:000079e4       ??_C@_0CE@HOCBBCP@Received?5out?5of?5sequence?5block?5?$CF@ 000189e4     oal_blserial:serfuncs.obj
 0001:00007a08       ??_C@_0BK@IPKIMKPH@Waiting?5for?5boot?5ack?4?4?4?$AN?6?$AA@ 00018a08     oal_blserial:serfuncs.obj
 0001:00007a24       ??_C@_0CK@DMEOPGMB@Got?5jump?5request?0?5KITL?5transport@ 00018a24     oal_blserial:serfuncs.obj
 0001:00007a50       ??_C@_0DG@MLEBFPEB@data?5checksum?5failure?4?5expected?5@ 00018a50     oal_blserial:serfuncs.obj
 0001:00007a88       ??_C@_0BN@FEFEJPIP@failed?5to?5read?5packet?5data?$AN?6?$AA@ 00018a88     oal_blserial:serfuncs.obj
 0001:00007aa8       ??_C@_0CM@DECDFMCF@insufficient?5buffer?5size?$DL?5ignori@ 00018aa8     oal_blserial:serfuncs.obj
 0001:00007ad4       ??_C@_0BL@MMGBDAGN@failed?5to?5receive?5header?$AN?6?$AA@ 00018ad4     oal_blserial:serfuncs.obj
 0001:00007af0       ??_C@_0BH@MJPKDDID@header?5checksum?5fail?$AN?6?$AA@ 00018af0     oal_blserial:serfuncs.obj
 0001:00007b08       ??_C@_0CA@LIHOEDHI@failed?5to?5receive?5header?5data?$AN?6?$AA@ 00018b08     oal_blserial:serfuncs.obj
 0001:00007b28       ??_C@_0CF@PODCGAIM@failed?5to?5receive?5header?5signatu@ 00018b28     oal_blserial:serfuncs.obj
 0001:00007b50       ??_C@_0CC@BCDLLINN@Host?5sent?5unhandled?5request?5type@ 00018b50     fsl_serial_pdd_common_topaz_v1:serial_dl.obj
 0001:00007b78       ??_C@_1MO@BCLNICFM@?$AAc?$AA?3?$AA?2?$AAw?$AAi?$AAn?$AAc?$AAe?$AAr?$AAo?$AAo?$AAt?$AAs?$AA?2?$AAt?$AAo?$AAp?$AAa?$AAz?$AA?2?$AAw?$AAi?$AAn?$AAc?$AAe?$AA7?$AA0?$AA0?$AA?2?$AAp?$AAl?$AAa@ 00018b78     fsl_serial_pdd_common_topaz_v1:serial_dl.obj
 0001:00007c48       ??_C@_0DA@KIPOMLGH@Host?5indicated?5an?5unsupported?5SE@ 00018c48     fsl_serial_pdd_common_topaz_v1:serial_dl.obj
 0001:00007c78       ??_C@_0BP@ONENEGJJ@Unhandled?5Get?5DESCRIPTOR_TYPE?$CB?$AA@ 00018c78     fsl_serial_pdd_common_topaz_v1:serial_dl.obj
 0001:00007c98       ??_C@_0CG@MDLKJKHE@PDD?5Signaled?5bogus?5transfer?5comp@ 00018c98     fsl_serial_pdd_common_topaz_v1:serial_dl.obj
 0001:00007cc0       ??_C@_0CN@LOCOBGOP@Endpoint?52?5has?5entered?5an?5unsupp@ 00018cc0     fsl_serial_pdd_common_topaz_v1:serial_dl.obj
 0001:00007cf0       ??_C@_1IK@NBNIIDPB@?$AAE?$AAR?$AAR?$AAO?$AAR?$AA?3?$AA?5?$AAP?$AAD?$AAD?$AA?5?$AAI?$AAn?$AAd?$AAi?$AAc?$AAa?$AAt?$AAe?$AAd?$AA?5?$AAt?$AAh?$AAe?$AAr?$AAe?$AA?5?$AAw?$AAa?$AAs?$AA?5?$AAa@ 00018cf0     fsl_serial_pdd_common_topaz_v1:serial_dl.obj
 0001:00007d80       ??_C@_1HE@HCMHOHD@?$AAE?$AAR?$AAR?$AAO?$AAR?$AA?3?$AA?5?$AAP?$AAD?$AAD?$AA?5?$AAI?$AAn?$AAd?$AAi?$AAc?$AAa?$AAt?$AAe?$AAd?$AA?5?$AAt?$AAh?$AAe?$AAr?$AAe?$AA?5?$AAw?$AAa?$AAs?$AA?5?$AAa@ 00018d80     fsl_serial_pdd_common_topaz_v1:serial_dl.obj
 0001:00007df8       ??_C@_1GC@EHFCFLNO@?$AAE?$AAR?$AAR?$AAO?$AAR?$AA?3?$AA?5?$AAS?$AAe?$AAn?$AAt?$AA?5?$AAd?$AAa?$AAt?$AAa?$AA?5?$AAd?$AAo?$AAe?$AAs?$AA?5?$AAn?$AAo?$AAt?$AA?5?$AAm?$AAa?$AAt?$AAc?$AAh?$AA?5@ 00018df8     fsl_serial_pdd_common_topaz_v1:serial_dl.obj
 0001:00007e60       ??_C@_1JG@LFGGGOHE@?$AAE?$AAR?$AAR?$AAO?$AAR?$AA?3?$AA?5?$AAP?$AAD?$AAD?$AA?5?$AAI?$AAn?$AAd?$AAi?$AAc?$AAa?$AAt?$AAe?$AAd?$AA?5?$AAR?$AAE?$AAC?$AAV?$AA?5?$AAc?$AAo?$AAm?$AAp?$AAl?$AAe@ 00018e60     fsl_serial_pdd_common_topaz_v1:serial_dl.obj
 0001:00007ef8       ??_C@_1HE@OMBLMFHA@?$AAE?$AAR?$AAR?$AAO?$AAR?$AA?3?$AA?5?$AAP?$AAD?$AAD?$AA?5?$AAI?$AAn?$AAd?$AAi?$AAc?$AAa?$AAt?$AAe?$AAd?$AA?5?$AAt?$AAh?$AAe?$AAr?$AAe?$AA?5?$AAw?$AAa?$AAs?$AA?5?$AAa@ 00018ef8     fsl_serial_pdd_common_topaz_v1:serial_dl.obj
 0001:00007f6c       ??_C@_1CI@OLENNHLD@?$AAU?$AAf?$AAn?$AAP?$AAd?$AAd?$AA_?$AAI?$AAn?$AAi?$AAt?$AA?5?$AAf?$AAa?$AAi?$AAl?$AAe?$AAd?$AA?$CB?$AA?$AA@ 00018f6c     fsl_serial_pdd_common_topaz_v1:serial_dl.obj
 0001:00007f98       ??_C@_1HG@HALKJNKP@?$AAE?$AAR?$AAR?$AAO?$AAR?$AA?3?$AA?5?$AAU?$AAS?$AAB?$AAS?$AAe?$AAr?$AAi?$AAa?$AAl?$AAI?$AAn?$AAi?$AAt?$AA?5?$AAc?$AAa?$AAl?$AAl?$AAe?$AAd?$AA?5?$AAa?$AAg?$AAa?$AAi@ 00018f98     fsl_serial_pdd_common_topaz_v1:serial_dl.obj
 0001:00008010       ??_C@_1GA@DBGLAADC@?$AAE?$AAR?$AAR?$AAO?$AAR?$AA?3?$AA?5?$AAP?$AAD?$AAD?$AA?5?$AAc?$AAa?$AAn?$AAn?$AAo?$AAt?$AA?5?$AAs?$AAu?$AAp?$AAp?$AAo?$AAr?$AAt?$AA?5?$AAl?$AAo?$AAg?$AAi?$AAc?$AAa@ 00019010     fsl_serial_pdd_common_topaz_v1:serial_dl.obj
 0001:00008070       ??_C@_1CG@HDEJOBAB@?$AAM?$AAa?$AAp?$AAp?$AAi?$AAn?$AAg?$AA?5?$AA?$CF?$AAd?$AA?5?$AAt?$AAo?$AA?5?$AA?$CF?$AAd?$AA?$AN?$AA?6?$AA?$AA@ 00019070     fsl_serial_pdd_common_topaz_v1:serial_dl.obj
 0001:00008098       ??_C@_1EO@JLDEGKNA@?$AAE?$AAR?$AAR?$AAO?$AAR?$AA?3?$AA?5?$AAP?$AAD?$AAD?$AA?5?$AAc?$AAa?$AAn?$AAn?$AAo?$AAt?$AA?5?$AAs?$AAu?$AAp?$AAp?$AAo?$AAr?$AAt?$AA?5?$AAe?$AAn?$AAd?$AAp?$AAo?$AAi@ 00019098     fsl_serial_pdd_common_topaz_v1:serial_dl.obj
 0001:000080e8       ??_C@_0CJ@BBDJGCGB@Unexpected?5Msg?5in?5HandlePDDNotif@ 000190e8     fsl_serial_pdd_common_topaz_v1:serial_dl.obj
 0001:00008114       ??_C@_1CO@ONOPPKFD@?$AAG?$AAo?$AAt?$AA?5?$AAS?$AAE?$AAT?$AAU?$AAP?$AA?5?$AAO?$AAU?$AAT?$AA?5?$AAp?$AAa?$AAc?$AAk?$AAe?$AAt?$AA?$AN?$AA?6?$AA?$AA@ 00019114     fsl_serial_pdd_common_topaz_v1:serial_dl.obj
 0001:00008144       ??_C@_0CI@BHALHJPB@Only?5GET_DESC?5and?5SET_CONFIG?5sup@ 00019144     fsl_serial_pdd_common_topaz_v1:serial_dl.obj
 0001:00008170       ??_C@_1GM@JEDJFMFC@?$AAE?$AAR?$AAR?$AAO?$AAR?$AA?3?$AA?5?$AAO?$AAE?$AAM?$AAS?$AAe?$AAr?$AAi?$AAa?$AAl?$AAS?$AAe?$AAn?$AAd?$AAR?$AAa?$AAw?$AA?5?$AAc?$AAa?$AAl?$AAl?$AAe?$AAd?$AA?5?$AAb@ 00019170     fsl_serial_pdd_common_topaz_v1:serial_dl.obj
 0001:000081dc       ??_C@_0DB@LKOJLGG@Serial?5Wrapper?5Circular?5Buffer?5O@ 000191dc     fsl_serial_pdd_common_topaz_v1:serial_dl.obj
 0001:00008210       ??_C@_0EA@FIJCBODK@Amount?5of?5transferred?5data?5in?5DW@ 00019210     fsl_serial_pdd_common_topaz_v1:serial_dl.obj
 0001:00008250       ??_C@_1DO@JIIKDGOP@?$AAE?$AAx?$AAi?$AAt?$AAi?$AAn?$AAg?$AA?5?$AAO?$AAE?$AAM?$AAS?$AAe?$AAr?$AAi?$AAa?$AAl?$AAR?$AAe?$AAc?$AAv?$AAR?$AAa?$AAw?$AA?4?$AA?4?$AA?4?$AA?4?$AA?$AN?$AA?6?$AA?$AA@ 00019250     fsl_serial_pdd_common_topaz_v1:serial_dl.obj
 0001:00008290       ??_C@_1HA@FEDIMNNJ@?$AAM?$AAu?$AAs?$AAt?$AA?5?$AAi?$AAn?$AAc?$AAr?$AAe?$AAa?$AAs?$AAe?$AA?5?$AAR?$AAE?$AAC?$AAV?$AA_?$AAB?$AAU?$AAF?$AAF?$AAE?$AAR?$AA_?$AAS?$AAI?$AAZ?$AAE?$AA?5?$AAt@ 00019290     fsl_serial_pdd_common_topaz_v1:serial_dl.obj
 0001:00008300       ??_C@_1GO@BNOBJNLF@?$AAE?$AAR?$AAR?$AAO?$AAR?$AA?3?$AA?5?$AAO?$AAE?$AAM?$AAS?$AAe?$AAr?$AAi?$AAa?$AAl?$AAR?$AAe?$AAc?$AAv?$AAR?$AAa?$AAw?$AA?5?$AAc?$AAa?$AAl?$AAl?$AAe?$AAr?$AA?5?$AAa@ 00019300     fsl_serial_pdd_common_topaz_v1:serial_dl.obj
 0001:00008370       ??_C@_1GM@DFDLJAKN@?$AAE?$AAR?$AAR?$AAO?$AAR?$AA?3?$AA?5?$AAO?$AAE?$AAM?$AAS?$AAe?$AAr?$AAi?$AAa?$AAl?$AAR?$AAe?$AAc?$AAv?$AAR?$AAa?$AAw?$AA?5?$AAc?$AAa?$AAl?$AAl?$AAe?$AAd?$AA?5?$AAb@ 00019370     fsl_serial_pdd_common_topaz_v1:serial_dl.obj
 0001:000083dc       ??_C@_0DG@ODLBGEPM@ERROR?3?5OEMSerialRecvRaw?5called?5b@ 000193dc     fsl_serial_pdd_common_topaz_v1:serial_dl.obj
 0001:00008414       ??_C@_0CM@FEMLNPOM@ERROR?3?5Unable?5to?5set?5block?5statu@ 00019414     nand_boot_common_topaz_v1:nandboot.obj
 0001:00008440       ??_C@_0DC@FINGMGAN@ERROR?3?5Unable?5to?5erase?5NAND?5flas@ 00019440     nand_boot_common_topaz_v1:nandboot.obj
 0001:00008474       ??_C@_0CL@JNFABMJO@INFO?3?5Found?5bad?5NAND?5flash?5block@ 00019474     nand_boot_common_topaz_v1:nandboot.obj
 0001:000084a0       ??_C@_0BN@PPPNLHLF@WARNING?3?5NANDBootInit?5fail?$AN?6?$AA@ 000194a0     nand_boot_common_topaz_v1:nandboot.obj
 0001:000084c0       ??_C@_0CP@MEMGALMB@ERROR?3?5Unable?5to?5get?5NAND?5flash?5@ 000194c0     nand_boot_common_topaz_v1:nandboot.obj
 0001:000084f0       ??_C@_0BO@PPFGHOP@ERROR?3?5Failed?5to?5verify?5NK?4?$AN?6?$AA@ 000194f0     nand_boot_common_topaz_v1:nandboot.obj
 0001:00008510       ??_C@_0DC@BCKCJKFP@WARNING?3?5Failed?5to?5write?5XLDR?5in@ 00019510     nand_boot_common_topaz_v1:nandboot.obj
 0001:00008544       ??_C@_0DG@BACIOMAB@Error?3?5No?5good?5block?5found?5?9?5una@ 00019544     nand_boot_common_topaz_v1:nandboot.obj
 0001:0000857c       ??_C@_0DO@KAJJOHBJ@ERROR?3?5XLDR?5size?5exceeds?5reserve@ 0001957c     nand_boot_common_topaz_v1:nandboot.obj
 0001:000085bc       ??_C@_0DE@DHNKGOFC@INFO?3?5Writing?5XLDR?5image?5to?5NAND@ 000195bc     nand_boot_common_topaz_v1:nandboot.obj
 0001:000085f0       ??_C@_0DO@NAFJLJJO@WARNING?3?5NAND?5device?5doesn?8t?5exi@ 000195f0     nand_boot_common_topaz_v1:nandboot.obj
 0001:00008630       ??_C@_0DO@IACNLFIB@INFO?3?5Updating?5of?5EBOOT?1SBOOT?5im@ 00019630     nand_boot_common_topaz_v1:nandboot.obj
 0001:00008670       ??_C@_0CB@PJJBOHIF@INFO?3?5Verifying?5image?5succeed?4?$AN?6@ 00019670     nand_boot_common_topaz_v1:nandboot.obj
 0001:00008694       ??_C@_0CL@HLKKIBHF@NAND?5flash?5block?5?$FL0x?$CFx?$FN?5isn?8t?5re@ 00019694     nand_boot_common_topaz_v1:nandboot.obj
 0001:000086c0       ??_C@_0CB@COMIICDO@ERROR?3?5Failed?5to?5verify?5image?4?$AN?6@ 000196c0     nand_boot_common_topaz_v1:nandboot.obj
 0001:000086e4       ??_C@_0DF@DMMPELAE@INFO?3?5Programming?5NAND?5flash?5blo@ 000196e4     nand_boot_common_topaz_v1:nandboot.obj
 0001:0000871c       ??_C@_0DO@LHIODLEE@ERROR?3?5Boot?5size?5exceeds?5reserve@ 0001971c     nand_boot_common_topaz_v1:nandboot.obj
 0001:0000875c       ??_C@_0DE@DFOAOGPK@INFO?3?5Writing?5Boot?5image?5to?5NAND@ 0001975c     nand_boot_common_topaz_v1:nandboot.obj
 0001:00008790       ??_C@_0DC@BGNPKHBI@INFO?3?5Updating?5of?5image?5complete@ 00019790     nand_boot_common_topaz_v1:nandboot.obj
 0001:000087c4       ??_C@_0CD@LBDDECMN@?$AN?6INFO?3?5Verifying?5image?5succeed?4@ 000197c4     nand_boot_common_topaz_v1:nandboot.obj
 0001:000087e8       ??_C@_0DK@BNDNAAAI@INFO?3?5Programming?5and?5Verifying?5@ 000197e8     nand_boot_common_topaz_v1:nandboot.obj
 0001:00008824       ??_C@_0CB@PAFJJGNA@ERROR?3?5Failed?5to?5update?5image?4?$AN?6@ 00019824     nand_boot_common_topaz_v1:nandboot.obj
 0001:00008848       ??_C@_0DF@NNJDPACB@INFO?3?5Programming?5NAND?5flash?5blo@ 00019848     nand_boot_common_topaz_v1:nandboot.obj
 0001:00008880       ??_C@_0DM@FFNMNECJ@ERROR?3?5NK?5size?5exceeds?5reserved?5@ 00019880     nand_boot_common_topaz_v1:nandboot.obj
 0001:000088bc       ??_C@_0DC@IBLKHNEB@INFO?3?5Writing?5NK?5image?5to?5NAND?5?$CI@ 000198bc     nand_boot_common_topaz_v1:nandboot.obj
 0001:000088f0       ??_C@_0DA@CFIHFKOJ@?$AN?6INFO?3?5Loading?5of?5NK?5completed?5@ 000198f0     nand_boot_common_topaz_v1:nandboot.obj
 0001:00008920       ??_C@_02GPIOPFAK@?$DO?$DO?$AA@ 00019920     nand_boot_common_topaz_v1:nandboot.obj
 0001:00008924       ??_C@_0CF@PLBLFIAH@ERROR?3?5Read?5sector?3?5?$FL0x?$CFx?$FN?5faile@ 00019924     nand_boot_common_topaz_v1:nandboot.obj
 0001:0000894c       ??_C@_0DC@PEELBEJC@INFO?3?5Reading?5NK?5image?5to?5NAND?5?$CI@ 0001994c     nand_boot_common_topaz_v1:nandboot.obj
 0001:00008980       ??_C@_0DN@FOBINPEN@WARNING?3?5NAND?5device?5doesn?8t?5exi@ 00019980     nand_boot_common_topaz_v1:nandboot.obj
 0001:000089c0       ??_C@_0CO@BJGFJAIH@WARNING?3?5Failed?5to?5Load?5configur@ 000199c0     nand_boot_common_topaz_v1:nandboot.obj
 0001:000089f0       ??_C@_0BO@PCFMGLDF@Error?3?5No?5good?5block?5found?$CB?$AN?6?$AA@ 000199f0     nand_boot_common_topaz_v1:nandboot.obj
 0001:00008a10       ??_C@_0CN@NHADDNNL@INFO?3?5Loading?5boot?5configuration@ 00019a10     nand_boot_common_topaz_v1:nandboot.obj
 0001:00008a40       ??_C@_0DI@OLNJMAJP@INFO?3?5Successfully?5stored?5boot?5c@ 00019a40     nand_boot_common_topaz_v1:nandboot.obj
 0001:00008a78       ??_C@_0DE@LLENDJKK@WARNING?3?5Failed?5to?5write?5boot?5co@ 00019a78     nand_boot_common_topaz_v1:nandboot.obj
 0001:00008aac       ??_C@_0DJ@HCHCAAAK@INFO?3?5Storing?5boot?5configuration@ 00019aac     nand_boot_common_topaz_v1:nandboot.obj
 0001:00008ae8       ??_C@_0ED@HDAKJGJP@Error?3?5No?5good?5block?5found?5?9?5una@ 00019ae8     nand_boot_common_topaz_v1:nandboot.obj
 0001:00008b2c       ??_C@_0DL@JLHJEAKF@?$AN?6INFO?3?5Format?5of?5NAND?5NK?5region@ 00019b2c     nand_boot_common_topaz_v1:nandboot.obj
 0001:00008b68       ??_C@_0CL@OKPLEKII@INFO?3?5Starting?5format?5of?5NAND?5NK@ 00019b68     nand_boot_common_topaz_v1:nandboot.obj
 0001:00008b94       ??_C@_0CO@FFMLABON@INFO?3?5Update?5of?5IPL?5completed?5su@ 00019b94     nand_boot_common_topaz_v1:nandboot.obj
 0001:00008bc4       ??_C@_0BP@DCNJBMKK@ERROR?3?5Failed?5to?5verify?5IPL?4?$AN?6?$AA@ 00019bc4     nand_boot_common_topaz_v1:nandboot.obj
 0001:00008be8       ??_C@_0EH@DDGBHFHG@INFO?3?5Programming?5IPL?5image?5from@ 00019be8     nand_boot_common_topaz_v1:nandboot.obj
 0001:00008c30       ??_C@_0DN@MHDNDODE@ERROR?3?5IPL?5size?5exceeds?5reserved@ 00019c30     nand_boot_common_topaz_v1:nandboot.obj
 0001:00008c70       ??_C@_0DD@FBNOANAB@INFO?3?5Writing?5IPL?5image?5to?5NAND?5@ 00019c70     nand_boot_common_topaz_v1:nandboot.obj
 0001:00008ca4       ??_C@_0CI@KOKADIKC@?$AN?6INFO?3?5Ready?5to?5write?5DIO?5image@ 00019ca4     nand_boot_common_topaz_v1:nandboot.obj
 0001:00008ccc       ??_C@_0BO@IMFCJLLN@INFO?3?5Erase?5is?5?$CFd?$CF?$CF?5complete?4?$AA@ 00019ccc     nand_boot_common_topaz_v1:nandboot.obj
 0001:00008cec       ??_C@_0DB@NKJDIEPK@INFO?3?5Erasing?5NAND?5flash?5blocks?5@ 00019cec     nand_boot_common_topaz_v1:nandboot.obj
 0001:00008d20       ??_C@_0ED@JNNBGIKF@ERROR?3?5DIO?5image?5size?5exceeds?5re@ 00019d20     nand_boot_common_topaz_v1:nandboot.obj
 0001:00008d68       ??_C@_0EG@LILMDEGK@WARN?3?5Block?5?$FL0x?$CFx?$FN?5?1?5sector?5?$FL0x?$CF@ 00019d68     nand_boot_common_topaz_v1:nandboot.obj
 0001:00008db0       ??_C@_0CH@DAJMGFOB@ERROR?3?5Writing?5sector?5?$FL0x?$CFx?$FN?5fai@ 00019db0     nand_boot_common_topaz_v1:nandboot.obj
 0001:00008dd8       ??_C@_0ED@MCLEPO@ERROR?3?5Incorrect?5or?5corrupted?5DI@ 00019dd8     nand_boot_common_topaz_v1:nandboot.obj
 0001:00008e1c       ??_C@_0DG@POHOAOBL@?$AN?6INFO?3?5Update?5of?5DIO?5image?5comp@ 00019e1c     nand_boot_common_topaz_v1:nandboot.obj
 0001:00008e54       ??_C@_0BL@KGENHFNE@?$AN?6INFO?3?5No?5NAND?5present?$CB?$AN?6?$AA@ 00019e54     nand_boot_common_topaz_v1:nandboot.obj
 0001:00008e70       ??_C@_0CM@MAKCJGJN@INFO?3?5Copy?5of?5IPL?5completed?5succ@ 00019e70     nand_boot_common_topaz_v1:nandboot.obj
 0001:00008e9c       ??_C@_0CO@DIGEHKBF@INFO?3?5Copying?5IPL?5image?5to?5RAM?5a@ 00019e9c     nand_boot_common_topaz_v1:nandboot.obj
 0001:00008ecc       ??_C@_0DF@OLHDGLNN@INFO?3?5Reading?5IPL?5image?5from?5NAN@ 00019ecc     nand_boot_common_topaz_v1:nandboot.obj
 0001:00008f04       ??_C@_0DN@CCBKKGDF@?$AN?6INFO?3?5Format?5of?5all?5NAND?5regio@ 00019f04     nand_boot_common_topaz_v1:nandboot.obj
 0001:00008f44       ??_C@_0BP@HLOCHMLD@INFO?3?5Format?5is?5?$CFd?$CF?$CF?5complete?4?$AA@ 00019f44     nand_boot_common_topaz_v1:nandboot.obj
 0001:00008f64       ??_C@_0DA@GHJFJAN@ERROR?3?5Unable?5to?5erase?5NAND?5flas@ 00019f64     nand_boot_common_topaz_v1:nandboot.obj
 0001:00008f94       ??_C@_0CN@CCDNFIGE@INFO?3?5Starting?5format?5of?5all?5NAN@ 00019f94     nand_boot_common_topaz_v1:nandboot.obj
 0001:00008fc4       ??_C@_1CK@OLHBCELJ@?$AAI?$AAn?$AAi?$AAt?$AAi?$AAa?$AAl?$AAi?$AAz?$AAe?$AAB?$AAB?$AAT?$AA?5?$AAF?$AAa?$AAi?$AAl?$AA?$AN?$AA?6?$AA?$AA@ 00019fc4     nand_common_topaz_v1:fmd.obj
 0001:00008ff0       ??_C@_1CE@GBLOPLJP@?$AAN?$AAu?$AAm?$AAb?$AAe?$AAr?$AAO?$AAf?$AAC?$AAh?$AAi?$AAp?$AA?$DN?$AA?$CF?$AAd?$AA?$AN?$AA?6?$AA?$AA@ 00019ff0     nand_common_topaz_v1:fmd.obj
 0001:00009018       ??_C@_1HM@GJHCPODI@?$AAF?$AAM?$AAD?$AA?3?$AA?3?$AAE?$AAR?$AAR?$AAO?$AAR?$AA?3?$AA?5?$AAN?$AAa?$AAn?$AAd?$AA?5?$AAc?$AAh?$AAi?$AAp?$AA?5?$AAt?$AAy?$AAp?$AAe?$AA?5?$AAs?$AAe?$AAl?$AAe?$AAc@ 0001a018     nand_common_topaz_v1:fmd.obj
 0001:00009094       ??_C@_1DA@NOCINKLA@?$AAn?$AAo?$AA?5?$AAN?$AAA?$AAN?$AAD?$AA?5?$AAt?$AAy?$AAp?$AAe?$AA?5?$AAm?$AAa?$AAt?$AAc?$AAh?$AAe?$AAd?$AA?$CB?$AA?$AN?$AA?6?$AA?$AA@ 0001a094     nand_common_topaz_v1:fmd.obj
 0001:000090c8       ??_C@_1OE@NKNGGBGA@?$AAc?$AA?3?$AA?2?$AAw?$AAi?$AAn?$AAc?$AAe?$AAr?$AAo?$AAo?$AAt?$AAs?$AA?2?$AAt?$AAo?$AAp?$AAa?$AAz?$AA?2?$AAw?$AAi?$AAn?$AAc?$AAe?$AA7?$AA0?$AA0?$AA?2?$AAp?$AAl?$AAa@ 0001a0c8     nand_common_topaz_v1:fmd.obj
 0001:000091ac       ??_C@_1DO@KBODJKMM@?$AAS?$AAe?$AAc?$AAt?$AAo?$AAr?$AA?1?$AAI?$AAn?$AAf?$AAo?$AA?5?$AAb?$AAu?$AAf?$AAf?$AAe?$AAr?$AAs?$AA?5?$AAa?$AAr?$AAe?$AA?5?$AAN?$AAU?$AAL?$AAL?$AA?$AN?$AA?6?$AA?$AA@ 0001a1ac     nand_common_topaz_v1:fmd.obj
 0001:000091f0       ??_C@_1EI@FGFOPHKM@?$AAB?$AAa?$AAd?$AA?5?$AAB?$AAl?$AAo?$AAc?$AAk?$AA?5?$AAf?$AAo?$AAu?$AAn?$AAd?$AA?3?$AA?5?$AAB?$AAl?$AAo?$AAc?$AAk?$AA?5?$AAN?$AAo?$AA?4?$AA?5?$AA?$DN?$AA?5?$AA0?$AAx?$AA?$CF@ 0001a1f0     nand_common_topaz_v1:fmd.obj
 0001:00009238       ??_C@_1DA@NBBNEODN@?$AAB?$AAL?$AAO?$AAC?$AAK?$AA_?$AAS?$AAT?$AAA?$AAT?$AAU?$AAS?$AA_?$AAR?$AAE?$AAS?$AAE?$AAR?$AAV?$AAE?$AAD?$AA?$AN?$AA?6?$AA?$AA@ 0001a238     nand_common_topaz_v1:fmd.obj
 0001:00009268       ??_C@_1DA@JEPFDADC@?$AAB?$AAL?$AAO?$AAC?$AAK?$AA_?$AAS?$AAT?$AAA?$AAT?$AAU?$AAS?$AA_?$AAR?$AAE?$AAA?$AAD?$AAO?$AAN?$AAL?$AAY?$AA?$AN?$AA?6?$AA?$AA@ 0001a268     nand_common_topaz_v1:fmd.obj
 0001:00009298       ??_C@_1IA@EECHOBPE@?$AAF?$AAM?$AAD?$AA_?$AAG?$AAe?$AAt?$AAB?$AAl?$AAo?$AAc?$AAk?$AAS?$AAt?$AAa?$AAt?$AAu?$AAs?$AA?5?$AA?3?$AA?5?$AAC?$AAS?$AAP?$AAN?$AAA?$AAN?$AAD?$AA_?$AAR?$AAe?$AAa@ 0001a298     nand_common_topaz_v1:fmd.obj
 0001:00009318       ??_C@_1EK@JMFCFNBO@?$AAG?$AAe?$AAt?$AAB?$AAl?$AAo?$AAc?$AAk?$AAB?$AAa?$AAd?$AAS?$AAt?$AAa?$AAt?$AAu?$AAs?$AA?5?$AA?3?$AA?5?$AAb?$AAa?$AAd?$AA?5?$AAb?$AAl?$AAo?$AAc?$AAk?$AA?5?$AA0?$AAx@ 0001a318     nand_common_topaz_v1:bbt.obj
 0001:00009368       ??_C@_1EK@BIPJPDEI@?$AAS?$AAe?$AAt?$AAB?$AAl?$AAo?$AAc?$AAk?$AAB?$AAa?$AAd?$AAS?$AAt?$AAa?$AAt?$AAu?$AAs?$AA?5?$AA?3?$AA?5?$AAb?$AAa?$AAd?$AA?5?$AAb?$AAl?$AAo?$AAc?$AAk?$AA?5?$AA0?$AAx@ 0001a368     nand_common_topaz_v1:bbt.obj
 0001:000093b4       ??_C@_1BO@FCAJAHJG@?$AAb?$AAl?$AAo?$AAc?$AAk?$AA?5?$AA?$DN?$AA?5?$AA0?$AAx?$AA?$CF?$AAX?$AA?$AN?$AA?6?$AA?$AA@ 0001a3b4     nand_common_topaz_v1:bbt.obj
 0001:000093d8       ??_C@_1EE@LDAGDDEG@?$AAC?$AAa?$AAl?$AAl?$AA?5?$AAB?$AAB?$AAT?$AA_?$AAS?$AAe?$AAt?$AAB?$AAl?$AAo?$AAc?$AAk?$AAR?$AAe?$AAs?$AAe?$AAr?$AAv?$AAe?$AAd?$AAS?$AAt?$AAa?$AAt?$AAu?$AAs?$AA?$AN@ 0001a3d8     nand_common_topaz_v1:bbt.obj
 0001:0000941c       ??_C@_1DC@OJPGNGKM@?$AAW?$AAr?$AAi?$AAt?$AAe?$AAB?$AAB?$AAT?$AA?5?$AA?3?$AA?5?$AAU?$AAp?$AAd?$AAa?$AAt?$AAe?$AA?5?$AAf?$AAa?$AAi?$AAl?$AA?$AN?$AA?6?$AA?$AA@ 0001a41c     nand_common_topaz_v1:bbt.obj
 0001:00009450       ??_C@_1HC@FCPIHGL@?$AAW?$AAr?$AAi?$AAt?$AAe?$AAB?$AAB?$AAT?$AA?5?$AAF?$AAo?$AAr?$AA?9?$AAl?$AAo?$AAo?$AAp?$AA?5?$AA?3?$AA?5?$AAd?$AAw?$AAS?$AAt?$AAa?$AAr?$AAt?$AAB?$AAl?$AAo?$AAc?$AAk@ 0001a450     nand_common_topaz_v1:bbt.obj
 0001:000094c8       ??_C@_1FM@PJOHFGIO@?$AAW?$AAr?$AAi?$AAt?$AAe?$AAB?$AAB?$AAT?$AA?5?$AA?3?$AA?5?$AAd?$AAw?$AAB?$AAB?$AAT?$AAB?$AAl?$AAo?$AAc?$AAk?$AA?5?$AA?$DN?$AA?5?$AA0?$AAx?$AA?$CF?$AAX?$AA?0?$AA?5?$AAd?$AAw@ 0001a4c8     nand_common_topaz_v1:bbt.obj
 0001:00009528       ??_C@_1JC@OKBDACKI@?$AAB?$AAB?$AAT?$AA_?$AAG?$AAe?$AAt?$AAB?$AAl?$AAo?$AAc?$AAk?$AAR?$AAe?$AAs?$AAe?$AAr?$AAv?$AAe?$AAd?$AAS?$AAt?$AAa?$AAt?$AAu?$AAs?$AA?5?$AA?3?$AA?5?$AAB?$AAB?$AAT@ 0001a528     nand_common_topaz_v1:bbt.obj
 0001:000095c0       ??_C@_1JA@JBPCDKFP@?$AAB?$AAB?$AAT?$AA_?$AAG?$AAe?$AAt?$AAB?$AAl?$AAo?$AAc?$AAk?$AAR?$AAe?$AAs?$AAe?$AAr?$AAv?$AAe?$AAd?$AAS?$AAt?$AAa?$AAt?$AAu?$AAs?$AA?5?$AA?3?$AA?5?$AAC?$AAS?$AAP@ 0001a5c0     nand_common_topaz_v1:bbt.obj
 0001:00009650       ??_C@_1GO@JJKIBJBN@?$AAB?$AAB?$AAT?$AA_?$AAS?$AAe?$AAt?$AAB?$AAl?$AAo?$AAc?$AAk?$AAR?$AAe?$AAs?$AAe?$AAr?$AAv?$AAe?$AAd?$AAS?$AAt?$AAa?$AAt?$AAu?$AAs?$AA?5?$AA?3?$AA?5?$AAB?$AAB?$AAT@ 0001a650     nand_common_topaz_v1:bbt.obj
 0001:000096c0       ??_C@_1FI@CHANIFCF@?$AAB?$AAB?$AAT?$AA_?$AAS?$AAe?$AAt?$AAB?$AAl?$AAo?$AAc?$AAk?$AAR?$AAe?$AAs?$AAe?$AAr?$AAv?$AAe?$AAd?$AAS?$AAt?$AAa?$AAt?$AAu?$AAs?$AA?5?$AA?3?$AA?5?$AAb?$AAl?$AAo@ 0001a6c0     nand_common_topaz_v1:bbt.obj
 0001:00009718       ??_C@_1DC@NMBGMIDN@?$AAW?$AAr?$AAi?$AAt?$AAe?$AAB?$AAB?$AAT?$AAS?$AAi?$AAg?$AAn?$AAa?$AAt?$AAu?$AAr?$AAe?$AA?5?$AAF?$AAa?$AAi?$AAl?$AA?$AN?$AA?6?$AA?$AA@ 0001a718     nand_common_topaz_v1:bbt.obj
 0001:00009750       ??_C@_1HM@GMJOILC@?$AAB?$AAB?$AAT?$AA_?$AAW?$AAr?$AAi?$AAt?$AAe?$AAO?$AAp?$AAe?$AAr?$AAa?$AAt?$AAi?$AAo?$AAn?$AA?5?$AA?3?$AA?5?$AAd?$AAw?$AAS?$AAt?$AAa?$AAr?$AAt?$AAB?$AAl?$AAo?$AAc@ 0001a750     nand_common_topaz_v1:bbt.obj
 0001:000097cc       ??_C@_1DE@BAILHGBL@?$AAB?$AAB?$AAT?$AA_?$AAE?$AAr?$AAa?$AAs?$AAe?$AAO?$AAp?$AAe?$AAr?$AAa?$AAt?$AAi?$AAo?$AAn?$AA?5?$AAF?$AAa?$AAi?$AAl?$AA?$AN?$AA?6?$AA?$AA@ 0001a7cc     nand_common_topaz_v1:bbt.obj
 0001:00009800       ??_C@_1DG@MLFLBPLM@?$AAC?$AAS?$AAP?$AAN?$AAA?$AAN?$AAD?$AA_?$AAW?$AAr?$AAi?$AAt?$AAe?$AAS?$AAe?$AAc?$AAt?$AAo?$AAr?$AA?5?$AAF?$AAa?$AAi?$AAl?$AA?$AN?$AA?6?$AA?$AA@ 0001a800     nand_common_topaz_v1:bbt.obj
 0001:00009838       ??_C@_1FO@JHBBKHC@?$AAB?$AAB?$AAT?$AA_?$AAW?$AAr?$AAi?$AAt?$AAe?$AAO?$AAp?$AAe?$AAr?$AAa?$AAt?$AAi?$AAo?$AAn?$AA?5?$AA?3?$AA?5?$AAB?$AAB?$AAT?$AA_?$AAE?$AAr?$AAa?$AAs?$AAe?$AAO?$AAp@ 0001a838     nand_common_topaz_v1:bbt.obj
 0001:00009898       ??_C@_1FA@CEMLDMBN@?$AAB?$AAB?$AAT?$AA_?$AAE?$AAr?$AAa?$AAs?$AAe?$AAO?$AAp?$AAe?$AAr?$AAa?$AAt?$AAi?$AAo?$AAn?$AA?5?$AAE?$AAn?$AAd?$AA?5?$AA?3?$AA?5?$AAb?$AAN?$AAu?$AAm?$AAb?$AAe?$AAr@ 0001a898     nand_common_topaz_v1:bbt.obj
 0001:000098e8       ??_C@_1DO@CFCFIEKM@?$AAC?$AAS?$AAP?$AAN?$AAA?$AAN?$AAD?$AA_?$AAE?$AAr?$AAa?$AAs?$AAe?$AAB?$AAl?$AAo?$AAc?$AAk?$AA?5?$AA0?$AAx?$AA?$CF?$AAX?$AA?5?$AAF?$AAa?$AAi?$AAl?$AA?$AN?$AA?6?$AA?$AA@ 0001a8e8     nand_common_topaz_v1:bbt.obj
 0001:00009928       ??_C@_1FE@DJOBLIFB@?$AAB?$AAB?$AAT?$AA_?$AAE?$AAr?$AAa?$AAs?$AAe?$AAO?$AAp?$AAe?$AAr?$AAa?$AAt?$AAi?$AAo?$AAn?$AA?5?$AAB?$AAe?$AAg?$AAi?$AAn?$AA?5?$AA?3?$AA?5?$AAb?$AAN?$AAu?$AAm?$AAb@ 0001a928     nand_common_topaz_v1:bbt.obj
 0001:0000997c       ??_C@_1CI@JPELOBJH@?$AAW?$AAr?$AAi?$AAt?$AAe?$AAB?$AAB?$AAT?$AAS?$AAi?$AAg?$AAn?$AAa?$AAt?$AAu?$AAr?$AAe?$AA?$AN?$AA?6?$AA?$AA@ 0001a97c     nand_common_topaz_v1:bbt.obj
 0001:000099a4       ??_C@_1BO@FDCJDGC@?$AAN?$AAo?$AA?5?$AAB?$AAB?$AAT?$AA?5?$AAF?$AAo?$AAu?$AAn?$AAd?$AA?$AN?$AA?6?$AA?$AA@ 0001a9a4     nand_common_topaz_v1:bbt.obj
 0001:000099c4       ??_C@_1DM@DIMCHKOP@?$AAB?$AAo?$AAt?$AAh?$AA?5?$AAB?$AAB?$AAT?$AA?5?$AAn?$AAe?$AAe?$AAd?$AA?5?$AAt?$AAo?$AA?5?$AAb?$AAe?$AA?5?$AAf?$AAl?$AAu?$AAs?$AAh?$AAe?$AAd?$AA?$AN?$AA?6?$AA?$AA@ 0001a9c4     nand_common_topaz_v1:bbt.obj
 0001:00009a00       ??_C@_1EI@NLCMEDKF@?$AAB?$AAB?$AAT?$AA?5?$AAD?$AAi?$AAf?$AAf?$AAe?$AAr?$AAe?$AAn?$AAc?$AAe?$AA?5?$AA?3?$AA?5?$AA?$CF?$AAd?$AA?5?$AA?3?$AA?5?$AA0?$AAx?$AA?$CF?$AAX?$AA?5?$AA?9?$AA?5?$AA0?$AAx?$AA?$CF@ 0001aa00     nand_common_topaz_v1:bbt.obj
 0001:00009a48       ??_C@_1GG@NPCKDGH@?$AAB?$AAB?$AAT?$AA_?$AAR?$AAe?$AAa?$AAd?$AAO?$AAp?$AAe?$AAr?$AAa?$AAt?$AAi?$AAo?$AAn?$AA?5?$AA?3?$AA?5?$AAB?$AAB?$AAT?$AA_?$AAE?$AAr?$AAa?$AAs?$AAe?$AAO?$AAp?$AAe@ 0001aa48     nand_common_topaz_v1:bbt.obj
 0001:00009ab0       ??_C@_1HK@DMNLDLPJ@?$AAB?$AAB?$AAT?$AA_?$AAR?$AAe?$AAa?$AAd?$AAO?$AAp?$AAe?$AAr?$AAa?$AAt?$AAi?$AAo?$AAn?$AA?5?$AA?3?$AA?5?$AAd?$AAw?$AAS?$AAt?$AAa?$AAr?$AAt?$AAB?$AAl?$AAo?$AAc?$AAk@ 0001aab0     nand_common_topaz_v1:bbt.obj
 0001:00009b30       ??_C@_1GA@PHEPAMKB@?$AAb?$AAB?$AAa?$AAd?$AAB?$AAl?$AAo?$AAc?$AAk?$AA?5?$AA?3?$AA?5?$AAE?$AAC?$AAC?$AA?5?$AAE?$AAn?$AAa?$AAb?$AAl?$AAe?$AA?5?$AA0?$AAx?$AA?$CF?$AAX?$AA?0?$AA?5?$AAE?$AAC?$AAC@ 0001ab30     nand_common_topaz_v1:bbt.obj
 0001:00009b90       ??_C@_1GO@BPBBFPFP@?$AAR?$AAe?$AAa?$AAd?$AAB?$AAl?$AAo?$AAc?$AAk?$AAB?$AAa?$AAd?$AAS?$AAt?$AAa?$AAt?$AAu?$AAs?$AA?5?$AA0?$AAx?$AA?$CF?$AAX?$AA?0?$AA?5?$AAE?$AAC?$AAC?$AA?5?$AAS?$AAt?$AAa@ 0001ab90     nand_common_topaz_v1:bbt.obj
 0001:00009c00       ??_C@_1DA@DJCDJBAL@?$AAN?$AAo?$AAt?$AA?5?$AAB?$AAB?$AAT?$AA_?$AAS?$AAI?$AAG?$AAN?$AA?5?$AA2?$AA?5?$AA?3?$AA?5?$AA0?$AAx?$AA?$CF?$AAX?$AA?$AN?$AA?6?$AA?$AA@ 0001ac00     nand_common_topaz_v1:bbt.obj
 0001:00009c30       ??_C@_1DA@FLDMEL@?$AAN?$AAo?$AAt?$AA?5?$AAB?$AAB?$AAT?$AA_?$AAS?$AAI?$AAG?$AAN?$AA?5?$AA1?$AA?5?$AA?3?$AA?5?$AA0?$AAx?$AA?$CF?$AAX?$AA?$AN?$AA?6?$AA?$AA@ 0001ac30     nand_common_topaz_v1:bbt.obj
 0001:00009c60       ??_C@_1GE@LMDHKNPP@?$AAR?$AAe?$AAa?$AAd?$AAB?$AAB?$AAT?$AAS?$AAi?$AAg?$AAn?$AAa?$AAt?$AAu?$AAr?$AAe?$AA?5?$AA?3?$AA?5?$AAB?$AAB?$AAT?$AA_?$AAE?$AAr?$AAa?$AAs?$AAe?$AAO?$AAp?$AAe?$AAr@ 0001ac60     nand_common_topaz_v1:bbt.obj
 0001:00009cc8       ??_C@_1IA@KFLDOLMH@?$AAC?$AAS?$AAP?$AAN?$AAA?$AAN?$AAD?$AA_?$AAR?$AAe?$AAa?$AAd?$AAS?$AAe?$AAc?$AAt?$AAo?$AAr?$AA?5?$AAF?$AAa?$AAi?$AAl?$AA?5?$AA?3?$AA?5?$AAs?$AAt?$AAa?$AAr?$AAt?$AAS@ 0001acc8     nand_common_topaz_v1:bbt.obj
 0001:00009d48       ??_C@_1EE@JIJBIFML@?$AAC?$AAr?$AAe?$AAa?$AAt?$AAe?$AAB?$AAB?$AAT?$AA?5?$AA?3?$AA?5?$AAN?$AAo?$AAn?$AA?9?$AAI?$AAn?$AAt?$AAe?$AAr?$AAl?$AAe?$AAa?$AAv?$AAe?$AA?5?$AAM?$AAo?$AAd?$AAe?$AA?$AN@ 0001ad48     nand_common_topaz_v1:bbt.obj
 0001:00009d8c       ??_C@_1DM@FMAPKBEC@?$AAC?$AAr?$AAe?$AAa?$AAt?$AAe?$AAB?$AAB?$AAT?$AA?5?$AA?3?$AA?5?$AAI?$AAn?$AAt?$AAe?$AAr?$AAl?$AAe?$AAa?$AAv?$AAe?$AA?5?$AAM?$AAo?$AAd?$AAe?$AA?$AN?$AA?6?$AA?$AA@ 0001ad8c     nand_common_topaz_v1:bbt.obj
 0001:00009dc8       ??_C@_1BO@FLNOHMKD@?$AA?9?$AA?5?$AAS?$AAD?$AAM?$AAM?$AAC?$AA_?$AAI?$AAn?$AAi?$AAt?$AA?$AN?$AA?6?$AA?$AA@ 0001adc8     sdmmc_boot_common_topaz_v1:sdfmd.obj
 0001:00009de8       ??_C@_1DK@OFGPADJD@?$AAI?$AAN?$AAF?$AAO?$AA?3?$AA?5?$AAI?$AAn?$AAi?$AAt?$AAi?$AAa?$AAl?$AAi?$AAz?$AAe?$AAd?$AA?5?$AAM?$AAM?$AAC?$AA?5?$AAC?$AAa?$AAr?$AAd?$AA?$AN?$AA?6?$AA?$AA@ 0001ade8     sdmmc_boot_common_topaz_v1:sdfmd.obj
 0001:00009e24       ??_C@_1DI@EGCEGKFN@?$AAI?$AAN?$AAF?$AAO?$AA?3?$AA?5?$AAI?$AAn?$AAi?$AAt?$AAi?$AAa?$AAl?$AAi?$AAz?$AAe?$AAd?$AA?5?$AAS?$AAD?$AA?5?$AAC?$AAa?$AAr?$AAd?$AA?$AN?$AA?6?$AA?$AA@ 0001ae24     sdmmc_boot_common_topaz_v1:sdfmd.obj
 0001:00009e5c       ??_C@_1DE@JKNKMHG@?$AAS?$AAD?$AAI?$AAn?$AAt?$AAe?$AAr?$AAf?$AAa?$AAc?$AAe?$AA_?$AAI?$AAn?$AAi?$AAt?$AA?5?$AAF?$AAa?$AAi?$AAl?$AAe?$AAd?$AA?$AN?$AA?6?$AA?$AA@ 0001ae5c     sdmmc_boot_common_topaz_v1:sdfmd.obj
 0001:00009e90       ??_C@_1BO@NCJMDGJD@?$AA?$CL?$AA?5?$AAS?$AAD?$AAM?$AAM?$AAC?$AA_?$AAI?$AAn?$AAi?$AAt?$AA?$AN?$AA?6?$AA?$AA@ 0001ae90     sdmmc_boot_common_topaz_v1:sdfmd.obj
 0001:00009eb0       ??_C@_1CE@OKBLGLBL@?$AA?9?$AA?5?$AAS?$AAD?$AAM?$AAM?$AAC?$AA_?$AAg?$AAe?$AAt?$AA_?$AAc?$AAi?$AAd?$AA?$AN?$AA?6?$AA?$AA@ 0001aeb0     sdmmc_boot_common_topaz_v1:sdfmd.obj
 0001:00009ed4       ??_C@_1CE@CDNLJMOH@?$AA?$CL?$AA?5?$AAS?$AAD?$AAM?$AAM?$AAC?$AA_?$AAg?$AAe?$AAt?$AA_?$AAc?$AAi?$AAd?$AA?$AN?$AA?6?$AA?$AA@ 0001aed4     sdmmc_boot_common_topaz_v1:sdfmd.obj
 0001:00009ef8       ??_C@_1EC@BMCFOHBM@?$AA?9?$AA?5?$AAS?$AAD?$AAM?$AAM?$AAC?$AA_?$AAs?$AAe?$AAt?$AA_?$AAd?$AAa?$AAt?$AAa?$AA_?$AAt?$AAr?$AAa?$AAn?$AAs?$AAf?$AAe?$AAr?$AA_?$AAm?$AAo?$AAd?$AAe?$AA?$AN?$AA?6@ 0001aef8     sdmmc_boot_common_topaz_v1:sdfmd.obj
 0001:00009f40       ??_C@_1EC@HDCBAPBP@?$AA?$CL?$AA?5?$AAS?$AAD?$AAM?$AAM?$AAC?$AA_?$AAs?$AAe?$AAt?$AA_?$AAd?$AAa?$AAt?$AAa?$AA_?$AAt?$AAr?$AAa?$AAn?$AAs?$AAf?$AAe?$AAr?$AA_?$AAm?$AAo?$AAd?$AAe?$AA?$AN?$AA?6@ 0001af40     sdmmc_boot_common_topaz_v1:sdfmd.obj
 0001:00009f84       ??_C@_1DM@BOLBGFFK@?$AA?9?$AA?5?$AAS?$AAD?$AAM?$AAM?$AAC?$AA_?$AAc?$AAa?$AAr?$AAd?$AA_?$AAs?$AAo?$AAf?$AAt?$AAw?$AAa?$AAr?$AAe?$AA_?$AAr?$AAe?$AAs?$AAe?$AAt?$AA?$AN?$AA?6?$AA?$AA@ 0001af84     sdmmc_boot_common_topaz_v1:sdfmd.obj
 0001:00009fc0       ??_C@_1DM@MNMLEILL@?$AA?$CL?$AA?5?$AAS?$AAD?$AAM?$AAM?$AAC?$AA_?$AAc?$AAa?$AAr?$AAd?$AA_?$AAs?$AAo?$AAf?$AAt?$AAw?$AAa?$AAr?$AAe?$AA_?$AAr?$AAe?$AAs?$AAe?$AAt?$AA?$AN?$AA?6?$AA?$AA@ 0001afc0     sdmmc_boot_common_topaz_v1:sdfmd.obj
 0001:00009ffc       ??_C@_1DG@LMAKMHFK@?$AA?9?$AA?5?$AAS?$AAD?$AAM?$AAM?$AAC?$AA_?$AAc?$AAa?$AAr?$AAd?$AA_?$AAs?$AAe?$AAn?$AAd?$AA_?$AAa?$AAp?$AAp?$AAc?$AAm?$AAd?$AA?$AN?$AA?6?$AA?$AA@ 0001affc     sdmmc_boot_common_topaz_v1:sdfmd.obj
 0001:0000a034       ??_C@_1DG@LJNHDCOO@?$AA?$CL?$AA?5?$AAS?$AAD?$AAM?$AAM?$AAC?$AA_?$AAc?$AAa?$AAr?$AAd?$AA_?$AAs?$AAe?$AAn?$AAd?$AA_?$AAa?$AAp?$AAp?$AAc?$AAm?$AAd?$AA?$AN?$AA?6?$AA?$AA@ 0001b034     sdmmc_boot_common_topaz_v1:sdfmd.obj
 0001:0000a06c       ??_C@_1CE@NKJHHKDK@?$AA?9?$AA?5?$AAS?$AAD?$AAM?$AAM?$AAC?$AA_?$AAg?$AAe?$AAt?$AA_?$AAc?$AAs?$AAd?$AA?$AN?$AA?6?$AA?$AA@ 0001b06c     sdmmc_boot_common_topaz_v1:sdfmd.obj
 0001:0000a090       ??_C@_1CE@BDFHINMG@?$AA?$CL?$AA?5?$AAS?$AAD?$AAM?$AAM?$AAC?$AA_?$AAg?$AAe?$AAt?$AA_?$AAc?$AAs?$AAd?$AA?$AN?$AA?6?$AA?$AA@ 0001b090     sdmmc_boot_common_topaz_v1:sdfmd.obj
 0001:0000a0b4       ??_C@_1CM@OJICGLDP@?$AA?9?$AA?5?$AAS?$AAD?$AAM?$AAM?$AAC?$AA_?$AAg?$AAe?$AAt?$AA_?$AAe?$AAx?$AAt?$AA_?$AAc?$AAs?$AAd?$AA?$AN?$AA?6?$AA?$AA@ 0001b0b4     sdmmc_boot_common_topaz_v1:sdfmd.obj
 0001:0000a0e0       ??_C@_1CM@BFHCPKHD@?$AA?$CL?$AA?5?$AAS?$AAD?$AAM?$AAM?$AAC?$AA_?$AAg?$AAe?$AAt?$AA_?$AAe?$AAx?$AAt?$AA_?$AAc?$AAs?$AAd?$AA?$AN?$AA?6?$AA?$AA@ 0001b0e0     sdmmc_boot_common_topaz_v1:sdfmd.obj
 0001:0000a10c       ??_C@_1DI@IFMKDPDF@?$AAC?$AAa?$AAr?$AAd?$AA?5?$AAC?$AAa?$AAp?$AAa?$AAc?$AAi?$AAt?$AAy?$AA?5?$AA?$CF?$AAd?$AA?5?$AA?$CI?$AAK?$AAb?$AAy?$AAt?$AAe?$AAs?$AA?$CJ?$AA?$AN?$AA?6?$AA?$AA@ 0001b10c     sdmmc_boot_common_topaz_v1:sdfmd.obj
 0001:0000a148       ??_C@_1FM@BKLIEMHK@?$AAE?$AAR?$AAR?$AAO?$AAR?$AA?3?$AA?5?$AAU?$AAn?$AAa?$AAb?$AAl?$AAe?$AA?5?$AAt?$AAo?$AA?5?$AAr?$AAe?$AAa?$AAd?$AA?5?$AAE?$AAX?$AAT?$AA_?$AAC?$AAS?$AAD?$AA?5?$AAf?$AAr@ 0001b148     sdmmc_boot_common_topaz_v1:sdfmd.obj
 0001:0000a1a4       ??_C@_1CO@MDKGHMCM@?$AA?9?$AA?5?$AAS?$AAD?$AAM?$AAM?$AAC?$AA_?$AAs?$AAe?$AAt?$AA_?$AAb?$AAl?$AAo?$AAc?$AAk?$AAl?$AAe?$AAn?$AA?$AN?$AA?6?$AA?$AA@ 0001b1a4     sdmmc_boot_common_topaz_v1:sdfmd.obj
 0001:0000a1d4       ??_C@_1CO@BIGCCDAH@?$AA?$CL?$AA?5?$AAS?$AAD?$AAM?$AAM?$AAC?$AA_?$AAs?$AAe?$AAt?$AA_?$AAb?$AAl?$AAo?$AAc?$AAk?$AAl?$AAe?$AAn?$AA?$AN?$AA?6?$AA?$AA@ 0001b1d4     sdmmc_boot_common_topaz_v1:sdfmd.obj
 0001:0000a204       ??_C@_1CG@PKGMFFOD@?$AA?9?$AA?5?$AAS?$AAD?$AAM?$AAM?$AAC?$AA_?$AAs?$AAe?$AAn?$AAd?$AA_?$AAr?$AAc?$AAa?$AA?$AN?$AA?6?$AA?$AA@ 0001b204     sdmmc_boot_common_topaz_v1:sdfmd.obj
 0001:0000a22c       ??_C@_1CG@GBLMFFCN@?$AA?$CL?$AA?5?$AAS?$AAD?$AAM?$AAM?$AAC?$AA_?$AAs?$AAe?$AAn?$AAd?$AA_?$AAr?$AAc?$AAa?$AA?$AN?$AA?6?$AA?$AA@ 0001b22c     sdmmc_boot_common_topaz_v1:sdfmd.obj
 0001:0000a254       ??_C@_1DA@IDDKHMO@?$AA?9?$AA?5?$AAS?$AAD?$AAM?$AAM?$AAC?$AA_?$AAR?$AA1?$AAb?$AA_?$AAb?$AAu?$AAs?$AAy?$AA_?$AAw?$AAa?$AAi?$AAt?$AA?$AN?$AA?6?$AA?$AA@ 0001b254     sdmmc_boot_common_topaz_v1:sdfmd.obj
 0001:0000a288       ??_C@_1EK@LIKKCIIF@?$AAR?$AA1?$AAb?$AA_?$AAb?$AAu?$AAs?$AAy?$AA_?$AAw?$AAa?$AAi?$AAt?$AA?5?$AAt?$AAi?$AAm?$AAe?$AAd?$AA?5?$AAo?$AAu?$AAt?$AA?5?$AAS?$AAt?$AAa?$AAt?$AAe?$AA?5?$AA?9?$AA?5@ 0001b288     sdmmc_boot_common_topaz_v1:sdfmd.obj
 0001:0000a2d4       ??_C@_1DA@IFJHMNAG@?$AA?$CL?$AA?5?$AAS?$AAD?$AAM?$AAM?$AAC?$AA_?$AAR?$AA1?$AAb?$AA_?$AAb?$AAu?$AAs?$AAy?$AA_?$AAw?$AAa?$AAi?$AAt?$AA?$AN?$AA?6?$AA?$AA@ 0001b2d4     sdmmc_boot_common_topaz_v1:sdfmd.obj
 0001:0000a308       ??_C@_1EC@JLIIGCHH@?$AAE?$AAR?$AAR?$AAO?$AAR?$AA?3?$AA?5?$AAc?$AAa?$AAr?$AAd?$AA?5?$AAi?$AAs?$AA?5?$AAw?$AAr?$AAi?$AAt?$AAe?$AA?9?$AAp?$AAr?$AAo?$AAt?$AAe?$AAc?$AAt?$AAe?$AAd?$AA?$AN?$AA?6@ 0001b308     sdmmc_boot_common_topaz_v1:sdfmd.obj
 0001:0000a34c       ??_C@_1CK@JMDODCBA@?$AA?9?$AA?5?$AAS?$AAD?$AAM?$AAM?$AAC?$AA_?$AAE?$AAr?$AAa?$AAs?$AAe?$AAB?$AAl?$AAo?$AAc?$AAk?$AA?$AN?$AA?6?$AA?$AA@ 0001b34c     sdmmc_boot_common_topaz_v1:sdfmd.obj
 0001:0000a378       ??_C@_1CK@GENHLLJN@?$AA?9?$AA?5?$AAS?$AAD?$AAM?$AAM?$AAC?$AA_?$AAR?$AAe?$AAa?$AAd?$AAS?$AAe?$AAc?$AAt?$AAo?$AAr?$AA?$AN?$AA?6?$AA?$AA@ 0001b378     sdmmc_boot_common_topaz_v1:sdfmd.obj
 0001:0000a3a4       ??_C@_1CK@BEKAKNHL@?$AA?$CL?$AA?5?$AAS?$AAD?$AAM?$AAM?$AAC?$AA_?$AAR?$AAe?$AAa?$AAd?$AAS?$AAe?$AAc?$AAt?$AAo?$AAr?$AA?$AN?$AA?6?$AA?$AA@ 0001b3a4     sdmmc_boot_common_topaz_v1:sdfmd.obj
 0001:0000a3d0       ??_C@_1CM@GNCJHEBI@?$AA?9?$AA?5?$AAS?$AAD?$AAM?$AAM?$AAC?$AA_?$AAW?$AAr?$AAi?$AAt?$AAe?$AAS?$AAe?$AAc?$AAt?$AAo?$AAr?$AA?$AN?$AA?6?$AA?$AA@ 0001b3d0     sdmmc_boot_common_topaz_v1:sdfmd.obj
 0001:0000a3fc       ??_C@_1CM@JBNJOFFE@?$AA?$CL?$AA?5?$AAS?$AAD?$AAM?$AAM?$AAC?$AA_?$AAW?$AAr?$AAi?$AAt?$AAe?$AAS?$AAe?$AAc?$AAt?$AAo?$AAr?$AA?$AN?$AA?6?$AA?$AA@ 0001b3fc     sdmmc_boot_common_topaz_v1:sdfmd.obj
 0001:0000a428       ??_C@_1FM@HGKBNLAK@?$AAI?$AAN?$AAF?$AAO?$AA?3?$AA?5?$AAU?$AAp?$AAd?$AAa?$AAt?$AAe?$AA?5?$AAo?$AAf?$AA?5?$AAX?$AAL?$AAD?$AAR?$AA?5?$AAc?$AAo?$AAm?$AAp?$AAl?$AAe?$AAt?$AAe?$AAd?$AA?5?$AAs@ 0001b428     sdmmc_boot_common_topaz_v1:sdboot.obj
 0001:0000a484       ??_C@_1DO@IPBABNAH@?$AAE?$AAR?$AAR?$AAO?$AAR?$AA?3?$AA?5?$AAF?$AAa?$AAi?$AAl?$AAe?$AAd?$AA?5?$AAt?$AAo?$AA?5?$AAv?$AAe?$AAr?$AAi?$AAf?$AAy?$AA?5?$AAX?$AAL?$AAD?$AAR?$AA?$AN?$AA?6?$AA?$AA@ 0001b484     sdmmc_boot_common_topaz_v1:sdboot.obj
 0001:0000a4c4       ??_C@_1DO@IEFCICMH@?$AAE?$AAR?$AAR?$AAO?$AAR?$AA?3?$AA?5?$AAF?$AAa?$AAi?$AAl?$AAe?$AAd?$AA?5?$AAt?$AAo?$AA?5?$AAu?$AAp?$AAd?$AAa?$AAt?$AAe?$AA?5?$AAX?$AAL?$AAD?$AAR?$AA?$AN?$AA?6?$AA?$AA@ 0001b4c4     sdmmc_boot_common_topaz_v1:sdboot.obj
 0001:0000a508       ??_C@_1IE@MIHIAOEN@?$AAI?$AAN?$AAF?$AAO?$AA?3?$AA?5?$AAU?$AAs?$AAi?$AAn?$AAg?$AA?5?$AAX?$AAL?$AAD?$AAR?$AA?5?$AAi?$AAm?$AAa?$AAg?$AAe?$AA?5?$AAf?$AAr?$AAo?$AAm?$AA?5?$AAf?$AAl?$AAa?$AAs@ 0001b508     sdmmc_boot_common_topaz_v1:sdboot.obj
 0001:0000a58c       ??_C@_1DK@GMPPEKDD@?$AAE?$AAR?$AAR?$AAO?$AAR?$AA?3?$AA?5?$AAX?$AAL?$AAD?$AAR?$AA?5?$AAe?$AAx?$AAc?$AAe?$AAe?$AAd?$AAs?$AA?5?$AA8?$AAK?$AAB?$AAy?$AAt?$AAe?$AA?$AN?$AA?6?$AA?$AA@ 0001b58c     sdmmc_boot_common_topaz_v1:sdboot.obj
 0001:0000a5c8       ??_C@_1FO@NFJLBPCM@?$AAE?$AAR?$AAR?$AAO?$AAR?$AA?3?$AA?5?$AAU?$AAn?$AAa?$AAb?$AAl?$AAe?$AA?5?$AAt?$AAo?$AA?5?$AAg?$AAe?$AAt?$AA?5?$AAS?$AAD?$AAH?$AAC?$AA?5?$AAf?$AAl?$AAa?$AAs?$AAh?$AA?5@ 0001b5c8     sdmmc_boot_common_topaz_v1:sdboot.obj
 0001:0000a628       ??_C@_1GI@PAGBENED@?$AAI?$AAN?$AAF?$AAO?$AA?3?$AA?5?$AAW?$AAr?$AAi?$AAt?$AAi?$AAn?$AAg?$AA?5?$AAX?$AAL?$AAD?$AAR?$AA?5?$AAi?$AAm?$AAa?$AAg?$AAe?$AA?5?$AAt?$AAo?$AA?5?$AAS?$AAD?$AAH?$AAC@ 0001b628     sdmmc_boot_common_topaz_v1:sdboot.obj
 0001:0000a690       ??_C@_1HM@GPHFIKP@?$AAW?$AAA?$AAR?$AAN?$AAI?$AAN?$AAG?$AA?3?$AA?5?$AAS?$AAD?$AAH?$AAC?$AA?5?$AAd?$AAe?$AAv?$AAi?$AAc?$AAe?$AA?5?$AAd?$AAo?$AAe?$AAs?$AAn?$AA?8?$AAt?$AA?5?$AAe?$AAx?$AAi@ 0001b690     sdmmc_boot_common_topaz_v1:sdboot.obj
 0001:0000a710       ??_C@_1GK@INEJNNDE@?$AAI?$AAN?$AAF?$AAO?$AA?3?$AA?5?$AAU?$AAp?$AAd?$AAa?$AAt?$AAe?$AA?5?$AAo?$AAf?$AA?5?$AAE?$AAB?$AAO?$AAO?$AAT?$AA?1?$AAS?$AAB?$AAO?$AAO?$AAT?$AA?5?$AAc?$AAo?$AAm?$AAp@ 0001b710     sdmmc_boot_common_topaz_v1:sdboot.obj
 0001:0000a77c       ??_C@_1DA@NFBIIBEK@?$AAI?$AAN?$AAF?$AAO?$AA?3?$AA?5?$AAV?$AAe?$AAr?$AAi?$AAf?$AAy?$AAi?$AAn?$AAg?$AA?5?$AAi?$AAm?$AAa?$AAg?$AAe?$AA?$AN?$AA?6?$AA?$AA@ 0001b77c     sdmmc_boot_common_topaz_v1:sdboot.obj
 0001:0000a7b0       ??_C@_1EM@CONNIEHK@?$AAE?$AAR?$AAR?$AAO?$AAR?$AA?3?$AA?5?$AAF?$AAa?$AAi?$AAl?$AAe?$AAd?$AA?5?$AAt?$AAo?$AA?5?$AAv?$AAe?$AAr?$AAi?$AAf?$AAy?$AA?5?$AAE?$AAB?$AAO?$AAO?$AAT?$AA?1?$AAS?$AAB@ 0001b7b0     sdmmc_boot_common_topaz_v1:sdboot.obj
 0001:0000a800       ??_C@_1EM@CAHDGELK@?$AAE?$AAR?$AAR?$AAO?$AAR?$AA?3?$AA?5?$AAF?$AAa?$AAi?$AAl?$AAe?$AAd?$AA?5?$AAt?$AAo?$AA?5?$AAu?$AAp?$AAd?$AAa?$AAt?$AAe?$AA?5?$AAE?$AAB?$AAO?$AAO?$AAT?$AA?1?$AAS?$AAB@ 0001b800     sdmmc_boot_common_topaz_v1:sdboot.obj
 0001:0000a850       ??_C@_1JO@FOINDKLK@?$AAI?$AAN?$AAF?$AAO?$AA?3?$AA?5?$AAP?$AAr?$AAo?$AAg?$AAr?$AAa?$AAm?$AAm?$AAi?$AAn?$AAg?$AA?5?$AAE?$AAB?$AAO?$AAO?$AAT?$AA?1?$AAS?$AAB?$AAO?$AAO?$AAT?$AA?5?$AAi?$AAm@ 0001b850     sdmmc_boot_common_topaz_v1:sdboot.obj
 0001:0000a8f0       ??_C@_1HM@DCFPNGII@?$AAE?$AAR?$AAR?$AAO?$AAR?$AA?3?$AA?5?$AAB?$AAo?$AAo?$AAt?$AA?5?$AAs?$AAi?$AAz?$AAe?$AA?5?$AAe?$AAx?$AAc?$AAe?$AAe?$AAd?$AAs?$AA?5?$AAr?$AAe?$AAs?$AAe?$AAr?$AAv?$AAe@ 0001b8f0     sdmmc_boot_common_topaz_v1:sdboot.obj
 0001:0000a970       ??_C@_1GI@NJJHBKOL@?$AAI?$AAN?$AAF?$AAO?$AA?3?$AA?5?$AAW?$AAr?$AAi?$AAt?$AAi?$AAn?$AAg?$AA?5?$AAB?$AAo?$AAo?$AAt?$AA?5?$AAi?$AAm?$AAa?$AAg?$AAe?$AA?5?$AAt?$AAo?$AA?5?$AAS?$AAD?$AAH?$AAC@ 0001b970     sdmmc_boot_common_topaz_v1:sdboot.obj
 0001:0000a9d8       ??_C@_1HK@PMKICAA@?$AAW?$AAA?$AAR?$AAN?$AAI?$AAN?$AAG?$AA?3?$AA?5?$AAS?$AAD?$AAH?$AAC?$AA?5?$AAd?$AAe?$AAv?$AAi?$AAc?$AAe?$AA?5?$AAd?$AAo?$AAe?$AAs?$AAn?$AA?8?$AAt?$AA?5?$AAe?$AAx?$AAi@ 0001b9d8     sdmmc_boot_common_topaz_v1:sdboot.obj
 0001:0000aa58       ??_C@_1FI@HDIKOHMP@?$AAI?$AAN?$AAF?$AAO?$AA?3?$AA?5?$AAU?$AAp?$AAd?$AAa?$AAt?$AAe?$AA?5?$AAo?$AAf?$AA?5?$AAN?$AAK?$AA?5?$AAc?$AAo?$AAm?$AAp?$AAl?$AAe?$AAt?$AAe?$AAd?$AA?5?$AAs?$AAu?$AAc@ 0001ba58     sdmmc_boot_common_topaz_v1:sdboot.obj
 0001:0000aab0       ??_C@_1DM@JEMNAJHC@?$AAI?$AAN?$AAF?$AAO?$AA?3?$AA?5?$AAv?$AAe?$AAr?$AAi?$AAf?$AAy?$AA?5?$AAi?$AAs?$AA?5?$AA?$CF?$AAd?$AA?$CF?$AA?$CF?$AA?5?$AAc?$AAo?$AAm?$AAp?$AAl?$AAe?$AAt?$AAe?$AA?$AA@ 0001bab0     sdmmc_boot_common_topaz_v1:sdboot.obj
 0001:0000aaec       ??_C@_1DK@IOAADILK@?$AAE?$AAR?$AAR?$AAO?$AAR?$AA?3?$AA?5?$AAF?$AAa?$AAi?$AAl?$AAe?$AAd?$AA?5?$AAt?$AAo?$AA?5?$AAv?$AAe?$AAr?$AAi?$AAf?$AAy?$AA?5?$AAN?$AAK?$AA?$AN?$AA?6?$AA?$AA@ 0001baec     sdmmc_boot_common_topaz_v1:sdboot.obj
 0001:0000ab28       ??_C@_1DE@CPANDEFA@?$AA?$AN?$AA?6?$AAI?$AAN?$AAF?$AAO?$AA?3?$AA?5?$AAV?$AAe?$AAr?$AAi?$AAf?$AAy?$AAi?$AAn?$AAg?$AA?5?$AAi?$AAm?$AAa?$AAg?$AAe?$AA?$AN?$AA?6?$AA?$AA@ 0001bb28     sdmmc_boot_common_topaz_v1:sdboot.obj
 0001:0000ab60       ??_C@_1GC@LOPKINJG@?$AA?$AN?$AA?6?$AAI?$AAN?$AAF?$AAO?$AA?3?$AA?5?$AAR?$AAe?$AAa?$AAd?$AAi?$AAn?$AAg?$AA?5?$AAi?$AAm?$AAa?$AAg?$AAe?$AA?5?$AAi?$AAn?$AA?5?$AAS?$AAD?$AAH?$AAC?$AA?5?$AAf?$AAo@ 0001bb60     sdmmc_boot_common_topaz_v1:sdboot.obj
 0001:0000abc4       ??_C@_1DO@GNNMCPKP@?$AAI?$AAN?$AAF?$AAO?$AA?3?$AA?5?$AAP?$AAr?$AAo?$AAg?$AAr?$AAa?$AAm?$AA?5?$AAi?$AAs?$AA?5?$AA?$CF?$AAd?$AA?$CF?$AA?$CF?$AA?5?$AAc?$AAo?$AAm?$AAp?$AAl?$AAe?$AAt?$AAe?$AA?$AA@ 0001bbc4     sdmmc_boot_common_topaz_v1:sdboot.obj
 0001:0000ac04       ??_C@_1DK@GKBEACFD@?$AAE?$AAR?$AAR?$AAO?$AAR?$AA?3?$AA?5?$AAF?$AAa?$AAi?$AAl?$AAe?$AAd?$AA?5?$AAt?$AAo?$AA?5?$AAu?$AAp?$AAd?$AAa?$AAt?$AAe?$AA?5?$AAN?$AAK?$AA?$AN?$AA?6?$AA?$AA@ 0001bc04     sdmmc_boot_common_topaz_v1:sdboot.obj
 0001:0000ac40       ??_C@_1IM@ILPGEKDA@?$AAI?$AAN?$AAF?$AAO?$AA?3?$AA?5?$AAP?$AAr?$AAo?$AAg?$AAr?$AAa?$AAm?$AAm?$AAi?$AAn?$AAg?$AA?5?$AAN?$AAK?$AA?5?$AAi?$AAm?$AAa?$AAg?$AAe?$AA?5?$AAf?$AAr?$AAo?$AAm?$AA?5@ 0001bc40     sdmmc_boot_common_topaz_v1:sdboot.obj
 0001:0000acd0       ??_C@_1HI@INNNJHLH@?$AAE?$AAR?$AAR?$AAO?$AAR?$AA?3?$AA?5?$AAN?$AAK?$AA?5?$AAs?$AAi?$AAz?$AAe?$AA?5?$AAe?$AAx?$AAc?$AAe?$AAe?$AAd?$AAs?$AA?5?$AAr?$AAe?$AAs?$AAe?$AAr?$AAv?$AAe?$AAd?$AA?5@ 0001bcd0     sdmmc_boot_common_topaz_v1:sdboot.obj
 0001:0000ad48       ??_C@_1FM@GMIEOAPE@?$AAE?$AAR?$AAR?$AAO?$AAR?$AA?3?$AA?5?$AAU?$AAn?$AAa?$AAb?$AAl?$AAe?$AA?5?$AAt?$AAo?$AA?5?$AAg?$AAe?$AAt?$AA?5?$AAS?$AAD?$AAH?$AAC?$AA?5?$AAf?$AAl?$AAa?$AAs?$AAh?$AA?5@ 0001bd48     sdmmc_boot_common_topaz_v1:sdboot.obj
 0001:0000ada8       ??_C@_1GE@DKMGNIPK@?$AAI?$AAN?$AAF?$AAO?$AA?3?$AA?5?$AAW?$AAr?$AAi?$AAt?$AAi?$AAn?$AAg?$AA?5?$AAN?$AAK?$AA?5?$AAi?$AAm?$AAa?$AAg?$AAe?$AA?5?$AAt?$AAo?$AA?5?$AAS?$AAD?$AAH?$AAC?$AA?5?$AA?$CI@ 0001bda8     sdmmc_boot_common_topaz_v1:sdboot.obj
 0001:0000ae10       ??_C@_1FI@CEHAOHOH@?$AA?$AN?$AA?6?$AAI?$AAN?$AAF?$AAO?$AA?3?$AA?5?$AAC?$AAo?$AAp?$AAy?$AA?5?$AAo?$AAf?$AA?5?$AAN?$AAK?$AA?5?$AAc?$AAo?$AAm?$AAp?$AAl?$AAe?$AAt?$AAe?$AAd?$AA?5?$AAs?$AAu?$AAc@ 0001be10     sdmmc_boot_common_topaz_v1:sdboot.obj
 0001:0000ae68       ??_C@_1DI@NDNNHKBF@?$AAI?$AAN?$AAF?$AAO?$AA?3?$AA?5?$AAR?$AAe?$AAa?$AAd?$AA?5?$AAi?$AAs?$AA?5?$AA?$CF?$AAd?$AA?$CF?$AA?$CF?$AA?5?$AAc?$AAo?$AAm?$AAp?$AAl?$AAe?$AAt?$AAe?$AA?$AA@ 0001be68     sdmmc_boot_common_topaz_v1:sdboot.obj
 0001:0000aea0       ??_C@_1FK@KMBLLLAA@?$AAI?$AAN?$AAF?$AAO?$AA?3?$AA?5?$AAC?$AAo?$AAp?$AAy?$AAi?$AAn?$AAg?$AA?5?$AAN?$AAK?$AA?5?$AAi?$AAm?$AAa?$AAg?$AAe?$AA?5?$AAt?$AAo?$AA?5?$AAR?$AAA?$AAM?$AA?5?$AAa?$AAd@ 0001bea0     sdmmc_boot_common_topaz_v1:sdboot.obj
 0001:0000af00       ??_C@_1GE@BKANAINO@?$AAI?$AAN?$AAF?$AAO?$AA?3?$AA?5?$AAR?$AAe?$AAa?$AAd?$AAi?$AAn?$AAg?$AA?5?$AAN?$AAK?$AA?5?$AAi?$AAm?$AAa?$AAg?$AAe?$AA?5?$AAt?$AAo?$AA?5?$AAS?$AAD?$AAH?$AAC?$AA?5?$AA?$CI@ 0001bf00     sdmmc_boot_common_topaz_v1:sdboot.obj
 0001:0000af68       ??_C@_1HI@KICDEAL@?$AAW?$AAA?$AAR?$AAN?$AAI?$AAN?$AAG?$AA?3?$AA?5?$AAS?$AAD?$AAH?$AAC?$AA?5?$AAd?$AAe?$AAv?$AAi?$AAc?$AAe?$AA?5?$AAd?$AAo?$AAe?$AAs?$AAn?$AA?8?$AAt?$AA?5?$AAe?$AAx?$AAi@ 0001bf68     sdmmc_boot_common_topaz_v1:sdboot.obj
 0001:0000afe0       ??_C@_1GE@GKLJAFOG@?$AA?$AN?$AA?6?$AAI?$AAN?$AAF?$AAO?$AA?3?$AA?5?$AAF?$AAo?$AAr?$AAm?$AAa?$AAt?$AA?5?$AAo?$AAf?$AA?5?$AAS?$AAD?$AA?1?$AAM?$AAM?$AAC?$AA?5?$AAc?$AAo?$AAm?$AAp?$AAl?$AAe?$AAt@ 0001bfe0     sdmmc_boot_common_topaz_v1:sdboot.obj
 0001:0000b044       ??_C@_1CC@LEGAKGAE@?$AAM?$AAB?$AAR?$AA?5?$AAC?$AAl?$AAe?$AAa?$AAr?$AA?5?$AAF?$AAa?$AAi?$AAl?$AA?$AN?$AA?6?$AA?$AA@ 0001c044     sdmmc_boot_common_topaz_v1:sdboot.obj
 0001:0000b068       ??_C@_1HC@PNJDDN@?$AAE?$AAR?$AAR?$AAO?$AAR?$AA?3?$AA?5?$AAU?$AAn?$AAa?$AAb?$AAl?$AAe?$AA?5?$AAt?$AAo?$AA?5?$AAe?$AAr?$AAa?$AAs?$AAe?$AA?5?$AAS?$AAD?$AAH?$AAC?$AA?5?$AA?5?$AAb?$AAl?$AAo@ 0001c068     sdmmc_boot_common_topaz_v1:sdboot.obj
 0001:0000b0e0       ??_C@_1EO@LDCMAOK@?$AAI?$AAN?$AAF?$AAO?$AA?3?$AA?5?$AAS?$AAt?$AAa?$AAr?$AAt?$AAi?$AAn?$AAg?$AA?5?$AAf?$AAo?$AAr?$AAm?$AAa?$AAt?$AA?5?$AAo?$AAf?$AA?5?$AAS?$AAD?$AA?1?$AAM?$AAM?$AAC?$AA?5@ 0001c0e0     sdmmc_boot_common_topaz_v1:sdboot.obj
 0001:0000b130       ??_C@_1HG@EOAOKIDM@?$AAE?$AAr?$AAr?$AAo?$AAr?$AA?5?$AAc?$AAr?$AAe?$AAa?$AAt?$AAi?$AAn?$AAg?$AA?5?$AAf?$AAi?$AAl?$AAe?$AA?5?$AAs?$AAy?$AAs?$AAt?$AAe?$AAm?$AA?5?$AAp?$AAa?$AAr?$AAt?$AAi@ 0001c130     sdmmc_boot_common_topaz_v1:sdboot.obj
 0001:0000b1a8       ??_C@_1JI@IILMJNEC@?$AA?5?$AAB?$AAo?$AAo?$AAt?$AA?5?$AAP?$AAa?$AAr?$AAt?$AAi?$AAt?$AAi?$AAo?$AAn?$AA?5?$AAs?$AAi?$AAz?$AAe?$AA?5?$AA?$DN?$AA?5?$AA?$CF?$AAd?$AA?5?$AAK?$AAb?$AAy?$AAt?$AAe?$AAs@ 0001c1a8     sdmmc_boot_common_topaz_v1:sdboot.obj
 0001:0000b240       ??_C@_1EK@OOHHLFLF@?$AAS?$AAu?$AAc?$AAc?$AAe?$AAs?$AAs?$AAf?$AAu?$AAl?$AAl?$AAy?$AA?5?$AAc?$AAr?$AAe?$AAa?$AAt?$AAe?$AAd?$AA?5?$AA2?$AA?5?$AAp?$AAa?$AAr?$AAt?$AAi?$AAt?$AAi?$AAo?$AAn@ 0001c240     sdmmc_boot_common_topaz_v1:sdboot.obj
 0001:0000b290       ??_C@_1LE@LFABDNNE@?$AA?$AN?$AA?6?$AAC?$AAa?$AAn?$AAn?$AAo?$AAt?$AA?5?$AAc?$AAr?$AAe?$AAa?$AAt?$AAe?$AA?5?$AAf?$AAi?$AAl?$AAe?$AA?5?$AAs?$AAy?$AAs?$AAt?$AAe?$AAm?$AA?5?$AAp?$AAa?$AAr?$AAi@ 0001c290     sdmmc_boot_common_topaz_v1:sdboot.obj
 0001:0000b348       ??_C@_1NA@NCJLFGCL@?$AA?$AN?$AA?6?$AAP?$AAl?$AAe?$AAa?$AAs?$AAe?$AA?5?$AAc?$AAr?$AAe?$AAa?$AAt?$AAe?$AA?5?$AAf?$AAi?$AAl?$AAe?$AA?5?$AAs?$AAy?$AAs?$AAt?$AAe?$AAm?$AA?5?$AAp?$AAa?$AAr?$AAt@ 0001c348     sdmmc_boot_common_topaz_v1:sdboot.obj
 0001:0000b418       ??_C@_1HC@CIAMDLCK@?$AAI?$AAN?$AAF?$AAO?$AA?3?$AA?5?$AAS?$AAu?$AAc?$AAc?$AAe?$AAs?$AAs?$AAf?$AAu?$AAl?$AAl?$AAy?$AA?5?$AAl?$AAo?$AAa?$AAd?$AAe?$AAd?$AA?5?$AAb?$AAo?$AAo?$AAt?$AA?5?$AAc@ 0001c418     sdmmc_boot_common_topaz_v1:sdboot.obj
 0001:0000b490       ??_C@_1GK@EOGIHKBG@?$AAE?$AAR?$AAR?$AAO?$AAR?$AA?3?$AA?5?$AAF?$AAa?$AAi?$AAl?$AAe?$AAd?$AA?5?$AAt?$AAo?$AA?5?$AAl?$AAo?$AAa?$AAd?$AA?5?$AAb?$AAo?$AAo?$AAt?$AA?5?$AAc?$AAo?$AAn?$AAf?$AAi@ 0001c490     sdmmc_boot_common_topaz_v1:sdboot.obj
 0001:0000b500       ??_C@_1FK@IEJDCBJC@?$AAI?$AAN?$AAF?$AAO?$AA?3?$AA?5?$AAL?$AAo?$AAa?$AAd?$AAi?$AAn?$AAg?$AA?5?$AAb?$AAo?$AAo?$AAt?$AA?5?$AAc?$AAo?$AAn?$AAf?$AAi?$AAg?$AAu?$AAr?$AAa?$AAt?$AAi?$AAo?$AAn@ 0001c500     sdmmc_boot_common_topaz_v1:sdboot.obj
 0001:0000b560       ??_C@_1GO@NKNNIIPK@?$AAI?$AAN?$AAF?$AAO?$AA?3?$AA?5?$AAS?$AAu?$AAc?$AAc?$AAe?$AAs?$AAs?$AAf?$AAu?$AAl?$AAl?$AAy?$AA?5?$AAs?$AAt?$AAo?$AAr?$AAe?$AAd?$AA?5?$AAb?$AAo?$AAo?$AAt?$AA?5?$AAc@ 0001c560     sdmmc_boot_common_topaz_v1:sdboot.obj
 0001:0000b5d0       ??_C@_1FK@CIBKLOOG@?$AAE?$AAR?$AAR?$AAO?$AAR?$AA?3?$AA?5?$AAF?$AAa?$AAi?$AAl?$AAe?$AAd?$AA?5?$AAt?$AAo?$AA?5?$AAu?$AAp?$AAd?$AAa?$AAt?$AAe?$AA?5?$AAB?$AAO?$AAO?$AAT?$AA?5?$AAc?$AAo?$AAn@ 0001c5d0     sdmmc_boot_common_topaz_v1:sdboot.obj
 0001:0000b630       ??_C@_1FG@KFKBJHMH@?$AAI?$AAN?$AAF?$AAO?$AA?3?$AA?5?$AAS?$AAt?$AAo?$AAr?$AAi?$AAn?$AAg?$AA?5?$AAb?$AAo?$AAo?$AAt?$AA?5?$AAc?$AAo?$AAn?$AAf?$AAi?$AAg?$AAu?$AAr?$AAa?$AAt?$AAi?$AAo?$AAn@ 0001c630     sdmmc_boot_common_topaz_v1:sdboot.obj
 0001:0000b688       ??_C@_1HI@KJHFFFK@?$AA?$AN?$AA?6?$AAC?$AAh?$AAa?$AAn?$AAg?$AAe?$AA?5?$AAb?$AAo?$AAo?$AAt?$AA?5?$AAp?$AAa?$AAr?$AAt?$AAi?$AAt?$AAi?$AAo?$AAn?$AA?5?$AAs?$AAi?$AAz?$AAe?$AA?5?$AAt?$AAo?$AA?5@ 0001c688     sdmmc_boot_common_topaz_v1:sdboot.obj
 0001:0000b700       ??_C@_1CM@NNNFPDLJ@?$AA?$AN?$AA?6?$AAe?$AAM?$AAM?$AAC?$AA?5?$AAn?$AAo?$AAt?$AA?5?$AAp?$AAr?$AAe?$AAs?$AAe?$AAn?$AAt?$AA?$CB?$AA?$AN?$AA?6?$AA?$AA@ 0001c700     sdmmc_boot_common_topaz_v1:sdboot.obj
 0001:0000b730       ??_C@_1KI@FPGGMGIK@?$AA?$AN?$AA?6?$AAE?$AAi?$AAt?$AAh?$AAe?$AAr?$AA?5?$AAt?$AAh?$AAi?$AAs?$AA?5?$AAi?$AAs?$AA?5?$AAn?$AAo?$AAt?$AA?5?$AAa?$AAn?$AA?5?$AAe?$AAM?$AAM?$AAC?$AA?5?$AA4?$AA?4?$AA3@ 0001c730     sdmmc_boot_common_topaz_v1:sdboot.obj
 0001:0000b7d8       ??_C@_1EO@EADFBCC@?$AA?$AN?$AA?6?$AAC?$AAh?$AAa?$AAn?$AAg?$AAi?$AAn?$AAg?$AA?5?$AAb?$AAo?$AAo?$AAt?$AA?5?$AAp?$AAa?$AAr?$AAt?$AAi?$AAt?$AAi?$AAo?$AAn?$AA?5?$AAs?$AAi?$AAz?$AAe?$AA?5?$AAt@ 0001c7d8     sdmmc_boot_common_topaz_v1:sdboot.obj
 0001:0000b828       ??_C@_1IE@FBCOHJCH@?$AAE?$AAi?$AAt?$AAh?$AAe?$AAr?$AA?5?$AAc?$AAa?$AAr?$AAd?$AA?5?$AAi?$AAs?$AA?5?$AAn?$AAo?$AAt?$AA?5?$AAe?$AAS?$AAD?$AA2?$AA?4?$AA1?$AA?0?$AA?5?$AAo?$AAr?$AA?5?$AAb?$AAo@ 0001c828     sdmmc_boot_common_topaz_v1:sdboot.obj
 0001:0000b8b0       ??_C@_1EI@GPPELNIK@?$AAF?$AAa?$AAi?$AAl?$AAe?$AAd?$AA?5?$AAt?$AAo?$AA?5?$AAs?$AAe?$AAt?$AA?5?$AAa?$AAc?$AAt?$AAi?$AAv?$AAe?$AA?5?$AAp?$AAa?$AAr?$AAt?$AAi?$AAt?$AAi?$AAo?$AAn?$AA?5?$AA?$CF@ 0001c8b0     sdmmc_boot_common_topaz_v1:sdboot.obj
 0001:0000b8f8       ??_C@_1CO@HLNOOPDD@?$AAP?$AAa?$AAr?$AAt?$AAi?$AAt?$AAi?$AAo?$AAn?$AA?5?$AA?$CF?$AAd?$AA?5?$AAe?$AAn?$AAa?$AAb?$AAl?$AAe?$AAd?$AA?$AN?$AA?6?$AA?$AA@ 0001c8f8     sdmmc_boot_common_topaz_v1:sdboot.obj
 0001:0000b928       ??_C@_1CK@BEDMMKID@?$AA?$AN?$AA?6?$AAe?$AAS?$AAD?$AA?5?$AAn?$AAo?$AAt?$AA?5?$AAp?$AAr?$AAe?$AAs?$AAe?$AAn?$AAt?$AA?$CB?$AA?$AN?$AA?6?$AA?$AA@ 0001c928     sdmmc_boot_common_topaz_v1:sdboot.obj
 0001:0000b958       ??_C@_1EE@CDLOKFNI@?$AAE?$AAR?$AAR?$AAO?$AAR?$AA?3?$AA?5?$AAF?$AAa?$AAi?$AAl?$AAe?$AAd?$AA?5?$AAt?$AAo?$AA?5?$AAr?$AAe?$AAa?$AAd?$AA?5?$AAf?$AAr?$AAo?$AAm?$AA?5?$AAS?$AAD?$AAH?$AAC?$AA?$AN@ 0001c958     sdmmc_boot_common_topaz_v1:sdboot.obj
 0001:0000b99c       ??_C@_1CK@CDKNMNLE@?$AAI?$AAN?$AAF?$AAO?$AA?3?$AA?5?$AAp?$AAB?$AAu?$AAf?$AAf?$AAe?$AAr?$AA?5?$AAN?$AAU?$AAL?$AAL?$AA?$AN?$AA?6?$AA?$AA@ 0001c99c     sdmmc_boot_common_topaz_v1:sdboot.obj
 0001:0000b9c8       ??_C@_1EI@EJJFEBCP@?$AAE?$AAR?$AAR?$AAO?$AAR?$AA?3?$AA?5?$AAc?$AAa?$AAn?$AAn?$AA?8?$AAt?$AA?5?$AAo?$AAp?$AAe?$AAn?$AA?5?$AAi?$AAm?$AAa?$AAg?$AAe?$AA?5?$AAf?$AAi?$AAl?$AAe?$AA?8?$AA?$CF?$AAS@ 0001c9c8     sdmmc_boot_common_topaz_v1:sdboot.obj
 0001:0000ba10       ??_C@_1EG@NDNAGFDE@?$AAS?$AAD?$AAM?$AAM?$AAC?$AAD?$AAo?$AAw?$AAn?$AAl?$AAo?$AAa?$AAd?$AA?5?$AA?3?$AA?5?$AAF?$AAA?$AAT?$AAI?$AAn?$AAi?$AAt?$AAD?$AAi?$AAs?$AAk?$AA?5?$AAF?$AAa?$AAi?$AAl@ 0001ca10     sdmmc_boot_common_topaz_v1:sdboot.obj
 0001:0000ba58       ??_C@_1EC@HHKHODCC@?$AAE?$AAR?$AAR?$AAO?$AAR?$AA?3?$AA?5?$AAr?$AAe?$AAa?$AAd?$AA?5?$AAi?$AAm?$AAa?$AAg?$AAe?$AA?5?$AAd?$AAa?$AAt?$AAa?$AA?5?$AAf?$AAa?$AAi?$AAl?$AAu?$AAr?$AAe?$AA?$AN?$AA?6@ 0001ca58     sdmmc_boot_common_topaz_v1:sdboot.obj
 0001:0000ba9c       ??_C@_13MOEPKPHB@?$AA?$DO?$AA?$AA@ 0001ca9c     sdmmc_boot_common_topaz_v1:sdboot.obj
 0001:0000baa0       ??_C@_1BI@GFBPCEKM@?$AA?9?$AA?5?$AAS?$AAD?$AA_?$AAI?$AAn?$AAi?$AAt?$AA?$AN?$AA?6?$AA?$AA@ 0001caa0     sdmmc_boot_common_topaz_v1:sd.obj
 0001:0000bab8       ??_C@_1DK@IPMKPGIA@?$AAS?$AAD?$AA?3?$AA?5?$AAS?$AAw?$AAi?$AAt?$AAc?$AAh?$AAe?$AAd?$AA?5?$AAt?$AAo?$AA?5?$AA4?$AA?5?$AAb?$AAi?$AAt?$AA?5?$AAm?$AAo?$AAd?$AAe?$AA?$AN?$AA?6?$AA?$AA@ 0001cab8     sdmmc_boot_common_topaz_v1:sd.obj
 0001:0000baf4       ??_C@_1BI@NFCCHGPM@?$AA?$CL?$AA?5?$AAS?$AAD?$AA_?$AAI?$AAn?$AAi?$AAt?$AA?$AN?$AA?6?$AA?$AA@ 0001caf4     sdmmc_boot_common_topaz_v1:sd.obj
 0001:0000bb0c       ??_C@_1DC@EDAIFJBN@?$AA?9?$AA?5?$AAS?$AAD?$AA_?$AAV?$AAo?$AAl?$AAt?$AAa?$AAg?$AAe?$AAV?$AAa?$AAl?$AAi?$AAd?$AAa?$AAt?$AAi?$AAo?$AAn?$AA?$AN?$AA?6?$AA?$AA@ 0001cb0c     sdmmc_boot_common_topaz_v1:sd.obj
 0001:0000bb40       ??_C@_1CM@KKGBLIBK@?$AAS?$AAD?$AA?5?$AAL?$AAo?$AAw?$AA?5?$AAD?$AAe?$AAn?$AAs?$AAi?$AAt?$AAy?$AA?5?$AAc?$AAa?$AAr?$AAd?$AA?$AN?$AA?6?$AA?$AA@ 0001cb40     sdmmc_boot_common_topaz_v1:sd.obj
 0001:0000bb6c       ??_C@_1CO@JHLEOIFJ@?$AAS?$AAD?$AA?5?$AAH?$AAi?$AAg?$AAh?$AA?5?$AAD?$AAe?$AAn?$AAs?$AAi?$AAt?$AAy?$AA?5?$AAc?$AAa?$AAr?$AAd?$AA?$AN?$AA?6?$AA?$AA@ 0001cb6c     sdmmc_boot_common_topaz_v1:sd.obj
 0001:0000bb9c       ??_C@_1CE@HCMHAKBK@?$AAS?$AAD?$AA?5?$AAO?$AAC?$AAR?$AA?5?$AAV?$AAa?$AAl?$AAu?$AAe?$AA?5?$AA?$CF?$AAx?$AA?$AN?$AA?6?$AA?$AA@ 0001cb9c     sdmmc_boot_common_topaz_v1:sd.obj
 0001:0000bbc0       ??_C@_1DC@ONEMABLJ@?$AA?$CL?$AA?5?$AAS?$AAD?$AA_?$AAV?$AAo?$AAl?$AAt?$AAa?$AAg?$AAe?$AAV?$AAa?$AAl?$AAi?$AAd?$AAa?$AAt?$AAi?$AAo?$AAn?$AA?$AN?$AA?6?$AA?$AA@ 0001cbc0     sdmmc_boot_common_topaz_v1:sd.obj
 0001:0000bbf4       ??_C@_1CC@IOCDEEML@?$AA?9?$AA?5?$AAS?$AAD?$AAG?$AAe?$AAt?$AAB?$AAi?$AAt?$AAM?$AAo?$AAd?$AAe?$AA?$AN?$AA?6?$AA?$AA@ 0001cbf4     sdmmc_boot_common_topaz_v1:sd.obj
 0001:0000bc18       ??_C@_1CC@FFCOKCHP@?$AA?$CL?$AA?5?$AAS?$AAD?$AAG?$AAe?$AAt?$AAB?$AAi?$AAt?$AAM?$AAo?$AAd?$AAe?$AA?$AN?$AA?6?$AA?$AA@ 0001cc18     sdmmc_boot_common_topaz_v1:sd.obj
 0001:0000bc3c       ??_C@_1CE@FOGAOHPA@?$AA?9?$AA?5?$AAS?$AAD?$AAS?$AAe?$AAt?$AAB?$AAu?$AAs?$AAW?$AAi?$AAd?$AAt?$AAh?$AA?$AN?$AA?6?$AA?$AA@ 0001cc3c     sdmmc_boot_common_topaz_v1:sd.obj
 0001:0000bc60       ??_C@_1CE@JHKABAAM@?$AA?$CL?$AA?5?$AAS?$AAD?$AAS?$AAe?$AAt?$AAB?$AAu?$AAs?$AAW?$AAi?$AAd?$AAt?$AAh?$AA?$AN?$AA?6?$AA?$AA@ 0001cc60     sdmmc_boot_common_topaz_v1:sd.obj
 0001:0000bc84       ??_C@_1BK@OMGCLANO@?$AA?9?$AA?5?$AAM?$AAM?$AAC?$AA_?$AAI?$AAn?$AAi?$AAt?$AA?$AN?$AA?6?$AA?$AA@ 0001cc84     sdmmc_boot_common_topaz_v1:mmc.obj
 0001:0000bca0       ??_C@_1EG@EENAJDPB@?$AAM?$AAM?$AAC?$AA_?$AAI?$AAn?$AAi?$AAt?$AA?3?$AA?5?$AAU?$AAn?$AAa?$AAb?$AAl?$AAe?$AA?5?$AAt?$AAo?$AA?5?$AAr?$AAe?$AAa?$AAd?$AA?5?$AAE?$AAX?$AAT?$AA_?$AAC?$AAS?$AAD@ 0001cca0     sdmmc_boot_common_topaz_v1:mmc.obj
 0001:0000bce8       ??_C@_1DM@OPCKEIJH@?$AAM?$AAM?$AAC?$AA?3?$AA?5?$AAS?$AAw?$AAi?$AAt?$AAc?$AAh?$AAe?$AAd?$AA?5?$AAt?$AAo?$AA?5?$AA4?$AA?5?$AAb?$AAi?$AAt?$AA?5?$AAm?$AAo?$AAd?$AAe?$AA?$AN?$AA?6?$AA?$AA@ 0001cce8     sdmmc_boot_common_topaz_v1:mmc.obj
 0001:0000bd24       ??_C@_1BK@NDLMGNGP@?$AA?$CL?$AA?5?$AAM?$AAM?$AAC?$AA_?$AAI?$AAn?$AAi?$AAt?$AA?$AN?$AA?6?$AA?$AA@ 0001cd24     sdmmc_boot_common_topaz_v1:mmc.obj
 0001:0000bd40       ??_C@_1DE@LEIOOFBI@?$AA?9?$AA?5?$AAM?$AAM?$AAC?$AA_?$AAV?$AAo?$AAl?$AAt?$AAa?$AAg?$AAe?$AAV?$AAa?$AAl?$AAi?$AAd?$AAa?$AAt?$AAi?$AAo?$AAn?$AA?$AN?$AA?6?$AA?$AA@ 0001cd40     sdmmc_boot_common_topaz_v1:mmc.obj
 0001:0000bd74       ??_C@_1CO@HJHBDFIM@?$AAM?$AAM?$AAC?$AA?5?$AAL?$AAo?$AAw?$AA?5?$AAD?$AAe?$AAn?$AAs?$AAi?$AAt?$AAy?$AA?5?$AAc?$AAa?$AAr?$AAd?$AA?$AN?$AA?6?$AA?$AA@ 0001cd74     sdmmc_boot_common_topaz_v1:mmc.obj
 0001:0000bda4       ??_C@_1DA@CDKGOJEI@?$AAM?$AAM?$AAC?$AA?5?$AAH?$AAi?$AAg?$AAh?$AA?5?$AAD?$AAe?$AAn?$AAs?$AAi?$AAt?$AAy?$AA?5?$AAc?$AAa?$AAr?$AAd?$AA?$AN?$AA?6?$AA?$AA@ 0001cda4     sdmmc_boot_common_topaz_v1:mmc.obj
 0001:0000bdd4       ??_C@_1DE@BLFFOLHH@?$AA?$CL?$AA?5?$AAM?$AAM?$AAC?$AA_?$AAV?$AAo?$AAl?$AAt?$AAa?$AAg?$AAe?$AAV?$AAa?$AAl?$AAi?$AAd?$AAa?$AAt?$AAi?$AAo?$AAn?$AA?$AN?$AA?6?$AA?$AA@ 0001cdd4     sdmmc_boot_common_topaz_v1:mmc.obj
 0001:0000be08       ??_C@_1DA@BDPILAEO@?$AA?$CL?$AA?5?$AAM?$AAM?$AAC?$AA?5?$AAS?$AAp?$AAe?$AAc?$AA?5?$AAV?$AAe?$AAr?$AAs?$AAi?$AAo?$AAn?$AA?5?$AA?$CF?$AAx?$AA?$AN?$AA?6?$AA?$AA@ 0001ce08     sdmmc_boot_common_topaz_v1:mmc.obj
 0001:0000be38       ??_C@_1CI@PFANDIPJ@?$AA?9?$AA?5?$AAM?$AAM?$AAC?$AA_?$AAS?$AAe?$AAt?$AAB?$AAu?$AAs?$AAW?$AAi?$AAd?$AAt?$AAh?$AA?$AN?$AA?6?$AA?$AA@ 0001ce38     sdmmc_boot_common_topaz_v1:mmc.obj
 0001:0000be60       ??_C@_1CI@KAHEFJOJ@?$AA?$CL?$AA?5?$AAM?$AAM?$AAC?$AA_?$AAS?$AAe?$AAt?$AAB?$AAu?$AAs?$AAW?$AAi?$AAd?$AAt?$AAh?$AA?$AN?$AA?6?$AA?$AA@ 0001ce60     sdmmc_boot_common_topaz_v1:mmc.obj
 0001:0000be88       ??_C@_1DM@NOJDJLBD@?$AAW?$AAa?$AAr?$AAn?$AAi?$AAn?$AAg?$AA?5?$AA?3?$AA?5?$AAE?$AAn?$AAd?$AAi?$AAn?$AAg?$AAH?$AAe?$AAa?$AAd?$AA?5?$AA?$DN?$AA?5?$AA0?$AAx?$AA?$CF?$AAX?$AA?$AN?$AA?6?$AA?$AA@ 0001ce88     sdmmc_boot_common_topaz_v1:sdfat.obj
 0001:0000bec4       ??_C@_00CNPNBAHC@?$AA@     0001cec4     sdmmc_boot_common_topaz_v1:sdfat.obj
 0001:0000bec8       ??_C@_02FEEPBPGD@A?3?$AA@  0001cec8     sdmmc_boot_common_topaz_v1:sdfat.obj
 0001:0000bed0       ??_C@_1HG@CJLDOBEO@?$AA?$HM?$AA?$CF?$AA3?$AAd?$AA?$HM?$AA?5?$AA?5?$AA?$CF?$AA0?$AA2?$AAX?$AA?$HM?$AA?$CF?$AA4?$AAu?$AA?1?$AA?$CF?$AA5?$AAu?$AA?1?$AA?$CF?$AA6?$AAu?$AA?5?$AA?5?$AA?$CF?$AA4?$AAu?$AA?1?$AA?$CF?$AA5?$AAu@ 0001ced0     sdmmc_boot_common_topaz_v1:sdfat.obj
 0001:0000bf48       ??_C@_1KI@GBNIFLCN@?$AA?$HM?$AAN?$AAo?$AA?4?$AA?$HM?$AAB?$AAo?$AAo?$AAt?$AA?$HM?$AAH?$AAe?$AAa?$AAd?$AA?1?$AAT?$AAr?$AAa?$AAc?$AAk?$AA?1?$AAS?$AAe?$AAc?$AAt?$AAo?$AAr?$AA?9?$AA?9?$AAH?$AAe?$AAa@ 0001cf48     sdmmc_boot_common_topaz_v1:sdfat.obj
 0001:0000bff0       ??_C@_1CC@IKMNJHMA@?$AAS?$AAi?$AAg?$AAn?$AAa?$AAt?$AAu?$AAr?$AAe?$AA?3?$AA?$CF?$AA0?$AA4?$AAX?$AA?$AN?$AA?6?$AA?$AA@ 0001cff0     sdmmc_boot_common_topaz_v1:sdfat.obj
 0001:0000c014       ??_C@_1DK@HJPJNBAK@?$AAS?$AAi?$AAg?$AAn?$AAa?$AAt?$AAu?$AAr?$AAe?$AA?5?$AA?5?$AA?5?$AA?5?$AA?5?$AA?5?$AA?5?$AA?5?$AA?5?$AA?5?$AA?5?$AA?3?$AA?5?$AA?$CF?$AA0?$AA4?$AAX?$AA?$AN?$AA?6?$AA?$AA@ 0001d014     sdmmc_boot_common_topaz_v1:sdfat.obj
 0001:0000c050       ??_C@_1DK@NEBIKGGI@?$AAF?$AAi?$AAl?$AAe?$AAS?$AAy?$AAs?$AAt?$AAe?$AAm?$AAT?$AAy?$AAp?$AAe?$AA?5?$AA?5?$AA?5?$AA?5?$AA?5?$AA?5?$AA?3?$AA?5?$AA?$CF?$AA?4?$AA8?$AAS?$AA?$AN?$AA?6?$AA?$AA@ 0001d050     sdmmc_boot_common_topaz_v1:sdfat.obj
 0001:0000c08c       ??_C@_1DM@FDBDEINO@?$AAV?$AAo?$AAl?$AAu?$AAm?$AAe?$AAL?$AAa?$AAb?$AAe?$AAl?$AA?5?$AA?5?$AA?5?$AA?5?$AA?5?$AA?5?$AA?5?$AA?5?$AA?5?$AA?3?$AA?5?$AA?$CF?$AA?4?$AA1?$AA1?$AAS?$AA?$AN?$AA?6?$AA?$AA@ 0001d08c     sdmmc_boot_common_topaz_v1:sdfat.obj
 0001:0000c0c8       ??_C@_1DK@DLNFCHHN@?$AAV?$AAo?$AAl?$AAu?$AAm?$AAe?$AAS?$AAe?$AAr?$AAi?$AAa?$AAl?$AAN?$AAu?$AAm?$AAb?$AAe?$AAr?$AA?5?$AA?5?$AA?3?$AA?5?$AA?$CF?$AA0?$AA8?$AAX?$AA?$AN?$AA?6?$AA?$AA@ 0001d0c8     sdmmc_boot_common_topaz_v1:sdfat.obj
 0001:0000c104       ??_C@_1DK@JAHCBLJK@?$AAE?$AAF?$AAD?$AAC?$AAS?$AAi?$AAg?$AAn?$AAa?$AAt?$AAu?$AAr?$AAe?$AA?5?$AA?5?$AA?5?$AA?5?$AA?5?$AA?5?$AA?5?$AA?3?$AA?5?$AA?$CF?$AA0?$AA2?$AAX?$AA?$AN?$AA?6?$AA?$AA@ 0001d104     sdmmc_boot_common_topaz_v1:sdfat.obj
 0001:0000c140       ??_C@_1DK@ONNKMJ@?$AAP?$AAh?$AAy?$AAs?$AAi?$AAc?$AAa?$AAl?$AAD?$AAi?$AAs?$AAk?$AAN?$AAu?$AAm?$AAb?$AAe?$AAr?$AA?5?$AA?5?$AA?3?$AA?5?$AA?$CF?$AA0?$AA2?$AAX?$AA?$AN?$AA?6?$AA?$AA@ 0001d140     sdmmc_boot_common_topaz_v1:sdfat.obj
 0001:0000c17c       ??_C@_1DG@HFBEDJMA@?$AAB?$AAa?$AAc?$AAk?$AAu?$AAp?$AAB?$AAo?$AAo?$AAt?$AAS?$AAe?$AAc?$AAt?$AAo?$AAr?$AA?5?$AA?5?$AA?5?$AA?5?$AA?3?$AA?5?$AA?$CF?$AAu?$AA?$AN?$AA?6?$AA?$AA@ 0001d17c     sdmmc_boot_common_topaz_v1:sdfat.obj
 0001:0000c1b4       ??_C@_1DG@MDDBKMHF@?$AAF?$AAi?$AAl?$AAe?$AAS?$AAy?$AAs?$AAt?$AAe?$AAm?$AAI?$AAn?$AAf?$AAo?$AAm?$AAa?$AAt?$AAi?$AAo?$AAn?$AA?3?$AA?5?$AA?$CF?$AAu?$AA?$AN?$AA?6?$AA?$AA@ 0001d1b4     sdmmc_boot_common_topaz_v1:sdfat.obj
 0001:0000c1ec       ??_C@_1DG@PIEFEGDE@?$AAR?$AAo?$AAo?$AAt?$AAE?$AAn?$AAt?$AAr?$AAy?$AAC?$AAl?$AAu?$AAs?$AAt?$AAe?$AAr?$AA?5?$AA?5?$AA?5?$AA?5?$AA?3?$AA?5?$AA?$CF?$AAu?$AA?$AN?$AA?6?$AA?$AA@ 0001d1ec     sdmmc_boot_common_topaz_v1:sdfat.obj
 0001:0000c224       ??_C@_1DK@NEIHAJBN@?$AAF?$AAi?$AAl?$AAe?$AAS?$AAy?$AAs?$AAt?$AAe?$AAm?$AAV?$AAe?$AAr?$AAs?$AAi?$AAo?$AAn?$AA?5?$AA?5?$AA?5?$AA?3?$AA?5?$AA?$CF?$AA0?$AA4?$AAX?$AA?$AN?$AA?6?$AA?$AA@ 0001d224     sdmmc_boot_common_topaz_v1:sdfat.obj
 0001:0000c260       ??_C@_1DK@NJGNFLGN@?$AAE?$AAx?$AAt?$AAe?$AAn?$AAt?$AAF?$AAl?$AAa?$AAg?$AA?5?$AA?5?$AA?5?$AA?5?$AA?5?$AA?5?$AA?5?$AA?5?$AA?5?$AA?5?$AA?3?$AA?5?$AA?$CF?$AA0?$AA4?$AAX?$AA?$AN?$AA?6?$AA?$AA@ 0001d260     sdmmc_boot_common_topaz_v1:sdfat.obj
 0001:0000c29c       ??_C@_1DG@HEHNBAMA@?$AAS?$AAe?$AAc?$AAt?$AAo?$AAr?$AAP?$AAe?$AAr?$AAF?$AAA?$AAT?$AA2?$AA?5?$AA?5?$AA?5?$AA?5?$AA?5?$AA?5?$AA?5?$AA?3?$AA?5?$AA?$CF?$AAu?$AA?$AN?$AA?6?$AA?$AA@ 0001d29c     sdmmc_boot_common_topaz_v1:sdfat.obj
 0001:0000c2d4       ??_C@_1DG@FEJNAMNL@?$AAT?$AAo?$AAt?$AAa?$AAl?$AAS?$AAe?$AAc?$AAt?$AAo?$AAr?$AA2?$AA?5?$AA?5?$AA?5?$AA?5?$AA?5?$AA?5?$AA?5?$AA?5?$AA?3?$AA?5?$AA?$CF?$AAu?$AA?$AN?$AA?6?$AA?$AA@ 0001d2d4     sdmmc_boot_common_topaz_v1:sdfat.obj
 0001:0000c30c       ??_C@_1DG@DPKDIDMO@?$AAN?$AAu?$AAm?$AAb?$AAe?$AAr?$AAO?$AAf?$AAH?$AAi?$AAd?$AAd?$AAe?$AAn?$AAS?$AAe?$AAc?$AAt?$AAo?$AAr?$AA?3?$AA?5?$AA?$CF?$AAu?$AA?$AN?$AA?6?$AA?$AA@ 0001d30c     sdmmc_boot_common_topaz_v1:sdfat.obj
 0001:0000c344       ??_C@_1DG@IHBHIAEC@?$AAN?$AAu?$AAm?$AAb?$AAe?$AAr?$AAO?$AAf?$AAS?$AAi?$AAd?$AAe?$AA?5?$AA?5?$AA?5?$AA?5?$AA?5?$AA?5?$AA?5?$AA?5?$AA?3?$AA?5?$AA?$CF?$AAu?$AA?$AN?$AA?6?$AA?$AA@ 0001d344     sdmmc_boot_common_topaz_v1:sdfat.obj
 0001:0000c37c       ??_C@_1DG@PGAICJDP@?$AAS?$AAe?$AAc?$AAt?$AAo?$AAr?$AAP?$AAe?$AAr?$AAT?$AAr?$AAa?$AAc?$AAk?$AA?5?$AA?5?$AA?5?$AA?5?$AA?5?$AA?5?$AA?3?$AA?5?$AA?$CF?$AAu?$AA?$AN?$AA?6?$AA?$AA@ 0001d37c     sdmmc_boot_common_topaz_v1:sdfat.obj
 0001:0000c3b4       ??_C@_1DG@HMFAOKNC@?$AAS?$AAe?$AAc?$AAt?$AAo?$AAr?$AAP?$AAe?$AAr?$AAF?$AAA?$AAT?$AA?5?$AA?5?$AA?5?$AA?5?$AA?5?$AA?5?$AA?5?$AA?5?$AA?3?$AA?5?$AA?$CF?$AAu?$AA?$AN?$AA?6?$AA?$AA@ 0001d3b4     sdmmc_boot_common_topaz_v1:sdfat.obj
 0001:0000c3ec       ??_C@_1DK@FCPCMDK@?$AAM?$AAe?$AAd?$AAi?$AAu?$AAm?$AAI?$AAd?$AA?5?$AA?5?$AA?5?$AA?5?$AA?5?$AA?5?$AA?5?$AA?5?$AA?5?$AA?5?$AA?5?$AA?5?$AA?3?$AA?5?$AA?$CF?$AA0?$AA2?$AAX?$AA?$AN?$AA?6?$AA?$AA@ 0001d3ec     sdmmc_boot_common_topaz_v1:sdfat.obj
 0001:0000c428       ??_C@_1DG@HBABGPCH@?$AAT?$AAo?$AAt?$AAa?$AAl?$AAS?$AAe?$AAc?$AAt?$AAo?$AAr?$AA?5?$AA?5?$AA?5?$AA?5?$AA?5?$AA?5?$AA?5?$AA?5?$AA?5?$AA?3?$AA?5?$AA?$CF?$AAu?$AA?$AN?$AA?6?$AA?$AA@ 0001d428     sdmmc_boot_common_topaz_v1:sdfat.obj
 0001:0000c460       ??_C@_1DG@OFONBFHD@?$AAN?$AAu?$AAm?$AAb?$AAe?$AAr?$AAO?$AAf?$AAR?$AAo?$AAo?$AAt?$AAE?$AAn?$AAt?$AAr?$AAy?$AA?5?$AA?5?$AA?5?$AA?3?$AA?5?$AA?$CF?$AAu?$AA?$AN?$AA?6?$AA?$AA@ 0001d460     sdmmc_boot_common_topaz_v1:sdfat.obj
 0001:0000c498       ??_C@_1DG@BGCBIOJA@?$AAN?$AAu?$AAm?$AAb?$AAe?$AAr?$AAO?$AAf?$AAF?$AAA?$AAT?$AA?5?$AA?5?$AA?5?$AA?5?$AA?5?$AA?5?$AA?5?$AA?5?$AA?5?$AA?3?$AA?5?$AA?$CF?$AAu?$AA?$AN?$AA?6?$AA?$AA@ 0001d498     sdmmc_boot_common_topaz_v1:sdfat.obj
 0001:0000c4d0       ??_C@_1DG@GDIAMPKD@?$AAR?$AAe?$AAs?$AAe?$AAr?$AAv?$AAe?$AAd?$AAS?$AAe?$AAc?$AAt?$AAo?$AAr?$AA?5?$AA?5?$AA?5?$AA?5?$AA?5?$AA?5?$AA?3?$AA?5?$AA?$CF?$AAu?$AA?$AN?$AA?6?$AA?$AA@ 0001d4d0     sdmmc_boot_common_topaz_v1:sdfat.obj
 0001:0000c508       ??_C@_1DG@MNDIIEKL@?$AAS?$AAe?$AAc?$AAt?$AAo?$AAr?$AAP?$AAe?$AAr?$AAC?$AAl?$AAu?$AAs?$AAt?$AAe?$AAr?$AA?5?$AA?5?$AA?5?$AA?5?$AA?3?$AA?5?$AA?$CF?$AAu?$AA?$AN?$AA?6?$AA?$AA@ 0001d508     sdmmc_boot_common_topaz_v1:sdfat.obj
 0001:0000c540       ??_C@_1DG@PONJPGFJ@?$AAS?$AAe?$AAc?$AAt?$AAo?$AAr?$AAS?$AAi?$AAz?$AAe?$AA?5?$AA?5?$AA?5?$AA?5?$AA?5?$AA?5?$AA?5?$AA?5?$AA?5?$AA?5?$AA?3?$AA?5?$AA?$CF?$AAu?$AA?$AN?$AA?6?$AA?$AA@ 0001d540     sdmmc_boot_common_topaz_v1:sdfat.obj
 0001:0000c578       ??_C@_1DK@MOPEPNKH@?$AAC?$AAr?$AAe?$AAa?$AAt?$AAo?$AAr?$AAI?$AAD?$AA?5?$AA?5?$AA?5?$AA?5?$AA?5?$AA?5?$AA?5?$AA?5?$AA?5?$AA?5?$AA?5?$AA?3?$AA?5?$AA?$CF?$AA?4?$AA8?$AAS?$AA?$AN?$AA?6?$AA?$AA@ 0001d578     sdmmc_boot_common_topaz_v1:sdfat.obj
 0001:0000c5b4       ??_C@_1DK@PBPLLOIJ@?$AAJ?$AAu?$AAm?$AAp?$AAC?$AAo?$AAd?$AAe?$AA?5?$AA?5?$AA?5?$AA?5?$AA?5?$AA?5?$AA?5?$AA?5?$AA?5?$AA?5?$AA?5?$AA?5?$AA?3?$AA?5?$AA?$CF?$AA0?$AA6?$AAX?$AA?$AN?$AA?6?$AA?$AA@ 0001d5b4     sdmmc_boot_common_topaz_v1:sdfat.obj
 0001:0000c5f0       ??_C@_1EA@FFGMJMNG@?$AAP?$AAa?$AAr?$AAt?$AAi?$AAt?$AAi?$AAo?$AAn?$AA?5?$AAN?$AAu?$AAm?$AAb?$AAe?$AAr?$AA?5?$AAb?$AAe?$AAy?$AAo?$AAn?$AAd?$AA?5?$AAs?$AAc?$AAo?$AAp?$AAe?$AA?$AN?$AA?6?$AA?$AA@ 0001d5f0     sdmmc_boot_common_topaz_v1:sdfat.obj
 0001:0000c630       ??_C@_1M@EEBCEMHK@?$AA?$CF?$AA0?$AA?$CK?$AAX?$AA?5?$AA?$AA@ 0001d630     sdmmc_boot_common_topaz_v1:sdfat.obj
 0001:0000c63c       ??_C@_1BA@DGPAFFOM@?$AA?$CF?$AA0?$AA4?$AAX?$AA?5?$AA?5?$AA?5?$AA?$AA@ 0001d63c     sdmmc_boot_common_topaz_v1:sdfat.obj
 0001:0000c650       ??_C@_1FC@LGLGMMJD@?$AAS?$AAt?$AAa?$AAr?$AAt?$AA?5?$AAp?$AAo?$AAs?$AAi?$AAt?$AAi?$AAo?$AAn?$AA?5?$AAb?$AAe?$AAy?$AAo?$AAn?$AAd?$AA?5?$AAF?$AAA?$AAT?$AA?5?$AAe?$AAn?$AAt?$AAr?$AAy?$AA?5@ 0001d650     sdmmc_boot_common_topaz_v1:sdfat.obj
 0001:0000c6a8       ??_C@_1PA@BNCCHDMH@?$AA?$CF?$AA0?$AA2?$AAu?$AA?1?$AA?$CF?$AA0?$AA2?$AAu?$AA?1?$AA?$CF?$AA0?$AA2?$AAu?$AA?9?$AA?$CF?$AA0?$AA2?$AAu?$AA?3?$AA?$CF?$AA0?$AA2?$AAu?$AA?3?$AA?$CF?$AA0?$AA2?$AAu?$AA?3?$AA?$CF?$AA0@ 0001d6a8     sdmmc_boot_common_topaz_v1:sdfat.obj
 0001:0000c798       ??_C@_1CE@IPBNILJ@?$AAF?$AAa?$AAi?$AAl?$AA?5?$AAt?$AAo?$AA?5?$AAr?$AAe?$AAa?$AAd?$AA?5?$AA?$CF?$AAS?$AA?$AN?$AA?6?$AA?$AA@ 0001d798     sdmmc_boot_common_topaz_v1:sdfat.obj
 0001:0000c7c0       ??_C@_1LM@LFBLGBLM@?$AAC?$AAr?$AAe?$AAa?$AAt?$AAe?$AAd?$AA?5?$AA?5?$AA?5?$AA?5?$AA?5?$AA?5?$AA?5?$AA?5?$AA?5?$AA?5?$AA?5?$AA?5?$AA?5?$AA?5?$AA?5?$AA?5?$AAM?$AAo?$AAd?$AAi?$AAf?$AAi?$AAe?$AAd?$AA?5@ 0001d7c0     sdmmc_boot_common_topaz_v1:sdfat.obj
 0001:0000c880       ??_C@_1FO@IBCJBBFN@?$AAS?$AAt?$AAa?$AAr?$AAt?$AA?5?$AAp?$AAo?$AAs?$AAi?$AAt?$AAi?$AAo?$AAn?$AA?5?$AAb?$AAe?$AAy?$AAo?$AAn?$AAd?$AA?5?$AAd?$AAi?$AAr?$AAe?$AAc?$AAt?$AAo?$AAr?$AAy?$AA?5@ 0001d880     sdmmc_boot_common_topaz_v1:sdfat.obj
 0001:0000c8e0       ??_C@_1CA@PKKJEAAM@?$AAC?$AAa?$AAn?$AA?8?$AAt?$AA?5?$AAo?$AAp?$AAe?$AAn?$AA?5?$AA?$CF?$AAS?$AA?$AN?$AA?6?$AA?$AA@ 0001d8e0     sdmmc_boot_common_topaz_v1:sdfat.obj
 0001:0000c900       ??_C@_1GK@JECCAOJF@?$AA?$CF?$AA0?$AA2?$AAu?$AA?1?$AA?$CF?$AA0?$AA2?$AAu?$AA?1?$AA?$CF?$AA0?$AA2?$AAu?$AA?9?$AA?$CF?$AA0?$AA2?$AAu?$AA?3?$AA?$CF?$AA0?$AA2?$AAu?$AA?3?$AA?$CF?$AA0?$AA2?$AAu?$AA?5?$AA?5?$AA?$CF@ 0001d900     sdmmc_boot_common_topaz_v1:sdfat.obj
 0001:0000c970       ??_C@_1GK@JJIDFIGI@?$AAM?$AAo?$AAd?$AAi?$AAf?$AAi?$AAe?$AAd?$AA?5?$AA?5?$AA?5?$AA?5?$AA?5?$AA?5?$AA?5?$AA?5?$AA?5?$AA?5?$AA?5?$AAA?$AAt?$AAt?$AA?5?$AAC?$AAl?$AAu?$AAs?$AAt?$AAe?$AAr?$AA?5?$AA?5@ 0001d970     sdmmc_boot_common_topaz_v1:sdfat.obj
 0001:0000c9dc       ??_C@_1CK@CMKNIHCM@?$AA?$CF?$AAS?$AA?5?$AAi?$AAs?$AAn?$AA?8?$AAt?$AA?5?$AAd?$AAi?$AAr?$AAe?$AAc?$AAt?$AAo?$AAr?$AAy?$AA?$AN?$AA?6?$AA?$AA@ 0001d9dc     sdmmc_boot_common_topaz_v1:sdfat.obj
 0001:0000ca08       ??_C@_1DC@OINNCOK@?$AA?$AN?$AA?6?$AAB?$AAu?$AAf?$AAf?$AAe?$AAr?$AAs?$AA?5?$AAa?$AAr?$AAe?$AA?5?$AAt?$AAh?$AAe?$AA?5?$AAs?$AAa?$AAm?$AAe?$AA?$AN?$AA?6?$AA?$AA@ 0001da08     oal_spifmd:cspifmd.obj
 0001:0000ca3c       ??_C@_1DK@IDFJNCDP@?$AA?$AN?$AA?6?$AAB?$AAu?$AAf?$AAf?$AAe?$AAr?$AAs?$AA?5?$AAa?$AAr?$AAe?$AA?5?$AAn?$AAo?$AAt?$AA?5?$AAt?$AAh?$AAe?$AA?5?$AAs?$AAa?$AAm?$AAe?$AA?$AN?$AA?6?$AA?$AA@ 0001da3c     oal_spifmd:cspifmd.obj
 0001:0000ca78       ??_C@_1CO@MDFNLLCG@?$AAS?$AAP?$AAI?$AAF?$AAM?$AAD?$AA_?$AAI?$AAn?$AAi?$AAt?$AA?3?$AA?5?$AAR?$AAE?$AAA?$AAD?$AAI?$AAN?$AAG?$AA?$AN?$AA?6?$AA?$AA@ 0001da78     oal_spifmd:cspifmd.obj
 0001:0000caa8       ??_C@_1DI@CGKKMABA@?$AAS?$AAP?$AAI?$AAF?$AAM?$AAD?$AA_?$AAI?$AAn?$AAi?$AAt?$AA?3?$AA?5?$AAW?$AAR?$AAI?$AAT?$AAI?$AAN?$AAG?$AA?5?$AA0?$AAx?$AAa?$AA5?$AA?$AN?$AA?6?$AA?$AA@ 0001daa8     oal_spifmd:cspifmd.obj
 0001:0000cae0       ??_C@_1CO@PAKGOKMG@?$AAS?$AAP?$AAI?$AAF?$AAM?$AAD?$AA_?$AAI?$AAn?$AAi?$AAt?$AA?3?$AA?5?$AAr?$AAe?$AAa?$AAd?$AAi?$AAn?$AAg?$AA?$AN?$AA?6?$AA?$AA@ 0001dae0     oal_spifmd:cspifmd.obj
 0001:0000cb10       ??_C@_1CO@DNNGCHKA@?$AAS?$AAP?$AAI?$AAF?$AAM?$AAD?$AA_?$AAI?$AAn?$AAi?$AAt?$AA?3?$AA?5?$AAe?$AAr?$AAa?$AAs?$AAi?$AAn?$AAg?$AA?$AN?$AA?6?$AA?$AA@ 0001db10     oal_spifmd:cspifmd.obj
 0001:0000cb40       ??_C@_1EG@JFGEONGL@?$AAS?$AAP?$AAI?$AAF?$AAM?$AAD?$AA_?$AAI?$AAn?$AAi?$AAt?$AA?3?$AA?5?$AAW?$AAr?$AAi?$AAt?$AAe?$AAE?$AAn?$AAa?$AAb?$AAl?$AAe?$AA?5?$AAf?$AAa?$AAi?$AAl?$AAe?$AAd?$AA?5@ 0001db40     oal_spifmd:cspifmd.obj
 0001:0000cb88       ??_C@_1GO@MHHJIKMG@?$AAS?$AAP?$AAI?$AAF?$AAM?$AAD?$AA_?$AAI?$AAn?$AAi?$AAt?$AA?3?$AA?5?$AAM?$AAa?$AAn?$AAu?$AAf?$AAa?$AAc?$AAt?$AAu?$AAr?$AAe?$AAr?$AA?5?$AAI?$AAD?$AA?5?$AA?$DN?$AA?5?$AA0@ 0001db88     oal_spifmd:cspifmd.obj
 0001:0000cc78       ??_C@_1EO@BIINPADA@?$AAO?$AAA?$AAL?$AAP?$AAm?$AAi?$AAc?$AAI?$AAn?$AAi?$AAt?$AA?3?$AA?5?$AAO?$AAA?$AAL?$AAP?$AAA?$AAt?$AAo?$AAU?$AAA?$AA?5?$AAr?$AAe?$AAt?$AAu?$AAr?$AAn?$AAe?$AAd?$AA?5@ 0001dc78     i2cutils:i2cutils.obj
 0001:0000ccc8       ??_C@_1EK@BGCNBCKF@?$AAO?$AAA?$AAL?$AAI?$AA2?$AAc?$AAI?$AAn?$AAi?$AAt?$AA?3?$AA?5?$AAI?$AAO?$AAM?$AAU?$AAX?$AAC?$AA?5?$AAm?$AAa?$AAp?$AAp?$AAi?$AAn?$AAg?$AA?5?$AAf?$AAa?$AAi?$AAl?$AAe@ 0001dcc8     i2cutils:i2cutils.obj
 0001:0000cd18       ??_C@_1FG@HMBKJBKF@?$AAO?$AAA?$AAL?$AAI?$AA2?$AAc?$AAI?$AAn?$AAi?$AAt?$AA?3?$AA?5?$AAT?$AAr?$AAy?$AAi?$AAn?$AAg?$AA?5?$AAt?$AAo?$AA?5?$AAi?$AAn?$AAi?$AAt?$AA?5?$AAI?$AA2?$AAC?$AA?5?$AAI@ 0001dd18     i2cutils:i2cutils.obj
 0001:0000cd70       ??_C@_1DK@MPINBAIN@?$AA?$CF?$AAs?$AA?3?$AA?5?$AAB?$AAu?$AAs?$AA?5?$AAb?$AAu?$AAs?$AAy?$AA?5?$AAf?$AAo?$AAr?$AA?5?$AA?$CF?$AAd?$AA?5?$AAc?$AAy?$AAc?$AAl?$AAe?$AAs?$AA?$AN?$AA?6?$AA?$AA@ 0001dd70     i2cutils:i2cutils.obj
 0001:0000cdac       ??_C@_1CI@JNEOMLK@?$AAO?$AAA?$AAL?$AAI?$AA2?$AAc?$AAG?$AAe?$AAn?$AAe?$AAr?$AAa?$AAt?$AAe?$AAS?$AAt?$AAa?$AAr?$AAt?$AA?$AA@ 0001ddac     i2cutils:i2cutils.obj
 0001:0000cdd8       ??_C@_1EI@LDHHPPEC@?$AA?$CF?$AAs?$AA?3?$AA?5?$AAB?$AAu?$AAs?$AA?5?$AAn?$AAo?$AAt?$AA?5?$AAc?$AAl?$AAe?$AAa?$AAr?$AAe?$AAd?$AA?5?$AAf?$AAo?$AAr?$AA?5?$AA?$CF?$AAd?$AA?5?$AAc?$AAy?$AAc?$AAl?$AAe@ 0001ddd8     i2cutils:i2cutils.obj
 0001:0000ce20       ??_C@_1CG@KGNMMGFF@?$AAO?$AAA?$AAL?$AAI?$AA2?$AAc?$AAG?$AAe?$AAn?$AAe?$AAr?$AAa?$AAt?$AAe?$AAS?$AAt?$AAo?$AAp?$AA?$AA@ 0001de20     i2cutils:i2cutils.obj
 0001:0000ce48       ??_C@_0BN@HCIGGCJK@Server?5Registration?5Failed?$AN?6?$AA@ 0001de48     eboot:ebsimp.obj
 0001:0000ce68       ??_C@_0CF@NJGKJDPK@EthDown?3?3Illegal?5Operation?5Code?5@ 0001de68     eboot:ebsimp.obj
 0001:0000ce90       ??_C@_0BK@BFELHAIB@EthDown?3?3TFTPD_OPEN?3?3?$CFs?$AN?6?$AA@ 0001de90     eboot:ebsimp.obj
 0001:0000ceac       ??_C@_0CC@OIEKENJI@EbootSimpleTFTP?5not?5initialized?$AN@ 0001deac     eboot:ebsimp.obj
 0001:0000ced0       ??_C@_0BM@GELEBJHM@EbootGratuitousARP?5failed?$AN?6?$AA@ 0001ded0     eboot:ebsimp.obj
 0001:0000ceec       ??_C@_0DG@LCJHGIIG@Some?5other?5station?5has?5IP?5Addres@ 0001deec     eboot:ebsimp.obj
 0001:0000cf24       ??_C@_0DG@KEGBCNMH@Some?5other?5station?5has?5IP?5Addres@ 0001df24     eboot:ebsimp.obj
 0001:0000cf5c       ??_C@_0DK@ECECEHHP@No?5ARP?5response?5in?5?$CFd?5seconds?0?5a@ 0001df5c     eboot:ebsimp.obj
 0001:0000cf98       ??_C@_0DA@PMFFKPM@Got?5Response?5from?5DHCP?5server?0?5I@ 0001df98     eboot:ebsimp.obj
 0001:0000cfc8       ??_C@_0CO@EJPPGFNA@DHCP?5server?5is?5not?5responding?5?$CB?$CB@ 0001dfc8     eboot:ebsimp.obj
 0001:0000cff8       ??_C@_0BL@PFCEMBID@Error?5On?5InitDHCP?$CI?$CJ?5Call?$AN?6?$AA@ 0001dff8     eboot:ebsimp.obj
 0001:0000d014       ??_C@_0CB@PCBFMPDH@?9EbootSendBootmeAndWaitForTftp?$AN?6@ 0001e014     eboot:ebsimp.obj
 0001:0000d038       ??_C@_0CB@EEDKKNBN@?$CLEbootSendBootmeAndWaitForTftp?$AN?6@ 0001e038     eboot:ebsimp.obj
 0001:0000d05c       ??_C@_0DF@HGBBKEBE@WARNING?3?5Some?5other?5station?5has?5@ 0001e05c     eboot:ebsimp.obj
 0001:0000d094       ??_C@_08NMEDJLNE@boot?4bin?$AA@ 0001e094     eboot:ebsimp.obj
 0001:0000d0a0       ??_C@_0CH@NEPGMPPP@Server?5Process?5Has?5UnRegistered?5@ 0001e0a0     eboot:tftpd.obj
 0001:0000d0c8       ??_C@_0CN@LGCIOIPF@There?5were?5no?5options?5detected?5i@ 0001e0c8     eboot:tftpd.obj
 0001:0000d0f8       ??_C@_0FJ@NDFKPFHG@Illegal?5TFTP?5Option?5?9?5An?5option?5@ 0001e0f8     eboot:tftpd.obj
 0001:0000d154       ??_C@_06CECHPPMB@?5?$CFd?4?$AN?6?$AA@ 0001e154     eboot:tftpd.obj
 0001:0000d15c       ??_C@_0DM@IIELHHA@with?5a?5value?5that?5is?5in?5range?4?$AN?6@ 0001e15c     eboot:tftpd.obj
 0001:0000d198       ??_C@_0DO@FNNPCMEI@with?5a?5value?5that?5is?5out?5of?5rang@ 0001e198     eboot:tftpd.obj
 0001:0000d1d8       ??_C@_0BL@FNDCPDJI@The?5option?8s?5value?5is?5?$CFs?$AN?6?$AA@ 0001e1d8     eboot:tftpd.obj
 0001:0000d1f4       ??_C@_07JPIGAOKK@blksize?$AA@ 0001e1f4     eboot:tftpd.obj
 0001:0000d1fc       ??_C@_0CC@KHJDBEOG@The?5packet?8s?5option?5name?5is?5?$CFs?4?$AN@ 0001e1fc     eboot:tftpd.obj
 0001:0000d220       ??_C@_0ED@FMPMEGBG@We?5currently?5only?5look?5at?5the?5fi@ 0001e220     eboot:tftpd.obj
 0001:0000d264       ??_C@_0CI@KEAAKLLA@This?5TFTP?5packet?5contains?5?$CFd?5opt@ 0001e264     eboot:tftpd.obj
 0001:0000d28c       ??_C@_0CG@JBBJIFDI@You?5must?5access?5files?5in?5binary?5@ 0001e28c     eboot:tftpd.obj
 0001:0000d2b4       ??_C@_05IIBPGMLM@octet?$AA@ 0001e2b4     eboot:tftpd.obj
 0001:0000d2bc       ??_C@_0DB@LKOCKFPL@Illegal?5TFTP?5Operation?5?9?5Read?1Wr@ 0001e2bc     eboot:tftpd.obj
 0001:0000d2f0       ??_C@_0CL@HCAEOMAE@Default?5TFTP?5block?5size?5set?5to?3?5@ 0001e2f0     eboot:tftpd.obj
 0001:0000d31c       ??_C@_0BF@MOPBEBEN@Dest?5IP?5?$CFs?5Port?5?$CFH?$AN?6?$AA@ 0001e31c     eboot:tftpd.obj
 0001:0000d334       ??_C@_0BF@JDGNCBEC@Src?5IP?5?$CFs?5Port?5?$CFH?5?5?5?$AA@ 0001e334     eboot:tftpd.obj
 0001:0000d34c       ??_C@_0BG@GIKNIKEH@Locked?5Down?5Link?5?$CFd?$AN?6?$AA@ 0001e34c     eboot:tftpd.obj
 0001:0000d364       ??_C@_0DB@OCKCBBAL@No?5Server?5Process?5Associated?5Wit@ 0001e364     eboot:tftpd.obj
 0001:0000d398       ??_C@_0CN@CMBNFGFO@TFTP?5packet?5could?5have?5?$CFd?5name?1v@ 0001e398     eboot:tftpd.obj
 0001:0000d3c8       ??_C@_0FD@OCECBKGJ@There?5must?5be?5an?5even?5number?0?5an@ 0001e3c8     eboot:tftpd.obj
 0001:0000d41c       ??_C@_06CBLHAGFD@?$FLNULL?$FN?$AA@ 0001e41c     eboot:tftpd.obj
 0001:0000d424       ??_C@_02HAOIJKIC@?$CFc?$AA@ 0001e424     eboot:tftpd.obj
 0001:0000d428       ??_C@_0CD@NDCILIIJ@Packet?5has?5the?5following?5data?3?$AN?6@ 0001e428     eboot:tftpd.obj
 0001:0000d44c       ??_C@_0CP@POPAOFAN@An?5OACK?5packet?5is?5the?5proper?5ack@ 0001e44c     eboot:tftpd.obj
 0001:0000d47c       ??_C@_0CG@OFKOPMJ@TftpReceiver?0?5port?3?50x?$CFX?0?5wkp?3?50@ 0001e47c     eboot:tftp.obj
 0001:0000d4a8       ??_C@_0EB@BKDEILKN@TFTP?5link?$FL?$CFu?$FN?3?5State?3?$CFu?0?5DestAdd@ 0001e4a8     eboot:tftp.obj
 0001:0000d4ec       ??_C@_0DC@EJGDJHJD@TFTPRetransmit?$CI?$CJ?5Slot?5?$CFu?0?5wDestT@ 0001e4ec     eboot:tftp.obj
 0001:0000d520       ??_C@_0BI@NOMLANFJ@Linked?5Timed?5Out?5By?5Odo?$AA@ 0001e520     eboot:tftp.obj
 0001:0000d538       ??_C@_0CM@MLNGGHPC@TFTPRetransmit?$CI?$CJ?3?3Error?5On?5SendU@ 0001e538     eboot:tftp.obj
 0001:0000d564       ??_C@_0DC@MHCCPLAO@TFtpStateMachine?3?3TFTP_STATE_CLO@ 0001e564     eboot:tftp.obj
 0001:0000d598       ??_C@_0DJ@MEFFBBAC@TFTP?3?5Desktop?5losing?5ACK?0?5block?5@ 0001e598     eboot:tftp.obj
 0001:0000d5d4       ??_C@_0CI@FJCIJAAP@TFTP?5Error?5Received?5From?5Host?5?$CFX@ 0001e5d4     eboot:tftp.obj
 0001:0000d5fc       ??_C@_0CA@DPHLAENA@?$CBTftpReturnCodes?0?5STATE_ERROR?$AN?6?$AA@ 0001e5fc     eboot:tftp.obj
 0001:0000d61c       ??_C@_0BD@LKENBIIO@?$CB?$CB?$CB?$CB?5TFTP?5Errror?$AN?6?$AA@ 0001e61c     eboot:tftp.obj
 0001:0000d630       ??_C@_0CJ@ICDDJIPJ@?$CBCheckUDP?3?5UDP?5header?5checksum?5f@ 0001e630     eboot:udp.obj
 0001:0000d65c       ??_C@_0CI@JJAKDMIL@?$CBCheckUDP?3?5IP?5header?5checksum?5fa@ 0001e65c     eboot:udp.obj
 0001:0000d684       ??_C@_0CE@JJEEIBJP@?$CBCheckUDP?3?5Not?5UDP?5?$CIproto?5?$DN?50x?$CFX@ 0001e684     eboot:udp.obj
 0001:0000d6a8       ??_C@_0IO@FOKDOCNJ@Duplicate?5IP?5Address?5Detected?3?$AN?6@ 0001e6a8     eboot:udp.obj
 0001:0000d738       ??_C@_0DO@EHKMGFMI@InitDHCP?$CI?$CJ?5Error?5?9?5First?5DHCP?5Op@ 0001e738     eboot:dhcp.obj
 0001:0000d778       ??_C@_0CF@NLOHFKBD@InitDHCP?$CI?$CJ?3?3?5Calling?5ProcessDHCP@ 0001e778     eboot:dhcp.obj
 0001:0000d7a0       ??_C@_0BJ@MEOPKMJJ@Lease?5time?3?5?$CFd?5seconds?$AN?6?$AA@ 0001e7a0     eboot:dhcp.obj
 0001:0000d7bc       ??_C@_0O@DFHLFDCO@netmask?3?5?$CFs?$AN?6?$AA@ 0001e7bc     eboot:dhcp.obj
 0001:0000d7cc       ??_C@_0DC@KHEOJACB@?$AN?6ProcessDHCP?$CI?$CJ?3?3DHCP?5IP?5Address@ 0001e7cc     eboot:dhcp.obj
 0001:0000d800       ??_C@_0FI@EHEELHEE@ProcessDHCP?$CI?$CJ?3?3DHCP_REQUESTING?3?3@ 0001e800     eboot:dhcp.obj
 0001:0000d858       ??_C@_0DC@EKKEKBDC@ProcessDHCP?$CI?$CJ?3?3DHCP_SELECTING?3?3S@ 0001e858     eboot:dhcp.obj
 0001:0000d890       ??_C@_0FK@JNLIFC@ProcessDHCP?$CI?$CJ?3?3DHCP_SELECTING?3?3D@ 0001e890     eboot:dhcp.obj
 0001:0000d8f0       ??_C@_0FI@KEBKGIEO@ProcessDHCP?$CI?$CJ?3?3DHCP_SELECTING?3?3D@ 0001e8f0     eboot:dhcp.obj
 0001:0000d948       ??_C@_0DK@EEIOPNMG@ProcessDHCP?$CI?$CJ?3?3DHCP_INIT?3?3SendDH@ 0001e948     eboot:dhcp.obj
 0001:0000d984       ??_C@_0BL@LBDFFECM@ProcessDHCP?$CI?$CJ?3?3DHCP_INIT?$AN?6?$AA@ 0001e984     eboot:dhcp.obj
 0001:0000d9a0       ??_C@_0DE@BHBNDGEJ@ProcessDHCP?$CI?$CJ?5Error?5?9?5No?5DHCP?5Me@ 0001e9a0     eboot:dhcp.obj
 0001:0000d9d4       ??_C@_0DI@NEOGOAKD@?$CLEbootProcessDHCP?3?5State?3?5?$CFu?0?5pM@ 0001e9d4     eboot:dhcp.obj
 0001:0000da0c       ??_C@_0CN@GEBEIIOD@SendDHCP?$CI?$CJ?3?3Error?5On?5DHCPRetrans@ 0001ea0c     eboot:dhcp.obj
 0001:0000da3c       ??_C@_0CG@GEIANEBC@SendDHCP?$CI?$CJ?3?3Error?5On?5SendUDP?$CI?$CJ?5C@ 0001ea3c     eboot:dhcp.obj
 0001:0000da64       ??_C@_0BH@NLCMGMCH@?$CLSendDHCP?0?5MsgType?3?5?$CFu?$AA@ 0001ea64     eboot:dhcp.obj
 0001:0000da7c       ??_C@_0DB@JKAMMNCP@EbootDHCPRetransmit?$CI?$CJ?3?3Error?5On?5@ 0001ea7c     eboot:dhcp.obj
 0001:0000dab0       ??_C@_0DK@FBGEAJFD@DHCPRetransmit?0?5retry?5count?5exce@ 0001eab0     eboot:dhcp.obj
 0001:0000daec       ??_C@_0CG@JNDKDABJ@?$CLDHCPRetransmit?3?5Retry?5?$CFu?0?5time?3@ 0001eaec     eboot:dhcp.obj
 0001:0000db14       ??_C@_0CO@FCHDJGDA@?$CLDHCPRetransmit?3?51st?5transmissio@ 0001eb14     eboot:dhcp.obj
 0001:0000db44       ??_C@_0DF@CLENMEEN@?$AN?6Enter?5new?5subnet?5mask?5or?5CR?5to@ 0001eb44     eboot:dhcp.obj
 0001:0000db7c       ??_C@_0CI@NDANHPBF@?$AN?6ReadSerialIP?$CI?$CJ?3?3Using?5IP?5Addre@ 0001eb7c     eboot:dhcp.obj
 0001:0000dba4       ??_C@_0BD@GIINPDL@Error?5in?5SendUDP?$AN?6?$AA@ 0001eba4     eboot:edbg.obj
 0001:0000dbb8       ??_C@_0CC@IFLECHKJ@Got?5EDBG_CMD_CONFIG?0?5flags?30x?$CFX?$AN@ 0001ebb8     eboot:edbg.obj
 0001:0000dbdc       ??_C@_0BH@EBGODALL@Got?5EDBG_CMD_JUMPIMG?$AN?6?$AA@ 0001ebdc     eboot:edbg.obj
 0001:0000dbf8       ??_C@_0EE@BGOJJHDN@TFTP?5download?5started?5previously@ 0001ebf8     eboot:edbg.obj
 0001:0000dc3c       ??_C@_0BE@MGGELJDD@Sent?5BOOTME?5to?5?$CFs?$AN?6?$AA@ 0001ec3c     eboot:edbg.obj
 0001:0000dc50       ??_C@_0CI@BKOJILAL@SendBootme?$CI?$CJ?3?3Error?5on?5SendUDP?$CI?$CJ@ 0001ec50     eboot:edbg.obj
 0001:0000dc78       ??_C@_1BBA@MLBOPNGI@?$AA?$AN?$AA?6?$AA?$CK?$AA?$CK?$AA?$CK?$AA?5?$AAA?$AAS?$AAS?$AAE?$AAR?$AAT?$AAI?$AAO?$AAN?$AA?5?$AAF?$AAA?$AAI?$AAL?$AAE?$AAD?$AA?5?$AAi?$AAn?$AA?5?$AAd?$AA?3?$AA?2?$AAc?$AAh?$AAe@ 0001ec78     fulllibc:strncpy_s.obj
 0001:0000dd88       ??_C@_1CI@HCPHDDLE@?$AAB?$AAu?$AAf?$AAf?$AAe?$AAr?$AA?5?$AAi?$AAs?$AA?5?$AAt?$AAo?$AAo?$AA?5?$AAs?$AAm?$AAa?$AAl?$AAl?$AA?$AA@ 0001ed88     fulllibc:strncpy_s.obj
 0001:0000ddb0       ??_C@_1PM@NHEEEKG@?$AA?$AN?$AA?6?$AA?$CK?$AA?$CK?$AA?$CK?$AA?5?$AAA?$AAS?$AAS?$AAE?$AAR?$AAT?$AAI?$AAO?$AAN?$AA?5?$AAF?$AAA?$AAI?$AAL?$AAE?$AAD?$AA?5?$AAi?$AAn?$AA?5?$AAd?$AA?3?$AA?2?$AAc?$AAh?$AAe@ 0001edb0     fulllibc:strncpy_s.obj
 0001:0000deb0       ??_C@_1PK@MLNBEAPB@?$AA?$AN?$AA?6?$AA?$CK?$AA?$CK?$AA?$CK?$AA?5?$AAA?$AAS?$AAS?$AAE?$AAR?$AAT?$AAI?$AAO?$AAN?$AA?5?$AAF?$AAA?$AAI?$AAL?$AAE?$AAD?$AA?5?$AAi?$AAn?$AA?5?$AAd?$AA?3?$AA?2?$AAc?$AAh?$AAe@ 0001eeb0     fulllibc:strncpy_s.obj
 0001:0000dfb0       ??_C@_1BCG@OOFNLCAK@?$AA?$AN?$AA?6?$AA?$CK?$AA?$CK?$AA?$CK?$AA?5?$AAA?$AAS?$AAS?$AAE?$AAR?$AAT?$AAI?$AAO?$AAN?$AA?5?$AAF?$AAA?$AAI?$AAL?$AAE?$AAD?$AA?5?$AAi?$AAn?$AA?5?$AAd?$AA?3?$AA?2?$AAc?$AAh?$AAe@ 0001efb0     fulllibc:strncpy_s.obj
 0001:0000e0d8       ??_C@_1BAO@KGHGEJLP@?$AA?$AN?$AA?6?$AA?$CK?$AA?$CK?$AA?$CK?$AA?5?$AAA?$AAS?$AAS?$AAE?$AAR?$AAT?$AAI?$AAO?$AAN?$AA?5?$AAF?$AAA?$AAI?$AAL?$AAE?$AAD?$AA?5?$AAi?$AAn?$AA?5?$AAd?$AA?3?$AA?2?$AAc?$AAh?$AAe@ 0001f0d8     fulllibc:strcpy_s.obj
 0001:0000e1e8       ??_C@_1PI@CMKALJAA@?$AA?$AN?$AA?6?$AA?$CK?$AA?$CK?$AA?$CK?$AA?5?$AAA?$AAS?$AAS?$AAE?$AAR?$AAT?$AAI?$AAO?$AAN?$AA?5?$AAF?$AAA?$AAI?$AAL?$AAE?$AAD?$AA?5?$AAi?$AAn?$AA?5?$AAd?$AA?3?$AA?2?$AAc?$AAh?$AAe@ 0001f1e8     fulllibc:strcpy_s.obj
 0001:0000e2e0       ??_C@_1BCE@JNDHDIBJ@?$AA?$AN?$AA?6?$AA?$CK?$AA?$CK?$AA?$CK?$AA?5?$AAA?$AAS?$AAS?$AAE?$AAR?$AAT?$AAI?$AAO?$AAN?$AA?5?$AAF?$AAA?$AAI?$AAL?$AAE?$AAD?$AA?5?$AAi?$AAn?$AA?5?$AAd?$AA?3?$AA?2?$AAc?$AAh?$AAe@ 0001f2e0     fulllibc:strcpy_s.obj
 0001:0000e408       ??_C@_1BAA@FKMLMOFD@?$AA?$AN?$AA?6?$AA?$CK?$AA?$CK?$AA?$CK?$AA?5?$AAA?$AAS?$AAS?$AAE?$AAR?$AAT?$AAI?$AAO?$AAN?$AA?5?$AAF?$AAA?$AAI?$AAL?$AAE?$AAD?$AA?5?$AAi?$AAn?$AA?5?$AAd?$AA?3?$AA?2?$AAc?$AAh?$AAe@ 0001f408     fulllibc:xtoas.obj
 0001:0000e508       ??_C@_1BAI@OHFFOLJE@?$AA?$AN?$AA?6?$AA?$CK?$AA?$CK?$AA?$CK?$AA?5?$AAA?$AAS?$AAS?$AAE?$AAR?$AAT?$AAI?$AAO?$AAN?$AA?5?$AAF?$AAA?$AAI?$AAL?$AAE?$AAD?$AA?5?$AAi?$AAn?$AA?5?$AAd?$AA?3?$AA?2?$AAc?$AAh?$AAe@ 0001f508     fulllibc:xtoas.obj
 0001:0000e610       ??_C@_1BCE@LLMIIAMI@?$AA?$AN?$AA?6?$AA?$CK?$AA?$CK?$AA?$CK?$AA?5?$AAA?$AAS?$AAS?$AAE?$AAR?$AAT?$AAI?$AAO?$AAN?$AA?5?$AAF?$AAA?$AAI?$AAL?$AAE?$AAD?$AA?5?$AAi?$AAn?$AA?5?$AAd?$AA?3?$AA?2?$AAc?$AAh?$AAe@ 0001f610     fulllibc:xtoas.obj
 0001:0000e738       ??_C@_1PG@CPEOIHDA@?$AA?$AN?$AA?6?$AA?$CK?$AA?$CK?$AA?$CK?$AA?5?$AAA?$AAS?$AAS?$AAE?$AAR?$AAT?$AAI?$AAO?$AAN?$AA?5?$AAF?$AAA?$AAI?$AAL?$AAE?$AAD?$AA?5?$AAi?$AAn?$AA?5?$AAd?$AA?3?$AA?2?$AAc?$AAh?$AAe@ 0001f738     fulllibc:xtoas.obj
 0001:0000e830       ??_C@_1OM@MKFMPGNL@?$AA?$AN?$AA?6?$AA?$CK?$AA?$CK?$AA?$CK?$AA?5?$AAA?$AAS?$AAS?$AAE?$AAR?$AAT?$AAI?$AAO?$AAN?$AA?5?$AAF?$AAA?$AAI?$AAL?$AAE?$AAD?$AA?5?$AAi?$AAn?$AA?5?$AAd?$AA?3?$AA?2?$AAc?$AAh?$AAe@ 0001f830     fulllibc:xtoas.obj
 0001:0000e920       ??_C@_1BAO@LCFFDMEN@?$AA?$AN?$AA?6?$AA?$CK?$AA?$CK?$AA?$CK?$AA?5?$AAA?$AAS?$AAS?$AAE?$AAR?$AAT?$AAI?$AAO?$AAN?$AA?5?$AAF?$AAA?$AAI?$AAL?$AAE?$AAD?$AA?5?$AAi?$AAn?$AA?5?$AAd?$AA?3?$AA?2?$AAc?$AAh?$AAe@ 0001f920     fulllibc:strcat_s.obj
 0001:0000ea30       ??_C@_1BCC@BBCJKABO@?$AA?$AN?$AA?6?$AA?$CK?$AA?$CK?$AA?$CK?$AA?5?$AAA?$AAS?$AAS?$AAE?$AAR?$AAT?$AAI?$AAO?$AAN?$AA?5?$AAF?$AAA?$AAI?$AAL?$AAE?$AAD?$AA?5?$AAi?$AAn?$AA?5?$AAd?$AA?3?$AA?2?$AAc?$AAh?$AAe@ 0001fa30     fulllibc:strcat_s.obj
 0001:0000eb54       ??_C@_1DM@FHLMIEG@?$AAS?$AAt?$AAr?$AAi?$AAn?$AAg?$AA?5?$AAi?$AAs?$AA?5?$AAn?$AAo?$AAt?$AA?5?$AAn?$AAu?$AAl?$AAl?$AA?5?$AAt?$AAe?$AAr?$AAm?$AAi?$AAn?$AAa?$AAt?$AAe?$AAd?$AA?$AA@ 0001fb54     fulllibc:strcat_s.obj
 0001:0000eb90       ??_C@_1PI@DLBBMBFO@?$AA?$AN?$AA?6?$AA?$CK?$AA?$CK?$AA?$CK?$AA?5?$AAA?$AAS?$AAS?$AAE?$AAR?$AAT?$AAI?$AAO?$AAN?$AA?5?$AAF?$AAA?$AAI?$AAL?$AAE?$AAD?$AA?5?$AAi?$AAn?$AA?5?$AAd?$AA?3?$AA?2?$AAc?$AAh?$AAe@ 0001fb90     fulllibc:strcat_s.obj
 0001:0000ec88       ??_C@_1BCE@LJDDLNGC@?$AA?$AN?$AA?6?$AA?$CK?$AA?$CK?$AA?$CK?$AA?5?$AAA?$AAS?$AAS?$AAE?$AAR?$AAT?$AAI?$AAO?$AAN?$AA?5?$AAF?$AAA?$AAI?$AAL?$AAE?$AAD?$AA?5?$AAi?$AAn?$AA?5?$AAd?$AA?3?$AA?2?$AAc?$AAh?$AAe@ 0001fc88     fulllibc:strcat_s.obj
 0001:0000edb0       ??_C@_1BCK@BANHEHIA@?$AA?$AN?$AA?6?$AA?$CK?$AA?$CK?$AA?$CK?$AA?5?$AAA?$AAS?$AAS?$AAE?$AAR?$AAT?$AAI?$AAO?$AAN?$AA?5?$AAF?$AAA?$AAI?$AAL?$AAE?$AAD?$AA?5?$AAi?$AAn?$AA?5?$AAd?$AA?3?$AA?2?$AAc?$AAh?$AAe@ 0001fdb0     fulllibc:strtol.obj
 0001:0000eee0       ??_C@_1PA@PKGOPLPJ@?$AA?$AN?$AA?6?$AA?$CK?$AA?$CK?$AA?$CK?$AA?5?$AAA?$AAS?$AAS?$AAE?$AAR?$AAT?$AAI?$AAO?$AAN?$AA?5?$AAF?$AAA?$AAI?$AAL?$AAE?$AAD?$AA?5?$AAi?$AAn?$AA?5?$AAd?$AA?3?$AA?2?$AAc?$AAh?$AAe@ 0001fee0     fulllibc:strtol.obj
 0001:0000efd0       pTOC                       0001ffd0     oal_blcommon:blcommon.obj
 0001:0000efd8       NKSignon                   0001ffd8     oal_blcommon:blcommon.obj
 0001:0000f034       ??_C@_0BI@OCFAEGPK@ROMHDR?5at?5Address?5?$CFXh?$AN?6?$AA@ 00020034     oal_blcommon:blcommon.obj
 0001:0000f04c       ??_C@_0CL@NOFKHKJC@System?5ready?$CB?$AN?6Preparing?5for?5dow@ 0002004c     oal_blcommon:blcommon.obj
 0001:0000f078       ??_C@_0FO@KDFAPMNM@?$CK?$CK?5Please?5update?5your?5Platform?5B@ 00020078     oal_blcommon:blcommon.obj
 0001:0000f0d8       ??_C@_0GI@NIAHKKOO@?$CK?$CK?5ERROR?3?5The?5X000FF?5packet?5is?5a@ 000200d8     oal_blcommon:blcommon.obj
 0001:0000f140       ??_C@_0EC@MIGFFFAC@?$CK?$CK?5ERROR?3?5This?5boot?5loader?5does?5@ 00020140     oal_blcommon:blcommon.obj
 0001:0000f184       ??_C@_04IPBEALME@?$CK?$CK?$AN?6?$AA@ 00020184     oal_blcommon:blcommon.obj
 0001:0000f190       ??_C@_0EC@NABDPCJO@?$CK?$CK?5ERROR?3?5This?5boot?5loader?5does?5@ 00020190     oal_blcommon:blcommon.obj
 0001:0000f1d4       ??_C@_06BEBGGBAB@?$AN?6?$CK?$CK?$AN?6?$AA@ 000201d4     oal_blcommon:blcommon.obj
 0001:0000f1dc       ??_C@_0BM@DKIOIAMD@?$AN?6BL_IMAGE_TYPE_UNKNOWN?$AN?6?$AN?6?$AA@ 000201dc     oal_blcommon:blcommon.obj
 0001:0000f1f8       ??_C@_0BP@KNNCEABF@?$AN?6BL_IMAGE_TYPE_SIGNED_NB0?$AN?6?$AN?6?$AA@ 000201f8     oal_blcommon:blcommon.obj
 0001:0000f218       ??_C@_07LAGBNAEN@R000FF?6?$AA@ 00020218     oal_blcommon:blcommon.obj
 0001:0000f220       ??_C@_0BP@MJFCGNBB@?$AN?6BL_IMAGE_TYPE_SIGNED_BIN?$AN?6?$AN?6?$AA@ 00020220     oal_blcommon:blcommon.obj
 0001:0000f240       ??_C@_07HMMLNAND@S000FF?6?$AA@ 00020240     oal_blcommon:blcommon.obj
 0001:0000f248       ??_C@_0BI@HBMHAEFD@?$AN?6BL_IMAGE_TYPE_BIN?$AN?6?$AN?6?$AA@ 00020248     oal_blcommon:blcommon.obj
 0001:0000f260       ??_C@_07MMNKOBGG@B000FF?6?$AA@ 00020260     oal_blcommon:blcommon.obj
 0001:0000f268       ??_C@_0BN@IHLEHBEK@?$AN?6BL_IMAGE_TYPE_MULTIXIP?$AN?6?$AN?6?$AA@ 00020268     oal_blcommon:blcommon.obj
 0001:0000f288       ??_C@_07CBKBMMIF@X000FF?6?$AA@ 00020288     oal_blcommon:blcommon.obj
 0001:0000f290       ??_C@_0BN@GCKOHOON@?$AN?6BL_IMAGE_TYPE_MANIFEST?$AN?6?$AN?6?$AA@ 00020290     oal_blcommon:blcommon.obj
 0001:0000f2b0       ??_C@_07JLHFPECJ@N000FF?6?$AA@ 000202b0     oal_blcommon:blcommon.obj
 0001:0000f2b8       ??_C@_0CL@OKMIEAHJ@?$AN?6ERROR?3?5Unable?5to?5read?5image?5si@ 000202b8     oal_blcommon:blcommon.obj
 0001:0000f2e8       ??_C@_0EC@LAKEOKID@?$AN?6ERROR?3?5Download?5manifest?5packe@ 000202e8     oal_blcommon:blcommon.obj
 0001:0000f32c       ??_C@_0DJ@PIPLIHFI@?$AN?6ERROR?3?5Unable?5to?5read?5download@ 0002032c     oal_blcommon:blcommon.obj
 0001:0000f368       ??_C@_0DG@DBBGHEAG@?$AN?6ERROR?3?5Unable?5to?5read?5download@ 00020368     oal_blcommon:blcommon.obj
 0001:0000f3a0       ??_C@_0DJ@LFHEGALA@ERROR?3?5Checksum?5failure?5?$CIexpecte@ 000203a0     oal_blcommon:blcommon.obj
 0001:0000f3dc       ??_C@_0DL@DCHMDHHD@ImageStart?5?$DN?50x?$CFx?0?5ImageLength?5?$DN@ 000203dc     oal_blcommon:blcommon.obj
 0001:0000f418       ??_C@_0BD@PHLGNLDI@rom_offset?$DN0x?$CFx?4?$AN?6?$AA@ 00020418     oal_blcommon:blcommon.obj
 0001:0000f42c       ??_C@_0DI@FDIIHFBA@?$CK?$CK?$CK?$CK?$CK?$CK?5Checksum?5failure?5on?5recor@ 0002042c     oal_blcommon:blcommon.obj
 0001:0000f464       ??_C@_0DD@KHJBCIED@?$CK?$CK?$CK?$CK?$CK?$CK?5Data?5record?5?$CFd?5corrupted?0@ 00020464     oal_blcommon:blcommon.obj
 0001:0000f498       ??_C@_0DG@MINKPHJL@?5?$DM?$DO?5Record?5?$FL?5?$CFd?5?$FN?5dwRecAddr?5?$DN?50x@ 00020498     oal_blcommon:blcommon.obj
 0001:0000f4d0       ??_C@_0BP@EOFEMPOO@Invalid?5flash?5address?1length?$AN?6?$AA@ 000204d0     oal_blcommon:blcommon.obj
 0001:0000f4f0       ??_C@_0CC@DNECAMLM@?$CBOEMVERIFYMEMORY?3?5Invalid?5image?$AN@ 000204f0     oal_blcommon:blcommon.obj
 0001:0000f514       ??_C@_0CE@NKAMCDHO@Unable?5to?5read?5image?5start?1lengt@ 00020514     oal_blcommon:blcommon.obj
 0001:0000f538       ??_C@_0CO@PFLGIDFG@ERROR?3?5failed?5when?5reading?5raw?5b@ 00020538     oal_blcommon:blcommon.obj
 0001:0000f568       ??_C@_0DH@GJCJAHAP@?$FL?$CFd?$FN?3?5Address?$DN0x?$CFx?5?5Length?$DN0x?$CFx?5@ 00020568     oal_blcommon:blcommon.obj
 0001:0000f5a0       ??_C@_03ILDADBHF@RAM?$AA@  000205a0     oal_blcommon:blcommon.obj
 0001:0000f5a4       ??_C@_05HPMNGINJ@FLASH?$AA@ 000205a4     oal_blcommon:blcommon.obj
 0001:0000f5b0       ??_C@_0FC@PGPOMBFM@?9?9?9?9?9?9?9?9?9?9?9?9?9?9?9?9?9?9?9?9?9?9?9?9?9?9?9?9?9?9?9?9@ 000205b0     oal_blcommon:blcommon.obj
 0001:0000f604       ??_C@_0BH@FIOKDOBJ@?$AN?6Completed?5file?$CIs?$CJ?3?$AN?6?$AA@ 00020604     oal_blcommon:blcommon.obj
 0001:0000f61c       ??_C@_0BP@GDIKDNGH@Checksum?5?$DN?50x?$CFx?5?$CI0x?$CFx?5bytes?$CJ?$AN?6?$AA@ 0002061c     oal_blcommon:blcommon.obj
 0001:0000f63c       ??_C@_0DF@LEIPBNDI@Computing?5checksum?3?5image?5start?5@ 0002063c     oal_blcommon:blcommon.obj
 0001:0000f674       ??_C@_06OLEINIPO@nk?4exe?$AA@ 00020674     oal_blcommon:blcommon.obj
 0001:0000f680       ??_C@_1GM@LBPDAPNJ@?$AAI?$AAN?$AAF?$AAO?$AA?3?$AAO?$AAA?$AAL?$AAL?$AAo?$AAg?$AAS?$AAe?$AAt?$AAZ?$AAo?$AAn?$AAe?$AAs?$AA?3?$AA?5?$AAd?$AAp?$AAC?$AAu?$AAr?$AAS?$AAe?$AAt?$AAt?$AAi?$AAn@ 00020680     oal_log:debug.obj
 0001:0000f6ec       ??_C@_0CF@FALACPBE@?9OALKitlCreateName?$CIpBuffer?5?$DN?5?8?$CFs@ 000206ec     oal_kitl:name.obj
 0001:0000f714       ??_C@_0CH@OGFCOEMI@?$CLOALKitlCreateName?$CI?8?$CFs?8?0?50x?$CFx?0?50@ 00020714     oal_kitl:name.obj
 0001:0000f73c       ??_C@_1BI@FCMLLAGN@?$AA?$CF?$AAd?$AA?4?$AA?$CF?$AAd?$AA?4?$AA?$CF?$AAd?$AA?4?$AA?$CF?$AAd?$AA?$AA@ 0002073c     oal_kitl:format.obj
 0001:0000f754       ??_C@_1DM@BKFFFBIH@?$AA?$CF?$AA0?$AA2?$AAx?$AA?3?$AA?$CF?$AA0?$AA2?$AAx?$AA?3?$AA?$CF?$AA0?$AA2?$AAx?$AA?3?$AA?$CF?$AA0?$AA2?$AAx?$AA?3?$AA?$CF?$AA0?$AA2?$AAx?$AA?3?$AA?$CF?$AA0?$AA2?$AAx?$AA?$AA@ 00020754     oal_kitl:format.obj
 0001:0000f790       ??_C@_1CE@LKOMNJFD@?$AAS?$AAD?$AAC?$AAo?$AAn?$AAf?$AAi?$AAg?$AAP?$AAi?$AAn?$AAs?$AA?3?$AA?5?$AA?5?$AA?$AN?$AA?6?$AA?$AA@ 00020790     bootcmn:esdhc.obj
 0001:0000f7b4       ??_C@_1CC@BIPKMMMN@?$AA?9?$AA?5?$AAS?$AAe?$AAt?$AAC?$AAl?$AAo?$AAc?$AAk?$AAR?$AAa?$AAt?$AAe?$AA?$AN?$AA?6?$AA?$AA@ 000207b4     bootcmn:esdhc.obj
 0001:0000f7d8       ??_C@_1II@FDLKPLJF@?$AAS?$AAe?$AAt?$AAC?$AAl?$AAo?$AAc?$AAk?$AAR?$AAa?$AAt?$AAe?$AA?5?$AA?9?$AA?5?$AAR?$AAe?$AAq?$AAu?$AAe?$AAs?$AAt?$AAe?$AAd?$AA?5?$AAR?$AAa?$AAt?$AAe?$AA?3?$AA?5?$AA?$CF@ 000207d8     bootcmn:esdhc.obj
 0001:0000f860       ??_C@_1GE@MNBEGPH@?$AAS?$AAD?$AAH?$AAC?$AAC?$AAm?$AAd?$AAC?$AAo?$AAn?$AAf?$AAi?$AAg?$AA?3?$AA?5?$AAC?$AAD?$AAI?$AAH?$AAB?$AA?5?$AAs?$AAe?$AAt?$AA?0?$AA?5?$AAc?$AAa?$AAn?$AA?8?$AAt?$AA?5@ 00020860     bootcmn:esdhc.obj
 0001:0000f8c8       ??_C@_1FI@ICPDGBFJ@?$AAS?$AAD?$AAH?$AAC?$AAC?$AAm?$AAd?$AAC?$AAo?$AAn?$AAf?$AAi?$AAg?$AA?3?$AA?5?$AAC?$AAI?$AAH?$AAB?$AA?5?$AAs?$AAe?$AAt?$AA?0?$AA?5?$AAc?$AAa?$AAn?$AA?8?$AAt?$AA?5?$AAS@ 000208c8     bootcmn:esdhc.obj
 0001:0000f920       ??_C@_1DG@ECDMKJHE@?$AA?9?$AA?5?$AAS?$AAD?$AAH?$AAC?$AAW?$AAa?$AAi?$AAt?$AAE?$AAn?$AAd?$AAC?$AAm?$AAd?$AAR?$AAe?$AAs?$AAp?$AAI?$AAn?$AAt?$AAr?$AA?$AN?$AA?6?$AA?$AA@ 00020920     bootcmn:esdhc.obj
 0001:0000f958       ??_C@_1EI@CNMHMOJJ@?$AAS?$AAD?$AAH?$AAC?$AAW?$AAa?$AAi?$AAt?$AAE?$AAn?$AAd?$AAC?$AAm?$AAd?$AAR?$AAe?$AAs?$AAp?$AAI?$AAn?$AAt?$AAr?$AA?5?$AAS?$AAt?$AAa?$AAt?$AAu?$AAs?$AA?3?$AA?5?$AA?$CF@ 00020958     bootcmn:esdhc.obj
 0001:0000f9a0       ??_C@_1DG@EHOBFMMA@?$AA?$CL?$AA?5?$AAS?$AAD?$AAH?$AAC?$AAW?$AAa?$AAi?$AAt?$AAE?$AAn?$AAd?$AAC?$AAm?$AAd?$AAR?$AAe?$AAs?$AAp?$AAI?$AAn?$AAt?$AAr?$AA?$AN?$AA?6?$AA?$AA@ 000209a0     bootcmn:esdhc.obj
 0001:0000f9d8       ??_C@_1CC@GIPLKAGC@?$AA?9?$AA?5?$AAS?$AAD?$AAH?$AAC?$AAD?$AAa?$AAt?$AAa?$AAR?$AAe?$AAa?$AAd?$AA?$AN?$AA?6?$AA?$AA@ 000209d8     bootcmn:esdhc.obj
 0001:0000f9fc       ??_C@_1CC@LDPGEGNG@?$AA?$CL?$AA?5?$AAS?$AAD?$AAH?$AAC?$AAD?$AAa?$AAt?$AAa?$AAR?$AAe?$AAa?$AAd?$AA?$AN?$AA?6?$AA?$AA@ 000209fc     bootcmn:esdhc.obj
 0001:0000fa20       ??_C@_1CI@HPFBCNOK@?$AA?$CL?$AA?5?$AAC?$AAh?$AAe?$AAc?$AAk?$AAD?$AAa?$AAt?$AAa?$AAS?$AAt?$AAa?$AAt?$AAu?$AAs?$AA?$AN?$AA?6?$AA?$AA@ 00020a20     bootcmn:esdhc.obj
 0001:0000fa48       ??_C@_1CK@NLHLPMPD@?$AA?9?$AA?5?$AAS?$AAD?$AAH?$AAC?$AAD?$AAa?$AAt?$AAa?$AAW?$AAr?$AAi?$AAt?$AAe?$AA?5?$AA?$CF?$AAd?$AA?$AN?$AA?6?$AA?$AA@ 00020a48     bootcmn:esdhc.obj
 0001:0000fa74       ??_C@_1CE@GBOPOCLE@?$AA?$CL?$AA?5?$AAS?$AAD?$AAH?$AAC?$AAD?$AAa?$AAt?$AAa?$AAW?$AAr?$AAi?$AAt?$AAe?$AA?$AN?$AA?6?$AA?$AA@ 00020a74     bootcmn:esdhc.obj
 0001:0000fa98       ??_C@_0DJ@BIKMIJAN@?$AN?6All?5the?5input?5parameters?5are?5s@ 00020a98     bootshell_common_topaz_v1:bootshell.obj
 0001:0000fad8       ??_C@_0EG@IMDNCDIO@?9?9?9?9?9?9?9?9?9?9?9?9?9?9?9?9?9?9?9?9?9?9?9?9?9?9?9?9?9?9?5E@ 00020ad8     bootshell_common_topaz_v1:bootshell.obj
 0001:0000fb20       ??_C@_0DM@EAFILELA@b?5RegAddress?5BitOffset?$CI0?931?$CJ?5Val@ 00020b20     bootshell_common_topaz_v1:bootshell.obj
 0001:0000fb5c       ??_C@_0DM@OGKFCBKC@s?5RegAddress?5RegValue?5?5?5?5?5?5?5?5?5?5?5@ 00020b5c     bootshell_common_topaz_v1:bootshell.obj
 0001:0000fb98       ??_C@_0DN@NGLAIDIN@d?5RegAddress?5?5?5?5?5?5?5?5?5?5?5?5?5?5?5?5?5?5?5?5@ 00020b98     bootshell_common_topaz_v1:bootshell.obj
 0001:0000fbd8       ??_C@_0DP@MKCEOKDD@e?5?5?5?5?5?5?5?5?5?5?5?5?5?5?5?5?5?5?5?5?5?5?5?5?5?5?5?5?5?5?5@ 00020bd8     bootshell_common_topaz_v1:bootshell.obj
 0001:0000fc18       ??_C@_0DJ@JLNEADMA@?$DP?5?5?5?5?5?5?5?5?5?5?5?5?5?5?5?5?5?5?5?5?5?5?5?5?5?5?5?5?5?5?5@ 00020c18     bootshell_common_topaz_v1:bootshell.obj
 0001:0000fc58       ??_C@_0EH@LPLMFKIL@?$AN?6?9?9?9?9?9?9?9?9?9?9?9?9?9?9?9?9?9?9?9?9?9?9?9?9?9?9?9?9?9?5@ 00020c58     bootshell_common_topaz_v1:bootshell.obj
 0001:0000fca0       ??_C@_0CM@CFBEBIAI@New?5Info?5?3?5?5Reg?5Addr?5?$DN?50x?$CFx?0Valu@ 00020ca0     bootshell_common_topaz_v1:bootshell.obj
 0001:0000fccc       ??_C@_0CH@NHPNKMID@Invalid?5Address?0Please?5Input?5Aga@ 00020ccc     bootshell_common_topaz_v1:bootshell.obj
 0001:0000fcf4       ??_C@_0CH@PFJMOMPP@Physical?5Reg?5Addr?5?$DN?5?$CFs?0Value?5?$DN?50@ 00020cf4     bootshell_common_topaz_v1:bootshell.obj
 0001:0000fd1c       ??_C@_0CL@FFJBHPMN@New?5Info?5?3?5Reg?5Addr?5?$DN?50x?$CFx?0Value@ 00020d1c     bootshell_common_topaz_v1:bootshell.obj
 0001:0000fd48       ??_C@_0CJ@JNGMHGML@Invalid?5Bit?5index?0Please?5Input?5A@ 00020d48     bootshell_common_topaz_v1:bootshell.obj
 0001:0000fd78       ??_C@_1EE@IBOLFELJ@?$AAN?$AAF?$AAC?$AAA?$AAl?$AAl?$AAo?$AAc?$AA?3?$AA?5?$AA?5?$AAM?$AAm?$AAM?$AAa?$AAp?$AAI?$AAo?$AAS?$AAp?$AAa?$AAc?$AAe?$AA?5?$AAf?$AAa?$AAi?$AAl?$AAe?$AAd?$AA?$CB?$AA?$AN@ 00020d78     nand_mx25_topaz_v1:cspnand.obj
 0001:0000fdc0       ??_C@_1EO@GCDKFDIC@?$AAN?$AAF?$AAC?$AAS?$AAe?$AAt?$AAP?$AAa?$AAg?$AAe?$AAs?$AAi?$AAz?$AAe?$AA?3?$AA?5?$AAM?$AAm?$AAM?$AAa?$AAp?$AAI?$AAo?$AAS?$AAp?$AAa?$AAc?$AAe?$AA?5?$AAf?$AAa?$AAi@ 00020dc0     nand_mx25_topaz_v1:cspnand.obj
 0001:0000fe10       ??_C@_1EK@GJMEEEMD@?$AAF?$AAM?$AAD?$AA_?$AAI?$AAn?$AAi?$AAt?$AA?3?$AA?5?$AAf?$AAa?$AAi?$AAl?$AAe?$AAd?$AA?5?$AAs?$AAe?$AAt?$AAt?$AAi?$AAn?$AAg?$AA?5?$AAp?$AAa?$AAg?$AAe?$AA?5?$AAs?$AAi@ 00020e10     nand_mx25_topaz_v1:cspnand.obj
 0001:0000fe60       ??_C@_1FK@CFMCDJKB@?$AAF?$AAM?$AAD?$AA_?$AAI?$AAn?$AAi?$AAt?$AA?3?$AA?5?$AAf?$AAa?$AAi?$AAl?$AAe?$AAd?$AA?5?$AAm?$AAe?$AAm?$AAo?$AAr?$AAy?$AA?5?$AAa?$AAl?$AAl?$AAo?$AAc?$AAa?$AAt?$AAi@ 00020e60     nand_mx25_topaz_v1:cspnand.obj
 0001:0000fec0       ??_C@_1KI@BGIGHJEB@?$AAc?$AA?3?$AA?2?$AAw?$AAi?$AAn?$AAc?$AAe?$AAr?$AAo?$AAo?$AAt?$AAs?$AA?2?$AAt?$AAo?$AAp?$AAa?$AAz?$AA?2?$AAw?$AAi?$AAn?$AAc?$AAe?$AA7?$AA0?$AA0?$AA?2?$AAp?$AAl?$AAa@ 00020ec0     nand_mx25_topaz_v1:cspnand.obj
 0001:0000ff68       ??_C@_1IC@MEAOLIC@?$AAS?$AAe?$AAc?$AAt?$AAo?$AAr?$AA?5?$AA0?$AAx?$AA?$CF?$AAX?$AA?5?$AA?9?$AA?9?$AA?9?$AA?5?$AAU?$AAn?$AAc?$AAo?$AAr?$AAr?$AAe?$AAc?$AAt?$AAa?$AAb?$AAl?$AAe?$AA?5?$AAE?$AAC@ 00020f68     nand_mx25_topaz_v1:cspnand.obj
 0001:0000fff0       ??_C@_1GC@GFMOIMEN@?$AAS?$AAe?$AAc?$AAt?$AAo?$AAr?$AA?5?$AA0?$AAx?$AA?$CF?$AAX?$AA?5?$AA?9?$AA?9?$AA?9?$AA?5?$AAU?$AAn?$AAc?$AAo?$AAr?$AAr?$AAe?$AAc?$AAt?$AAa?$AAb?$AAl?$AAe?$AA?5?$AAE?$AAC@ 00020ff0     nand_mx25_topaz_v1:cspnand.obj
 0001:00010058       ??_C@_1EK@DNEGBDKK@?$AAN?$AAA?$AAN?$AAD?$AA?5?$AAe?$AAr?$AAa?$AAs?$AAe?$AA?5?$AAf?$AAa?$AAi?$AAl?$AAe?$AAd?$AA?5?$AA?$CI?$AAb?$AAl?$AAo?$AAc?$AAk?$AAI?$AAD?$AA?5?$AA?$DN?$AA?5?$AA0?$AAx?$AA?$CF@ 00021058     nand_mx25_topaz_v1:cspnand.obj
 0001:000100a8       ??_C@_1FE@OJPAKAII@?$AAN?$AAA?$AAN?$AAD?$AA?5?$AAp?$AAr?$AAo?$AAg?$AAr?$AAa?$AAm?$AA?5?$AAf?$AAa?$AAi?$AAl?$AAe?$AAd?$AA?5?$AA?$CI?$AAS?$AAe?$AAc?$AAt?$AAo?$AAr?$AAa?$AAd?$AAd?$AAr?$AA?5@ 000210a8     nand_mx25_topaz_v1:cspnand.obj
 0001:00010120       OEMBootInit                00021120 f   eboot.obj
 0001:00010158       OEMGetMagicNumber          00021158 f   eboot.obj
 0001:00010174       GetPreDownloadInfo         00021174 f   eboot.obj
 0001:00010398       GetLaunchInfo              00021398 f   eboot.obj
 0001:00010578       OEMReadData                00021578 f   eboot.obj
 0001:00010604       ResetDefaultBootCFG        00021604 f   eboot.obj
 0001:00010898       OEMEthGetFrame             00021898 f   eboot.obj
 0001:000108e0       OEMEthSendFrame            000218e0 f   eboot.obj
 0001:00010b74       BLMenu                     00021b74 f   menu.obj
 0001:00011280       KITLOutputDebugString      00022280 f   oal_blnk:wrappersa.obj
 0001:00011304       NKsprintfA                 00022304 f   oal_blnk:wrappersa.obj
 0001:00011344       inet_ntoa                  00022344 f   oal_blnk:ipformata.obj
 0001:000113b8       inet_addr                  000223b8 f   oal_blnk:ipformata.obj
 0001:000114b8       NKvsprintfA                000224b8 f   oal_blnk:formata.obj
 0001:00012910       OALPAtoVA                  00023910 f   oal_blmemory_arm:memory.obj
 0001:00012a98       OALVAtoPA                  00023a98 f   oal_blmemory_arm:memory.obj
 0001:00012c64       OALSerialInit              00023c64 f   bspcmn:debugserial.obj
 0001:00012cdc       OEMInitDebugSerial         00023cdc f   bspcmn:debugserial.obj
 0001:00012f00       OEMWriteDebugByte          00023f00 f   bspcmn:debugserial.obj
 0001:00012f58       OEMReadDebugByte           00023f58 f   bspcmn:debugserial.obj
 0001:00012fa8       OEMWriteDebugLED           00023fa8 f   bspcmn:debugserial.obj
 0001:00012fb8       OALBspArgsInit             00023fb8 f   bspcmn:bspargs.obj
 0001:0001378c       OALBspArgsPrint            0002478c f   bspcmn:bspargs.obj
 0001:00013d10       main                       00024d10 f   bootcmn:main.obj
 0001:00013d3c       OEMDebugInit               00024d3c f   bootcmn:main.obj
 0001:00013d5c       OEMPlatformInit            00024d5c f   bootcmn:main.obj
 0001:00014190       OEMPreDownload             00025190 f   bootcmn:main.obj
 0001:000143e8       OEMLaunch                  000253e8 f   bootcmn:main.obj
 0001:000144f4       OEMMultiBINNotify          000254f4 f   bootcmn:main.obj
 0001:00014ad8       OEMReportError             00025ad8 f   bootcmn:main.obj
 0001:00014b0c       OEMVerifyMemory            00025b0c f   bootcmn:main.obj
 0001:00014ebc       StoreBootCFG               00025ebc f   bootcmn:main.obj
 0001:00014f14       LoadBootCFG                00025f14 f   bootcmn:main.obj
 0001:00014fd0       ConfigBootCFG              00025fd0 f   bootcmn:main.obj
 0001:00015150       InitSpecifiedEthDevice     00026150 f   bootcmn:ether.obj
 0001:00015634       OALKitlInitEthIrq          00026634 f   bootcmn:ether.obj
 0001:0001564c       OALKitlClearEthIrq         0002664c f   bootcmn:ether.obj
 0001:00015650       OALKitlSendEthSelfReset    00026650 f   bootcmn:ether.obj
 0001:00015668       OEMReset                   00026668 f   bootcmn:utils.obj
 0001:000156b8       SpinForever                000266b8 f   bootcmn:utils.obj
 0001:00015710       OEMShowProgress            00026710 f   bootcmn:utils.obj
 0001:00015720       BootTimerInit              00026720 f   bootcmn:utils.obj
 0001:000157a4       OALClockSetGatingMode      000267a4 f   bootcmn:utils.obj
 0001:00015834       SetBootMe                  00026834 f   bootcmn:utils.obj
 0001:00015a1c       SetDelay                   00026a1c f   bootcmn:utils.obj
 0001:00015bf0       NKCreateStaticMapping      00026bf0 f   bootcmn:utils.obj
 0001:00015c28       OEMIsFlashAddr             00026c28 f   bootcmn:flash.obj
 0001:00015ca0       OEMMapMemAddr              00026ca0 f   bootcmn:flash.obj
 0001:00015d70       OEMStartEraseFlash         00026d70 f   bootcmn:flash.obj
 0001:00015ddc       OEMContinueEraseFlash      00026ddc f   bootcmn:flash.obj
 0001:00015e2c       OEMFinishEraseFlash        00026e2c f   bootcmn:flash.obj
 0001:00015e88       OEMWriteFlash              00026e88 f   bootcmn:flash.obj
 0001:00016194       FlashLoadBootCFG           00027194 f   bootcmn:flash.obj
 0001:0001624c       FlashStoreBootCFG          0002724c f   bootcmn:flash.obj
 0001:00016304       SPIWriteXldr               00027304 f   bootcmn:cspi_flash.obj
 0001:0001653c       SPIWriteBoot               0002753c f   bootcmn:cspi_flash.obj
 0001:0001694c       SPILoadBootCFG             0002794c f   bootcmn:cspi_flash.obj
 0001:00016ab8       SPIStoreBootCFG            00027ab8 f   bootcmn:cspi_flash.obj
 0001:00016cc4       I2CEEPROMWriteXldr         00027cc4 f   bootcmn:i2c_eeprom.obj
 0001:00016f0c       PageWrite                  00027f0c f   bootcmn:i2c_eeprom.obj
 0001:00017020       PageRead                   00028020 f   bootcmn:i2c_eeprom.obj
 0001:00017168       IsWriteOperationComplete   00028168 f   bootcmn:i2c_eeprom.obj
 0001:00017218       OALConfigSerialUART        00028218 f   serialutils:serialutils.obj
 0001:00017658       OALConfigSerialIOMUX       00028658 f   serialutils:serialutils.obj
 0001:00017754       OALStall                   00028754 f   ethdrv:ethdrv.obj
 0001:000179d4       OEMEthGetSecs              000289d4 f   ethdrv:ethdrv.obj
 0001:000179f8       OEMKitlGetSecs             000289f8 f   ethdrv:ethdrv.obj
 0001:00017bbc       BLMenuShow                 00028bbc f   blmenu_common_topaz_v1:menu.obj
 0001:00017f84       BLMenuEnableDisable        00028f84 f   blmenu_common_topaz_v1:menu.obj
 0001:000180d8       BLMenuSetMacAddress        000290d8 f   blmenu_common_topaz_v1:menu.obj
 0001:00018284       BLMenuSetIpAddress         00029284 f   blmenu_common_topaz_v1:menu.obj
 0001:000183f4       BLMenuSetIpMask            000293f4 f   blmenu_common_topaz_v1:menu.obj
 0001:0001855c       BLMenuReadLine             0002955c f   blmenu_common_topaz_v1:menu.obj
 0001:00018694       BLMenuPrintData            00029694 f   blmenu_common_topaz_v1:menu.obj
 0001:00018a88       BLMenuBootShell            00029a88 f   blmenu_common_topaz_v1:menu.obj
 0001:00018ab0       BLMenuSaveSettings         00029ab0 f   blmenu_common_topaz_v1:menu.obj
 0001:00018b04       BLMenuReset                00029b04 f   blmenu_common_topaz_v1:menu.obj
 0001:00018b2c       BLMenuLaunchFlashImage     00029b2c f   blmenu_common_topaz_v1:menu.obj
 0001:00018b60       BLMenuBootDelay            00029b60 f   blmenu_common_topaz_v1:menu.obj
 0001:00018ba4       BLMenuResetConfiguration   00029ba4 f   blmenu_common_topaz_v1:menu.obj
 0001:00018bd8       BLMenuDownloadImageNow     00029bd8 f   blmenu_common_topaz_v1:menu.obj
 0001:00018c0c       BLMenuFormatNandOS         00029c0c f   blmenu_common_topaz_v1:menu.obj
 0001:00018c98       BLMenuFormatAllNand        00029c98 f   blmenu_common_topaz_v1:menu.obj
 0001:00018d30       BLMenuMMCSDUtilities       00029d30 f   blmenu_common_topaz_v1:menu.obj
 0001:00018d60       BLMenuEMMCToggleBP         00029d60 f   blmenu_common_topaz_v1:menu.obj
 0001:00018da4       BLMenuEMMCBPSize           00029da4 f   blmenu_common_topaz_v1:menu.obj
 0001:00018e58       BLMenuESDBPEnable          00029e58 f   blmenu_common_topaz_v1:menu.obj
 0001:00018e80       BLMenuESDBPSize            00029e80 f   blmenu_common_topaz_v1:menu.obj
 0001:00018f34       BLMenuFormatAllSDMMC       00029f34 f   blmenu_common_topaz_v1:menu.obj
 0001:00018fcc       BLMenuCreateFileSystemOnSDMMC 00029fcc f   blmenu_common_topaz_v1:menu.obj
 0001:00019080       BLMenuReturn               0002a080 f   blmenu_common_topaz_v1:menu.obj
 0001:000190a4       BspBootShell               0002a0a4 f   bsp_bootshell:bspbootshell.obj
 0001:000197d0       MIIREAD                    0002a7d0 f   oal_ethdrv_fec_common_topaz_v1:fec.obj
 0001:000198e0       MIIWRITE                   0002a8e0 f   oal_ethdrv_fec_common_topaz_v1:fec.obj
 0001:00019968       CalculateHashValue         0002a968 f   oal_ethdrv_fec_common_topaz_v1:fec.obj
 0001:00019a64       FECEnableInts              0002aa64 f   oal_ethdrv_fec_common_topaz_v1:fec.obj
 0001:00019b10       FECDisableInts             0002ab10 f   oal_ethdrv_fec_common_topaz_v1:fec.obj
 0001:00019bbc       FECInitDMABuffer           0002abbc f   oal_ethdrv_fec_common_topaz_v1:fec.obj
 0001:00019f98       FECInit                    0002af98 f   oal_ethdrv_fec_common_topaz_v1:fec.obj
 0001:0001aa6c       FECSendFrame               0002ba6c f   oal_ethdrv_fec_common_topaz_v1:fec.obj
 0001:0001ad20       FECGetFrame                0002bd20 f   oal_ethdrv_fec_common_topaz_v1:fec.obj
 0001:0001afbc       FECCurrentPacketFilter     0002bfbc f   oal_ethdrv_fec_common_topaz_v1:fec.obj
 0001:0001b0ec       FECMulticastList           0002c0ec f   oal_ethdrv_fec_common_topaz_v1:fec.obj
 0001:0001b2ec       OALKitlGetFECDmaBuffer     0002c2ec f   bspfec:bspfec.obj
 0001:0001b308       OALKitlFECBSPInit          0002c308 f   bspfec:bspfec.obj
 0001:0001b6b4       BSPFECusesRMII             0002c6b4 f   bspfec:bspfec.obj
 0001:0001b6cc       RndisRestart               0002c6cc f   fsl_rne_mdd_common_topaz_v1:rndis.obj
 0001:0001b75c       RndisPrepareRndisPacket    0002c75c f   fsl_rne_mdd_common_topaz_v1:rndis.obj
 0001:0001b8cc       PDD_IsPacketSend           0002c8cc f   fsl_rne_mdd_common_topaz_v1:rndis.obj
 0001:0001b8ec       MddSendRndisPacketComplete 0002c8ec f   fsl_rne_mdd_common_topaz_v1:rndis.obj
 0001:0001b90c       RndisEDbgSendFrame         0002c90c f   fsl_rne_mdd_common_topaz_v1:rndis.obj
 0001:0001bb0c       MddSendRndisMessageComplete 0002cb0c f   fsl_rne_mdd_common_topaz_v1:rndis.obj
 0001:0001bb50       RndisSendRndisMessage      0002cb50 f   fsl_rne_mdd_common_topaz_v1:rndis.obj
 0001:0001c02c       RndisProcessMessage        0002d02c f   fsl_rne_mdd_common_topaz_v1:rndis.obj
 0001:0001c538       RndisEDbgGetFrame          0002d538 f   fsl_rne_mdd_common_topaz_v1:rndis.obj
 0001:0001c71c       RndisProcessPacket         0002d71c f   fsl_rne_mdd_common_topaz_v1:rndis.obj
 0001:0001c988       RndisInit                  0002d988 f   fsl_rne_mdd_common_topaz_v1:rndis.obj
 0001:0001cc40       RndisGetIrq                0002dc40 f   fsl_rne_mdd_common_topaz_v1:rndis.obj
 0001:0001cc60       RndisGetPCICard            0002dc60 f   fsl_rne_mdd_common_topaz_v1:rndis.obj
 0001:0001cc98       RndisDeInit                0002dc98 f   fsl_rne_mdd_common_topaz_v1:rndis.obj
 0001:0001cc9c       RndisCurrentPacketFilter   0002dc9c f   fsl_rne_mdd_common_topaz_v1:rndis.obj
 0001:0001ccac       RndisMulticastList         0002dcac f   fsl_rne_mdd_common_topaz_v1:rndis.obj
 0001:0001ccd0       RndisEnableInts            0002dcd0 f   fsl_rne_mdd_common_topaz_v1:rndis.obj
 0001:0001ccf4       RndisDisableInts           0002dcf4 f   fsl_rne_mdd_common_topaz_v1:rndis.obj
 0001:0001cd18       RndisSetOptions            0002dd18 f   fsl_rne_mdd_common_topaz_v1:rndis.obj
 0001:0001cd3c       MddInitializeCriticalSection 0002dd3c f   fsl_rne_mdd_common_topaz_v1:rndis.obj
 0001:0001cd4c       MddDeleteCriticalSection   0002dd4c f   fsl_rne_mdd_common_topaz_v1:rndis.obj
 0001:0001cd5c       MddEnterCriticalSection    0002dd5c f   fsl_rne_mdd_common_topaz_v1:rndis.obj
 0001:0001cd6c       MddLeaveCriticalSection    0002dd6c f   fsl_rne_mdd_common_topaz_v1:rndis.obj
 0001:0001cd7c       RndisMiniCeLogMsg          0002dd7c f   fsl_rne_mdd_common_topaz_v1:rndis.obj
 0001:0001cd8c       HostMiniQueryInformation   0002dd8c f   fsl_rne_mdd_common_topaz_v1:hostmini.obj
 0001:0001d1f8       HostMiniSetInformation     0002e1f8 f   fsl_rne_mdd_common_topaz_v1:hostmini.obj
 0001:0001d3fc       MddIndicateRndisMessage    0002e3fc f   fsl_rne_mdd_common_topaz_v1:hostmini.obj
 0001:0001d414       MddIndicateRndisPacket     0002e414 f   fsl_rne_mdd_common_topaz_v1:hostmini.obj
 0001:0001d43c       MDDAllocDataWrapper        0002e43c f   fsl_rne_mdd_common_topaz_v1:hostmini.obj
 0001:0001d4b4       MDDAllocMem                0002e4b4 f   fsl_rne_mdd_common_topaz_v1:hostmini.obj
 0001:0001d4d0       MDDFreeMem                 0002e4d0 f   fsl_rne_mdd_common_topaz_v1:hostmini.obj
 0001:0001d4e0       MDDFreeDataWrapper         0002e4e0 f   fsl_rne_mdd_common_topaz_v1:hostmini.obj
 0001:0001d500       MddDisconnect              0002e500 f   fsl_rne_mdd_common_topaz_v1:hostmini.obj
 0001:0001d51c       HostMiniInit               0002e51c f   fsl_rne_mdd_common_topaz_v1:hostmini.obj
 0001:0001d578       HostMiniDeInit             0002e578 f   fsl_rne_mdd_common_topaz_v1:hostmini.obj
 0001:0001d594       InitBuffer                 0002e594 f   fsl_rne_mdd_common_topaz_v1:util.obj
 0001:0001d690       AvaiableBufferSize         0002e690 f   fsl_rne_mdd_common_topaz_v1:util.obj
 0001:0001d76c       AllocBuffer                0002e76c f   fsl_rne_mdd_common_topaz_v1:util.obj
 0001:0001d9e8       FreeBuffer                 0002e9e8 f   fsl_rne_mdd_common_topaz_v1:util.obj
 0001:0001dd2c       GetFirstUsedBuffer         0002ed2c f   fsl_rne_mdd_common_topaz_v1:util.obj
 0001:0001de3c       PDD_GetDescriptor          0002ee3c f   fsl_rne_pdd_common_topaz_v1:rndis_pdd.obj
 0001:0001e1c0       PDD_DoVendorCommand        0002f1c0 f   fsl_rne_pdd_common_topaz_v1:rndis_pdd.obj
 0001:0001e548       setupDataOutTransfer       0002f548 f   fsl_rne_pdd_common_topaz_v1:rndis_pdd.obj
 0001:0001e6fc       HandleSetupPacket          0002f6fc f   fsl_rne_pdd_common_topaz_v1:rndis_pdd.obj
 0001:0001eb90       TxComplete                 0002fb90 f   fsl_rne_pdd_common_topaz_v1:rndis_pdd.obj
 0001:0001ec64       NotifyHandler              0002fc64 f   fsl_rne_pdd_common_topaz_v1:rndis_pdd.obj
 0001:0001f9a4       PDDInit                    000309a4 f   fsl_rne_pdd_common_topaz_v1:rndis_pdd.obj
 0001:0001fcc4       PDDDeinit                  00030cc4 f   fsl_rne_pdd_common_topaz_v1:rndis_pdd.obj
 0001:0001fd58       PDD_SendRndisMessage       00030d58 f   fsl_rne_pdd_common_topaz_v1:rndis_pdd.obj
 0001:0001ff0c       PDD_SendRndisPacket        00030f0c f   fsl_rne_pdd_common_topaz_v1:rndis_pdd.obj
 0001:00020124       PDD_Set                    00031124 f   fsl_rne_pdd_common_topaz_v1:rndis_pdd.obj
 0001:00020404       PDD_Get                    00031404 f   fsl_rne_pdd_common_topaz_v1:rndis_pdd.obj
 0001:00020640       PDD_ISR                    00031640 f   fsl_rne_pdd_common_topaz_v1:rndis_pdd.obj
 0001:00020674       PDD_IndicateRndisPacketComplete 00031674 f   fsl_rne_pdd_common_topaz_v1:rndis_pdd.obj
 0001:00020728       SetRNDISMACAddress         00031728 f   fsl_rne_pdd_common_topaz_v1:rndis_pdd.obj
 0001:00020744       SetRNDISSerialNumber       00031744 f   fsl_rne_pdd_common_topaz_v1:rndis_pdd.obj
 0001:000208cc       IsListEmpty                000318cc f i fsl_rne_pdd_common_topaz_v1:rndis_pdd.obj
 0001:00020918       RemoveHeadList             00031918 f i fsl_rne_pdd_common_topaz_v1:rndis_pdd.obj
 0001:0002095c       CheckListEntry             0003195c f i fsl_rne_pdd_common_topaz_v1:rndis_pdd.obj
 0001:00020b04       RemoveEntryList            00031b04 f i fsl_rne_pdd_common_topaz_v1:rndis_pdd.obj
 0001:00020b78       InitializeListHead         00031b78 f i fsl_rne_pdd_common_topaz_v1:rndis_pdd.obj
 0001:00020bb8       InsertTailList             00031bb8 f i fsl_rne_pdd_common_topaz_v1:rndis_pdd.obj
 0001:00020be0       InsertEntryList            00031be0 f i fsl_rne_pdd_common_topaz_v1:rndis_pdd.obj
 0001:00020c70       DescriptorPhy              00031c70 f   usb_usbfn_mx25_topaz_v1:i_pdd.obj
 0001:00020cc4       DescriptorVirtual          00031cc4 f   usb_usbfn_mx25_topaz_v1:i_pdd.obj
 0001:00020d18       ClearUsbstsUI              00031d18 f   usb_usbfn_mx25_topaz_v1:i_pdd.obj
 0001:00020d94       UfnPdd_PowerDown           00031d94 f   usb_usbfn_mx25_topaz_v1:i_pdd.obj
 0001:000214c0       UfnPdd_PowerUp             000324c0 f   usb_usbfn_mx25_topaz_v1:i_pdd.obj
 0001:00021a10       UpdateDevicePower          00032a10 f   usb_usbfn_mx25_topaz_v1:i_pdd.obj
 0001:00021d18       SetupEvent                 00032d18 f   usb_usbfn_mx25_topaz_v1:i_pdd.obj
 0001:00022468       DumpDeviceState            00033468 f   usb_usbfn_mx25_topaz_v1:i_pdd.obj
 0001:0002292c       DumpInterruptSource        0003392c f   usb_usbfn_mx25_topaz_v1:i_pdd.obj
 0001:00022ac4       CopyFromUncachedBuffer     00033ac4 f   usb_usbfn_mx25_topaz_v1:i_pdd.obj
 0001:00022d50       CheckEndpoint              00033d50 f   usb_usbfn_mx25_topaz_v1:i_pdd.obj
 0001:000242cc       InterruptHandle            000352cc f   usb_usbfn_mx25_topaz_v1:i_pdd.obj
 0001:000257e8       UfnPdd_IssueTransfer       000367e8 f   usb_usbfn_mx25_topaz_v1:i_pdd.obj
 0001:000275cc       UfnPdd_AbortTransfer       000385cc f   usb_usbfn_mx25_topaz_v1:i_pdd.obj
 0001:00027c94       UfnPdd_StallEndpoint       00038c94 f   usb_usbfn_mx25_topaz_v1:i_pdd.obj
 0001:00027e4c       UfnPdd_ClearEndpointStall  00038e4c f   usb_usbfn_mx25_topaz_v1:i_pdd.obj
 0001:0002804c       UfnPdd_IsEndpointHalted    0003904c f   usb_usbfn_mx25_topaz_v1:i_pdd.obj
 0001:00028218       UfnPdd_SendControlStatusHandshake 00039218 f   usb_usbfn_mx25_topaz_v1:i_pdd.obj
 0001:00028be0       UfnPdd_InitiateRemoteWakeup 00039be0 f   usb_usbfn_mx25_topaz_v1:i_pdd.obj
 0001:00028c64       SetPowerState              00039c64 f   usb_usbfn_mx25_topaz_v1:i_pdd.obj
 0001:00029018       UfnPdd_IOControl           0003a018 f   usb_usbfn_mx25_topaz_v1:i_pdd.obj
 0001:0002959c       UfnPdd_Deinit              0003a59c f   usb_usbfn_mx25_topaz_v1:i_pdd.obj
 0001:000295c8       UfnPdd_DeregisterDevice    0003a5c8 f   usb_usbfn_mx25_topaz_v1:i_pdd.obj
 0001:000295ec       UfnPdd_Stop                0003a5ec f   usb_usbfn_mx25_topaz_v1:i_pdd.obj
 0001:00029718       UfnPdd_DeinitEndpoint      0003a718 f   usb_usbfn_mx25_topaz_v1:i_pdd.obj
 0001:00029970       UfnPdd_InitEndpoint        0003a970 f   usb_usbfn_mx25_topaz_v1:i_pdd.obj
 0001:00029dfc       UfnPdd_SetAddress          0003adfc f   usb_usbfn_mx25_topaz_v1:i_pdd.obj
 0001:00029e6c       UfnPdd_Start               0003ae6c f   usb_usbfn_mx25_topaz_v1:i_pdd.obj
 0001:0002ab40       UfnPdd_RegisterDevice      0003bb40 f   usb_usbfn_mx25_topaz_v1:i_pdd.obj
 0001:0002b010       UfnPdd_IsEndpointSupportable 0003c010 f   usb_usbfn_mx25_topaz_v1:i_pdd.obj
 0001:0002b0a8       UfnPdd_IsConfigurationSupportable 0003c0a8 f   usb_usbfn_mx25_topaz_v1:i_pdd.obj
 0001:0002b3d4       UfnPdd_Init                0003c3d4 f   usb_usbfn_mx25_topaz_v1:i_pdd.obj
 0001:0002bc24       UfnPdd_DllEntry            0003cc24 f   usb_usbfn_mx25_topaz_v1:i_pdd.obj
 0001:0002bc48       FslUfnGetUsbFnPdd          0003cc48 f   usb_usbfn_eboot_mx25_topaz_v1:i_stub.obj
 0001:0002bc64       FslUfnRequestIrq           0003cc64 f   usb_usbfn_eboot_mx25_topaz_v1:i_stub.obj
 0001:0002bc88       FslUfnIsUSBKitlEnable      0003cc88 f   usb_usbfn_eboot_mx25_topaz_v1:i_stub.obj
 0001:0002bca0       FslUfnCreateThread         0003cca0 f   usb_usbfn_eboot_mx25_topaz_v1:i_stub.obj
 0001:0002bcc4       UsbFnInterruptThread       0003ccc4 f   usb_usbfn_eboot_mx25_topaz_v1:i_stub.obj
 0001:0002bd04       FslUfnTrigIrq              0003cd04 f   usb_usbfn_eboot_mx25_topaz_v1:i_stub.obj
 0001:0002bd1c       FslUfnDeinit               0003cd1c f   usb_usbfn_eboot_mx25_topaz_v1:i_stub.obj
 0001:0002bd2c       FslUfnGetDMABuffer         0003cd2c f   usb_usbfn_eboot_mx25_topaz_v1:i_stub.obj
 0001:0002be54       BSPUSBClockSwitch          0003ce54 f   usb_usbfn_eboot_mx25_topaz_v1:i_stub.obj
 0001:0002be78       BSPUSBClockCreateFileMapping 0003ce78 f   usb_usbfn_eboot_mx25_topaz_v1:i_stub.obj
 0001:0002be90       GetDeviceRegistryParams    0003ce90 f   usb_usbfn_eboot_mx25_topaz_v1:i_stub.obj
 0001:0002bee0       SetInterruptEvent          0003cee0 f   usb_usbfn_eboot_mx25_topaz_v1:i_stub.obj
 0001:0002bf10       FslUfnGetPageNumber        0003cf10 f   usb_usbfn_eboot_mx25_topaz_v1:i_stub.obj
 0001:0002bf54       FslUfnGetPageSize          0003cf54 f   usb_usbfn_eboot_mx25_topaz_v1:i_stub.obj
 0001:0002bf6c       FslUfnGetPageShift         0003cf6c f   usb_usbfn_eboot_mx25_topaz_v1:i_stub.obj
 0001:0002bf84       FslInitializeCriticalSection 0003cf84 f   usb_usbfn_eboot_mx25_topaz_v1:i_stub.obj
 0001:0002bf94       FslEnterCriticalSection    0003cf94 f   usb_usbfn_eboot_mx25_topaz_v1:i_stub.obj
 0001:0002bfa4       FslLeaveCriticalSection    0003cfa4 f   usb_usbfn_eboot_mx25_topaz_v1:i_stub.obj
 0001:0002bfb4       LocalFree                  0003cfb4 f   usb_usbfn_eboot_mx25_topaz_v1:i_stub.obj
 0001:0002bfd8       CreateBusAccessHandle      0003cfd8 f   usb_usbfn_eboot_mx25_topaz_v1:i_stub.obj
 0001:0002bffc       CloseBusAccessHandle       0003cffc f   usb_usbfn_eboot_mx25_topaz_v1:i_stub.obj
 0001:0002c00c       CloseHandle                0003d00c f   usb_usbfn_eboot_mx25_topaz_v1:i_stub.obj
 0001:0002c030       MmUnmapIoSpace             0003d030 f   usb_usbfn_eboot_mx25_topaz_v1:i_stub.obj
 0001:0002c040       CeLogData                  0003d040 f   usb_usbfn_eboot_mx25_topaz_v1:i_stub.obj
 0001:0002c050       InterruptInitialize        0003d050 f   usb_usbfn_eboot_mx25_topaz_v1:i_stub.obj
 0001:0002c074       InterruptDone              0003d074 f   usb_usbfn_eboot_mx25_topaz_v1:i_stub.obj
 0001:0002c084       MmMapIoSpace               0003d084 f   usb_usbfn_eboot_mx25_topaz_v1:i_stub.obj
 0001:0002c0bc       InterruptDisable           0003d0bc f   usb_usbfn_eboot_mx25_topaz_v1:i_stub.obj
 0001:0002c0cc       CacheSync                  0003d0cc f   usb_usbfn_eboot_mx25_topaz_v1:i_stub.obj
 0001:0002c0e4       LockPages                  0003d0e4 f   usb_usbfn_eboot_mx25_topaz_v1:i_stub.obj
 0001:0002c120       GetLastError               0003d120 f   usb_usbfn_eboot_mx25_topaz_v1:i_stub.obj
 0001:0002c138       UnlockPages                0003d138 f   usb_usbfn_eboot_mx25_topaz_v1:i_stub.obj
 0001:0002c15c       CeOpenCallerBuffer         0003d15c f   usb_usbfn_eboot_mx25_topaz_v1:i_stub.obj
 0001:0002c18c       CeCloseCallerBuffer        0003d18c f   usb_usbfn_eboot_mx25_topaz_v1:i_stub.obj
 0001:0002c1b0       StringCchLengthW           0003d1b0 f   usb_usbfn_eboot_mx25_topaz_v1:i_stub.obj
 0001:0002c1ec       StringCchVPrintfW          0003d1ec f   usb_usbfn_eboot_mx25_topaz_v1:i_stub.obj
 0001:0002c210       SetDevicePowerState        0003d210 f   usb_usbfn_eboot_mx25_topaz_v1:i_stub.obj
 0001:0002c234       Sleep                      0003d234 f   usb_usbfn_eboot_mx25_topaz_v1:i_stub.obj
 0001:0002c24c       FslNKDbgPrintfW            0003d24c f   usb_usbfn_eboot_mx25_topaz_v1:i_stub.obj
 0001:0002c2a4       CacheRangeFlush            0003d2a4 f   usb_usbfn_eboot_mx25_topaz_v1:i_stub.obj
 0001:0002c358       SerialReadData             0003d358 f   oal_blserial:serfuncs.obj
 0001:0002c5b8       ?CalcChksum@@YAEPAEG@Z     0003d5b8 f   oal_blserial:serfuncs.obj
 0001:0002c654       SerialSendBootRequest      0003d654 f   oal_blserial:serfuncs.obj
 0001:0002c770       SerialSendBlockAck         0003d770 f   oal_blserial:serfuncs.obj
 0001:0002c8c8       SerialWaitForBootAck       0003d8c8 f   oal_blserial:serfuncs.obj
 0001:0002c9c4       SerialWaitForJump          0003d9c4 f   oal_blserial:serfuncs.obj
 0001:0002caac       RecvPacket                 0003daac f   oal_blserial:serfuncs.obj
 0001:0002cc88       RecvHeader                 0003dc88 f   oal_blserial:serfuncs.obj
 0001:0002cdf4       ?HandleClassRequest@@YAXPAU_USB_DEVICE_REQUEST@@PAU_EP0_REQUEST@@@Z 0003ddf4 f   fsl_serial_pdd_common_topaz_v1:serial_dl.obj
 0001:0002cf20       ?HandleGetDescriptor@@YAXPAU_USB_DEVICE_REQUEST@@PAU_EP0_REQUEST@@@Z 0003df20 f   fsl_serial_pdd_common_topaz_v1:serial_dl.obj
 0001:0002d0ec       ?HandleTransferComplete@@YAXPAU_STransfer@@@Z 0003e0ec f   fsl_serial_pdd_common_topaz_v1:serial_dl.obj
 0001:0002d574       USBSerialInit              0003e574 f   fsl_serial_pdd_common_topaz_v1:serial_dl.obj
 0001:0002e2e0       OEMSerialSendRaw           0003f2e0 f   fsl_serial_pdd_common_topaz_v1:serial_dl.obj
 0001:0002e4bc       OEMSerialRecvRaw           0003f4bc f   fsl_serial_pdd_common_topaz_v1:serial_dl.obj
 0001:0002ea70       USBKitlSerialInit          0003fa70 f   fsl_serial_pdd_common_topaz_v1:serial_dl.obj
 0001:0002eaac       USBKitlSerialRecv          0003faac f   fsl_serial_pdd_common_topaz_v1:serial_dl.obj
 0001:0002ec60       USBKitlSerialSend          0003fc60 f   fsl_serial_pdd_common_topaz_v1:serial_dl.obj
 0001:0002ecb4       USBKitlSerialEnableInts    0003fcb4 f   fsl_serial_pdd_common_topaz_v1:serial_dl.obj
 0001:0002ecb8       USBKitlSerialDisableInts   0003fcb8 f   fsl_serial_pdd_common_topaz_v1:serial_dl.obj
 0001:0002ecbc       GetRNDISMACAddress         0003fcbc f   fsl_usbfn_rndiskitl_mx25_topaz_v1:hwinit.obj
 0001:0002ed04       controllerSetup            0003fd04 f   fsl_usbfn_rndiskitl_mx25_topaz_v1:hwinit.obj
 0001:0002eebc       USBClockInit               0003febc f   fsl_usbfn_rndiskitl_mx25_topaz_v1:hwinit.obj
 0001:0002eee4       HardwareInitialize         0003fee4 f   fsl_usbfn_rndiskitl_mx25_topaz_v1:hwinit.obj
 0001:0002f118       PowerDownSchemeExist       00040118 f   fsl_usbfn_rndiskitl_mx25_topaz_v1:hwinit.obj
 0001:0002f130       BSPUsbXvrEnableVBUSIntr    00040130 f   fsl_usbfn_rndiskitl_mx25_topaz_v1:hwinit.obj
 0001:0002f1ac       BSPUsbResetPHY             000401ac f   fsl_usbfn_rndiskitl_mx25_topaz_v1:hwinit.obj
 0001:0002f1bc       BSPUsbSetBusConfig         000401bc f   fsl_usbfn_rndiskitl_mx25_topaz_v1:hwinit.obj
 0001:0002f1fc       BSPUSBInterruptControl     000401fc f   fsl_usbfn_rndiskitl_mx25_topaz_v1:hwinit.obj
 0001:0002f20c       BSPPhyShowDevDiscon        0004020c f   fsl_usbfn_rndiskitl_mx25_topaz_v1:hwinit.obj
 0001:0002f224       BSPUsbSetCurrentLimitation 00040224 f   fsl_usbfn_rndiskitl_mx25_topaz_v1:hwinit.obj
 0001:0002f234       FslUfnGetKitlDMABuffer     00040234 f   fsl_usbfn_rndiskitl_mx25_topaz_v1:stub.obj
 0001:0002f250       NANDBootReserved           00040250 f   nand_boot_common_topaz_v1:nandboot.obj
 0001:0002f440       GetNextGoodBlock           00040440 f   nand_boot_common_topaz_v1:nandboot.obj
 0001:0002f4c0       GetPhyBlkAddr              000404c0 f   nand_boot_common_topaz_v1:nandboot.obj
 0001:0002f578       NANDWriteXldr              00040578 f   nand_boot_common_topaz_v1:nandboot.obj
 0001:0002fb54       NANDWriteBoot              00040b54 f   nand_boot_common_topaz_v1:nandboot.obj
 0001:00030080       NANDWriteNK                00041080 f   nand_boot_common_topaz_v1:nandboot.obj
 0001:00030694       NANDLoadNK                 00041694 f   nand_boot_common_topaz_v1:nandboot.obj
 0001:00030914       NANDLoadBootCFG            00041914 f   nand_boot_common_topaz_v1:nandboot.obj
 0001:00030aa0       NANDStoreBootCFG           00041aa0 f   nand_boot_common_topaz_v1:nandboot.obj
 0001:00030ccc       NANDFormatNK               00041ccc f   nand_boot_common_topaz_v1:nandboot.obj
 0001:00030e8c       NANDWriteIPL               00041e8c f   nand_boot_common_topaz_v1:nandboot.obj
 0001:000313c8       IsSectorEmpty              000423c8 f   nand_boot_common_topaz_v1:nandboot.obj
 0001:00031494       NANDStartWriteBinDIO       00042494 f   nand_boot_common_topaz_v1:nandboot.obj
 0001:00031728       NANDContinueWriteBinDIO    00042728 f   nand_boot_common_topaz_v1:nandboot.obj
 0001:00031b5c       NANDFinishWriteBinDIO      00042b5c f   nand_boot_common_topaz_v1:nandboot.obj
 0001:00031bb0       NANDLoadIPL                00042bb0 f   nand_boot_common_topaz_v1:nandboot.obj
 0001:00031dec       NANDFormatAll              00042dec f   nand_boot_common_topaz_v1:nandboot.obj
 0001:00031f80       NANDLowLevelFormat         00042f80 f   nand_boot_common_topaz_v1:nandboot.obj
 0001:000320bc       FMD_Init                   000430bc f   nand_common_topaz_v1:fmd.obj
 0001:0003241c       FMD_Deinit                 0004341c f   nand_common_topaz_v1:fmd.obj
 0001:00032454       FMD_ReadSector             00043454 f   nand_common_topaz_v1:fmd.obj
 0001:00032734       FMD_EraseBlock             00043734 f   nand_common_topaz_v1:fmd.obj
 0001:00032828       FMD_WriteSector            00043828 f   nand_common_topaz_v1:fmd.obj
 0001:00032a24       FMD_PowerUp                00043a24 f   nand_common_topaz_v1:fmd.obj
 0001:00032a28       FMD_PowerDown              00043a28 f   nand_common_topaz_v1:fmd.obj
 0001:00032a2c       FMD_OEMIoControl           00043a2c f   nand_common_topaz_v1:fmd.obj
 0001:00032a78       FMD_GetInfo                00043a78 f   nand_common_topaz_v1:fmd.obj
 0001:00032bd0       FMD_GetBlockStatus         00043bd0 f   nand_common_topaz_v1:fmd.obj
 0001:00032d44       FMD_SetBlockStatus         00043d44 f   nand_common_topaz_v1:fmd.obj
 0001:00032e9c       ?BBT_GetBlockBadStatus@@YAHKK@Z 00043e9c f   nand_common_topaz_v1:bbt.obj
 0001:00032fe4       ?BBT_SetBlockBadStatus@@YAXKK@Z 00043fe4 f   nand_common_topaz_v1:bbt.obj
 0001:00033c18       ?BBT_Init@@YAHXZ           00044c18 f   nand_common_topaz_v1:bbt.obj
 0001:00034994       BSPNAND_GetFlashInfo       00045994 f   nandfmd_lib:nandbsp.obj
 0001:00034b88       BSPNAND_GetBufferPointer   00045b88 f   nandfmd_lib:nandbsp.obj
 0001:00034c20       SDMMC_Init                 00045c20 f   sdmmc_boot_common_topaz_v1:sdfmd.obj
 0001:00034dd4       SDMMC_Deinit               00045dd4 f   sdmmc_boot_common_topaz_v1:sdfmd.obj
 0001:00034df4       SDMMC_get_cid              00045df4 f   sdmmc_boot_common_topaz_v1:sdfmd.obj
 0001:00034f10       SDMMC_set_data_transfer_mode 00045f10 f   sdmmc_boot_common_topaz_v1:sdfmd.obj
 0001:0003501c       SDMMC_card_software_reset  0004601c f   sdmmc_boot_common_topaz_v1:sdfmd.obj
 0001:000350f4       SDMMC_card_send_appcmd     000460f4 f   sdmmc_boot_common_topaz_v1:sdfmd.obj
 0001:000351ec       SDMMC_get_csd              000461ec f   sdmmc_boot_common_topaz_v1:sdfmd.obj
 0001:0003531c       SDMMC_get_ext_csd          0004631c f   sdmmc_boot_common_topaz_v1:sdfmd.obj
 0001:00035444       SDMMC_GetCardCapacity      00046444 f   sdmmc_boot_common_topaz_v1:sdfmd.obj
 0001:00035644       SDMMC_set_blocklen         00046644 f   sdmmc_boot_common_topaz_v1:sdfmd.obj
 0001:00035744       SDMMC_send_rca             00046744 f   sdmmc_boot_common_topaz_v1:sdfmd.obj
 0001:00035904       SDMMC_R1b_busy_wait        00046904 f   sdmmc_boot_common_topaz_v1:sdfmd.obj
 0001:00035ad0       SDCard_command_config      00046ad0 f   sdmmc_boot_common_topaz_v1:sdfmd.obj
 0001:00035b20       SDMMC_GetInfo              00046b20 f   sdmmc_boot_common_topaz_v1:sdfmd.obj
 0001:00035bcc       SDMMC_EraseBlock           00046bcc f   sdmmc_boot_common_topaz_v1:sdfmd.obj
 0001:00035dfc       SDMMC_ReadSector           00046dfc f   sdmmc_boot_common_topaz_v1:sdfmd.obj
 0001:00035f9c       SDMMC_WriteSector          00046f9c f   sdmmc_boot_common_topaz_v1:sdfmd.obj
 0001:00036168       SDHCWriteXldr              00047168 f   sdmmc_boot_common_topaz_v1:sdboot.obj
 0001:00036394       SDHCWriteBoot              00047394 f   sdmmc_boot_common_topaz_v1:sdboot.obj
 0001:000365bc       SDHCWriteNK                000475bc f   sdmmc_boot_common_topaz_v1:sdboot.obj
 0001:000369e8       SDHCLoadNK                 000479e8 f   sdmmc_boot_common_topaz_v1:sdboot.obj
 0001:00036c28       SDHCFormatAll              00047c28 f   sdmmc_boot_common_topaz_v1:sdboot.obj
 0001:00036e78       SDHCCreateFileSystemPartition 00047e78 f   sdmmc_boot_common_topaz_v1:sdboot.obj
 0001:000370bc       SDHCLoadBootCFG            000480bc f   sdmmc_boot_common_topaz_v1:sdboot.obj
 0001:00037288       SDHCStoreBootCFG           00048288 f   sdmmc_boot_common_topaz_v1:sdboot.obj
 0001:0003745c       SDHCDisableBP              0004845c f   sdmmc_boot_common_topaz_v1:sdboot.obj
 0001:000374a8       EMMCToggleBP               000484a8 f   sdmmc_boot_common_topaz_v1:sdboot.obj
 0001:00037668       EMMCToggleBPSize           00048668 f   sdmmc_boot_common_topaz_v1:sdboot.obj
 0001:0003791c       ESDSetActivePartition      0004891c f   sdmmc_boot_common_topaz_v1:sdboot.obj
 0001:00037b00       ESDQueryPartitionSize      00048b00 f   sdmmc_boot_common_topaz_v1:sdboot.obj
 0001:00037bb4       ESDToggleBP                00048bb4 f   sdmmc_boot_common_topaz_v1:sdboot.obj
 0001:00037ca0       ESDToggleBPSize            00048ca0 f   sdmmc_boot_common_topaz_v1:sdboot.obj
 0001:00037eb0       SDReadDataBlock            00048eb0 f   sdmmc_boot_common_topaz_v1:sdboot.obj
 0001:000381b4       SDMMCDownload              000491b4 f   sdmmc_boot_common_topaz_v1:sdboot.obj
 0001:00038268       SDMMCReadData              00049268 f   sdmmc_boot_common_topaz_v1:sdboot.obj
 0001:00038328       SD_Init                    00049328 f   sdmmc_boot_common_topaz_v1:sd.obj
 0001:00038518       SD_VoltageValidation       00049518 f   sdmmc_boot_common_topaz_v1:sd.obj
 0001:00038af4       MMC_Init                   00049af4 f   sdmmc_boot_common_topaz_v1:mmc.obj
 0001:00039118       MMC_Send_Switch_Cmd        0004a118 f   sdmmc_boot_common_topaz_v1:mmc.obj
 0001:000391ac       FATInitDisk                0004a1ac f   sdmmc_boot_common_topaz_v1:sdfat.obj
 0001:0003a40c       FATGetDiskSize             0004b40c f   sdmmc_boot_common_topaz_v1:sdfat.obj
 0001:0003a424       FATReadDisk                0004b424 f   sdmmc_boot_common_topaz_v1:sdfat.obj
 0001:0003a4d8       FATGetPartitionNumber      0004b4d8 f   sdmmc_boot_common_topaz_v1:sdfat.obj
 0001:0003a4f8       FATGetPartitionSize        0004b4f8 f   sdmmc_boot_common_topaz_v1:sdfat.obj
 0001:0003a564       FATReadPartition           0004b564 f   sdmmc_boot_common_topaz_v1:sdfat.obj
 0001:0003a670       FATOpenFile                0004b670 f   sdmmc_boot_common_topaz_v1:sdfat.obj
 0001:0003c354       FATCloseFile               0004d354 f   sdmmc_boot_common_topaz_v1:sdfat.obj
 0001:0003c380       FATIsReadOnly              0004d380 f   sdmmc_boot_common_topaz_v1:sdfat.obj
 0001:0003c3cc       FATIsHidden                0004d3cc f   sdmmc_boot_common_topaz_v1:sdfat.obj
 0001:0003c418       FATIsSystem                0004d418 f   sdmmc_boot_common_topaz_v1:sdfat.obj
 0001:0003c464       FATIsVolumeLabel           0004d464 f   sdmmc_boot_common_topaz_v1:sdfat.obj
 0001:0003c4b0       FATIsDirectory             0004d4b0 f   sdmmc_boot_common_topaz_v1:sdfat.obj
 0001:0003c4fc       FATIsArchive               0004d4fc f   sdmmc_boot_common_topaz_v1:sdfat.obj
 0001:0003c548       FATEndOfFile               0004d548 f   sdmmc_boot_common_topaz_v1:sdfat.obj
 0001:0003c5a0       FATGetFileSize             0004d5a0 f   sdmmc_boot_common_topaz_v1:sdfat.obj
 0001:0003c5cc       FATGetFilePos              0004d5cc f   sdmmc_boot_common_topaz_v1:sdfat.obj
 0001:0003c5f8       FATSetFilePos              0004d5f8 f   sdmmc_boot_common_topaz_v1:sdfat.obj
 0001:0003c7e0       FATReadFile                0004d7e0 f   sdmmc_boot_common_topaz_v1:sdfat.obj
 0001:0003caf4       FATReadFileEx              0004daf4 f   sdmmc_boot_common_topaz_v1:sdfat.obj
 0001:0003cb5c       DumpMasterBootRecord       0004db5c f   sdmmc_boot_common_topaz_v1:sdfat.obj
 0001:0003cf08       DumpPartitionBootSector    0004df08 f   sdmmc_boot_common_topaz_v1:sdfat.obj
 0001:0003d66c       DumpFATTable               0004e66c f   sdmmc_boot_common_topaz_v1:sdfat.obj
 0001:0003d894       DumpDirectory              0004e894 f   sdmmc_boot_common_topaz_v1:sdfat.obj
 0001:0003db94       DumpDirectoryEx            0004eb94 f   sdmmc_boot_common_topaz_v1:sdfat.obj
 0001:0003dd30       PrepareBuffer              0004ed30 f   oal_spifmd:cspifmd.obj
 0001:0003df54       SPIFMD_Init                0004ef54 f   oal_spifmd:cspifmd.obj
 0001:0003e89c       SPIFMD_Deinit              0004f89c f   oal_spifmd:cspifmd.obj
 0001:0003e918       SPIFMD_GetInfo             0004f918 f   oal_spifmd:cspifmd.obj
 0001:0003e9bc       SPIFMD_GetBlockStatus      0004f9bc f   oal_spifmd:cspifmd.obj
 0001:0003e9e0       SPIFMD_SetBlockStatus      0004f9e0 f   oal_spifmd:cspifmd.obj
 0001:0003ea04       SPIFMD_EraseBlock          0004fa04 f   oal_spifmd:cspifmd.obj
 0001:0003eaa4       SPIFMD_ReadSector          0004faa4 f   oal_spifmd:cspifmd.obj
 0001:0003ebf0       SPIFMD_WriteSector         0004fbf0 f   oal_spifmd:cspifmd.obj
 0001:0003ed38       OALI2cInit                 0004fd38 f   i2cutils:i2cutils.obj
 0001:0003ef64       OALI2cEnable               0004ff64 f   i2cutils:i2cutils.obj
 0001:0003f030       OALI2cDisable              00050030 f   i2cutils:i2cutils.obj
 0001:0003f064       OALI2cCalculateClkRateDiv  00050064 f   i2cutils:i2cutils.obj
 0001:0003f36c       OALI2cGenerateStart        0005036c f   i2cutils:i2cutils.obj
 0001:0003f638       OALI2cRepeatedStart        00050638 f   i2cutils:i2cutils.obj
 0001:0003f894       OALI2cWriteData            00050894 f   i2cutils:i2cutils.obj
 0001:0003fb34       OALI2cReadData             00050b34 f   i2cutils:i2cutils.obj
 0001:0003fe2c       OALI2cSetReceiveMode       00050e2c f   i2cutils:i2cutils.obj
 0001:0003feb4       OALI2cSetTxAck             00050eb4 f   i2cutils:i2cutils.obj
 0001:0003ff3c       OALI2cPutData              00050f3c f   i2cutils:i2cutils.obj
 0001:000401a8       OALI2cGetData              000511a8 f   i2cutils:i2cutils.obj
 0001:000403a0       OALI2cGenerateStop         000513a0 f   i2cutils:i2cutils.obj
 0001:00040618       EbootInitTftpSimple        00051618 f   eboot:ebsimp.obj
 0001:00040758       EbootEtherReadData         00051758 f   eboot:ebsimp.obj
 0001:000409b4       EbootCheckIP               000519b4 f   eboot:ebsimp.obj
 0001:00040ad8       EbootGetDHCPAddr           00051ad8 f   eboot:ebsimp.obj
 0001:00040d48       EbootSendBootmeAndWaitForTftp 00051d48 f   eboot:ebsimp.obj
 0001:00040f94       EbootWaitForHostConnect    00051f94 f   eboot:ebsimp.obj
 0001:00041170       EbootInitEtherTransport    00052170 f   eboot:ebsimp.obj
 0001:00041300       EbootInitTFtpd             00052300 f   eboot:tftpd.obj
 0001:00041354       tolower                    00052354 f   eboot:tftpd.obj
 0001:000413ac       EbootTFtpdServerRegister   000523ac f   eboot:tftpd.obj
 0001:000414c0       EbootTFtpdServerUnRegister 000524c0 f   eboot:tftpd.obj
 0001:0004160c       GenerateSrcPort            0005260c f   eboot:tftpd.obj
 0001:00041628       TFtpdFormNewLink           00052628 f   eboot:tftpd.obj
 0001:00041e58       TFtpdCallBack              00052e58 f   eboot:tftpd.obj
 0001:00042720       EbootInitTFtp              00053720 f   eboot:tftp.obj
 0001:000427b4       EbootTFtpReceiver          000537b4 f   eboot:tftp.obj
 0001:00042a94       TFTPRetransmit             00053a94 f   eboot:tftp.obj
 0001:00042cd4       TFtpKillLink               00053cd4 f   eboot:tftp.obj
 0001:00042f2c       TFtpStateMachine           00053f2c f   eboot:tftp.obj
 0001:000436a4       TFtpOpen                   000546a4 f   eboot:tftp.obj
 0001:00043bc0       TFtpRead                   00054bc0 f   eboot:tftp.obj
 0001:00043f60       TFtpWrite                  00054f60 f   eboot:tftp.obj
 0001:00044304       SrcAddrFromFrame           00055304 f   eboot:udp.obj
 0001:00044420       EbootProcessARP            00055420 f   eboot:udp.obj
 0001:000448ac       EbootGratuitousARP         000558ac f   eboot:udp.obj
 0001:00044b68       EbootSendUDP               00055b68 f   eboot:udp.obj
 0001:000450b8       SetPromiscuousIP           000560b8 f   eboot:udp.obj
 0001:000450cc       ClearPromiscuousIP         000560cc f   eboot:udp.obj
 0001:000450e0       EbootCheckUDP              000560e0 f   eboot:udp.obj
 0001:00045700       EbootInitDHCP              00056700 f   eboot:dhcp.obj
 0001:00045784       EbootProcessDHCP           00056784 f   eboot:dhcp.obj
 0001:00045dd8       SendDHCP                   00056dd8 f   eboot:dhcp.obj
 0001:00046664       DHCPBuildOps               00057664 f   eboot:dhcp.obj
 0001:00046ba0       DHCPFindOption             00057ba0 f   eboot:dhcp.obj
 0001:00046cc8       DHCPParseField             00057cc8 f   eboot:dhcp.obj
 0001:00046d40       EbootDHCPRetransmit        00057d40 f   eboot:dhcp.obj
 0001:00046f84       EbootDHCPDecline           00057f84 f   eboot:dhcp.obj
 0001:0004705c       EbootReadSerialIP          0005805c f   eboot:dhcp.obj
 0001:000472b8       EbootProcessEDBG           000582b8 f   eboot:edbg.obj
 0001:0004755c       EbootSendBootme            0005855c f   eboot:edbg.obj
 0001:000478c4       __security_init_cookie     000588c4 f   gsnull:gsnull.obj
 0001:000478ec       __report_gsfailure         000588ec f   gsnull:gsnull.obj
 0001:00047900       memcpy                     00058900 f   fulllibc:memcpy.obj
 0001:000482a0       memset                     000592a0     fulllibc:memset.obj
 0001:00048328       __GSHandlerCheck           00059328 f   fulllibc:gshandler.obj
 0001:0004836c       __GSHandlerCheckCommon     0005936c f   fulllibc:gshandler.obj
 0001:00048410       __security_check_cookie    00059410 f   fulllibc:armsecgs.obj
 0001:00048420       __gsfailure                00059420     fulllibc:armsecgs.obj
 0001:00048464       memcmp                     00059464     fulllibc:memcmp.obj
 0001:00048530       atol                       00059530 f   fulllibc:atox.obj
 0001:00048568       atoi                       00059568 f   fulllibc:atox.obj
 0001:00048598       __rt_udivrem64by64         00059598     fulllibc:mdsdiv64.obj
 0001:00048690       __rt_divrem64by64          00059690     fulllibc:mdsdiv64.obj
 0001:000486e0       __rt_udiv64by64            000596e0     fulllibc:mdsdiv64.obj
 0001:000486f0       __rt_urem64by64            000596f0     fulllibc:mdsdiv64.obj
 0001:00048708       __rt_sdiv64by64            00059708     fulllibc:mdsdiv64.obj
 0001:00048718       __rt_srem64by64            00059718     fulllibc:mdsdiv64.obj
 0001:00048730       __rt_udiv                  00059730 f   fulllibc:__udiv.obj
 0001:000487f4       strncmp                    000597f4     fulllibc:astrncmp.obj
 0001:00048824       strlen                     00059824     fulllibc:mdsstrlen.obj
 0001:00048888       __rt_sdiv                  00059888 f   fulllibc:__div.obj
 0001:00048964       memmove                    00059964     fulllibc:memmove.obj
 0001:000490f4       memmovebigblk              0005a0f4     fulllibc:memmove.obj
 0001:00049b8c       strncpy_s                  0005ab8c f   fulllibc:strncpy_s.obj
 0001:00049ef8       toupper                    0005aef8 f   fulllibc:toupper.obj
 0001:00049f50       strcpy                     0005af50     fulllibc:strcpy.obj
 0001:00049fd4       strcat                     0005afd4     fulllibc:mdsstrcat.obj
 0001:00049ffc       strcpy_s                   0005affc f   fulllibc:strcpy_s.obj
 0001:0004a230       strcmp                     0005b230     fulllibc:mdsstrcmp.obj
 0001:0004a320       _itoa_s                    0005b320 f   fulllibc:xtoas.obj
 0001:0004a7f0       _ltoa_s                    0005b7f0 f   fulllibc:xtoas.obj
 0001:0004a860       _ultoa_s                   0005b860 f   fulllibc:xtoas.obj
 0001:0004a8a4       strcat_s                   0005b8a4 f   fulllibc:strcat_s.obj
 0001:0004aba8       strtol                     0005bba8 f   fulllibc:strtol.obj
 0001:0004b138       strtoul                    0005c138 f   fulllibc:strtol.obj
 0001:0004b174       __raise_int_divide_by_zero 0005c174 f   fulllibc:diverr.obj
 0001:0004b194       __raise_int_overflow       0005c194 f   fulllibc:diverr.obj
 0001:0004b1b4       _initp_misc_invarg         0005c1b4 f   fulllibc:invarg.obj
 0001:0004b1d4       _invalid_parameter         0005c1d4 f   fulllibc:invarg.obj
 0001:0004b25c       _invalid_parameter_noinfo  0005c25c f   fulllibc:invarg.obj
 0001:0004b288       _set_invalid_parameter_handler 0005c288 f   fulllibc:invarg.obj
 0001:0004b2f8       _get_invalid_parameter_handler 0005c2f8 f   fulllibc:invarg.obj
 0001:0004b340       __crtRaiseException        0005c340 f   fulllibc:raiseexc.obj
 0001:0004b37c       _encode_pointer            0005c37c f   fulllibc:encptr.obj
 0001:0004b3a0       _encoded_null              0005c3a0 f   fulllibc:encptr.obj
 0001:0004b3c8       _decode_pointer            0005c3c8 f   fulllibc:encptr.obj
 0001:0004b3ec       OALFlushDCache             0005c3ec f   oal_cache_arm926:flushdc.obj
 0001:0004b3f8       OALCleanDCache             0005c3f8 f   oal_cache_arm926:cleandc.obj
 0001:0004b404       OALFlushDCacheLines        0005c404 f   oal_cache_arm926:flushdclines.obj
 0001:0004b424       NKDbgPrintfW               0005c424 f   oal_blnk:wrappers.obj
 0001:0004b45c       NKvDbgPrintfW              0005c45c f   oal_blnk:wrappers.obj
 0001:0004b48c       NKwvsprintfW               0005c48c f   oal_blnk:format.obj
 0001:0004c7d4       BootloaderMain             0005d7d4 f   oal_blcommon:blcommon.obj
 0001:0004dd18       Nib2HexChar                0005ed18 f   oal_blcommon:blcommon.obj
 0001:0004dd90       OALLogSetZones             0005ed90 f   oal_log:debug.obj
 0001:0004ddf8       OALLogSerial               0005edf8 f   oal_log:log.obj
 0001:0004de50       OALLogPrintf               0005ee50 f   oal_log:log.obj
 0001:0004de88       OALKitlCreateName          0005ee88 f   oal_kitl:name.obj
 0001:0004e0bc       OALKitlIPtoString          0005f0bc f   oal_kitl:format.obj
 0001:0004e130       OALKitlMACtoString         0005f130 f   oal_kitl:format.obj
 0001:0004e1d8       OALKitlStringToIP          0005f1d8 f   oal_kitl:format.obj
 0001:0004e328       OALKitlStringToMAC         0005f328 f   oal_kitl:format.obj
 0001:0004e5a4       OEMWriteDebugString        0005f5a4 f   oal_other:debug.obj
 0001:0004e5f4       BSP_GetNANDBufferPointer   0005f5f4 f   bootcmn:nand.obj
 0001:0004e624       BSP_GetNANDImageCfg        0005f624 f   bootcmn:nand.obj
 0001:0004e6f4       BSP_OEMIoControl           0005f6f4 f   bootcmn:nand.obj
 0001:0004e720       SDConfigPins               0005f720 f   bootcmn:esdhc.obj
 0001:0004e900       SDInterface_Init           0005f900 f   bootcmn:esdhc.obj
 0001:0004ea54       SDHC_IsCardPresent         0005fa54 f   bootcmn:esdhc.obj
 0001:0004ea94       SDHC_IsCardWriteProtected  0005fa94 f   bootcmn:esdhc.obj
 0001:0004ead4       SetClockRate               0005fad4 f   bootcmn:esdhc.obj
 0001:0004eea0       SDHCSendCmdWaitResp        0005fea0 f   bootcmn:esdhc.obj
 0001:0004f464       SDHCReadResponse           00060464 f   bootcmn:esdhc.obj
 0001:0004f5b8       SDHCDataRead               000605b8 f   bootcmn:esdhc.obj
 0001:0004f7c8       SDHCDataWrite              000607c8 f   bootcmn:esdhc.obj
 0001:0004f958       BSP_MMC4BitSupported       00060958 f   bootcmn:esdhc.obj
 0001:0004f970       BSP_GetSDImageCfg          00060970 f   bootcmn:esdhc.obj
 0001:0004fa20       OutputHelpInformation      00060a20 f   bootshell_common_topaz_v1:bootshell.obj
 0001:0004fa88       SetReg                     00060a88 f   bootshell_common_topaz_v1:bootshell.obj
 0001:0004fb4c       ShowReg                    00060b4c f   bootshell_common_topaz_v1:bootshell.obj
 0001:0004fbf4       SetBit                     00060bf4 f   bootshell_common_topaz_v1:bootshell.obj
 0001:0004fd44       HexString2Hex              00060d44 f   bootshell_common_topaz_v1:bootshell.obj
 0001:000502b0       OffsetString2Decimal       000612b0 f   bootshell_common_topaz_v1:bootshell.obj
 0001:00050318       DebugGetLine               00061318 f   bootshell_common_topaz_v1:bootshell.obj
 0001:00050414       OEMWaitAndReadDebugByte    00061414 f   bootshell_common_topaz_v1:bootshell.obj
 0001:00050454       ?SwapBBI@@YAXXZ            00061454 f   nand_mx25_topaz_v1:cspnand.obj
 0001:000505bc       ?NFCAlloc@@YAHXZ           000615bc f   nand_mx25_topaz_v1:cspnand.obj
 0001:00050638       ?NFCSetPagesize@@YAHI@Z    00061638 f   nand_mx25_topaz_v1:cspnand.obj
 0001:000507b0       ?NFCWait@@YAXXZ            000617b0 f   nand_mx25_topaz_v1:cspnand.obj
 0001:00050810       CSPNAND_Reset              00061810 f   nand_mx25_topaz_v1:cspnand.obj
 0001:000508f0       CSPNAND_ReadID             000618f0 f   nand_mx25_topaz_v1:cspnand.obj
 0001:000509bc       CSPNAND_EnableECC          000619bc f   nand_mx25_topaz_v1:cspnand.obj
 0001:00050a54       CSPNAND_ILSupport          00061a54 f   nand_mx25_topaz_v1:cspnand.obj
 0001:00050a6c       CSPNAND_PostInit           00061a6c f   nand_mx25_topaz_v1:cspnand.obj
 0001:00050a7c       CSPNAND_Init               00061a7c f   nand_mx25_topaz_v1:cspnand.obj
 0001:00050d60       CSPNAND_Deinit             00061d60 f   nand_mx25_topaz_v1:cspnand.obj
 0001:00050d84       CSPNAND_ReadSector         00061d84 f   nand_mx25_topaz_v1:cspnand.obj
 0001:000516b0       CSPNAND_EraseBlock         000626b0 f   nand_mx25_topaz_v1:cspnand.obj
 0001:0005193c       CSPNAND_WriteSector        0006293c f   nand_mx25_topaz_v1:cspnand.obj
 0001:00051f8c       CSPNAND_GetECCStatus       00062f8c f   nand_mx25_topaz_v1:cspnand.obj
 0001:00052020       RdPageAlign4               00063020 f   nand_mx25_topaz_v1:nfcrw.obj
 0001:00052044       RdPageAlign1               00063044 f   nand_mx25_topaz_v1:nfcrw.obj
 0001:000520b4       RdPageAlign2               000630b4 f   nand_mx25_topaz_v1:nfcrw.obj
 0001:0005211c       RdPageAlign3               0006311c f   nand_mx25_topaz_v1:nfcrw.obj
 0001:0005218c       WrPageAlign4               0006318c f   nand_mx25_topaz_v1:nfcrw.obj
 0001:000521b0       WrPageAlign1               000631b0 f   nand_mx25_topaz_v1:nfcrw.obj
 0001:00052220       WrPageAlign2               00063220 f   nand_mx25_topaz_v1:nfcrw.obj
 0001:00052288       WrPageAlign3               00063288 f   nand_mx25_topaz_v1:nfcrw.obj
 0001:000522fc       __crt_unrecoverable_error  000632fc f   eboot:crtsupp.obj
 0001:00052310       BSPNAND_SetClock           00063310 f   bootcmn:nfc_boot.obj
 0001:00052334       BSPNAND_ConfigIOMUX        00063334 f   bootcmn:nfc_boot.obj
 0001:00052344       BSPNAND_RemapRegister      00063344 f   bootcmn:nfc_boot.obj
 0002:00000000       EthDevice                  00064000     eboot.obj
 0002:00000270       g_DownloadImage            00064270     bootcmn:main.obj
 0002:00000350       Am79c874Info               00064350     oal_ethdrv_fec_common_topaz_v1:fec.obj
 0002:00000554       PhyInfo                    00064554     oal_ethdrv_fec_common_topaz_v1:fec.obj
 0002:00000568       LAN8700Info                00064568     oal_ethdrv_fec_common_topaz_v1:fec.obj
 0002:00000770       Dp83640Info                00064770     oal_ethdrv_fec_common_topaz_v1:fec.obj
 0002:00000978       KSZ8041NLInfo              00064978     oal_ethdrv_fec_common_topaz_v1:fec.obj
 0002:00000b7c       bRndisSendPacketEmpty      00064b7c     fsl_rne_mdd_common_topaz_v1:rndis.obj
 0002:00000bb0       RNdisMddSupportedOids      00064bb0     fsl_rne_mdd_common_topaz_v1:hostmini.obj
 0002:00000c40       g_InterruptData            00064c40     fsl_rne_pdd_common_topaz_v1:rndis_pdd.obj
 0002:00001000       g_serial_rev_buf           00065000     fsl_rne_pdd_common_topaz_v1:buffer.obj
 0002:00001000       g_rndis_ep2_buf            00065000     fsl_rne_pdd_common_topaz_v1:buffer.obj
 0002:00003000       g_serial_send_buf          00067000     fsl_rne_pdd_common_topaz_v1:buffer.obj
 0002:00003000       g_rndis_ep3_buf            00067000     fsl_rne_pdd_common_topaz_v1:buffer.obj
 0002:00005000       g_rndis_ep0_buf            00069000     fsl_rne_pdd_common_topaz_v1:buffer.obj
 0002:00005440       ?ChipInfo@@3PAU_NandChipInfo@@A 00069440     nand_common_topaz_v1:fmd.obj
 0002:00005570       __security_cookie          00069570     gsnull:gsnull.obj
 0002:00005574       __security_cookie_complement 00069574     gsnull:gsnull.obj
 0002:000055c0       initialOALLogZones         000695c0     oal_log:debug.obj
 0002:000055c8       dpCurSettings              000695c8     oal_log:debug.obj
 0002:00005bb0       g_bNandBootloader          00069bb0     bootcmn:main.obj
 0002:00005bb4       g_bNandExist               00069bb4     bootcmn:main.obj
 0002:00005bb8       g_bSDHCBootloader          00069bb8     bootcmn:main.obj
 0002:00005bbc       g_bSDHCExist               00069bbc     bootcmn:main.obj
 0002:00005bc0       g_bSpiBootloader           00069bc0     bootcmn:main.obj
 0002:00005bc4       g_bSpiExist                00069bc4     bootcmn:main.obj
 0002:00005bc8       g_SerialUSBDownload        00069bc8     bootcmn:main.obj
 0002:00005c08       bCFGChanged                00069c08     blmenu_common_topaz_v1:menu.obj
 0002:00005c0c       PrintSoc                   00069c0c     blmenu_common_topaz_v1:menu.obj
 0002:0000fb40       g_pEP3DataWrapper          00073b40     fsl_rne_pdd_common_topaz_v1:rndis_pdd.obj
 0002:0000fb44       g_devState                 00073b44     fsl_rne_pdd_common_topaz_v1:rndis_pdd.obj
 0002:0000fb48       g_EP0TransferState         00073b48     fsl_rne_pdd_common_topaz_v1:rndis_pdd.obj
 0002:0000fb4c       g_EP2TransferState         00073b4c     fsl_rne_pdd_common_topaz_v1:rndis_pdd.obj
 0002:00010ea8       ?g_buffer@@3PAEA           00074ea8     oal_blserial:serfuncs.obj
 0002:00011ac8       ?g_mddInterface@@3U_UFN_MDD_INTERFACE_INFO@@A 00075ac8     fsl_serial_pdd_common_topaz_v1:serial_dl.obj
 0002:00011ad0       ?g_EP1Transfer@@3U_STransfer@@A 00075ad0     fsl_serial_pdd_common_topaz_v1:serial_dl.obj
 0002:00011af0       ?g_RecvBuffer@@3PAEA       00075af0     fsl_serial_pdd_common_topaz_v1:serial_dl.obj
 0002:00011b10       ?g_pddInterface@@3U_UFN_PDD_INTERFACE_INFO@@A 00075b10     fsl_serial_pdd_common_topaz_v1:serial_dl.obj
 0002:00011b70       ?g_EP2Transfer@@3U_STransfer@@A 00075b70     fsl_serial_pdd_common_topaz_v1:serial_dl.obj
 0002:00011b90       ?g_EP0Transfer@@3U_STransfer@@A 00075b90     fsl_serial_pdd_common_topaz_v1:serial_dl.obj
 0002:00011bf4       ?g_DeviceState@@3W4DEVICE_STATE@@A 00075bf4     fsl_serial_pdd_common_topaz_v1:serial_dl.obj
 0002:00011bf8       ?g_EP0State@@3W4TRANSFER_STATE@@A 00075bf8     fsl_serial_pdd_common_topaz_v1:serial_dl.obj
 0002:00011bfc       ?g_EP1State@@3W4TRANSFER_STATE@@A 00075bfc     fsl_serial_pdd_common_topaz_v1:serial_dl.obj
 0002:00011c00       ?g_EP2State@@3W4TRANSFER_STATE@@A 00075c00     fsl_serial_pdd_common_topaz_v1:serial_dl.obj
 0002:00011c04       ?g_RecvBufferHead@@3GA     00075c04     fsl_serial_pdd_common_topaz_v1:serial_dl.obj
 0002:00011c08       ?g_RecvBufferTail@@3GA     00075c08     fsl_serial_pdd_common_topaz_v1:serial_dl.obj
 0002:00011c6c       ?g_FlashInfoExt@@3U_FlashInfoExt@@A 00075c6c     nand_common_topaz_v1:fmd.obj
 0002:00011ca4       ?g_bInterLeaveMode@@3HA    00075ca4     nand_common_topaz_v1:fmd.obj
 0002:00011cd0       ?g_SectorBuf@@3PAEA        00075cd0     nandfmd_lib:nandbsp.obj
 0002:000124d0       ?g_BBTSecondBuf@@3PAEA     000764d0     nandfmd_lib:nandbsp.obj
 0002:00012cd0       ?g_BBTFirstBuf@@3PAEA      00076cd0     nandfmd_lib:nandbsp.obj
 0002:000134d0       ?BBMarkPage@@3PAEA         000774d0     nandfmd_lib:nandbsp.obj
 0002:000134d4       Card_rca                   000774d4     sdmmc_boot_common_topaz_v1:sdfmd.obj
 0002:000134d8       bHighDensityCard           000774d8     sdmmc_boot_common_topaz_v1:sdfmd.obj
 0002:000134dc       mmcSpecVersion             000774dc     sdmmc_boot_common_topaz_v1:sdfmd.obj
 0002:000134e0       eSDBPEnabled               000774e0     sdmmc_boot_common_topaz_v1:sdboot.obj
 0002:000134e8       bCacheBuffer               000774e8     sdmmc_boot_common_topaz_v1:sdboot.obj
 0002:000136e8       eSDBootPartitionSize       000776e8     sdmmc_boot_common_topaz_v1:sd.obj
 0002:0001fdf8       bDoLaunch                  00083df8     eboot:tftpd.obj
 0002:0001fdfc       TftpPeerAddr               00083dfc     eboot:tftpd.obj
 0002:00021e30       bLastCmdRead               00085e30     bootcmn:esdhc.obj
 0002:00021e34       ?bECCMode@@3_NA            00085e34     nand_mx25_topaz_v1:cspnand.obj
 0002:00021e38       ?g_CSPfi@@3U_FlashInfoExt@@A 00085e38     nand_mx25_topaz_v1:cspnand.obj
 0002:00021e70       g_pNFC                     00085e70     nand_mx25_topaz_v1:cspnand.obj
 0002:00021e80       g_DeviceAddr               00085e80     <common>
 0002:00021ea0       g_oalCacheInfo             00085ea0     <common>
 0002:00021ee8       g_pOEMVerifyMemory         00085ee8     <common>
 0002:00021eec       g_dwROMOffset              00085eec     <common>
 0002:00021ef0       g_pOEMReportError          00085ef0     <common>
 0002:00021ef4       g_pOEMMultiBINNotify       00085ef4     <common>
 0002:00021ef8       g_pOEMCheckSignature       00085ef8     <common>
 0002:00021efc       g_pDdkClkConfig            00085efc     <common>
 0002:00021f00       g_pUART                    00085f00     <common>
 0002:00021f04       g_pIOMUX                   00085f04     <common>
 0002:00021f08       g_pCRM                     00085f08     <common>
 0002:00021f0c       dwVVN                      00085f0c     <common>
 0002:00021f10       g_pESDHCReg                00085f10     <common>
 0002:00021f14       g_pGPIO4                   00085f14     <common>
 0002:00021f20       sectorBuf                  00085f20     <common>
 0002:00022f20       pfnEDbgDisableInts         00086f20     <common>
 0002:00022f24       pfnEDbgGetFrame            00086f24     <common>
 0002:00022f28       pfnEDbgEnableInts          00086f28     <common>
 0002:00022f2c       pfnEDbgInit                00086f2c     <common>
 0002:00022f30       pfnEDbgSendFrame           00086f30     <common>
 0002:00022f34       pfnEDbgInitDMABuffer       00086f34     <common>
 0002:00022f38       g_pBSPArgs                 00086f38     <common>
 0002:00022f3c       g_ImageType                00086f3c     <common>
 0002:00022f40       g_ImageMemory              00086f40     <common>
 0002:00022f44       g_DefaultRamAddress        00086f44     <common>
 0002:00022f50       g_BinDIO                   00086f50     <common>
 0002:00022f60       g_BootCFG                  00086f60     <common>
 0002:00022fbc       SetBitFlag                 00086fbc     <common>
 0002:00022fc0       SetRegFlag                 00086fc0     <common>
 0002:00022fc4       ExitingShellFlag           00086fc4     <common>
 0002:00022fc8       ShowRegFlag                00086fc8     <common>
 0002:00022fd0       BspValueSet                00086fd0     <common>
 0002:00022fda       BspBitSet                  00086fda     <common>
 0002:00022fe0       Linebuffer                 00086fe0     <common>
 0002:000231e0       BspAddrSet                 000871e0     <common>
 0002:00023200       RndisMdd                   00087200     <common>
 0002:000232d0       g_EP0DataWrapper           000872d0     <common>
 0002:000232e0       MDDZONE5                   000872e0     <common>
 0002:000232e8       g_mddInterface             000872e8     <common>
 0002:00023300       g_EP1Transfer              00087300     <common>
 0002:00023320       g_RndisKitlDev             00087320     <common>
 0002:00023768       g_udr                      00087768     <common>
 0002:00023770       MDDZONE4                   00087770     <common>
 0002:00023774       PDDZONE                    00087774     <common>
 0002:00023780       g_EP3Transfer              00087780     <common>
 0002:000237a0       g_pddInterface             000877a0     <common>
 0002:00023800       MDDZONE3                   00087800     <common>
 0002:00023820       g_EP2Transfer              00087820     <common>
 0002:00023840       PDDZONE0                   00087840     <common>
 0002:00023860       g_EP0Transfer              00087860     <common>
 0002:00023880       MDDZONE0                   00087880     <common>
 0002:00023884       MDDZONE                    00087884     <common>
 0002:00023888       MDDZONE2                   00087888     <common>
 0002:000238a0       g_csRegister               000878a0     <common>
 0002:000238c0       SDController               000878c0     <common>
 0002:00023980       g_fnFileInfo               00087980     <common>
 0002:000239a0       extCSDBuffer               000879a0     <common>
 0002:00023ba0       sdCardReg                  00087ba0     <common>
 0002:00023be0       SDImageCfg                 00087be0     <common>
 0002:00023c0c       g_pCspi                    00087c0c     <common>
 0002:00023c20       TFtpLinks                  00087c20     <common>
 0002:000244e0       wOdoWellKnownServerPort    000884e0     <common>
 0002:000244e2       wHostWellKnownServerPort   000884e2     <common>
 0002:000244e4       nNumTFtpLinksInUse         000884e4     <common>
 0002:00024500       TFTPFrameBuffer            00088500     <common>
 0002:00024940       TFtpdServerRegistry        00088940     <common>
 0002:00024a08       __pInvalidArgHandler       00088a08     <common>

 entry point at        0001:00000000

 Static symbols

 0001:0001097c       SelectEtherDevice          0002197c f   menu.obj
 0001:00010a24       SelectSerialDebug          00021a24 f   menu.obj
 0001:00010ae8       SelectBootDevice           00021ae8 f   menu.obj
 0001:000110c8       PrintData                  000220c8 f   menu.obj
 0001:0001279c       GetFormatValue             0002379c f   oal_blnk:formata.obj
 0001:00012884       Reverse                    00023884 f   oal_blnk:formata.obj
 0001:00012e58       InitGlobals                00023e58 f   bspcmn:debugserial.obj
 0001:0001542c       InitUSBRNDISDevice         0002642c f   bootcmn:ether.obj
 0001:00019378       ParseCommand               0002a378 f   bsp_bootshell:bspbootshell.obj
 0001:0001e41c       PDD_SendNotification       0002f41c f   fsl_rne_pdd_common_topaz_v1:rndis_pdd.obj
 0001:0001e498       PDD_RecvNotification       0002f498 f   fsl_rne_pdd_common_topaz_v1:rndis_pdd.obj
 0001:0001f6cc       RegisterUSBDevice          000306cc f   fsl_rne_pdd_common_topaz_v1:rndis_pdd.obj
 0001:0002037c       PDD_DiscardPendingMessages 0003137c f   fsl_rne_pdd_common_topaz_v1:rndis_pdd.obj
 0001:000213e8       CeLogMsg                   000323e8 f   usb_usbfn_mx25_topaz_v1:i_pdd.obj
 0001:00022040       GetSetupPacket             00033040 f   usb_usbfn_mx25_topaz_v1:i_pdd.obj
 0001:00024f1c       HandleUSBReset             00035f1c f   usb_usbfn_mx25_topaz_v1:i_pdd.obj
 0001:00025408       DevStatEvent               00036408 f   usb_usbfn_mx25_topaz_v1:i_pdd.obj
 0001:000254cc       USBControllerRun           000364cc f   usb_usbfn_mx25_topaz_v1:i_pdd.obj
 0001:00026dec       BuildTdBufferList          00037dec f   usb_usbfn_mx25_topaz_v1:i_pdd.obj
 0001:00027b2c       FlushEndpoint              00038b2c f   usb_usbfn_mx25_topaz_v1:i_pdd.obj
 0001:000283a0       PrimeQh0ForZeroTransfer    000393a0 f   usb_usbfn_mx25_topaz_v1:i_pdd.obj
 0001:00028db4       SetDeviceTestMode          00039db4 f   usb_usbfn_mx25_topaz_v1:i_pdd.obj
 0001:0002a114       InitQh0                    0003b114 f   usb_usbfn_mx25_topaz_v1:i_pdd.obj
 0001:0002b350       Log2                       0003c350 f   usb_usbfn_mx25_topaz_v1:i_pdd.obj
 0001:0002d728       ?HandleUSBDeviceRegistration@@YAXXZ 0003e728 f   fsl_serial_pdd_common_topaz_v1:serial_dl.obj
 0001:0002dcf8       ?HandlePDDNotification@@YAHPAXKK@Z 0003ecf8 f   fsl_serial_pdd_common_topaz_v1:serial_dl.obj
 0001:0002e0a8       ?HandleSetupPkt@@YAXPAU_USB_DEVICE_REQUEST@@PAU_EP0_REQUEST@@@Z 0003f0a8 f   fsl_serial_pdd_common_topaz_v1:serial_dl.obj
 0001:0002ef78       InitializeMux              0003ff78 f   fsl_usbfn_rndiskitl_mx25_topaz_v1:hwinit.obj
 0001:0002ef90       InitializeTransceiver      0003ff90 f   fsl_usbfn_rndiskitl_mx25_topaz_v1:hwinit.obj
 0001:0002f3bc       NANDBootInit               000403bc f   nand_boot_common_topaz_v1:nandboot.obj
 0001:0003264c       ?CalcSector@@YAKAAK@Z      0004364c f   nand_common_topaz_v1:fmd.obj
 0001:00032784       ?CalcBlock@@YAKAAK@Z       00043784 f   nand_common_topaz_v1:fmd.obj
 0001:00032f18       ?GetBlockBadStatus@@YAHK@Z 00043f18 f   nand_common_topaz_v1:bbt.obj
 0001:0003304c       ?SetBlockBadStatus@@YAXK@Z 0004404c f   nand_common_topaz_v1:bbt.obj
 0001:000330f0       ?WriteBBT@@YAHKK@Z         000440f0 f   nand_common_topaz_v1:bbt.obj
 0001:00033364       ?BBT_GetBlockReservedStatus@@YAHKK@Z 00044364 f   nand_common_topaz_v1:bbt.obj
 0001:00033454       ?BBT_SetBlockReservedStatus@@YAHKK@Z 00044454 f   nand_common_topaz_v1:bbt.obj
 0001:00033594       ?BBT_WriteOperation@@YAHKKPAE@Z 00044594 f   nand_common_topaz_v1:bbt.obj
 0001:000338b8       ?BBT_GetNumSector@@YAKXZ   000448b8 f   nand_common_topaz_v1:bbt.obj
 0001:00033900       ?BBT_GetSectorAddr@@YAKK@Z 00044900 f   nand_common_topaz_v1:bbt.obj
 0001:000339b0       ?BBT_EraseOperation@@YAHKK@Z 000449b0 f   nand_common_topaz_v1:bbt.obj
 0001:00033ad0       ?WriteBBTSignature@@YAHKK@Z 00044ad0 f   nand_common_topaz_v1:bbt.obj
 0001:00033cac       ?OpenBBT@@YAHXZ            00044cac f   nand_common_topaz_v1:bbt.obj
 0001:00033e2c       ?ReadBBT@@YAHXZ            00044e2c f   nand_common_topaz_v1:bbt.obj
 0001:00034170       ?BBT_ReadOperation@@YAHKKPAE@Z 00045170 f   nand_common_topaz_v1:bbt.obj
 0001:00034368       ?ReadBlockBadStatus@@YAHKK@Z 00045368 f   nand_common_topaz_v1:bbt.obj
 0001:000345f4       ?ReadBBTSignature@@YAHKK@Z 000455f4 f   nand_common_topaz_v1:bbt.obj
 0001:000347dc       ?CreateBBT@@YAHXZ          000457dc f   nand_common_topaz_v1:bbt.obj
 0001:000387e8       SDGetBitMode               000497e8 f   sdmmc_boot_common_topaz_v1:sd.obj
 0001:000389a0       SDSetBusWidth              000499a0 f   sdmmc_boot_common_topaz_v1:sd.obj
 0001:00038d78       MMC_VoltageValidation      00049d78 f   sdmmc_boot_common_topaz_v1:mmc.obj
 0001:00038fb0       MMC_GetSpecVersion         00049fb0 f   sdmmc_boot_common_topaz_v1:mmc.obj
 0001:0003902c       MMC_SetBusWidth            0004a02c f   sdmmc_boot_common_topaz_v1:mmc.obj
 0001:00039238       InitPartition              0004a238 f   sdmmc_boot_common_topaz_v1:sdfat.obj
 0001:00039b54       InitMasterBootRecord       0004ab54 f   sdmmc_boot_common_topaz_v1:sdfat.obj
 0001:0003a3f4       GetDefaultSectorSize       0004b3f4 f   sdmmc_boot_common_topaz_v1:sdfat.obj
 0001:0003a734       ClearFileInfo              0004b734 f   sdmmc_boot_common_topaz_v1:sdfat.obj
 0001:0003a7a0       FindRootDirEntry           0004b7a0 f   sdmmc_boot_common_topaz_v1:sdfat.obj
 0001:0003a9bc       InitFileInfo               0004b9bc f   sdmmc_boot_common_topaz_v1:sdfat.obj
 0001:0003aa8c       CalculateFATEntries        0004ba8c f   sdmmc_boot_common_topaz_v1:sdfat.obj
 0001:0003ab20       IsAllocFATEntry            0004bb20 f   sdmmc_boot_common_topaz_v1:sdfat.obj
 0001:0003ac90       IsEndFATEntry              0004bc90 f   sdmmc_boot_common_topaz_v1:sdfat.obj
 0001:0003adcc       GetFATEntry                0004bdcc f   sdmmc_boot_common_topaz_v1:sdfat.obj
 0001:0003b1bc       FillCacheFATEntries        0004c1bc f   sdmmc_boot_common_topaz_v1:sdfat.obj
 0001:0003b31c       GetFATEntryBytes           0004c31c f   sdmmc_boot_common_topaz_v1:sdfat.obj
 0001:0003b374       GetFATEntryBits            0004c374 f   sdmmc_boot_common_topaz_v1:sdfat.obj
 0001:0003b40c       ConvertBytesToFATEntries   0004c40c f   sdmmc_boot_common_topaz_v1:sdfat.obj
 0001:0003b4d4       ConvertFATEntriesToBytes   0004c4d4 f   sdmmc_boot_common_topaz_v1:sdfat.obj
 0001:0003b59c       CompareFileName            0004c59c f   sdmmc_boot_common_topaz_v1:sdfat.obj
 0001:0003b6b4       FindNextDirEntry           0004c6b4 f   sdmmc_boot_common_topaz_v1:sdfat.obj
 0001:0003b77c       GetDirEntryEx              0004c77c f   sdmmc_boot_common_topaz_v1:sdfat.obj
 0001:0003ba30       GetDirEntry                0004ca30 f   sdmmc_boot_common_topaz_v1:sdfat.obj
 0001:0003c2b0       ComputeCheckSum            0004d2b0 f   sdmmc_boot_common_topaz_v1:sdfat.obj
 0001:0003db54       GetDirEntryNumber          0004eb54 f   sdmmc_boot_common_topaz_v1:sdfat.obj
 0001:0003e228       CalcClockDiv               0004f228 f   oal_spifmd:cspifmd.obj
 0001:0003e2c0       CSPI_ClockEnable           0004f2c0 f   oal_spifmd:cspifmd.obj
 0001:0003e30c       CSPI_GpioMux               0004f30c f   oal_spifmd:cspifmd.obj
 0001:0003e398       TransactMessage            0004f398 f   oal_spifmd:cspifmd.obj
 0001:0003e75c       WriteEnable                0004f75c f   oal_spifmd:cspifmd.obj
 0001:0003e7d0       FlashIsWriteable           0004f7d0 f   oal_spifmd:cspifmd.obj
 0001:0003e838       WriteInProgress            0004f838 f   oal_spifmd:cspifmd.obj
 0001:0004069c       EbootSimpleCallback        0005169c f   eboot:ebsimp.obj
 0001:00045510       DuplicateIPWarning         00056510 f   eboot:udp.obj
 0001:00045598       CRC                        00056598 f   eboot:udp.obj
 0001:000469f4       FormatDHCPName             000579f4 f   eboot:dhcp.obj
 0001:00046ae8       HexToChar                  00057ae8 f   eboot:dhcp.obj
 0001:0004a3b8       xtoa_s                     0005b3b8 f   fulllibc:xtoas.obj
 0001:0004abe4       strtoxl                    0005bbe4 f   fulllibc:strtol.obj
 0001:0004b0d8       __ascii_isspace            0005c0d8 f   fulllibc:strtol.obj
 0001:0004c65c       GetFormatValue             0005d65c f   oal_blnk:format.obj
 0001:0004c744       Reverse                    0005d744 f   oal_blnk:format.obj
 0001:0004c9f0       HALT                       0005d9f0 f   oal_blcommon:blcommon.obj
 0001:0004ca2c       KernelRelocate             0005da2c f   oal_blcommon:blcommon.obj
 0001:0004cb54       DownloadImage              0005db54 f   oal_blcommon:blcommon.obj
 0001:0004cd58       GetImageType               0005dd58 f   oal_blcommon:blcommon.obj
 0001:0004cef0       CheckImageManifest         0005def0 f   oal_blcommon:blcommon.obj
 0001:0004cfe0       VerifyChecksum             0005dfe0 f   oal_blcommon:blcommon.obj
 0001:0004d0a0       DownloadBin                0005e0a0 f   oal_blcommon:blcommon.obj
 0001:0004d6e0       DownloadNB0                0005e6e0 f   oal_blcommon:blcommon.obj
 0001:0004d950       WriteImageToFlash          0005e950 f   oal_blcommon:blcommon.obj
 0001:0004da88       ComputeChecksum            0005ea88 f   oal_blcommon:blcommon.obj
 0001:0004db8c       IsKernelRegion             0005eb8c f   oal_blcommon:blcommon.obj
 0001:0004eee4       SDHCCmdConfig              0005fee4 f   bootcmn:esdhc.obj
 0001:0004f350       SDHCWaitEndCmdRespIntr     00060350 f   bootcmn:esdhc.obj
 0001:0004f740       SDHCCheckDataStatus        00060740 f   bootcmn:esdhc.obj
 0001:00050868       ?SetCs@@YAXK@Z             00061868 f   nand_mx25_topaz_v1:cspnand.obj
 0001:00051598       ?NFCReadMain@@YAXPAE@Z     00062598 f   nand_mx25_topaz_v1:cspnand.obj
 0001:0005161c       ?NFCReadSpare@@YAXPAU_SectorInfo@@@Z 0006261c f   nand_mx25_topaz_v1:cspnand.obj
 0001:00051db4       ?NFCWriteMain@@YAXPAE@Z    00062db4 f   nand_mx25_topaz_v1:cspnand.obj
 0001:00051e38       ?NFCWriteSpare@@YAXPAU_SectorInfo@@@Z 00062e38 f   nand_mx25_topaz_v1:cspnand.obj
 0001:00051edc       ?NFCClearSpare@@YAXXZ      00062edc f   nand_mx25_topaz_v1:cspnand.obj
